################################################################################
#                                                                              #
#      IAR Universal Linker V6.2.2.68                                          #
#                                                                              #
#           Link time     =  08/Sep/2015  11:52:24                             #
#           Target CPU    =  x51                                               #
#           List file     =  C:\ble\BLE-CC254x-1.4.1.43908\Projects\ble\Simple #
#                            BLEBroadcaster-usb\CC2540\CC2540USB\List\HostTest #
#                            Release.map                                       #
#           Output file 1 =  C:\ble\BLE-CC254x-1.4.1.43908\Projects\ble\Simple #
#                            BLEBroadcaster-usb\CC2540\CC2540USB\Exe\HostTestR #
#                            elease.d51                                        #
#                            Format: ubrof10                                   #
#                            UBROF version 10.0.6                              #
#                            Using library modules for C-SPY (-rt)             #
#           Output file 2 =  C:\ble\BLE-CC254x-1.4.1.43908\Projects\ble\Simple #
#                            BLEBroadcaster-usb\CC2540\hex\HostTestReleaseCC25 #
#                            40Usb.hex                                         #
#                            Format: intel-extended                            #
#           Command line  =  "-IC:\Program Files\IAR Systems\Embedded Workbenc #
#                            h 7.2\8051\CONFIG\"                               #
#                            -D_NR_OF_BANKS=0x07 -D_CODEBANK_END=0xFFFF        #
#                            -D_CODEBANK_START=0x8000 -D?CBANK_MASK=0xFF       #
#                            -D?CBANK=0x9F                                     #
#                            C:\ble\BLE-CC254x-1.4.1.43908\Projects\ble\Simple #
#                            BLEBroadcaster-usb\CC2540\CC2540USB\Obj\broadcast #
#                            er.r51                                            #
#                            C:\ble\BLE-CC254x-1.4.1.43908\Projects\ble\Librar #
#                            ies\CC2540DB\bin\CC2540_BLE_bcast.lib             #
#                            C:\ble\BLE-CC254x-1.4.1.43908\Projects\ble\Librar #
#                            ies\Common\bin\CC254x_BLE_HCI_TL_bcast.lib        #
#                            C:\ble\BLE-CC254x-1.4.1.43908\Projects\ble\Simple #
#                            BLEBroadcaster-usb\CC2540\CC2540USB\Obj\gap.r51   #
#                            C:\ble\BLE-CC254x-1.4.1.43908\Projects\ble\Simple #
#                            BLEBroadcaster-usb\CC2540\CC2540USB\Obj\gattserva #
#                            pp_util.r51                                       #
#                            C:\ble\BLE-CC254x-1.4.1.43908\Projects\ble\Simple #
#                            BLEBroadcaster-usb\CC2540\CC2540USB\Obj\hal_adc.r #
#                            51                                                #
#                            C:\ble\BLE-CC254x-1.4.1.43908\Projects\ble\Simple #
#                            BLEBroadcaster-usb\CC2540\CC2540USB\Obj\hal_aes.r #
#                            51                                                #
#                            C:\ble\BLE-CC254x-1.4.1.43908\Projects\ble\Simple #
#                            BLEBroadcaster-usb\CC2540\CC2540USB\Obj\hal_asser #
#                            t.r51                                             #
#                            C:\ble\BLE-CC254x-1.4.1.43908\Projects\ble\Simple #
#                            BLEBroadcaster-usb\CC2540\CC2540USB\Obj\hal_dma.r #
#                            51                                                #
#                            C:\ble\BLE-CC254x-1.4.1.43908\Projects\ble\Simple #
#                            BLEBroadcaster-usb\CC2540\CC2540USB\Obj\hal_drive #
#                            rs.r51                                            #
#                            C:\ble\BLE-CC254x-1.4.1.43908\Projects\ble\Simple #
#                            BLEBroadcaster-usb\CC2540\CC2540USB\Obj\hal_flash #
#                            .r51                                              #
#                            C:\ble\BLE-CC254x-1.4.1.43908\Projects\ble\Simple #
#                            BLEBroadcaster-usb\CC2540\CC2540USB\Obj\hal_key.r #
#                            51                                                #
#                            C:\ble\BLE-CC254x-1.4.1.43908\Projects\ble\Simple #
#                            BLEBroadcaster-usb\CC2540\CC2540USB\Obj\hal_lcd.r #
#                            51                                                #
#                            C:\ble\BLE-CC254x-1.4.1.43908\Projects\ble\Simple #
#                            BLEBroadcaster-usb\CC2540\CC2540USB\Obj\hal_led.r #
#                            51                                                #
#                            C:\ble\BLE-CC254x-1.4.1.43908\Projects\ble\Simple #
#                            BLEBroadcaster-usb\CC2540\CC2540USB\Obj\hal_sleep #
#                            .r51                                              #
#                            C:\ble\BLE-CC254x-1.4.1.43908\Projects\ble\Simple #
#                            BLEBroadcaster-usb\CC2540\CC2540USB\Obj\hal_start #
#                            up.r51                                            #
#                            C:\ble\BLE-CC254x-1.4.1.43908\Projects\ble\Simple #
#                            BLEBroadcaster-usb\CC2540\CC2540USB\Obj\hal_timer #
#                            .r51                                              #
#                            C:\ble\BLE-CC254x-1.4.1.43908\Projects\ble\Simple #
#                            BLEBroadcaster-usb\CC2540\CC2540USB\Obj\hal_uart. #
#                            r51                                               #
#                            C:\ble\BLE-CC254x-1.4.1.43908\Projects\ble\Simple #
#                            BLEBroadcaster-usb\CC2540\CC2540USB\Obj\npi.r51   #
#                            C:\ble\BLE-CC254x-1.4.1.43908\Projects\ble\Simple #
#                            BLEBroadcaster-usb\CC2540\CC2540USB\Obj\OnBoard.r #
#                            51                                                #
#                            C:\ble\BLE-CC254x-1.4.1.43908\Projects\ble\Simple #
#                            BLEBroadcaster-usb\CC2540\CC2540USB\Obj\OSAL.r51  #
#                            C:\ble\BLE-CC254x-1.4.1.43908\Projects\ble\Simple #
#                            BLEBroadcaster-usb\CC2540\CC2540USB\Obj\osal_bufm #
#                            gr.r51                                            #
#                            C:\ble\BLE-CC254x-1.4.1.43908\Projects\ble\Simple #
#                            BLEBroadcaster-usb\CC2540\CC2540USB\Obj\osal_cbti #
#                            mer.r51                                           #
#                            C:\ble\BLE-CC254x-1.4.1.43908\Projects\ble\Simple #
#                            BLEBroadcaster-usb\CC2540\CC2540USB\Obj\OSAL_Cloc #
#                            kBLE.r51                                          #
#                            C:\ble\BLE-CC254x-1.4.1.43908\Projects\ble\Simple #
#                            BLEBroadcaster-usb\CC2540\CC2540USB\Obj\OSAL_Memo #
#                            ry.r51                                            #
#                            C:\ble\BLE-CC254x-1.4.1.43908\Projects\ble\Simple #
#                            BLEBroadcaster-usb\CC2540\CC2540USB\Obj\OSAL_PwrM #
#                            gr.r51                                            #
#                            C:\ble\BLE-CC254x-1.4.1.43908\Projects\ble\Simple #
#                            BLEBroadcaster-usb\CC2540\CC2540USB\Obj\OSAL_Simp #
#                            leBLEBroadcaster.r51                              #
#                            C:\ble\BLE-CC254x-1.4.1.43908\Projects\ble\Simple #
#                            BLEBroadcaster-usb\CC2540\CC2540USB\Obj\osal_snv. #
#                            r51                                               #
#                            C:\ble\BLE-CC254x-1.4.1.43908\Projects\ble\Simple #
#                            BLEBroadcaster-usb\CC2540\CC2540USB\Obj\OSAL_Time #
#                            rs.r51                                            #
#                            C:\ble\BLE-CC254x-1.4.1.43908\Projects\ble\Simple #
#                            BLEBroadcaster-usb\CC2540\CC2540USB\Obj\serialInt #
#                            erface.r51                                        #
#                            C:\ble\BLE-CC254x-1.4.1.43908\Projects\ble\Simple #
#                            BLEBroadcaster-usb\CC2540\CC2540USB\Obj\simpleBLE #
#                            Broadcaster.r51                                   #
#                            C:\ble\BLE-CC254x-1.4.1.43908\Projects\ble\Simple #
#                            BLEBroadcaster-usb\CC2540\CC2540USB\Obj\SimpleBLE #
#                            Broadcaster_Main.r51                              #
#                            C:\ble\BLE-CC254x-1.4.1.43908\Projects\ble\Simple #
#                            BLEBroadcaster-usb\CC2540\CC2540USB\Obj\usb_cdc_d #
#                            escriptor.r51                                     #
#                            C:\ble\BLE-CC254x-1.4.1.43908\Projects\ble\Simple #
#                            BLEBroadcaster-usb\CC2540\CC2540USB\Obj\usb_cdc_h #
#                            ooks.r51                                          #
#                            C:\ble\BLE-CC254x-1.4.1.43908\Projects\ble\Simple #
#                            BLEBroadcaster-usb\CC2540\CC2540USB\Obj\usb_descr #
#                            iptor_parser.r51                                  #
#                            C:\ble\BLE-CC254x-1.4.1.43908\Projects\ble\Simple #
#                            BLEBroadcaster-usb\CC2540\CC2540USB\Obj\usb_firmw #
#                            are_library_config.r51                            #
#                            C:\ble\BLE-CC254x-1.4.1.43908\Projects\ble\Simple #
#                            BLEBroadcaster-usb\CC2540\CC2540USB\Obj\usb_frame #
#                            work.r51                                          #
#                            C:\ble\BLE-CC254x-1.4.1.43908\Projects\ble\Simple #
#                            BLEBroadcaster-usb\CC2540\CC2540USB\Obj\usb_inter #
#                            rupt.r51                                          #
#                            C:\ble\BLE-CC254x-1.4.1.43908\Projects\ble\Simple #
#                            BLEBroadcaster-usb\CC2540\CC2540USB\Obj\usb_stand #
#                            ard_requests.r51                                  #
#                            C:\ble\BLE-CC254x-1.4.1.43908\Projects\ble\Simple #
#                            BLEBroadcaster-usb\CC2540\CC2540USB\Obj\usb_suspe #
#                            nd.r51                                            #
#                            -o                                                #
#                            C:\ble\BLE-CC254x-1.4.1.43908\Projects\ble\Simple #
#                            BLEBroadcaster-usb\CC2540\CC2540USB\Exe\HostTestR #
#                            elease.d51                                        #
#                            -l                                                #
#                            C:\ble\BLE-CC254x-1.4.1.43908\Projects\ble\Simple #
#                            BLEBroadcaster-usb\CC2540\CC2540USB\List\HostTest #
#                            Release.map                                       #
#                            -xmsn -f                                          #
#                            C:\ble\BLE-CC254x-1.4.1.43908\Projects\ble\Simple #
#                            BLEBroadcaster-usb\CC2540\..\..\common\cc2540\ti_ #
#                            51ew_cc2540b.xcl                                  #
#                            (-D_IDATA_END=0xFF -D_PDATA_START=0x1E00          #
#                            -D_PDATA_END=0x1EFF -D_IXDATA_START=0x0001        #
#                            -D_IXDATA_END=0x1EFF                              #
#                            -D_XDATA_START=_IXDATA_START                      #
#                            -D_XDATA_END=_IXDATA_END -D_CODE_START=0x0000     #
#                            -D_CODE_END=0x7FFF -D_FIRST_BANK_ADDR=0x10000     #
#                            -D_NEAR_CODE_END=_CODE_END -D?REGISTER_BANK=0     #
#                            -D_REGISTER_BANK_START=0 -D?PBANK_NUMBER=0x1E     #
#                            -D_BREG_START=0x00 -D?VB=0x20                     #
#                            -D_FAR_DATA_NR_OF_BANKS=0x0E                      #
#                            -D_FAR_DATA_START=0x010001                        #
#                            -D_FAR_DATA_END=0xFFFFFF                          #
#                            -D_FAR_CODE_START=_CODE_START                     #
#                            -D_FAR_CODE_END=_CODE_END                         #
#                            -Z(BIT)BREG=_BREG_START -Z(BIT)BIT_N=0-7F         #
#                            -Z(DATA)REGISTERS+8=_REGISTER_BANK_START          #
#                            -Z(DATA)BDATA_Z,BDATA_N,BDATA_I=20-2F             #
#                            -Z(DATA)VREG=08-7F -Z(DATA)PSP,XSP=08-7F          #
#                            -Z(DATA)DOVERLAY=08-7F                            #
#                            -Z(DATA)DATA_I,DATA_Z,DATA_N=08-7F                #
#                            -U(IDATA)0-7F=(DATA)0-7F                          #
#                            -Z(IDATA)IDATA_I,IDATA_Z,IDATA_N=08-_IDATA_END    #
#                            -Z(IDATA)ISTACK+_IDATA_STACK_SIZE#08-_IDATA_END   #
#                            -Z(IDATA)IOVERLAY=08-FF                           #
#                            -Z(CODE)INTVEC=_CODE_START                        #
#                            -Z(CODE)CSTART=_CODE_START-_CODE_END              #
#                            -Z(CODE)BIT_ID,BDATA_ID,DATA_ID,IDATA_ID,IXDATA_I #
#                            D,PDATA_ID,XDATA_ID=_CODE_START-_CODE_END         #
#                            -Z(CODE)HUGE_ID=_FAR_CODE_START-_FAR_CODE_END     #
#                            -D_SLEEP_CODE_SPACE_START=(_CODE_END-7)           #
#                            -D_SLEEP_CODE_SPACE_END=(_CODE_END)               #
#                            -Z(CODE)SLEEP_CODE=_SLEEP_CODE_SPACE_START-_SLEEP #
#                            _CODE_SPACE_END                                   #
#                            -Z(CODE)BANK_RELAYS,RCODE,DIFUNCT,CODE_N,NEAR_COD #
#                            E=_CODE_START-_CODE_END                           #
#                            -P(CODE)CODE_C=_CODE_START-_CODE_END              #
#                            -P(CONST)XDATA_ROM_C=0x8000-0xFFFF                #
#                            -P(CODE)XDATA_ROM_C_FLASH=0x18000-0x1FFFF         #
#                            -QXDATA_ROM_C=XDATA_ROM_C_FLASH                   #
#                            -P(CODE)BANKED_CODE=_CODE_START-_CODE_END,[(_CODE #
#                            BANK_START+_FIRST_BANK_ADDR)-(_CODEBANK_END+_FIRS #
#                            T_BANK_ADDR)]*_NR_OF_BANKS+10000                  #
#                            -P(CODE)FAR_CODE_C,FAR_CODE_N,FAR_CODE=[_FAR_CODE #
#                            _START-_FAR_CODE_END]/10000                       #
#                            -P(CODE)HUGE_CODE_C=_FAR_CODE_START-_FAR_CODE_END #
#                            -Z(CODE)CHECKSUM#_CODE_END                        #
#                            -Z(XDATA)EXT_STACK+_EXTENDED_STACK_SIZE=_EXTENDED #
#                            _STACK_START                                      #
#                            -Z(XDATA)PSTACK+_PDATA_STACK_SIZE=_PDATA_START-_P #
#                            DATA_END                                          #
#                            -Z(XDATA)XSTACK+_XDATA_STACK_SIZE=_XDATA_START-_X #
#                            DATA_END                                          #
#                            -Z(XDATA)PDATA_Z,PDATA_I=_PDATA_START-_PDATA_END  #
#                            -P(XDATA)PDATA_N=_PDATA_START-_PDATA_END          #
#                            -Z(XDATA)IXDATA_Z,IXDATA_I=_IXDATA_START-_IXDATA_ #
#                            END                                               #
#                            -P(XDATA)IXDATA_N=_IXDATA_START-_IXDATA_END       #
#                            -Z(XDATA)XDATA_Z,XDATA_I=_XDATA_START-_XDATA_END  #
#                            -P(XDATA)XDATA_N=_XDATA_START-_XDATA_END          #
#                            -Z(XDATA)XDATA_HEAP+_XDATA_HEAP_SIZE=_XDATA_START #
#                            -_XDATA_END                                       #
#                            -Z(XDATA)FAR_Z=[_FAR_DATA_START-_FAR_DATA_END]/10 #
#                            000                                               #
#                            -Z(XDATA)FAR_I=[_FAR_DATA_START-_FAR_DATA_END]/10 #
#                            000                                               #
#                            -Z(CODE)FAR_ID=[_FAR_CODE_START-_FAR_CODE_END]/10 #
#                            000                                               #
#                            -Z(XDATA)FAR_HEAP+_FAR_HEAP_SIZE=[_FAR_DATA_START #
#                            -_FAR_DATA_END]/10000                             #
#                            -P(XDATA)FAR_N=[_FAR_DATA_START-_FAR_DATA_END]*_F #
#                            AR_DATA_NR_OF_BANKS+10000                         #
#                            -P(CONST)FAR_ROM_C=[_FAR_DATA_START-_FAR_DATA_END #
#                            ]*_FAR_DATA_NR_OF_BANKS+10000                     #
#                            -Z(XDATA)HUGE_Z,HUGE_I=_FAR_DATA_START-_FAR_DATA_ #
#                            END                                               #
#                            -P(XDATA)HUGE_N=_FAR_DATA_START-_FAR_DATA_END     #
#                            -Z(XDATA)HUGE_HEAP+_HUGE_HEAP_SIZE=_FAR_DATA_STAR #
#                            T-_FAR_DATA_END                                   #
#                            -Z(CONST)HUGE_ROM_C=_FAR_DATA_START-_FAR_DATA_END #
#                            -cx51 -D_BLENV_ADDRESS_SPACE_START=0x7E800        #
#                            -D_BLENV_ADDRESS_SPACE_END=0x7F7FF                #
#                            -Z(CODE)BLENV_ADDRESS_SPACE=_BLENV_ADDRESS_SPACE_ #
#                            START-_BLENV_ADDRESS_SPACE_END                    #
#                            -D_BANK0_START=0x00000 -D_BANK0_END=0x07FFF       #
#                            -D_BANK1_START=0x18000 -D_BANK1_END=0x1FFFF       #
#                            -D_BANK2_START=0x28000 -D_BANK2_END=0x2FFFF       #
#                            -D_BANK3_START=0x38000 -D_BANK3_END=0x3FFFF       #
#                            -D_BANK4_START=0x48000 -D_BANK4_END=0x4FFFF       #
#                            -D_BANK5_START=0x58000 -D_BANK5_END=0x5FFFF       #
#                            -D_BANK6_START=0x68000 -D_BANK6_END=0x6FFFF       #
#                            -D_BANK7_START=0x78000                            #
#                            -D_BANK7_END=(_BLENV_ADDRESS_SPACE_START-1)       #
#                            -P(CODE)BANK0=_BANK0_START-_BANK0_END             #
#                            -P(CODE)BANK1=_BANK1_START-_BANK1_END             #
#                            -P(CODE)BANK2=_BANK2_START-_BANK2_END             #
#                            -P(CODE)BANK3=_BANK3_START-_BANK3_END             #
#                            -P(CODE)BANK4=_BANK4_START-_BANK4_END             #
#                            -P(CODE)BANK5=_BANK5_START-_BANK5_END             #
#                            -P(CODE)BANK6=_BANK6_START-_BANK6_END             #
#                            -P(CODE)BANK7=_BANK7_START-_BANK7_END             #
#                            -M(CODE)[(_CODEBANK_START+_FIRST_BANK_ADDR)-(_COD #
#                            EBANK_END+_FIRST_BANK_ADDR)]*_NR_OF_BANKS+0x10000 #
#                            =0x8000                                           #
#                            -ww69=i                                           #
#                            -D_FLASH_LOCK_BITS_START=((_NR_OF_BANKS*_FIRST_BA #
#                            NK_ADDR)+0xFFF0)                                  #
#                            -D_FLASH_LOCK_BITS_END=((_NR_OF_BANKS*_FIRST_BANK #
#                            _ADDR)+0xFFFF)                                    #
#                            -Z(CODE)FLASH_LOCK_BITS=_FLASH_LOCK_BITS_START-_F #
#                            LASH_LOCK_BITS_END                                #
#                            -U(CODE)0x0000=(CODE)_FLASH_LOCK_BITS_START-_FLAS #
#                            H_LOCK_BITS_END)                                  #
#                            -D_NR_OF_VIRTUAL_REGISTERS=10 -D?PBANK=0x93       #
#                            -e?BCALL_FF=?BCALL -e?BRET_FF=?BRET               #
#                            -e?BDISPATCH_FF=?BDISPATCH                        #
#                            -e_small_write=_formatted_write                   #
#                            -e_medium_read=_formatted_read -rt                #
#                            -Ointel-extended=C:\ble\BLE-CC254x-1.4.1.43908\Pr #
#                            ojects\ble\SimpleBLEBroadcaster-usb\CC2540\hex\Ho #
#                            stTestReleaseCC2540Usb.hex                        #
#                            -s __program_start                                #
#                            "C:\Program Files\IAR Systems\Embedded Workbench  #
#                            7.2\8051\LIB\CLIB\cl-pli-blxd-1e16x01.r51"        #
#                            -D_IDATA_STACK_SIZE=0xC0 -D?ESP=0 -D?ESP_MASK=0   #
#                            -D_EXTENDED_STACK_START=0                         #
#                            -D_EXTENDED_STACK_SIZE=0                          #
#                            -D_PDATA_STACK_SIZE=0x00                          #
#                            -D_XDATA_STACK_SIZE=0x280                         #
#                            -D_XDATA_HEAP_SIZE=0xFF -D_FAR_HEAP_SIZE=0xFFF    #
#                            -D_HUGE_HEAP_SIZE=0xFFF                           #
#                            -D_FAR22_HEAP_SIZE=0xFFF                          #
#                                                                              #
#                           Copyright (C) 1987-2015 IAR Systems AB.            #
################################################################################





                ****************************************
                *                                      *
                *           CROSS REFERENCE            *
                *                                      *
                ****************************************

       Program entry at : CODE      00000107  Relocatable, from module : CSTARTUP




                ****************************************
                *                                      *
                *            RUNTIME MODEL             *
                *                                      *
                ****************************************

  __SystemLibrary          = CLib
  __calling_convention     = xdata_reentrant
  __code_model             = banked
  __core                   = plain
  __data_model             = large
  __dptr_size              = 16
  __extended_stack         = disabled
  __location_for_constants = data
  __number_of_dptrs        = 1
  __rt_version             = 1

                ****************************************
                *                                      *
                *    AUTOMATIC SYMBOL REDIRECTIONS     *
                *                                      *
                ****************************************

                  There are no automatic symbol redirections.



                ****************************************
                *                                      *
                *              MODULE MAP              *
                *                                      *
                ****************************************


  DEFINED ABSOLUTE ENTRIES
    *************************************************************************

  DEFINED ABSOLUTE ENTRIES
  PROGRAM MODULE, NAME : ?ABS_ENTRY_MOD

Absolute parts
           ENTRY                   ADDRESS         REF BY
           =====                   =======         ======
           _FAR22_HEAP_SIZE        00000FFF 
           _HUGE_HEAP_SIZE         00000FFF 
           _FAR_HEAP_SIZE          00000FFF 
           _XDATA_HEAP_SIZE        000000FF 
           _XDATA_STACK_SIZE       00000280 
           _PDATA_STACK_SIZE       00000000 
           _EXTENDED_STACK_SIZE    00000000 
           _EXTENDED_STACK_START   00000000 
           ?ESP_MASK               00000000 
           ?ESP                    00000000 
           _IDATA_STACK_SIZE       000000C0 
           ?PBANK                  00000093 
           _NR_OF_VIRTUAL_REGISTERS
                                   00000010 
           _FLASH_LOCK_BITS_END    0003FFFF 
           _FLASH_LOCK_BITS_START
                                   0003FFF0 
           _BANK7_END              0003E7FF 
           _BANK7_START            00038000 
           _BANK6_END              00037FFF 
           _BANK6_START            00030000 
           _BANK5_END              0002FFFF 
           _BANK5_START            00028000 
           _BANK4_END              00027FFF 
           _BANK4_START            00020000 
           _BANK3_END              0001FFFF 
           _BANK3_START            00018000 
           _BANK2_END              00017FFF 
           _BANK2_START            00010000 
           _BANK1_END              0000FFFF 
           _BANK1_START            00008000 
           _BANK0_END              00007FFF 
           _BANK0_START            00000000 
           _BLENV_ADDRESS_SPACE_END
                                   0003F7FF 
           _BLENV_ADDRESS_SPACE_START
                                   0003E800 
           _SLEEP_CODE_SPACE_END   00007FFF 
           _SLEEP_CODE_SPACE_START
                                   00007FF8 
           _FAR_CODE_END           00007FFF 
           _FAR_CODE_START         00000000 
           _FAR_DATA_END           00FFFFFF 
           _FAR_DATA_START         00010001 
           _FAR_DATA_NR_OF_BANKS   0000000E 
           ?VB                     00000020        ?BANKED_ENTER_XDATA (?BANKED_ENTER_XDATA)
                                                   ?BANKED_LEAVE_XDATA (?BANKED_LEAVE_XDATA)
                                                   ?FUNC_ENTER_XDATA (?FUNC_ENTER_XDATA)
                                                   ?FUNC_LEAVE_XDATA (?FUNC_LEAVE_XDATA)
                                                   ?INTERRUPT_ENTER_XSP (?INTERRUPT_ENTER_XSP)
                                                   ?INTERRUPT_LEAVE_XSP (?INTERRUPT_LEAVE_XSP)
           _BREG_START             00000000 
           ?PBANK_NUMBER           0000001E 
           _REGISTER_BANK_START    00000000 
           ?REGISTER_BANK          00000000        Segment part 6 (CSTARTUP)
           _NEAR_CODE_END          00007FFF 
           _FIRST_BANK_ADDR        00010000 
           _CODE_END               00007FFF 
           _CODE_START             00000000 
           _XDATA_END              00001EFF 
           _XDATA_START            00000001 
           _IXDATA_END             00001EFF 
           _IXDATA_START           00000001 
           _PDATA_END              00001EFF 
           _PDATA_START            00001E00 
           _IDATA_END              000000FF 
           ?CBANK                  0000009F        ?RESET_CODE_BANK (CSTARTUP)
                                                   Segment part 0 (?BANKED_CODE_SUPPORT)
           ?CBANK_MASK             000000FF 
           _CODEBANK_START         00008000 
           _CODEBANK_END           0000FFFF 
           _NR_OF_BANKS            00000007 
    *************************************************************************

  FILE NAME : C:\ble\BLE-CC254x-1.4.1.43908\Projects\ble\SimpleBLEBroadcaster-usb\CC2540\CC2540USB\Obj\broadcaster.r51
  PROGRAM MODULE, NAME : broadcaster

  SEGMENTS IN THE MODULE
  ======================
XDATA_Z
  Relative segment, address: XDATA 00000281 - 00000281 (0x1 bytes), align: 0
  Segment part 6.             Intra module refs:   GAPRole_Init
                                                   GAPRole_ProcessEvent
                                                   GAPRole_SetParameter
                                                   gapRole_ProcessGAPMsg
                                                   gapRole_SetupGAP
           LOCAL                   ADDRESS         
           =====                   =======         
           gapRole_TaskID          00000281 
    -------------------------------------------------------------------------
XDATA_Z
  Relative segment, address: XDATA 00000282 - 00000282 (0x1 bytes), align: 0
  Segment part 7.             Intra module refs:   GAPRole_Init
                                                   GAPRole_ProcessEvent
                                                   GAPRole_SetParameter
                                                   GAPRole_StartDevice
                                                   gapRole_ProcessGAPMsg
           LOCAL                   ADDRESS         
           =====                   =======         
           gapRole_state           00000282 
    -------------------------------------------------------------------------
XDATA_Z
  Relative segment, address: XDATA 00000283 - 00000283 (0x1 bytes), align: 0
  Segment part 8.             Intra module refs:   GAPRole_GetParameter
                                                   GAPRole_Init
                                                   gapRole_SetupGAP
           LOCAL                   ADDRESS         
           =====                   =======         
           gapRole_profileRole     00000283 
    -------------------------------------------------------------------------
XDATA_Z
  Relative segment, address: XDATA 00000284 - 00000289 (0x6 bytes), align: 0
  Segment part 9.             Intra module refs:   GAPRole_GetParameter
                                                   gapRole_ProcessGAPMsg
           LOCAL                   ADDRESS         
           =====                   =======         
           gapRole_bdAddr          00000284 
    -------------------------------------------------------------------------
XDATA_I
  Relative segment, address: XDATA 0000105B - 0000105B (0x1 bytes), align: 0
  Segment part 10.            Intra module refs:   GAPRole_GetParameter
                                                   GAPRole_ProcessEvent
                                                   GAPRole_SetParameter
                                                   gapRole_ProcessGAPMsg
           LOCAL                   ADDRESS         
           =====                   =======         
           gapRole_AdvEnabled      0000105B 
    -------------------------------------------------------------------------
XDATA_I
  Relative segment, address: XDATA 0000105C - 0000105D (0x2 bytes), align: 0
  Segment part 12.            Intra module refs:   GAPRole_GetParameter
                                                   GAPRole_SetParameter
                                                   gapRole_ProcessGAPMsg
           LOCAL                   ADDRESS         
           =====                   =======         
           gapRole_AdvertOffTime   0000105C 
    -------------------------------------------------------------------------
XDATA_I
  Relative segment, address: XDATA 0000105E - 0000105E (0x1 bytes), align: 0
  Segment part 14.            Intra module refs:   GAPRole_GetParameter
                                                   GAPRole_SetParameter
                                                   gapRole_ProcessGAPMsg
           LOCAL                   ADDRESS         
           =====                   =======         
           gapRole_AdvertDataLen   0000105E 
    -------------------------------------------------------------------------
XDATA_I
  Relative segment, address: XDATA 0000105F - 0000107D (0x1f bytes), align: 0
  Segment part 16.            Intra module refs:   GAPRole_GetParameter
                                                   GAPRole_SetParameter
                                                   gapRole_ProcessGAPMsg
           LOCAL                   ADDRESS         
           =====                   =======         
           gapRole_AdvertData      0000105F 
    -------------------------------------------------------------------------
XDATA_Z
  Relative segment, address: XDATA 0000028A - 0000028A (0x1 bytes), align: 0
  Segment part 18.            Intra module refs:   GAPRole_GetParameter
                                                   GAPRole_SetParameter
                                                   gapRole_ProcessGAPMsg
           LOCAL                   ADDRESS         
           =====                   =======         
           gapRole_ScanRspDataLen
                                   0000028A 
    -------------------------------------------------------------------------
XDATA_Z
  Relative segment, address: XDATA 0000028B - 000002A9 (0x1f bytes), align: 0
  Segment part 19.            Intra module refs:   GAPRole_GetParameter
                                                   GAPRole_SetParameter
                                                   gapRole_ProcessGAPMsg
           LOCAL                   ADDRESS         
           =====                   =======         
           gapRole_ScanRspData     0000028B 
    -------------------------------------------------------------------------
XDATA_Z
  Relative segment, address: XDATA 000002AA - 000002AA (0x1 bytes), align: 0
  Segment part 20.            Intra module refs:   GAPRole_GetParameter
                                                   GAPRole_Init
                                                   GAPRole_ProcessEvent
                                                   GAPRole_SetParameter
           LOCAL                   ADDRESS         
           =====                   =======         
           gapRole_AdvEventType    000002AA 
    -------------------------------------------------------------------------
XDATA_Z
  Relative segment, address: XDATA 000002AB - 000002AB (0x1 bytes), align: 0
  Segment part 21.            Intra module refs:   GAPRole_GetParameter
                                                   GAPRole_Init
                                                   GAPRole_ProcessEvent
                                                   GAPRole_SetParameter
           LOCAL                   ADDRESS         
           =====                   =======         
           gapRole_AdvDirectType   000002AB 
    -------------------------------------------------------------------------
XDATA_Z
  Relative segment, address: XDATA 000002AC - 000002B1 (0x6 bytes), align: 0
  Segment part 22.            Intra module refs:   GAPRole_GetParameter
                                                   GAPRole_ProcessEvent
                                                   GAPRole_SetParameter
           LOCAL                   ADDRESS         
           =====                   =======         
           gapRole_AdvDirectAddr   000002AC 
    -------------------------------------------------------------------------
XDATA_Z
  Relative segment, address: XDATA 000002B2 - 000002B2 (0x1 bytes), align: 0
  Segment part 23.            Intra module refs:   GAPRole_GetParameter
                                                   GAPRole_Init
                                                   GAPRole_ProcessEvent
                                                   GAPRole_SetParameter
           LOCAL                   ADDRESS         
           =====                   =======         
           gapRole_AdvChanMap      000002B2 
    -------------------------------------------------------------------------
XDATA_Z
  Relative segment, address: XDATA 000002B3 - 000002B3 (0x1 bytes), align: 0
  Segment part 24.            Intra module refs:   GAPRole_GetParameter
                                                   GAPRole_Init
                                                   GAPRole_ProcessEvent
                                                   GAPRole_SetParameter
           LOCAL                   ADDRESS         
           =====                   =======         
           gapRole_AdvFilterPolicy
                                   000002B3 
    -------------------------------------------------------------------------
XDATA_Z
  Relative segment, address: XDATA 000002B4 - 000002B5 (0x2 bytes), align: 0
  Segment part 25.            Intra module refs:   GAPRole_ProcessEvent
                                                   GAPRole_StartDevice
                                                   gapRole_ProcessGAPMsg
           LOCAL                   ADDRESS         
           =====                   =======         
           pGapRoles_AppCGs        000002B4 
    -------------------------------------------------------------------------
<BANKED_CODE,CODE_C> 1 (was BANKED_CODE)
  Relative segment, address: CODE 00005121 - 00005381 (0x261 bytes), align: 0
  Segment part 26.            Intra module refs:   GAPRole_SetParameter::?relay
           ENTRY                   ADDRESS         REF BY
           =====                   =======         ======
           GAPRole_SetParameter    00005121 
               calls direct
               XSTACK = 00000000 ( 00000014 )
    -------------------------------------------------------------------------
<BANKED_CODE,CODE_C> 1 (was BANKED_CODE)
  Relative segment, address: CODE 00005382 - 000054F3 (0x172 bytes), align: 0
  Segment part 28.            Intra module refs:   GAPRole_GetParameter::?relay
           ENTRY                   ADDRESS         REF BY
           =====                   =======         ======
           GAPRole_GetParameter    00005382 
               calls direct
               XSTACK = 00000000 ( 00000010 )
               ISTACK = 00000000 ( 00000001 )
    -------------------------------------------------------------------------
<BANKED_CODE,CODE_C> 1 (was BANKED_CODE)
  Relative segment, address: CODE 000054F4 - 0000551C (0x29 bytes), align: 0
  Segment part 30.            Intra module refs:   GAPRole_StartDevice::?relay
           ENTRY                   ADDRESS         REF BY
           =====                   =======         ======
           GAPRole_StartDevice     000054F4 
               calls direct
               XSTACK = 00000000 ( 00000009 )
    -------------------------------------------------------------------------
<BANKED_CODE,CODE_C> 1 (was BANKED_CODE)
  Relative segment, address: CODE 0000551D - 00005559 (0x3d bytes), align: 0
  Segment part 32.            Intra module refs:   GAPRole_Init::?relay
           ENTRY                   ADDRESS         REF BY
           =====                   =======         ======
           GAPRole_Init            0000551D 
               calls direct
               XSTACK = 00000000 ( 00000009 )
    -------------------------------------------------------------------------
<BANKED_CODE,CODE_C> 1 (was BANKED_CODE)
  Relative segment, address: CODE 0000555A - 00005693 (0x13a bytes), align: 0
  Segment part 34.            Intra module refs:   GAPRole_ProcessEvent::?relay
           ENTRY                   ADDRESS         REF BY
           =====                   =======         ======
           GAPRole_ProcessEvent    0000555A 
               calls direct
               XSTACK = 00000000 ( 0000001B )
               ISTACK = 00000000 ( 00000001 )
    -------------------------------------------------------------------------
<BANKED_CODE,CODE_C> 1 (was BANKED_CODE)
  Relative segment, address: CODE 00005694 - 000056B5 (0x22 bytes), align: 0
  Segment part 36.            Intra module refs:   gapRole_ProcessOSALMsg::?relay
           LOCAL                   ADDRESS         
           =====                   =======         
           gapRole_ProcessOSALMsg
                                   00005694 
               calls direct
               XSTACK = 00000019 ( 00000009 )
    -------------------------------------------------------------------------
<BANKED_CODE,CODE_C> 1 (was BANKED_CODE)
  Relative segment, address: CODE 000056B6 - 00005876 (0x1c1 bytes), align: 0
  Segment part 38.            Intra module refs:   gapRole_ProcessGAPMsg::?relay
           LOCAL                   ADDRESS         
           =====                   =======         
           gapRole_ProcessGAPMsg   000056B6 
               calls direct
               XSTACK = 00000009 ( 00000014 )
               ISTACK = 00000000 ( 00000001 )
    -------------------------------------------------------------------------
<BANKED_CODE,CODE_C> 1 (was BANKED_CODE)
  Relative segment, address: CODE 00005877 - 000058AD (0x37 bytes), align: 0
  Segment part 40.            Intra module refs:   gapRole_SetupGAP::?relay
           LOCAL                   ADDRESS         
           =====                   =======         
           gapRole_SetupGAP        00005877 
               calls direct
               XSTACK = 00000009 ( 0000000E )
    -------------------------------------------------------------------------
XDATA_ID
  Relative segment, address: CODE 00000137 - 00000137 (0x1 bytes), align: 0
  Segment part 11.            Intra module refs:   gapRole_AdvEnabled
    -------------------------------------------------------------------------
XDATA_ID
  Relative segment, address: CODE 00000138 - 00000139 (0x2 bytes), align: 0
  Segment part 13.            Intra module refs:   gapRole_AdvertOffTime
    -------------------------------------------------------------------------
XDATA_ID
  Relative segment, address: CODE 0000013A - 0000013A (0x1 bytes), align: 0
  Segment part 15.            Intra module refs:   gapRole_AdvertDataLen
    -------------------------------------------------------------------------
XDATA_ID
  Relative segment, address: CODE 0000013B - 00000159 (0x1f bytes), align: 0
  Segment part 17.            Intra module refs:   gapRole_AdvertData
    -------------------------------------------------------------------------
BANK_RELAYS
  Relative segment, address: CODE 0000022A - 0000022F (0x6 bytes), align: 0
  Segment part 27.
           ENTRY                   ADDRESS         REF BY
           =====                   =======         ======
           GAPRole_SetParameter::?relay
                                   0000022A        Application_StartAdvertise (simpleBLEBroadcaster)
                                                   Application_StopAdvertise (simpleBLEBroadcaster)
                                                   Application_UpdateAdv (simpleBLEBroadcaster)
                                                   Application_UpdateRsp (simpleBLEBroadcaster)
                                                   SimpleBLEBroadcaster_Init (simpleBLEBroadcaster)
    -------------------------------------------------------------------------
BANK_RELAYS
  Relative segment, address: CODE 00000230 - 00000235 (0x6 bytes), align: 0
  Segment part 29.
           ENTRY                   ADDRESS         REF BY
           =====                   =======         ======
           GAPRole_GetParameter::?relay
                                   00000230        Application_StartAdvertise (simpleBLEBroadcaster)
                                                   Application_StopAdvertise (simpleBLEBroadcaster)
                                                   peripheralStateNotificationCB (simpleBLEBroadcaster)
    -------------------------------------------------------------------------
BANK_RELAYS
  Relative segment, address: CODE 00000236 - 0000023B (0x6 bytes), align: 0
  Segment part 31.
           ENTRY                   ADDRESS         REF BY
           =====                   =======         ======
           GAPRole_StartDevice::?relay
                                   00000236        SimpleBLEBroadcaster_ProcessEvent (simpleBLEBroadcaster)
    -------------------------------------------------------------------------
BANK_RELAYS
  Relative segment, address: CODE 0000023C - 00000241 (0x6 bytes), align: 0
  Segment part 33.
           ENTRY                   ADDRESS         REF BY
           =====                   =======         ======
           GAPRole_Init::?relay    0000023C        osalInitTasks (OSAL_SimpleBLEBroadcaster)
    -------------------------------------------------------------------------
BANK_RELAYS
  Relative segment, address: CODE 00000242 - 00000247 (0x6 bytes), align: 0
  Segment part 35.
           ENTRY                   ADDRESS         REF BY
           =====                   =======         ======
           GAPRole_ProcessEvent::?relay
                                   00000242        tasksArr (OSAL_SimpleBLEBroadcaster)
    -------------------------------------------------------------------------
BANK_RELAYS
  Relative segment, address: CODE 00000248 - 0000024D (0x6 bytes), align: 0
  Segment part 37.            Intra module refs:   GAPRole_ProcessEvent
           LOCAL                   ADDRESS         
           =====                   =======         
           gapRole_ProcessOSALMsg::?relay
                                   00000248 
    -------------------------------------------------------------------------
BANK_RELAYS
  Relative segment, address: CODE 0000024E - 00000253 (0x6 bytes), align: 0
  Segment part 39.            Intra module refs:   gapRole_ProcessOSALMsg
           LOCAL                   ADDRESS         
           =====                   =======         
           gapRole_ProcessGAPMsg::?relay
                                   0000024E 
    -------------------------------------------------------------------------
BANK_RELAYS
  Relative segment, address: CODE 00000254 - 00000259 (0x6 bytes), align: 0
  Segment part 41.            Intra module refs:   GAPRole_StartDevice
           LOCAL                   ADDRESS         
           =====                   =======         
           gapRole_SetupGAP::?relay
                                   00000254 

    *************************************************************************

  FILE NAME : C:\ble\BLE-CC254x-1.4.1.43908\Projects\ble\Libraries\CC2540DB\bin\CC2540_BLE_bcast.lib
  LIBRARY MODULE, NAME : gap_configmgr

  SEGMENTS IN THE MODULE
  ======================
XDATA_I
  Relative segment, address: XDATA 0000107E - 0000107E (0x1 bytes), align: 0
  Segment part 6.             Intra module refs:   GAP_ParamsInit
                                                   gapProcessRandomAddrComplete
                                                   gapSendDeviceInitDoneEvent
           ENTRY                   ADDRESS         REF BY
           =====                   =======         ======
           gapAppTaskID            0000107E 
    -------------------------------------------------------------------------
XDATA_Z
  Relative segment, address: XDATA 000002B6 - 000002B6 (0x1 bytes), align: 0
  Segment part 8.             Intra module refs:   GAP_ParamsInit
           ENTRY                   ADDRESS         REF BY
           =====                   =======         ======
           gapProfileRole          000002B6        GAP_MakeDiscoverable (gap_peridevmgr)
                                                   GAP_PeriDevMgrInit (gap_peridevmgr)
                                                   GAP_UpdateAdvertisingData (gap_peridevmgr)
                                                   gapProcessAdvertisingEvt (gap_peridevmgr)
    -------------------------------------------------------------------------
XDATA_Z
  Relative segment, address: XDATA 000002B7 - 000002B7 (0x1 bytes), align: 0
  Segment part 9.             Intra module refs:   gapProcessRandomAddrComplete
           ENTRY                   ADDRESS         REF BY
           =====                   =======         ======
           gapDeviceAddrMode       000002B7        GAP_MakeDiscoverable (gap_peridevmgr)
                                                   gapSetAdvParams (gap_peridevmgr)
    -------------------------------------------------------------------------
XDATA_Z
  Relative segment, address: XDATA 000002B8 - 000002B9 (0x2 bytes), align: 0
  Segment part 10.
           ENTRY                   ADDRESS         REF BY
           =====                   =======         ======
           gapPrivateAddrChangeTimeout
                                   000002B8        GAP_EndDiscoverable (gap_peridevmgr)
                                                   GAP_MakeDiscoverable (gap_peridevmgr)
    -------------------------------------------------------------------------
XDATA_Z
  Relative segment, address: XDATA 000002BA - 000002BA (0x1 bytes), align: 0
  Segment part 11.            Intra module refs:   gapProcessRandomAddrComplete
           ENTRY                   ADDRESS         REF BY
           =====                   =======         ======
           gapAutoAdvPrivateAddrChange
                                   000002BA        gapProcessAdvertisingEvt (gap_peridevmgr)
                                                   gapWriteAdvEnableStatus (gap_peridevmgr)
    -------------------------------------------------------------------------
XDATA_Z
  Relative segment, address: XDATA 000002BB - 000002CA (0x10 bytes), align: 0
  Segment part 12.            Intra module refs:   GAP_ParamsInit
                                                   gapReadBD_ADDRStatus
                                                   gapReadBufSizeCmdStatus
                                                   gapSendDeviceInitDoneEvent
    -------------------------------------------------------------------------
XDATA_I
  Relative segment, address: XDATA 0000107F - 000010CC (0x4e bytes), align: 0
  Segment part 13.            Intra module refs:   Segment part 22
    -------------------------------------------------------------------------
XDATA_Z
  Relative segment, address: XDATA 000002CB - 000002D0 (0x6 bytes), align: 0
  Segment part 15.            Intra module refs:   gapProcessRandomAddrComplete
    -------------------------------------------------------------------------
<BANKED_CODE,XDATA_ROM_C_FLASH> 1 (was BANKED_CODE)
  Relative segment, address: CODE 0000B127 - 0000B14E (0x28 bytes), align: 0
  Segment part 18.            Intra module refs:   GAP_SetParamValue::?relay
           ENTRY                   ADDRESS         REF BY
           =====                   =======         ======
           GAP_SetParamValue       0000B127 
               ISTACK = 00000000 ( 00000002 )
    -------------------------------------------------------------------------
<BANKED_CODE,XDATA_ROM_C_FLASH> 1 (was BANKED_CODE)
  Relative segment, address: CODE 0000B14F - 0000B16A (0x1c bytes), align: 0
  Segment part 20.            Intra module refs:   GAP_GetParamValue::?relay
           ENTRY                   ADDRESS         REF BY
           =====                   =======         ======
           GAP_GetParamValue       0000B14F 
               XSTACK = 00000014 ( 00000000 )
               ISTACK = 00000000 ( 00000002 )
    -------------------------------------------------------------------------
<BANKED_CODE,XDATA_ROM_C_FLASH> 1 (was BANKED_CODE)
  Relative segment, address: CODE 0000B16B - 0000B17B (0x11 bytes), align: 0
  Segment part 22.            Intra module refs:   GAP_GetParamValue
                                                   GAP_SetParamValue
    -------------------------------------------------------------------------
<BANKED_CODE,XDATA_ROM_C_FLASH> 1 (was BANKED_CODE)
  Relative segment, address: CODE 0000B17C - 0000B1AE (0x33 bytes), align: 0
  Segment part 23.            Intra module refs:   GAP_ParamsInit::?relay
           ENTRY                   ADDRESS         REF BY
           =====                   =======         ======
           GAP_ParamsInit          0000B17C 
               calls direct
               XSTACK = 00000000 ( 00000009 )
    -------------------------------------------------------------------------
<BANKED_CODE,XDATA_ROM_C_FLASH> 1 (was BANKED_CODE)
  Relative segment, address: CODE 0000B1AF - 0000B1B3 (0x5 bytes), align: 0
  Segment part 25.            Intra module refs:   GAP_ParamsInit
    -------------------------------------------------------------------------
<BANKED_CODE,XDATA_ROM_C_FLASH> 1 (was BANKED_CODE)
  Relative segment, address: CODE 0000B1B4 - 0000B1F8 (0x45 bytes), align: 0
  Segment part 30.            Intra module refs:   gapReadBD_ADDRStatus::?relay
           ENTRY                   ADDRESS         REF BY
           =====                   =======         ======
           gapReadBD_ADDRStatus    0000B1B4 
               calls direct
               XSTACK = 00000000 ( 0000000C )
    -------------------------------------------------------------------------
<BANKED_CODE,XDATA_ROM_C_FLASH> 1 (was BANKED_CODE)
  Relative segment, address: CODE 0000B1F9 - 0000B1FA (0x2 bytes), align: 0
  Segment part 32.            Intra module refs:   gapReadBD_ADDRStatus
                                                   gapReadBufSizeCmdStatus
    -------------------------------------------------------------------------
<BANKED_CODE,XDATA_ROM_C_FLASH> 1 (was BANKED_CODE)
  Relative segment, address: CODE 0000B1FB - 0000B1FF (0x5 bytes), align: 0
  Segment part 33.            Intra module refs:   Segment part 32
    -------------------------------------------------------------------------
<BANKED_CODE,XDATA_ROM_C_FLASH> 1 (was BANKED_CODE)
  Relative segment, address: CODE 0000B200 - 0000B24B (0x4c bytes), align: 0
  Segment part 34.            Intra module refs:   gapReadBufSizeCmdStatus::?relay
           ENTRY                   ADDRESS         REF BY
           =====                   =======         ======
           gapReadBufSizeCmdStatus
                                   0000B200 
               calls direct
               XSTACK = 00000000 ( 0000000A )
    -------------------------------------------------------------------------
<BANKED_CODE,XDATA_ROM_C_FLASH> 1 (was BANKED_CODE)
  Relative segment, address: CODE 0000B24C - 0000B27E (0x33 bytes), align: 0
  Segment part 38.            Intra module refs:   gapAddAddrAdj::?relay
           ENTRY                   ADDRESS         REF BY
           =====                   =======         ======
           gapAddAddrAdj           0000B24C 
               XSTACK = 0000000A ( 00000000 )
               ISTACK = 00000000 ( 00000002 )
    -------------------------------------------------------------------------
<BANKED_CODE,XDATA_ROM_C_FLASH> 1 (was BANKED_CODE)
  Relative segment, address: CODE 0000B27F - 0000B285 (0x7 bytes), align: 0
  Segment part 41.            Intra module refs:   GAP_GetParamValue
                                                   GAP_SetParamValue
                                                   gapAddAddrAdj
    -------------------------------------------------------------------------
<BANKED_CODE,XDATA_ROM_C_FLASH> 1 (was BANKED_CODE)
  Relative segment, address: CODE 0000B286 - 0000B28B (0x6 bytes), align: 0
  Segment part 43.            Intra module refs:   GAP_GetParamValue
    -------------------------------------------------------------------------
<BANKED_CODE,XDATA_ROM_C_FLASH> 1 (was BANKED_CODE)
  Relative segment, address: CODE 0000B28C - 0000B32A (0x9f bytes), align: 0
  Segment part 46.            Intra module refs:   gapProcessRandomAddrComplete::?relay
           ENTRY                   ADDRESS         REF BY
           =====                   =======         ======
           gapProcessRandomAddrComplete
                                   0000B28C 
               calls direct
               XSTACK = 00000000 ( 00000010 )
               ISTACK = 00000000 ( 00000001 )
    -------------------------------------------------------------------------
<BANKED_CODE,XDATA_ROM_C_FLASH> 1 (was BANKED_CODE)
  Relative segment, address: CODE 0000B32B - 0000B32F (0x5 bytes), align: 0
  Segment part 48.            Intra module refs:   gapProcessRandomAddrComplete
                                                   gapSendDeviceInitDoneEvent
    -------------------------------------------------------------------------
<BANKED_CODE,XDATA_ROM_C_FLASH> 1 (was BANKED_CODE)
  Relative segment, address: CODE 0000B330 - 0000B335 (0x6 bytes), align: 0
  Segment part 49.            Intra module refs:   gapProcessRandomAddrComplete
                                                   gapSendDeviceInitDoneEvent
    -------------------------------------------------------------------------
<BANKED_CODE,XDATA_ROM_C_FLASH> 1 (was BANKED_CODE)
  Relative segment, address: CODE 0000B336 - 0000B3B1 (0x7c bytes), align: 0
  Segment part 63.            Intra module refs:   gapSendDeviceInitDoneEvent::?relay
           LOCAL                   ADDRESS         
           =====                   =======         
           gapSendDeviceInitDoneEvent
                                   0000B336 
               calls direct
               XSTACK = 0000000A ( 0000000E )
               ISTACK = 00000000 ( 00000001 )
    -------------------------------------------------------------------------
<BANKED_CODE,XDATA_ROM_C_FLASH> 1 (was BANKED_CODE)
  Relative segment, address: CODE 0000B3B2 - 0000B3C3 (0x12 bytes), align: 0
  Segment part 65.            Intra module refs:   gapProcessRandomAddrComplete
                                                   gapSendDeviceInitDoneEvent
    -------------------------------------------------------------------------
XDATA_ID
  Relative segment, address: CODE 0000015A - 0000015A (0x1 bytes), align: 0
  Segment part 7.             Intra module refs:   gapAppTaskID
    -------------------------------------------------------------------------
XDATA_ID
  Relative segment, address: CODE 0000015B - 000001A8 (0x4e bytes), align: 0
  Segment part 14.            Intra module refs:   Segment part 13
    -------------------------------------------------------------------------
<XDATA_ROM_C> 1 (was XDATA_ROM_C)
  Relative segment, address: CONST 00008FE4 - 00008FE7 (0x4 bytes), align: 0
  Segment part 16.            Intra module refs:   GAP_MakeDiscoverable (gap_peridevmgr)
                                                   gapProcessRandomAddrComplete
                                                   gapWriteAdvEnableStatus (gap_peridevmgr)
           ENTRY                   ADDRESS         REF BY
           =====                   =======         ======
           __Constant_ea60         00008FE4 
    -------------------------------------------------------------------------
BANK_RELAYS
  Relative segment, address: CODE 0000025A - 0000025F (0x6 bytes), align: 0
  Segment part 19.
           ENTRY                   ADDRESS         REF BY
           =====                   =======         ======
           GAP_SetParamValue::?relay
                                   0000025A        GAPRole_SetParameter (broadcaster)
                                                   SimpleBLEBroadcaster_Init (simpleBLEBroadcaster)
    -------------------------------------------------------------------------
BANK_RELAYS
  Relative segment, address: CODE 00000260 - 00000265 (0x6 bytes), align: 0
  Segment part 21.
           ENTRY                   ADDRESS         REF BY
           =====                   =======         ======
           GAP_GetParamValue::?relay
                                   00000260        GAPRole_GetParameter (broadcaster)
                                                   GAP_MakeDiscoverable (gap_peridevmgr)
                                                   gapSetAdvParams (gap_peridevmgr)
                                                   gapWriteAdvEnableStatus (gap_peridevmgr)
    -------------------------------------------------------------------------
BANK_RELAYS
  Relative segment, address: CODE 00000266 - 0000026B (0x6 bytes), align: 0
  Segment part 24.
           ENTRY                   ADDRESS         REF BY
           =====                   =======         ======
           GAP_ParamsInit::?relay
                                   00000266        GAP_DeviceInit (gap)
    -------------------------------------------------------------------------
BANK_RELAYS
  Relative segment, address: CODE 0000026C - 00000271 (0x6 bytes), align: 0
  Segment part 31.
           ENTRY                   ADDRESS         REF BY
           =====                   =======         ======
           gapReadBD_ADDRStatus::?relay
                                   0000026C        gapProcessHCICmdCompleteEvt (gap_simpletask)
    -------------------------------------------------------------------------
BANK_RELAYS
  Relative segment, address: CODE 00000272 - 00000277 (0x6 bytes), align: 0
  Segment part 35.
           ENTRY                   ADDRESS         REF BY
           =====                   =======         ======
           gapReadBufSizeCmdStatus::?relay
                                   00000272        gapProcessHCICmdCompleteEvt (gap_simpletask)
    -------------------------------------------------------------------------
BANK_RELAYS
  Relative segment, address: CODE 00000278 - 0000027D (0x6 bytes), align: 0
  Segment part 39.
           ENTRY                   ADDRESS         REF BY
           =====                   =======         ======
           gapAddAddrAdj::?relay   00000278        gapSetAdvParams (gap_peridevmgr)
    -------------------------------------------------------------------------
BANK_RELAYS
  Relative segment, address: CODE 0000027E - 00000283 (0x6 bytes), align: 0
  Segment part 47.
           ENTRY                   ADDRESS         REF BY
           =====                   =======         ======
           gapProcessRandomAddrComplete::?relay
                                   0000027E        gapProcessHCICmdCompleteEvt (gap_simpletask)
    -------------------------------------------------------------------------
BANK_RELAYS
  Relative segment, address: CODE 00000284 - 00000289 (0x6 bytes), align: 0
  Segment part 64.            Intra module refs:   gapReadBD_ADDRStatus
                                                   gapReadBufSizeCmdStatus
           LOCAL                   ADDRESS         
           =====                   =======         
           gapSendDeviceInitDoneEvent::?relay
                                   00000284 
    -------------------------------------------------------------------------
<BANKED_CODE,XDATA_ROM_C_FLASH> 1 (was XDATA_ROM_C_FLASH)
  Relative segment, address: CODE 00008FE4 - 00008FE7 (0x4 bytes), align: 0
  Segment part 66.            Intra module refs:   __Constant_ea60

    -------------------------------------------------------------------------
  LIBRARY MODULE, NAME : gap_devmgr

  SEGMENTS IN THE MODULE
  ======================
XDATA_Z
  Relative segment, address: XDATA 000002D1 - 000002D2 (0x2 bytes), align: 0
  Segment part 7.
           ENTRY                   ADDRESS         REF BY
           =====                   =======         ======
           pGapAdvertState         000002D1        GAP_MakeDiscoverable (gap_peridevmgr)
                                                   Segment part 19 (gap_peridevmgr)
                                                   Segment part 73 (gap_peridevmgr)
                                                   Segment part 90 (gap_peridevmgr)
                                                   gapFreeAdvertState (gap_peridevmgr)
                                                   gapSendMakeDiscEvent (gap_peridevmgr)
                                                   gapSetAdvParams (gap_peridevmgr)
                                                   gapWriteAdvEnableStatus (gap_peridevmgr)
    -------------------------------------------------------------------------
<BANKED_CODE,XDATA_ROM_C_FLASH> 1 (was BANKED_CODE)
  Relative segment, address: CODE 0000C37F - 0000C395 (0x17 bytes), align: 0
  Segment part 15.            Intra module refs:   gapValidADType::?relay
           ENTRY                   ADDRESS         REF BY
           =====                   =======         ======
           gapValidADType          0000C37F 
               XSTACK = 0000000F ( 00000000 )
    -------------------------------------------------------------------------
<BANKED_CODE,XDATA_ROM_C_FLASH> 1 (was BANKED_CODE)
  Relative segment, address: CODE 0000C396 - 0000C41B (0x86 bytes), align: 0
  Segment part 17.            Intra module refs:   gapFindADType::?relay
           ENTRY                   ADDRESS         REF BY
           =====                   =======         ======
           gapFindADType           0000C396 
               calls direct
               XSTACK = 00000002 ( 0000000F )
               ISTACK = 00000000 ( 00000001 )
    -------------------------------------------------------------------------
<BANKED_CODE,XDATA_ROM_C_FLASH> 1 (was BANKED_CODE)
  Relative segment, address: CODE 0000C41C - 0000C425 (0xa bytes), align: 0
  Segment part 19.            Intra module refs:   gapFindADType
    -------------------------------------------------------------------------
BANK_RELAYS
  Relative segment, address: CODE 0000028A - 0000028F (0x6 bytes), align: 0
  Segment part 16.            Intra module refs:   gapFindADType
           ENTRY                   ADDRESS         REF BY
           =====                   =======         ======
           gapValidADType::?relay
                                   0000028A 
    -------------------------------------------------------------------------
BANK_RELAYS
  Relative segment, address: CODE 00000290 - 00000295 (0x6 bytes), align: 0
  Segment part 18.
           ENTRY                   ADDRESS         REF BY
           =====                   =======         ======
           gapFindADType::?relay   00000290        isLimitedDiscoverableMode (gap_peridevmgr)

    -------------------------------------------------------------------------
  LIBRARY MODULE, NAME : gap_peridevmgr

  SEGMENTS IN THE MODULE
  ======================
XDATA_I
  Relative segment, address: XDATA 000010CD - 000010CD (0x1 bytes), align: 0
  Segment part 6.             Intra module refs:   GAP_UpdateAdvertisingData
                                                   gapWriteAdvDataStatus
    -------------------------------------------------------------------------
XDATA_Z
  Relative segment, address: XDATA 000002D3 - 000002D4 (0x2 bytes), align: 0
  Segment part 9.             Intra module refs:   GAP_MakeDiscoverable
                                                   GAP_PeriDevMgrInit
                                                   GAP_UpdateAdvertisingData
                                                   Segment part 37
                                                   Segment part 41
                                                   Segment part 67
                                                   isLimitedDiscoverableMode
    -------------------------------------------------------------------------
XDATA_Z
  Relative segment, address: XDATA 000002D5 - 000002D6 (0x2 bytes), align: 0
  Segment part 10.            Intra module refs:   GAP_PeriDevMgrInit
                                                   GAP_UpdateAdvertisingData
    -------------------------------------------------------------------------
XDATA_Z
  Relative segment, address: XDATA 000002D7 - 000002D8 (0x2 bytes), align: 0
  Segment part 11.            Intra module refs:   GAP_EndDiscoverable
                                                   gapProcessAdvertisingEvt
                                                   gapWriteAdvEnableStatus
    -------------------------------------------------------------------------
XDATA_I
  Relative segment, address: XDATA 000010CE - 000010D3 (0x6 bytes), align: 0
  Segment part 12.            Intra module refs:   GAP_PeriDevMgrInit
    -------------------------------------------------------------------------
<BANKED_CODE,CODE_C> 1 (was BANKED_CODE)
  Relative segment, address: CODE 000058AE - 00005986 (0xd9 bytes), align: 0
  Segment part 16.            Intra module refs:   GAP_MakeDiscoverable::?relay
           ENTRY                   ADDRESS         REF BY
           =====                   =======         ======
           GAP_MakeDiscoverable    000058AE 
               calls direct
               XSTACK = 00000000 ( 00000010 )
               ISTACK = 00000000 ( 00000001 )
    -------------------------------------------------------------------------
<BANKED_CODE,CODE_C> 1 (was BANKED_CODE)
  Relative segment, address: CODE 00005987 - 00005987 (0x1 bytes), align: 0
  Segment part 18.            Intra module refs:   GAP_EndDiscoverable
                                                   GAP_MakeDiscoverable
    -------------------------------------------------------------------------
<BANKED_CODE,CODE_C> 1 (was BANKED_CODE)
  Relative segment, address: CODE 00005988 - 0000598E (0x7 bytes), align: 0
  Segment part 19.            Intra module refs:   Segment part 18
                                                   gapSetAdvParams
                                                   gapWriteAdvEnableStatus
    -------------------------------------------------------------------------
<BANKED_CODE,CODE_C> 1 (was BANKED_CODE)
  Relative segment, address: CODE 0000598F - 00005997 (0x9 bytes), align: 0
  Segment part 20.            Intra module refs:   Segment part 19
    -------------------------------------------------------------------------
<BANKED_CODE,CODE_C> 1 (was BANKED_CODE)
  Relative segment, address: CODE 00005998 - 00005A42 (0xab bytes), align: 0
  Segment part 21.            Intra module refs:   GAP_UpdateAdvertisingData::?relay
           ENTRY                   ADDRESS         REF BY
           =====                   =======         ======
           GAP_UpdateAdvertisingData
                                   00005998 
               calls direct
               XSTACK = 00000000 ( 00000014 )
               ISTACK = 00000000 ( 00000001 )
    -------------------------------------------------------------------------
<BANKED_CODE,CODE_C> 1 (was BANKED_CODE)
  Relative segment, address: CODE 00005A43 - 00005A8C (0x4a bytes), align: 0
  Segment part 23.            Intra module refs:   GAP_EndDiscoverable::?relay
           ENTRY                   ADDRESS         REF BY
           =====                   =======         ======
           GAP_EndDiscoverable     00005A43 
               calls direct
               XSTACK = 0000000C ( 00000009 )
    -------------------------------------------------------------------------
<BANKED_CODE,CODE_C> 1 (was BANKED_CODE)
  Relative segment, address: CODE 00005A8D - 00005A93 (0x7 bytes), align: 0
  Segment part 33.            Intra module refs:   gapFreeAdvertState
    -------------------------------------------------------------------------
<BANKED_CODE,CODE_C> 1 (was BANKED_CODE)
  Relative segment, address: CODE 00005A94 - 00005B35 (0xa2 bytes), align: 0
  Segment part 34.            Intra module refs:   GAP_PeriDevMgrInit::?relay
           ENTRY                   ADDRESS         REF BY
           =====                   =======         ======
           GAP_PeriDevMgrInit      00005A94 
               calls direct
               XSTACK = 00000000 ( 00000009 )
    -------------------------------------------------------------------------
<BANKED_CODE,CODE_C> 1 (was BANKED_CODE)
  Relative segment, address: CODE 00005B36 - 00005B3A (0x5 bytes), align: 0
  Segment part 36.            Intra module refs:   GAP_EndDiscoverable
                                                   GAP_PeriDevMgrInit
                                                   gapSetAdvParamsStatus
    -------------------------------------------------------------------------
<BANKED_CODE,CODE_C> 1 (was BANKED_CODE)
  Relative segment, address: CODE 00005B3B - 00005B3D (0x3 bytes), align: 0
  Segment part 37.            Intra module refs:   GAP_PeriDevMgrInit
    -------------------------------------------------------------------------
<BANKED_CODE,CODE_C> 1 (was BANKED_CODE)
  Relative segment, address: CODE 00005B3E - 00005B43 (0x6 bytes), align: 0
  Segment part 38.            Intra module refs:   GAP_MakeDiscoverable
                                                   GAP_PeriDevMgrInit
                                                   Segment part 37
    -------------------------------------------------------------------------
<BANKED_CODE,CODE_C> 1 (was BANKED_CODE)
  Relative segment, address: CODE 00005B44 - 00005BA9 (0x66 bytes), align: 0
  Segment part 39.            Intra module refs:   gapPeriProcessHCICmdCompleteEvt::?relay
           LOCAL                   ADDRESS         
           =====                   =======         
           gapPeriProcessHCICmdCompleteEvt
                                   00005B44 
               calls direct, is indirectly called
               XSTACK = 00000000 ( 0000000A )
    -------------------------------------------------------------------------
<BANKED_CODE,CODE_C> 1 (was BANKED_CODE)
  Relative segment, address: CODE 00005BAA - 00005BAC (0x3 bytes), align: 0
  Segment part 41.            Intra module refs:   isLimitedDiscoverableMode
    -------------------------------------------------------------------------
<BANKED_CODE,CODE_C> 1 (was BANKED_CODE)
  Relative segment, address: CODE 00005BAD - 00005BAF (0x3 bytes), align: 0
  Segment part 42.            Intra module refs:   Segment part 41
                                                   gapPeriProcessHCICmdCompleteEvt
    -------------------------------------------------------------------------
<BANKED_CODE,CODE_C> 1 (was BANKED_CODE)
  Relative segment, address: CODE 00005BB0 - 00005BB4 (0x5 bytes), align: 0
  Segment part 43.            Intra module refs:   GAP_EndDiscoverable
                                                   GAP_MakeDiscoverable
                                                   Segment part 42
                                                   gapProcessAdvertisingEvt
    -------------------------------------------------------------------------
<BANKED_CODE,CODE_C> 1 (was BANKED_CODE)
  Relative segment, address: CODE 00005BB5 - 00005C8D (0xd9 bytes), align: 0
  Segment part 44.            Intra module refs:   gapSetAdvParams::?relay
           ENTRY                   ADDRESS         REF BY
           =====                   =======         ======
           gapSetAdvParams         00005BB5 
               calls direct, is indirectly called
               XSTACK = 0000000C ( 00000014 )
    -------------------------------------------------------------------------
<BANKED_CODE,CODE_C> 1 (was BANKED_CODE)
  Relative segment, address: CODE 00005C8E - 00005C99 (0xc bytes), align: 0
  Segment part 46.            Intra module refs:   gapSetAdvParams
    -------------------------------------------------------------------------
<BANKED_CODE,CODE_C> 1 (was BANKED_CODE)
  Relative segment, address: CODE 00005C9A - 00005CC2 (0x29 bytes), align: 0
  Segment part 47.            Intra module refs:   gapSetAdvParamsStatus::?relay
           ENTRY                   ADDRESS         REF BY
           =====                   =======         ======
           gapSetAdvParamsStatus   00005C9A 
               calls direct
               XSTACK = 0000000A ( 00000009 )
    -------------------------------------------------------------------------
<BANKED_CODE,CODE_C> 1 (was BANKED_CODE)
  Relative segment, address: CODE 00005CC3 - 00005CC7 (0x5 bytes), align: 0
  Segment part 49.            Intra module refs:   gapSetAdvParams
                                                   gapSetAdvParamsStatus
                                                   gapWriteAdvEnableStatus
    -------------------------------------------------------------------------
<BANKED_CODE,CODE_C> 1 (was BANKED_CODE)
  Relative segment, address: CODE 00005CC8 - 00005CCD (0x6 bytes), align: 0
  Segment part 50.            Intra module refs:   GAP_MakeDiscoverable
                                                   Segment part 43
                                                   Segment part 49
                                                   Segment part 84
    -------------------------------------------------------------------------
<BANKED_CODE,CODE_C> 1 (was BANKED_CODE)
  Relative segment, address: CODE 00005CCE - 00005DB5 (0xe8 bytes), align: 0
  Segment part 51.            Intra module refs:   gapWriteAdvEnableStatus::?relay
           ENTRY                   ADDRESS         REF BY
           =====                   =======         ======
           gapWriteAdvEnableStatus
                                   00005CCE 
               calls direct
               XSTACK = 0000000A ( 00000014 )
               ISTACK = 00000000 ( 00000001 )
    -------------------------------------------------------------------------
<BANKED_CODE,CODE_C> 1 (was BANKED_CODE)
  Relative segment, address: CODE 00005DB6 - 00005DBD (0x8 bytes), align: 0
  Segment part 53.            Intra module refs:   gapSendMakeDiscEvent
                                                   gapWriteAdvEnableStatus
    -------------------------------------------------------------------------
<BANKED_CODE,CODE_C> 1 (was BANKED_CODE)
  Relative segment, address: CODE 00005DBE - 00005DC6 (0x9 bytes), align: 0
  Segment part 54.            Intra module refs:   Segment part 53
                                                   gapWriteAdvDataStatus
    -------------------------------------------------------------------------
<BANKED_CODE,CODE_C> 1 (was BANKED_CODE)
  Relative segment, address: CODE 00005DC7 - 00005E03 (0x3d bytes), align: 0
  Segment part 55.            Intra module refs:   gapWriteAdvDataStatus::?relay
           ENTRY                   ADDRESS         REF BY
           =====                   =======         ======
           gapWriteAdvDataStatus   00005DC7 
               calls direct
               XSTACK = 0000000A ( 0000000A )
               ISTACK = 00000000 ( 00000001 )
    -------------------------------------------------------------------------
<BANKED_CODE,CODE_C> 1 (was BANKED_CODE)
  Relative segment, address: CODE 00005E04 - 00005EC4 (0xc1 bytes), align: 0
  Segment part 57.            Intra module refs:   gapProcessAdvertisingEvt::?relay
           LOCAL                   ADDRESS         
           =====                   =======         
           gapProcessAdvertisingEvt
                                   00005E04 
               calls direct, is indirectly called
               XSTACK = 00000000 ( 00000010 )
    -------------------------------------------------------------------------
<BANKED_CODE,CODE_C> 1 (was BANKED_CODE)
  Relative segment, address: CODE 00005EC5 - 00005EC9 (0x5 bytes), align: 0
  Segment part 61.            Intra module refs:   GAP_MakeDiscoverable
                                                   gapProcessAdvertisingEvt
    -------------------------------------------------------------------------
<BANKED_CODE,CODE_C> 1 (was BANKED_CODE)
  Relative segment, address: CODE 00005ECA - 00005ECE (0x5 bytes), align: 0
  Segment part 64.            Intra module refs:   gapPeriProcessHCICmdCompleteEvt
                                                   gapSendMakeDiscEvent
                                                   gapWriteAdvDataStatus
                                                   isLimitedDiscoverableMode
    -------------------------------------------------------------------------
<BANKED_CODE,CODE_C> 1 (was BANKED_CODE)
  Relative segment, address: CODE 00005ECF - 00005ED1 (0x3 bytes), align: 0
  Segment part 67.            Intra module refs:   GAP_PeriDevMgrInit
    -------------------------------------------------------------------------
<BANKED_CODE,CODE_C> 1 (was BANKED_CODE)
  Relative segment, address: CODE 00005ED2 - 00005ED7 (0x6 bytes), align: 0
  Segment part 68.            Intra module refs:   GAP_PeriDevMgrInit
                                                   Segment part 67
                                                   gapFreeAdvertState
    -------------------------------------------------------------------------
<BANKED_CODE,CODE_C> 1 (was BANKED_CODE)
  Relative segment, address: CODE 00005ED8 - 00005EDA (0x3 bytes), align: 0
  Segment part 73.            Intra module refs:   gapSetAdvParams
    -------------------------------------------------------------------------
<BANKED_CODE,CODE_C> 1 (was BANKED_CODE)
  Relative segment, address: CODE 00005EDB - 00005EDF (0x5 bytes), align: 0
  Segment part 74.            Intra module refs:   Segment part 20
                                                   Segment part 73
                                                   Segment part 91
    -------------------------------------------------------------------------
<BANKED_CODE,CODE_C> 1 (was BANKED_CODE)
  Relative segment, address: CODE 00005EE0 - 00005F0C (0x2d bytes), align: 0
  Segment part 81.            Intra module refs:   gapSendMakeDiscEvent::?relay
           LOCAL                   ADDRESS         
           =====                   =======         
           gapSendMakeDiscEvent    00005EE0 
               calls direct
               XSTACK = 00000010 ( 0000000A )
               ISTACK = 00000000 ( 00000001 )
    -------------------------------------------------------------------------
<BANKED_CODE,CODE_C> 1 (was BANKED_CODE)
  Relative segment, address: CODE 00005F0D - 00005F15 (0x9 bytes), align: 0
  Segment part 83.            Intra module refs:   gapPeriProcessHCICmdCompleteEvt
    -------------------------------------------------------------------------
<BANKED_CODE,CODE_C> 1 (was BANKED_CODE)
  Relative segment, address: CODE 00005F16 - 00005F1E (0x9 bytes), align: 0
  Segment part 84.            Intra module refs:   Segment part 83
                                                   gapSendMakeDiscEvent
                                                   gapWriteAdvEnableStatus
    -------------------------------------------------------------------------
<BANKED_CODE,CODE_C> 1 (was BANKED_CODE)
  Relative segment, address: CODE 00005F1F - 00005F3A (0x1c bytes), align: 0
  Segment part 85.            Intra module refs:   gapFreeAdvertState::?relay
           LOCAL                   ADDRESS         
           =====                   =======         
           gapFreeAdvertState      00005F1F 
               calls direct
               XSTACK = 00000010 ( 00000000 )
               ISTACK = 00000000 ( 00000002 )
    -------------------------------------------------------------------------
<BANKED_CODE,CODE_C> 1 (was BANKED_CODE)
  Relative segment, address: CODE 00005F3B - 00005F8F (0x55 bytes), align: 0
  Segment part 87.            Intra module refs:   isLimitedDiscoverableMode::?relay
           LOCAL                   ADDRESS         
           =====                   =======         
           isLimitedDiscoverableMode
                                   00005F3B 
               calls direct
               XSTACK = 00000010 ( 0000000D )
    -------------------------------------------------------------------------
<BANKED_CODE,CODE_C> 1 (was BANKED_CODE)
  Relative segment, address: CODE 00005F90 - 00005F91 (0x2 bytes), align: 0
  Segment part 89.            Intra module refs:   GAP_EndDiscoverable
                                                   gapSendMakeDiscEvent
                                                   gapSetAdvParamsStatus
                                                   gapWriteAdvEnableStatus
    -------------------------------------------------------------------------
<BANKED_CODE,CODE_C> 1 (was BANKED_CODE)
  Relative segment, address: CODE 00005F92 - 00005F94 (0x3 bytes), align: 0
  Segment part 90.            Intra module refs:   GAP_MakeDiscoverable
                                                   Segment part 89
                                                   gapFreeAdvertState
                                                   gapProcessAdvertisingEvt
                                                   gapSetAdvParams
    -------------------------------------------------------------------------
<BANKED_CODE,CODE_C> 1 (was BANKED_CODE)
  Relative segment, address: CODE 00005F95 - 00005F9B (0x7 bytes), align: 0
  Segment part 91.            Intra module refs:   GAP_MakeDiscoverable
                                                   GAP_PeriDevMgrInit
                                                   GAP_UpdateAdvertisingData
                                                   Segment part 90
                                                   gapProcessAdvertisingEvt
                                                   isLimitedDiscoverableMode
    -------------------------------------------------------------------------
XDATA_ID
  Relative segment, address: CODE 000001A9 - 000001A9 (0x1 bytes), align: 0
  Segment part 7.             Intra module refs:   Segment part 6
    -------------------------------------------------------------------------
XDATA_ID
  Relative segment, address: CODE 000001AA - 000001AF (0x6 bytes), align: 0
  Segment part 13.            Intra module refs:   Segment part 12
    -------------------------------------------------------------------------
<XDATA_ROM_C> 1 (was XDATA_ROM_C)
  Relative segment, address: CONST 00008FD0 - 00008FD3 (0x4 bytes), align: 0
  Segment part 15.            Intra module refs:   gapWriteAdvEnableStatus
           ENTRY                   ADDRESS         REF BY
           =====                   =======         ======
           __Constant_3e8          00008FD0 
    -------------------------------------------------------------------------
BANK_RELAYS
  Relative segment, address: CODE 00000296 - 0000029B (0x6 bytes), align: 0
  Segment part 17.
           ENTRY                   ADDRESS         REF BY
           =====                   =======         ======
           GAP_MakeDiscoverable::?relay
                                   00000296        GAPRole_ProcessEvent (broadcaster)
    -------------------------------------------------------------------------
BANK_RELAYS
  Relative segment, address: CODE 0000029C - 000002A1 (0x6 bytes), align: 0
  Segment part 22.
           ENTRY                   ADDRESS         REF BY
           =====                   =======         ======
           GAP_UpdateAdvertisingData::?relay
                                   0000029C        GAPRole_SetParameter (broadcaster)
                                                   gapRole_ProcessGAPMsg (broadcaster)
    -------------------------------------------------------------------------
BANK_RELAYS
  Relative segment, address: CODE 000002A2 - 000002A7 (0x6 bytes), align: 0
  Segment part 24.            Intra module refs:   gapProcessAdvertisingEvt
           ENTRY                   ADDRESS         REF BY
           =====                   =======         ======
           GAP_EndDiscoverable::?relay
                                   000002A2        GAPRole_SetParameter (broadcaster)
    -------------------------------------------------------------------------
BANK_RELAYS
  Relative segment, address: CODE 000002A8 - 000002AD (0x6 bytes), align: 0
  Segment part 35.
           ENTRY                   ADDRESS         REF BY
           =====                   =======         ======
           GAP_PeriDevMgrInit::?relay
                                   000002A8        GAP_DeviceInit (gap)
    -------------------------------------------------------------------------
BANK_RELAYS
  Relative segment, address: CODE 000002AE - 000002B3 (0x6 bytes), align: 0
  Segment part 40.            Intra module refs:   Segment part 13
           LOCAL                   ADDRESS         
           =====                   =======         
           gapPeriProcessHCICmdCompleteEvt::?relay
                                   000002AE 
    -------------------------------------------------------------------------
BANK_RELAYS
  Relative segment, address: CODE 000002B4 - 000002B9 (0x6 bytes), align: 0
  Segment part 45.            Intra module refs:   GAP_MakeDiscoverable
                                                   Segment part 13
           ENTRY                   ADDRESS         REF BY
           =====                   =======         ======
           gapSetAdvParams::?relay
                                   000002B4 
    -------------------------------------------------------------------------
BANK_RELAYS
  Relative segment, address: CODE 000002BA - 000002BF (0x6 bytes), align: 0
  Segment part 48.            Intra module refs:   gapPeriProcessHCICmdCompleteEvt
           ENTRY                   ADDRESS         REF BY
           =====                   =======         ======
           gapSetAdvParamsStatus::?relay
                                   000002BA 
    -------------------------------------------------------------------------
BANK_RELAYS
  Relative segment, address: CODE 000002C0 - 000002C5 (0x6 bytes), align: 0
  Segment part 52.            Intra module refs:   gapPeriProcessHCICmdCompleteEvt
           ENTRY                   ADDRESS         REF BY
           =====                   =======         ======
           gapWriteAdvEnableStatus::?relay
                                   000002C0 
    -------------------------------------------------------------------------
BANK_RELAYS
  Relative segment, address: CODE 000002C6 - 000002CB (0x6 bytes), align: 0
  Segment part 56.            Intra module refs:   gapPeriProcessHCICmdCompleteEvt
           ENTRY                   ADDRESS         REF BY
           =====                   =======         ======
           gapWriteAdvDataStatus::?relay
                                   000002C6 
    -------------------------------------------------------------------------
BANK_RELAYS
  Relative segment, address: CODE 000002CC - 000002D1 (0x6 bytes), align: 0
  Segment part 58.            Intra module refs:   Segment part 13
           LOCAL                   ADDRESS         
           =====                   =======         
           gapProcessAdvertisingEvt::?relay
                                   000002CC 
    -------------------------------------------------------------------------
BANK_RELAYS
  Relative segment, address: CODE 000002D2 - 000002D7 (0x6 bytes), align: 0
  Segment part 82.            Intra module refs:   gapSetAdvParamsStatus
                                                   gapWriteAdvEnableStatus
           LOCAL                   ADDRESS         
           =====                   =======         
           gapSendMakeDiscEvent::?relay
                                   000002D2 
    -------------------------------------------------------------------------
BANK_RELAYS
  Relative segment, address: CODE 000002D8 - 000002DD (0x6 bytes), align: 0
  Segment part 86.            Intra module refs:   GAP_MakeDiscoverable
                                                   gapProcessAdvertisingEvt
                                                   gapSendMakeDiscEvent
                                                   gapWriteAdvEnableStatus
           LOCAL                   ADDRESS         
           =====                   =======         
           gapFreeAdvertState::?relay
                                   000002D8 
    -------------------------------------------------------------------------
BANK_RELAYS
  Relative segment, address: CODE 000002DE - 000002E3 (0x6 bytes), align: 0
  Segment part 88.            Intra module refs:   gapSetAdvParams
                                                   gapWriteAdvEnableStatus
           LOCAL                   ADDRESS         
           =====                   =======         
           isLimitedDiscoverableMode::?relay
                                   000002DE 
    -------------------------------------------------------------------------
<BANKED_CODE,XDATA_ROM_C_FLASH> 1 (was XDATA_ROM_C_FLASH)
  Relative segment, address: CODE 00008FD0 - 00008FD3 (0x4 bytes), align: 0
  Segment part 93.            Intra module refs:   __Constant_3e8

    -------------------------------------------------------------------------
  LIBRARY MODULE, NAME : gap_simpletask

  SEGMENTS IN THE MODULE
  ======================
XDATA_Z
  Relative segment, address: XDATA 000002D9 - 000002D9 (0x1 bytes), align: 0
  Segment part 6.             Intra module refs:   GAP_Init
                                                   GAP_ProcessEvent
           ENTRY                   ADDRESS         REF BY
           =====                   =======         ======
           gapTaskID               000002D9        GAP_EndDiscoverable (gap_peridevmgr)
                                                   GAP_MakeDiscoverable (gap_peridevmgr)
                                                   gapProcessAdvertisingEvt (gap_peridevmgr)
                                                   gapProcessRandomAddrComplete (gap_configmgr)
                                                   gapWriteAdvEnableStatus (gap_peridevmgr)
    -------------------------------------------------------------------------
XDATA_I
  Relative segment, address: XDATA 000010D4 - 000010D4 (0x1 bytes), align: 0
  Segment part 7.             Intra module refs:   GAP_ProcessEvent
                                                   GAP_RegisterForMsgs
           ENTRY                   ADDRESS         REF BY
           =====                   =======         ======
           gapUnwantedTaskID       000010D4 
    -------------------------------------------------------------------------
XDATA_Z
  Relative segment, address: XDATA 000002DA - 000002DB (0x2 bytes), align: 0
  Segment part 9.             Intra module refs:   GAP_ProcessEvent
                                                   gapProcessHCICmdCompleteEvt
                                                   gapRegisterPeripheral
           ENTRY                   ADDRESS         REF BY
           =====                   =======         ======
           pfnPeripheralCBs        000002DA        gapProcessRandomAddrComplete (gap_configmgr)
    -------------------------------------------------------------------------
XDATA_Z
  Relative segment, address: XDATA 000002DC - 000002DD (0x2 bytes), align: 0
  Segment part 10.            Intra module refs:   Segment part 27
    -------------------------------------------------------------------------
<BANKED_CODE,XDATA_ROM_C_FLASH> 1 (was BANKED_CODE)
  Relative segment, address: CODE 0000B80F - 0000B819 (0xb bytes), align: 0
  Segment part 11.            Intra module refs:   GAP_RegisterForMsgs::?relay
           ENTRY                   ADDRESS         REF BY
           =====                   =======         ======
           GAP_RegisterForMsgs     0000B80F 
               ISTACK = 00000000 ( 00000002 )
    -------------------------------------------------------------------------
<BANKED_CODE,XDATA_ROM_C_FLASH> 1 (was BANKED_CODE)
  Relative segment, address: CODE 0000B81A - 0000B82B (0x12 bytes), align: 0
  Segment part 13.            Intra module refs:   GAP_Init::?relay
           ENTRY                   ADDRESS         REF BY
           =====                   =======         ======
           GAP_Init                0000B81A 
               calls direct
               XSTACK = 00000000 ( 00000009 )
    -------------------------------------------------------------------------
<BANKED_CODE,XDATA_ROM_C_FLASH> 1 (was BANKED_CODE)
  Relative segment, address: CODE 0000B82C - 0000B8F1 (0xc6 bytes), align: 0
  Segment part 15.            Intra module refs:   GAP_ProcessEvent::?relay
           ENTRY                   ADDRESS         REF BY
           =====                   =======         ======
           GAP_ProcessEvent        0000B82C 
               calls direct
               XSTACK = 00000000 ( 0000000C )
    -------------------------------------------------------------------------
<BANKED_CODE,XDATA_ROM_C_FLASH> 1 (was BANKED_CODE)
  Relative segment, address: CODE 0000B8F2 - 0000B8F6 (0x5 bytes), align: 0
  Segment part 17.            Intra module refs:   GAP_ProcessEvent
                                                   gapProcessHCICmdCompleteEvt
    -------------------------------------------------------------------------
<BANKED_CODE,XDATA_ROM_C_FLASH> 1 (was BANKED_CODE)
  Relative segment, address: CODE 0000B8F7 - 0000B8FB (0x5 bytes), align: 0
  Segment part 18.            Intra module refs:   GAP_ProcessEvent
    -------------------------------------------------------------------------
<BANKED_CODE,XDATA_ROM_C_FLASH> 1 (was BANKED_CODE)
  Relative segment, address: CODE 0000B8FC - 0000B903 (0x8 bytes), align: 0
  Segment part 19.            Intra module refs:   Segment part 18
                                                   gapProcessHCICmdCompleteEvt
    -------------------------------------------------------------------------
<BANKED_CODE,XDATA_ROM_C_FLASH> 1 (was BANKED_CODE)
  Relative segment, address: CODE 0000B904 - 0000B908 (0x5 bytes), align: 0
  Segment part 20.            Intra module refs:   GAP_NumActiveConnections::?relay
           ENTRY                   ADDRESS         REF BY
           =====                   =======         ======
           GAP_NumActiveConnections
                                   0000B904 
    -------------------------------------------------------------------------
<BANKED_CODE,XDATA_ROM_C_FLASH> 1 (was BANKED_CODE)
  Relative segment, address: CODE 0000B909 - 0000B9C1 (0xb9 bytes), align: 0
  Segment part 22.            Intra module refs:   gapProcessHCICmdCompleteEvt::?relay
           LOCAL                   ADDRESS         
           =====                   =======         
           gapProcessHCICmdCompleteEvt
                                   0000B909 
               calls direct
               XSTACK = 0000000C ( 0000000C )
    -------------------------------------------------------------------------
<BANKED_CODE,XDATA_ROM_C_FLASH> 1 (was BANKED_CODE)
  Relative segment, address: CODE 0000B9C2 - 0000B9CB (0xa bytes), align: 0
  Segment part 24.            Intra module refs:   Segment part 19
                                                   gapProcessHCICmdCompleteEvt
    -------------------------------------------------------------------------
<BANKED_CODE,XDATA_ROM_C_FLASH> 1 (was BANKED_CODE)
  Relative segment, address: CODE 0000B9CC - 0000B9D1 (0x6 bytes), align: 0
  Segment part 25.            Intra module refs:   Segment part 18
                                                   Segment part 26
                                                   gapProcessHCICmdCompleteEvt
    -------------------------------------------------------------------------
<BANKED_CODE,XDATA_ROM_C_FLASH> 1 (was BANKED_CODE)
  Relative segment, address: CODE 0000B9D2 - 0000B9E2 (0x11 bytes), align: 0
  Segment part 26.            Intra module refs:   gapProcessHCICmdCompleteEvt
    -------------------------------------------------------------------------
<BANKED_CODE,XDATA_ROM_C_FLASH> 1 (was BANKED_CODE)
  Relative segment, address: CODE 0000B9E3 - 0000B9E5 (0x3 bytes), align: 0
  Segment part 27.            Intra module refs:   GAP_ProcessEvent
                                                   gapProcessHCICmdCompleteEvt
    -------------------------------------------------------------------------
<BANKED_CODE,XDATA_ROM_C_FLASH> 1 (was BANKED_CODE)
  Relative segment, address: CODE 0000B9E6 - 0000B9ED (0x8 bytes), align: 0
  Segment part 28.            Intra module refs:   GAP_ProcessEvent
                                                   Segment part 27
                                                   gapProcessHCICmdCompleteEvt
    -------------------------------------------------------------------------
<BANKED_CODE,XDATA_ROM_C_FLASH> 1 (was BANKED_CODE)
  Relative segment, address: CODE 0000B9EE - 0000B9F1 (0x4 bytes), align: 0
  Segment part 31.            Intra module refs:   gapRegisterPeripheral
    -------------------------------------------------------------------------
<BANKED_CODE,XDATA_ROM_C_FLASH> 1 (was BANKED_CODE)
  Relative segment, address: CODE 0000B9F2 - 0000B9F9 (0x8 bytes), align: 0
  Segment part 32.            Intra module refs:   GAP_RegisterForMsgs
                                                   Segment part 31
    -------------------------------------------------------------------------
<BANKED_CODE,XDATA_ROM_C_FLASH> 1 (was BANKED_CODE)
  Relative segment, address: CODE 0000B9FA - 0000BA02 (0x9 bytes), align: 0
  Segment part 33.            Intra module refs:   gapRegisterPeripheral::?relay
           ENTRY                   ADDRESS         REF BY
           =====                   =======         ======
           gapRegisterPeripheral   0000B9FA 
               ISTACK = 00000000 ( 00000002 )
    -------------------------------------------------------------------------
XDATA_ID
  Relative segment, address: CODE 000001B0 - 000001B0 (0x1 bytes), align: 0
  Segment part 8.             Intra module refs:   gapUnwantedTaskID
    -------------------------------------------------------------------------
BANK_RELAYS
  Relative segment, address: CODE 000002E4 - 000002E9 (0x6 bytes), align: 0
  Segment part 12.
           ENTRY                   ADDRESS         REF BY
           =====                   =======         ======
           GAP_RegisterForMsgs::?relay
                                   000002E4        GAPRole_Init (broadcaster)
    -------------------------------------------------------------------------
BANK_RELAYS
  Relative segment, address: CODE 000002EA - 000002EF (0x6 bytes), align: 0
  Segment part 14.
           ENTRY                   ADDRESS         REF BY
           =====                   =======         ======
           GAP_Init::?relay        000002EA        osalInitTasks (OSAL_SimpleBLEBroadcaster)
    -------------------------------------------------------------------------
BANK_RELAYS
  Relative segment, address: CODE 000002F0 - 000002F5 (0x6 bytes), align: 0
  Segment part 16.
           ENTRY                   ADDRESS         REF BY
           =====                   =======         ======
           GAP_ProcessEvent::?relay
                                   000002F0        tasksArr (OSAL_SimpleBLEBroadcaster)
    -------------------------------------------------------------------------
BANK_RELAYS
  Relative segment, address: CODE 000002F6 - 000002FB (0x6 bytes), align: 0
  Segment part 21.
           ENTRY                   ADDRESS         REF BY
           =====                   =======         ======
           GAP_NumActiveConnections::?relay
                                   000002F6        GAP_MakeDiscoverable (gap_peridevmgr)
                                                   gapSetAdvParams (gap_peridevmgr)
    -------------------------------------------------------------------------
BANK_RELAYS
  Relative segment, address: CODE 000002FC - 00000301 (0x6 bytes), align: 0
  Segment part 23.            Intra module refs:   GAP_ProcessEvent
           LOCAL                   ADDRESS         
           =====                   =======         
           gapProcessHCICmdCompleteEvt::?relay
                                   000002FC 
    -------------------------------------------------------------------------
BANK_RELAYS
  Relative segment, address: CODE 00000302 - 00000307 (0x6 bytes), align: 0
  Segment part 34.
           ENTRY                   ADDRESS         REF BY
           =====                   =======         ======
           gapRegisterPeripheral::?relay
                                   00000302        GAP_PeriDevMgrInit (gap_peridevmgr)

    -------------------------------------------------------------------------
  LIBRARY MODULE, NAME : hci

  SEGMENTS IN THE MODULE
  ======================
XDATA_Z
  Relative segment, address: XDATA 000002DE - 000002DE (0x1 bytes), align: 0
  Segment part 8.
           ENTRY                   ADDRESS         REF BY
           =====                   =======         ======
           hciPTMenabled           000002DE        HCI_CommandCompleteEvent (hci_event)
                                                   HCI_Init (hci_tl)
                                                   HCI_VendorSpecifcCommandCompleteEvent (hci_event_PATCH)
    -------------------------------------------------------------------------
XDATA_Z
  Relative segment, address: XDATA 000002DF - 000002DF (0x1 bytes), align: 0
  Segment part 9.
           ENTRY                   ADDRESS         REF BY
           =====                   =======         ======
           ctrlToHostEnable        000002DF        HCI_ResetCmd (hci_PATCH)
    -------------------------------------------------------------------------
XDATA_Z
  Relative segment, address: XDATA 000002E0 - 000002E1 (0x2 bytes), align: 0
  Segment part 10.
           ENTRY                   ADDRESS         REF BY
           =====                   =======         ======
           numHostBufs             000002E0        HCI_ResetCmd (hci_PATCH)
    -------------------------------------------------------------------------
<BANKED_CODE,CODE_C> 1 (was BANKED_CODE)
  Relative segment, address: CODE 00003ED3 - 00003EDC (0xa bytes), align: 0
  Segment part 11.            Intra module refs:   HCI_bm_alloc::?relay
           ENTRY                   ADDRESS         REF BY
           =====                   =======         ======
           HCI_bm_alloc            00003ED3 
               calls direct
               ISTACK = 00000000 ( 00000002 )
    -------------------------------------------------------------------------
<BANKED_CODE,CODE_C> 1 (was BANKED_CODE)
  Relative segment, address: CODE 00003EDD - 00003F25 (0x49 bytes), align: 0
  Segment part 13.            Intra module refs:   HCI_SetEventMaskCmd::?relay
           ENTRY                   ADDRESS         REF BY
           =====                   =======         ======
           HCI_SetEventMaskCmd     00003EDD 
               calls direct
               XSTACK = 00000000 ( 0000000D )
    -------------------------------------------------------------------------
<BANKED_CODE,CODE_C> 1 (was BANKED_CODE)
  Relative segment, address: CODE 00003F26 - 00003FD0 (0xab bytes), align: 0
  Segment part 15.            Intra module refs:   HCI_ReadLocalVersionInfoCmd::?relay
           ENTRY                   ADDRESS         REF BY
           =====                   =======         ======
           HCI_ReadLocalVersionInfoCmd
                                   00003F26 
               calls direct
               XSTACK = 00000000 ( 0000001A )
               ISTACK = 00000000 ( 00000001 )
    -------------------------------------------------------------------------
<BANKED_CODE,CODE_C> 1 (was BANKED_CODE)
  Relative segment, address: CODE 00003FD1 - 00003FF3 (0x23 bytes), align: 0
  Segment part 17.            Intra module refs:   HCI_ReadLocalSupportedFeaturesCmd::?relay
           ENTRY                   ADDRESS         REF BY
           =====                   =======         ======
           HCI_ReadLocalSupportedFeaturesCmd
                                   00003FD1 
               calls direct
               XSTACK = 00000000 ( 00000009 )
               ISTACK = 00000000 ( 00000002 )
    -------------------------------------------------------------------------
<BANKED_CODE,CODE_C> 1 (was BANKED_CODE)
  Relative segment, address: CODE 00003FF4 - 00003FF5 (0x2 bytes), align: 0
  Segment part 19.            Intra module refs:   HCI_LE_ReadLocalSupportedFeaturesCmd
                                                   HCI_LE_ReadSupportedStatesCmd
    -------------------------------------------------------------------------
<BANKED_CODE,CODE_C> 1 (was BANKED_CODE)
  Relative segment, address: CODE 00003FF6 - 00003FF8 (0x3 bytes), align: 0
  Segment part 20.            Intra module refs:   HCI_ReadLocalSupportedFeaturesCmd
                                                   Segment part 19
    -------------------------------------------------------------------------
<BANKED_CODE,CODE_C> 1 (was BANKED_CODE)
  Relative segment, address: CODE 00003FF9 - 00003FFF (0x7 bytes), align: 0
  Segment part 21.            Intra module refs:   HCI_LE_RandCmd
                                                   Segment part 20
    -------------------------------------------------------------------------
<BANKED_CODE,CODE_C> 1 (was BANKED_CODE)
  Relative segment, address: CODE 00004000 - 00004027 (0x28 bytes), align: 0
  Segment part 22.            Intra module refs:   HCI_ReadBDADDRCmd::?relay
           ENTRY                   ADDRESS         REF BY
           =====                   =======         ======
           HCI_ReadBDADDRCmd       00004000 
               calls direct
               XSTACK = 00000000 ( 00000007 )
               ISTACK = 00000000 ( 00000003 )
    -------------------------------------------------------------------------
<BANKED_CODE,CODE_C> 1 (was BANKED_CODE)
  Relative segment, address: CODE 00004028 - 00004062 (0x3b bytes), align: 0
  Segment part 24.            Intra module refs:   HCI_ReadRssiCmd::?relay
           ENTRY                   ADDRESS         REF BY
           =====                   =======         ======
           HCI_ReadRssiCmd         00004028 
               calls direct
               XSTACK = 00000000 ( 0000000D )
               ISTACK = 00000000 ( 00000001 )
    -------------------------------------------------------------------------
<BANKED_CODE,CODE_C> 1 (was BANKED_CODE)
  Relative segment, address: CODE 00004063 - 00004069 (0x7 bytes), align: 0
  Segment part 26.            Intra module refs:   HCI_EXT_SetRxGainCmd
                                                   HCI_EXT_SetTxPowerCmd
                                                   HCI_ReadRssiCmd
    -------------------------------------------------------------------------
<BANKED_CODE,CODE_C> 1 (was BANKED_CODE)
  Relative segment, address: CODE 0000406A - 00004096 (0x2d bytes), align: 0
  Segment part 27.            Intra module refs:   HCI_LE_SetEventMaskCmd::?relay
           ENTRY                   ADDRESS         REF BY
           =====                   =======         ======
           HCI_LE_SetEventMaskCmd
                                   0000406A 
               calls direct
               XSTACK = 00000000 ( 00000001 )
               ISTACK = 00000000 ( 00000002 )
    -------------------------------------------------------------------------
<BANKED_CODE,CODE_C> 1 (was BANKED_CODE)
  Relative segment, address: CODE 00004097 - 0000409E (0x8 bytes), align: 0
  Segment part 29.            Intra module refs:   HCI_LE_SetEventMaskCmd
                                                   HCI_SetEventMaskCmd
    -------------------------------------------------------------------------
<BANKED_CODE,CODE_C> 1 (was BANKED_CODE)
  Relative segment, address: CODE 0000409F - 000040C0 (0x22 bytes), align: 0
  Segment part 30.            Intra module refs:   HCI_LE_ReadLocalSupportedFeaturesCmd::?relay
           ENTRY                   ADDRESS         REF BY
           =====                   =======         ======
           HCI_LE_ReadLocalSupportedFeaturesCmd
                                   0000409F 
               calls direct
               XSTACK = 00000000 ( 00000009 )
               ISTACK = 00000000 ( 00000003 )
    -------------------------------------------------------------------------
<BANKED_CODE,CODE_C> 1 (was BANKED_CODE)
  Relative segment, address: CODE 000040C1 - 000040C8 (0x8 bytes), align: 0
  Segment part 32.            Intra module refs:   HCI_LE_ReadLocalSupportedFeaturesCmd
                                                   HCI_ReadLocalSupportedFeaturesCmd
    -------------------------------------------------------------------------
<BANKED_CODE,CODE_C> 1 (was BANKED_CODE)
  Relative segment, address: CODE 000040C9 - 000040F1 (0x29 bytes), align: 0
  Segment part 33.            Intra module refs:   HCI_LE_SetRandomAddressCmd::?relay
           ENTRY                   ADDRESS         REF BY
           =====                   =======         ======
           HCI_LE_SetRandomAddressCmd
                                   000040C9 
               calls direct
               XSTACK = 00000000 ( 00000001 )
               ISTACK = 00000000 ( 00000003 )
    -------------------------------------------------------------------------
<BANKED_CODE,CODE_C> 1 (was BANKED_CODE)
  Relative segment, address: CODE 000040F2 - 0000413F (0x4e bytes), align: 0
  Segment part 35.            Intra module refs:   HCI_LE_SetAdvParamCmd::?relay
           ENTRY                   ADDRESS         REF BY
           =====                   =======         ======
           HCI_LE_SetAdvParamCmd   000040F2 
               calls direct
               XSTACK = 00000006 ( 00000010 )
               ISTACK = 00000000 ( 00000001 )
    -------------------------------------------------------------------------
<BANKED_CODE,CODE_C> 1 (was BANKED_CODE)
  Relative segment, address: CODE 00004140 - 00004145 (0x6 bytes), align: 0
  Segment part 37.            Intra module refs:   HCI_LE_SetAdvParamCmd
    -------------------------------------------------------------------------
<BANKED_CODE,CODE_C> 1 (was BANKED_CODE)
  Relative segment, address: CODE 00004146 - 0000415A (0x15 bytes), align: 0
  Segment part 38.            Intra module refs:   HCI_LE_SetAdvDataCmd::?relay
           ENTRY                   ADDRESS         REF BY
           =====                   =======         ======
           HCI_LE_SetAdvDataCmd    00004146 
               calls direct
               XSTACK = 00000000 ( 0000000A )
               ISTACK = 00000000 ( 00000001 )
    -------------------------------------------------------------------------
<BANKED_CODE,CODE_C> 1 (was BANKED_CODE)
  Relative segment, address: CODE 0000415B - 0000416F (0x15 bytes), align: 0
  Segment part 40.            Intra module refs:   HCI_LE_SetScanRspDataCmd::?relay
           ENTRY                   ADDRESS         REF BY
           =====                   =======         ======
           HCI_LE_SetScanRspDataCmd
                                   0000415B 
               calls direct
               XSTACK = 00000000 ( 0000000A )
               ISTACK = 00000000 ( 00000001 )
    -------------------------------------------------------------------------
<BANKED_CODE,CODE_C> 1 (was BANKED_CODE)
  Relative segment, address: CODE 00004170 - 00004184 (0x15 bytes), align: 0
  Segment part 42.            Intra module refs:   HCI_LE_SetAdvEnableCmd::?relay
           ENTRY                   ADDRESS         REF BY
           =====                   =======         ======
           HCI_LE_SetAdvEnableCmd
                                   00004170 
               calls direct
               XSTACK = 00000000 ( 0000000A )
               ISTACK = 00000000 ( 00000001 )
    -------------------------------------------------------------------------
<BANKED_CODE,CODE_C> 1 (was BANKED_CODE)
  Relative segment, address: CODE 00004185 - 000041A0 (0x1c bytes), align: 0
  Segment part 44.            Intra module refs:   HCI_LE_ReadAdvChanTxPowerCmd::?relay
           ENTRY                   ADDRESS         REF BY
           =====                   =======         ======
           HCI_LE_ReadAdvChanTxPowerCmd
                                   00004185 
               calls direct
               XSTACK = 00000000 ( 00000002 )
               ISTACK = 00000000 ( 00000003 )
    -------------------------------------------------------------------------
<BANKED_CODE,CODE_C> 1 (was BANKED_CODE)
  Relative segment, address: CODE 000041A1 - 000041AC (0xc bytes), align: 0
  Segment part 46.            Intra module refs:   HCI_LE_ReadAdvChanTxPowerCmd
                                                   HCI_LE_ReadWhiteListSizeCmd
    -------------------------------------------------------------------------
<BANKED_CODE,CODE_C> 1 (was BANKED_CODE)
  Relative segment, address: CODE 000041AD - 000041B3 (0x7 bytes), align: 0
  Segment part 47.            Intra module refs:   HCI_LE_ReadAdvChanTxPowerCmd
                                                   HCI_LE_ReadSupportedStatesCmd
                                                   HCI_LE_ReadWhiteListSizeCmd
                                                   HCI_ReadBDADDRCmd
    -------------------------------------------------------------------------
<BANKED_CODE,CODE_C> 1 (was BANKED_CODE)
  Relative segment, address: CODE 000041B4 - 000041B7 (0x4 bytes), align: 0
  Segment part 48.            Intra module refs:   HCI_ReadRssiCmd
                                                   Segment part 47
    -------------------------------------------------------------------------
<BANKED_CODE,CODE_C> 1 (was BANKED_CODE)
  Relative segment, address: CODE 000041B8 - 000041BD (0x6 bytes), align: 0
  Segment part 49.            Intra module refs:   Segment part 101
                                                   Segment part 29
                                                   Segment part 32
                                                   Segment part 48
                                                   Segment part 55
    -------------------------------------------------------------------------
<BANKED_CODE,CODE_C> 1 (was BANKED_CODE)
  Relative segment, address: CODE 000041BE - 000041DB (0x1e bytes), align: 0
  Segment part 50.            Intra module refs:   HCI_LE_ReadWhiteListSizeCmd::?relay
           ENTRY                   ADDRESS         REF BY
           =====                   =======         ======
           HCI_LE_ReadWhiteListSizeCmd
                                   000041BE 
               calls direct
               XSTACK = 00000000 ( 00000002 )
               ISTACK = 00000000 ( 00000003 )
    -------------------------------------------------------------------------
<BANKED_CODE,CODE_C> 1 (was BANKED_CODE)
  Relative segment, address: CODE 000041DC - 000041EF (0x14 bytes), align: 0
  Segment part 52.            Intra module refs:   HCI_LE_ClearWhiteListCmd::?relay
           ENTRY                   ADDRESS         REF BY
           =====                   =======         ======
           HCI_LE_ClearWhiteListCmd
                                   000041DC 
               calls direct
               XSTACK = 00000000 ( 00000001 )
               ISTACK = 00000000 ( 00000003 )
    -------------------------------------------------------------------------
<BANKED_CODE,CODE_C> 1 (was BANKED_CODE)
  Relative segment, address: CODE 000041F0 - 000041F6 (0x7 bytes), align: 0
  Segment part 54.            Intra module refs:   HCI_LE_AddWhiteListCmd
                                                   HCI_LE_ClearWhiteListCmd
                                                   HCI_LE_ReceiverTestCmd
                                                   HCI_LE_RemoveWhiteListCmd
                                                   HCI_LE_SetAdvDataCmd
                                                   HCI_LE_SetAdvEnableCmd
                                                   HCI_LE_SetAdvParamCmd
                                                   HCI_LE_SetScanRspDataCmd
                                                   HCI_LE_TransmitterTestCmd
    -------------------------------------------------------------------------
<BANKED_CODE,CODE_C> 1 (was BANKED_CODE)
  Relative segment, address: CODE 000041F7 - 000041FC (0x6 bytes), align: 0
  Segment part 55.            Intra module refs:   HCI_LE_SetRandomAddressCmd
                                                   Segment part 54
    -------------------------------------------------------------------------
<BANKED_CODE,CODE_C> 1 (was BANKED_CODE)
  Relative segment, address: CODE 000041FD - 00004211 (0x15 bytes), align: 0
  Segment part 56.            Intra module refs:   HCI_LE_AddWhiteListCmd::?relay
           ENTRY                   ADDRESS         REF BY
           =====                   =======         ======
           HCI_LE_AddWhiteListCmd
                                   000041FD 
               calls direct
               XSTACK = 00000000 ( 0000000A )
               ISTACK = 00000000 ( 00000001 )
    -------------------------------------------------------------------------
<BANKED_CODE,CODE_C> 1 (was BANKED_CODE)
  Relative segment, address: CODE 00004212 - 00004226 (0x15 bytes), align: 0
  Segment part 58.            Intra module refs:   HCI_LE_RemoveWhiteListCmd::?relay
           ENTRY                   ADDRESS         REF BY
           =====                   =======         ======
           HCI_LE_RemoveWhiteListCmd
                                   00004212 
               calls direct
               XSTACK = 00000000 ( 0000000A )
               ISTACK = 00000000 ( 00000001 )
    -------------------------------------------------------------------------
<BANKED_CODE,CODE_C> 1 (was BANKED_CODE)
  Relative segment, address: CODE 00004227 - 00004279 (0x53 bytes), align: 0
  Segment part 60.            Intra module refs:   HCI_LE_EncryptCmd::?relay
           ENTRY                   ADDRESS         REF BY
           =====                   =======         ======
           HCI_LE_EncryptCmd       00004227 
               calls direct
               XSTACK = 00000000 ( 0000001D )
               ISTACK = 00000000 ( 00000001 )
    -------------------------------------------------------------------------
<BANKED_CODE,CODE_C> 1 (was BANKED_CODE)
  Relative segment, address: CODE 0000427A - 00004281 (0x8 bytes), align: 0
  Segment part 62.            Intra module refs:   HCI_EXT_DecryptCmd
                                                   HCI_LE_EncryptCmd
                                                   HCI_ReadLocalVersionInfoCmd
                                                   HCI_SetEventMaskCmd
                                                   LL_RandCback
    -------------------------------------------------------------------------
<BANKED_CODE,CODE_C> 1 (was BANKED_CODE)
  Relative segment, address: CODE 00004282 - 000042BB (0x3a bytes), align: 0
  Segment part 63.            Intra module refs:   HCI_LE_RandCmd::?relay
           ENTRY                   ADDRESS         REF BY
           =====                   =======         ======
           HCI_LE_RandCmd          00004282 
               calls direct
               XSTACK = 00000000 ( 00000009 )
               ISTACK = 00000000 ( 00000003 )
    -------------------------------------------------------------------------
<BANKED_CODE,CODE_C> 1 (was BANKED_CODE)
  Relative segment, address: CODE 000042BC - 000042E5 (0x2a bytes), align: 0
  Segment part 65.            Intra module refs:   HCI_LE_ReadSupportedStatesCmd::?relay
           ENTRY                   ADDRESS         REF BY
           =====                   =======         ======
           HCI_LE_ReadSupportedStatesCmd
                                   000042BC 
               calls direct
               XSTACK = 00000000 ( 00000009 )
               ISTACK = 00000000 ( 00000003 )
    -------------------------------------------------------------------------
<BANKED_CODE,CODE_C> 1 (was BANKED_CODE)
  Relative segment, address: CODE 000042E6 - 000042FA (0x15 bytes), align: 0
  Segment part 67.            Intra module refs:   HCI_LE_ReceiverTestCmd::?relay
           ENTRY                   ADDRESS         REF BY
           =====                   =======         ======
           HCI_LE_ReceiverTestCmd
                                   000042E6 
               calls direct
               XSTACK = 00000000 ( 0000000A )
               ISTACK = 00000000 ( 00000001 )
    -------------------------------------------------------------------------
<BANKED_CODE,CODE_C> 1 (was BANKED_CODE)
  Relative segment, address: CODE 000042FB - 0000430F (0x15 bytes), align: 0
  Segment part 69.            Intra module refs:   HCI_LE_TransmitterTestCmd::?relay
           ENTRY                   ADDRESS         REF BY
           =====                   =======         ======
           HCI_LE_TransmitterTestCmd
                                   000042FB 
               calls direct
               XSTACK = 00000000 ( 0000000A )
               ISTACK = 00000000 ( 00000001 )
    -------------------------------------------------------------------------
<BANKED_CODE,CODE_C> 1 (was BANKED_CODE)
  Relative segment, address: CODE 00004310 - 00004340 (0x31 bytes), align: 0
  Segment part 71.            Intra module refs:   HCI_LE_TestEndCmd::?relay
           ENTRY                   ADDRESS         REF BY
           =====                   =======         ======
           HCI_LE_TestEndCmd       00004310 
               calls direct
               XSTACK = 00000000 ( 00000003 )
               ISTACK = 00000000 ( 00000002 )
    -------------------------------------------------------------------------
<BANKED_CODE,CODE_C> 1 (was BANKED_CODE)
  Relative segment, address: CODE 00004341 - 00004345 (0x5 bytes), align: 0
  Segment part 73.            Intra module refs:   HCI_EXT_EndModemTestCmd
                                                   HCI_EXT_ModemHopTestTxCmd
                                                   HCI_EXT_SaveFreqTuneCmd
                                                   HCI_EXT_SetLocalSupportedFeaturesCmd
    -------------------------------------------------------------------------
<BANKED_CODE,CODE_C> 1 (was BANKED_CODE)
  Relative segment, address: CODE 00004346 - 00004347 (0x2 bytes), align: 0
  Segment part 74.            Intra module refs:   HCI_EXT_SetBDADDRCmd
                                                   HCI_LE_TestEndCmd
                                                   Segment part 73
    -------------------------------------------------------------------------
<BANKED_CODE,CODE_C> 1 (was BANKED_CODE)
  Relative segment, address: CODE 00004348 - 0000434C (0x5 bytes), align: 0
  Segment part 75.            Intra module refs:   Segment part 131
                                                   Segment part 74
    -------------------------------------------------------------------------
<BANKED_CODE,CODE_C> 1 (was BANKED_CODE)
  Relative segment, address: CODE 0000434D - 0000438E (0x42 bytes), align: 0
  Segment part 76.            Intra module refs:   HCI_EXT_SetRxGainCmd::?relay
           ENTRY                   ADDRESS         REF BY
           =====                   =======         ======
           HCI_EXT_SetRxGainCmd    0000434D 
               calls direct
               XSTACK = 00000000 ( 0000000D )
               ISTACK = 00000000 ( 00000001 )
    -------------------------------------------------------------------------
<BANKED_CODE,CODE_C> 1 (was BANKED_CODE)
  Relative segment, address: CODE 0000438F - 000043D0 (0x42 bytes), align: 0
  Segment part 78.            Intra module refs:   HCI_EXT_SetTxPowerCmd::?relay
           ENTRY                   ADDRESS         REF BY
           =====                   =======         ======
           HCI_EXT_SetTxPowerCmd   0000438F 
               calls direct
               XSTACK = 00000000 ( 0000000D )
               ISTACK = 00000000 ( 00000001 )
    -------------------------------------------------------------------------
<BANKED_CODE,CODE_C> 1 (was BANKED_CODE)
  Relative segment, address: CODE 000043D1 - 000043D7 (0x7 bytes), align: 0
  Segment part 80.            Intra module refs:   HCI_EXT_ExtendRfRangeCmd
                                                   HCI_EXT_SetRxGainCmd
                                                   HCI_EXT_SetTxPowerCmd
    -------------------------------------------------------------------------
<BANKED_CODE,CODE_C> 1 (was BANKED_CODE)
  Relative segment, address: CODE 000043D8 - 000043E0 (0x9 bytes), align: 0
  Segment part 81.            Intra module refs:   HCI_ReadLocalVersionInfoCmd
                                                   Segment part 80
    -------------------------------------------------------------------------
<BANKED_CODE,CODE_C> 1 (was BANKED_CODE)
  Relative segment, address: CODE 000043E1 - 000043E9 (0x9 bytes), align: 0
  Segment part 82.            Intra module refs:   HCI_LE_AddWhiteListCmd
                                                   HCI_LE_ReceiverTestCmd
                                                   HCI_LE_RemoveWhiteListCmd
                                                   HCI_LE_SetAdvDataCmd
                                                   HCI_LE_SetAdvEnableCmd
                                                   HCI_LE_SetAdvParamCmd
                                                   HCI_LE_SetScanRspDataCmd
                                                   HCI_LE_TransmitterTestCmd
    -------------------------------------------------------------------------
<BANKED_CODE,CODE_C> 1 (was BANKED_CODE)
  Relative segment, address: CODE 000043EA - 000043EC (0x3 bytes), align: 0
  Segment part 83.            Intra module refs:   HCI_EXT_BuildRevisionCmd
                                                   Segment part 112
                                                   Segment part 26
                                                   Segment part 82
    -------------------------------------------------------------------------
<BANKED_CODE,CODE_C> 1 (was BANKED_CODE)
  Relative segment, address: CODE 000043ED - 000043F1 (0x5 bytes), align: 0
  Segment part 84.            Intra module refs:   Segment part 83
    -------------------------------------------------------------------------
<BANKED_CODE,CODE_C> 1 (was BANKED_CODE)
  Relative segment, address: CODE 000043F2 - 0000441C (0x2b bytes), align: 0
  Segment part 85.            Intra module refs:   HCI_EXT_ClkDivOnHaltCmd::?relay
           ENTRY                   ADDRESS         REF BY
           =====                   =======         ======
           HCI_EXT_ClkDivOnHaltCmd
                                   000043F2 
               calls direct
               XSTACK = 00000000 ( 0000000C )
               ISTACK = 00000000 ( 00000001 )
    -------------------------------------------------------------------------
<BANKED_CODE,CODE_C> 1 (was BANKED_CODE)
  Relative segment, address: CODE 0000441D - 00004447 (0x2b bytes), align: 0
  Segment part 87.            Intra module refs:   HCI_EXT_DeclareNvUsageCmd::?relay
           ENTRY                   ADDRESS         REF BY
           =====                   =======         ======
           HCI_EXT_DeclareNvUsageCmd
                                   0000441D 
               calls direct
               XSTACK = 00000000 ( 0000000C )
               ISTACK = 00000000 ( 00000001 )
    -------------------------------------------------------------------------
<BANKED_CODE,CODE_C> 1 (was BANKED_CODE)
  Relative segment, address: CODE 00004448 - 000044AD (0x66 bytes), align: 0
  Segment part 89.            Intra module refs:   HCI_EXT_DecryptCmd::?relay
           ENTRY                   ADDRESS         REF BY
           =====                   =======         ======
           HCI_EXT_DecryptCmd      00004448 
               calls direct
               XSTACK = 00000000 ( 0000001F )
               ISTACK = 00000000 ( 00000001 )
    -------------------------------------------------------------------------
<BANKED_CODE,CODE_C> 1 (was BANKED_CODE)
  Relative segment, address: CODE 000044AE - 000044D7 (0x2a bytes), align: 0
  Segment part 91.            Intra module refs:   HCI_EXT_SetLocalSupportedFeaturesCmd::?relay
           ENTRY                   ADDRESS         REF BY
           =====                   =======         ======
           HCI_EXT_SetLocalSupportedFeaturesCmd
                                   000044AE 
               calls direct
               XSTACK = 00000000 ( 00000003 )
               ISTACK = 00000000 ( 00000003 )
    -------------------------------------------------------------------------
<BANKED_CODE,CODE_C> 1 (was BANKED_CODE)
  Relative segment, address: CODE 000044D8 - 000044E0 (0x9 bytes), align: 0
  Segment part 93.            Intra module refs:   HCI_LE_ClearWhiteListCmd
                                                   HCI_LE_SetEventMaskCmd
                                                   HCI_LE_SetRandomAddressCmd
    -------------------------------------------------------------------------
<BANKED_CODE,CODE_C> 1 (was BANKED_CODE)
  Relative segment, address: CODE 000044E1 - 000044E3 (0x3 bytes), align: 0
  Segment part 94.            Intra module refs:   HCI_EXT_ExtendRfRangeCmd
                                                   HCI_ReadBDADDRCmd
                                                   Segment part 21
                                                   Segment part 46
                                                   Segment part 75
                                                   Segment part 93
    -------------------------------------------------------------------------
<BANKED_CODE,CODE_C> 1 (was BANKED_CODE)
  Relative segment, address: CODE 000044E4 - 000044EA (0x7 bytes), align: 0
  Segment part 95.            Intra module refs:   HCI_bm_alloc
                                                   Segment part 94
    -------------------------------------------------------------------------
<BANKED_CODE,CODE_C> 1 (was BANKED_CODE)
  Relative segment, address: CODE 000044EB - 00004515 (0x2b bytes), align: 0
  Segment part 96.            Intra module refs:   HCI_EXT_ModemTestTxCmd::?relay
           ENTRY                   ADDRESS         REF BY
           =====                   =======         ======
           HCI_EXT_ModemTestTxCmd
                                   000044EB 
               calls direct
               XSTACK = 00000000 ( 0000000C )
               ISTACK = 00000000 ( 00000001 )
    -------------------------------------------------------------------------
<BANKED_CODE,CODE_C> 1 (was BANKED_CODE)
  Relative segment, address: CODE 00004516 - 0000453F (0x2a bytes), align: 0
  Segment part 98.            Intra module refs:   HCI_EXT_ModemHopTestTxCmd::?relay
           ENTRY                   ADDRESS         REF BY
           =====                   =======         ======
           HCI_EXT_ModemHopTestTxCmd
                                   00004516 
               calls direct
               XSTACK = 00000000 ( 00000003 )
               ISTACK = 00000000 ( 00000003 )
    -------------------------------------------------------------------------
<BANKED_CODE,CODE_C> 1 (was BANKED_CODE)
  Relative segment, address: CODE 00004540 - 00004540 (0x1 bytes), align: 0
  Segment part 100.           Intra module refs:   HCI_EXT_ClkDivOnHaltCmd
                                                   HCI_EXT_DeclareNvUsageCmd
                                                   HCI_EXT_EndModemTestCmd
                                                   HCI_EXT_HaltDuringRfCmd
                                                   HCI_EXT_MapPmIoPortCmd
                                                   HCI_EXT_ModemHopTestTxCmd
                                                   HCI_EXT_ModemTestRxCmd
                                                   HCI_EXT_ModemTestTxCmd
                                                   HCI_EXT_SaveFreqTuneCmd
                                                   HCI_EXT_SetBDADDRCmd
                                                   HCI_EXT_SetFreqTuneCmd
                                                   HCI_EXT_SetLocalSupportedFeaturesCmd
                                                   HCI_EXT_SetMaxDtmTxPowerCmd
    -------------------------------------------------------------------------
<BANKED_CODE,CODE_C> 1 (was BANKED_CODE)
  Relative segment, address: CODE 00004541 - 00004546 (0x6 bytes), align: 0
  Segment part 101.           Intra module refs:   HCI_EXT_DecryptCmd
                                                   HCI_LE_TestEndCmd
                                                   LL_EXT_ExtendRfRangeCback
                                                   LL_EXT_SetRxGainCback
                                                   LL_EXT_SetTxPowerCback
                                                   Segment part 100
    -------------------------------------------------------------------------
<BANKED_CODE,CODE_C> 1 (was BANKED_CODE)
  Relative segment, address: CODE 00004547 - 00004571 (0x2b bytes), align: 0
  Segment part 102.           Intra module refs:   HCI_EXT_ModemTestRxCmd::?relay
           ENTRY                   ADDRESS         REF BY
           =====                   =======         ======
           HCI_EXT_ModemTestRxCmd
                                   00004547 
               calls direct
               XSTACK = 00000000 ( 0000000C )
               ISTACK = 00000000 ( 00000001 )
    -------------------------------------------------------------------------
<BANKED_CODE,CODE_C> 1 (was BANKED_CODE)
  Relative segment, address: CODE 00004572 - 0000459B (0x2a bytes), align: 0
  Segment part 104.           Intra module refs:   HCI_EXT_EndModemTestCmd::?relay
           ENTRY                   ADDRESS         REF BY
           =====                   =======         ======
           HCI_EXT_EndModemTestCmd
                                   00004572 
               calls direct
               XSTACK = 00000000 ( 00000003 )
               ISTACK = 00000000 ( 00000003 )
    -------------------------------------------------------------------------
<BANKED_CODE,CODE_C> 1 (was BANKED_CODE)
  Relative segment, address: CODE 0000459C - 000045D8 (0x3d bytes), align: 0
  Segment part 106.           Intra module refs:   HCI_EXT_SetBDADDRCmd::?relay
           ENTRY                   ADDRESS         REF BY
           =====                   =======         ======
           HCI_EXT_SetBDADDRCmd    0000459C 
               calls direct
               XSTACK = 00000000 ( 00000003 )
               ISTACK = 00000000 ( 00000003 )
    -------------------------------------------------------------------------
<BANKED_CODE,CODE_C> 1 (was BANKED_CODE)
  Relative segment, address: CODE 000045D9 - 00004600 (0x28 bytes), align: 0
  Segment part 110.           Intra module refs:   HCI_EXT_SetFreqTuneCmd::?relay
           ENTRY                   ADDRESS         REF BY
           =====                   =======         ======
           HCI_EXT_SetFreqTuneCmd
                                   000045D9 
               calls direct
               XSTACK = 00000000 ( 0000000C )
               ISTACK = 00000000 ( 00000001 )
    -------------------------------------------------------------------------
<BANKED_CODE,CODE_C> 1 (was BANKED_CODE)
  Relative segment, address: CODE 00004601 - 0000460C (0xc bytes), align: 0
  Segment part 112.           Intra module refs:   HCI_EXT_ClkDivOnHaltCmd
                                                   HCI_EXT_DeclareNvUsageCmd
                                                   HCI_EXT_HaltDuringRfCmd
                                                   HCI_EXT_MapPmIoPortCmd
                                                   HCI_EXT_ModemTestRxCmd
                                                   HCI_EXT_ModemTestTxCmd
                                                   HCI_EXT_SetFreqTuneCmd
                                                   HCI_EXT_SetMaxDtmTxPowerCmd
    -------------------------------------------------------------------------
<BANKED_CODE,CODE_C> 1 (was BANKED_CODE)
  Relative segment, address: CODE 0000460D - 00004636 (0x2a bytes), align: 0
  Segment part 113.           Intra module refs:   HCI_EXT_SaveFreqTuneCmd::?relay
           ENTRY                   ADDRESS         REF BY
           =====                   =======         ======
           HCI_EXT_SaveFreqTuneCmd
                                   0000460D 
               calls direct
               XSTACK = 00000000 ( 00000003 )
               ISTACK = 00000000 ( 00000003 )
    -------------------------------------------------------------------------
<BANKED_CODE,CODE_C> 1 (was BANKED_CODE)
  Relative segment, address: CODE 00004637 - 00004660 (0x2a bytes), align: 0
  Segment part 115.           Intra module refs:   HCI_EXT_SetMaxDtmTxPowerCmd::?relay
           ENTRY                   ADDRESS         REF BY
           =====                   =======         ======
           HCI_EXT_SetMaxDtmTxPowerCmd
                                   00004637 
               calls direct
               XSTACK = 00000000 ( 0000000C )
               ISTACK = 00000000 ( 00000001 )
    -------------------------------------------------------------------------
<BANKED_CODE,CODE_C> 1 (was BANKED_CODE)
  Relative segment, address: CODE 00004661 - 0000468B (0x2b bytes), align: 0
  Segment part 117.           Intra module refs:   HCI_EXT_MapPmIoPortCmd::?relay
           ENTRY                   ADDRESS         REF BY
           =====                   =======         ======
           HCI_EXT_MapPmIoPortCmd
                                   00004661 
               calls direct
               XSTACK = 00000000 ( 0000000C )
               ISTACK = 00000000 ( 00000001 )
    -------------------------------------------------------------------------
<BANKED_CODE,CODE_C> 1 (was BANKED_CODE)
  Relative segment, address: CODE 0000468C - 000046D1 (0x46 bytes), align: 0
  Segment part 119.           Intra module refs:   HCI_EXT_ExtendRfRangeCmd::?relay
           ENTRY                   ADDRESS         REF BY
           =====                   =======         ======
           HCI_EXT_ExtendRfRangeCmd
                                   0000468C 
               calls direct
               XSTACK = 00000000 ( 00000004 )
               ISTACK = 00000000 ( 00000003 )
    -------------------------------------------------------------------------
<BANKED_CODE,CODE_C> 1 (was BANKED_CODE)
  Relative segment, address: CODE 000046D2 - 000046FC (0x2b bytes), align: 0
  Segment part 121.           Intra module refs:   HCI_EXT_HaltDuringRfCmd::?relay
           ENTRY                   ADDRESS         REF BY
           =====                   =======         ======
           HCI_EXT_HaltDuringRfCmd
                                   000046D2 
               calls direct
               XSTACK = 00000000 ( 0000000C )
               ISTACK = 00000000 ( 00000001 )
    -------------------------------------------------------------------------
<BANKED_CODE,CODE_C> 1 (was BANKED_CODE)
  Relative segment, address: CODE 000046FD - 0000475C (0x60 bytes), align: 0
  Segment part 125.           Intra module refs:   HCI_EXT_BuildRevisionCmd::?relay
           ENTRY                   ADDRESS         REF BY
           =====                   =======         ======
           HCI_EXT_BuildRevisionCmd
                                   000046FD 
               calls direct
               XSTACK = 00000000 ( 00000010 )
               ISTACK = 00000000 ( 00000001 )
    -------------------------------------------------------------------------
<BANKED_CODE,CODE_C> 1 (was BANKED_CODE)
  Relative segment, address: CODE 0000475D - 0000479F (0x43 bytes), align: 0
  Segment part 127.           Intra module refs:   LL_RandCback::?relay
           ENTRY                   ADDRESS         REF BY
           =====                   =======         ======
           LL_RandCback            0000475D 
               calls direct
               XSTACK = 00000000 ( 00000015 )
    -------------------------------------------------------------------------
<BANKED_CODE,CODE_C> 1 (was BANKED_CODE)
  Relative segment, address: CODE 000047A0 - 000047C1 (0x22 bytes), align: 0
  Segment part 129.           Intra module refs:   LL_EXT_SetRxGainCback::?relay
           ENTRY                   ADDRESS         REF BY
           =====                   =======         ======
           LL_EXT_SetRxGainCback   000047A0 
               calls direct
               XSTACK = 00000000 ( 00000003 )
               ISTACK = 00000000 ( 00000002 )
    -------------------------------------------------------------------------
<BANKED_CODE,CODE_C> 1 (was BANKED_CODE)
  Relative segment, address: CODE 000047C2 - 000047C9 (0x8 bytes), align: 0
  Segment part 131.           Intra module refs:   LL_EXT_ExtendRfRangeCback
                                                   LL_EXT_SetRxGainCback
                                                   LL_EXT_SetTxPowerCback
    -------------------------------------------------------------------------
<BANKED_CODE,CODE_C> 1 (was BANKED_CODE)
  Relative segment, address: CODE 000047CA - 000047EE (0x25 bytes), align: 0
  Segment part 132.           Intra module refs:   LL_EXT_SetTxPowerCback::?relay
           ENTRY                   ADDRESS         REF BY
           =====                   =======         ======
           LL_EXT_SetTxPowerCback
                                   000047CA 
               calls direct
               XSTACK = 00000000 ( 00000003 )
               ISTACK = 00000000 ( 00000002 )
    -------------------------------------------------------------------------
<BANKED_CODE,CODE_C> 1 (was BANKED_CODE)
  Relative segment, address: CODE 000047EF - 00004816 (0x28 bytes), align: 0
  Segment part 136.           Intra module refs:   LL_EXT_ExtendRfRangeCback::?relay
           ENTRY                   ADDRESS         REF BY
           =====                   =======         ======
           LL_EXT_ExtendRfRangeCback
                                   000047EF 
               calls direct
               XSTACK = 00000000 ( 00000003 )
               ISTACK = 00000000 ( 00000002 )
    -------------------------------------------------------------------------
BANK_RELAYS
  Relative segment, address: CODE 00000308 - 0000030D (0x6 bytes), align: 0
  Segment part 12.
           ENTRY                   ADDRESS         REF BY
           =====                   =======         ======
           HCI_bm_alloc::?relay    00000308        hciSerialPacketParser (hci_tl)
    -------------------------------------------------------------------------
BANK_RELAYS
  Relative segment, address: CODE 0000030E - 00000313 (0x6 bytes), align: 0
  Segment part 14.
           ENTRY                   ADDRESS         REF BY
           =====                   =======         ======
           HCI_SetEventMaskCmd::?relay
                                   0000030E        hciSetEventMask (hci_tl)
    -------------------------------------------------------------------------
BANK_RELAYS
  Relative segment, address: CODE 00000314 - 00000319 (0x6 bytes), align: 0
  Segment part 16.
           ENTRY                   ADDRESS         REF BY
           =====                   =======         ======
           HCI_ReadLocalVersionInfoCmd::?relay
                                   00000314        hciReadLocalVersionInfo (hci_tl)
    -------------------------------------------------------------------------
BANK_RELAYS
  Relative segment, address: CODE 0000031A - 0000031F (0x6 bytes), align: 0
  Segment part 18.
           ENTRY                   ADDRESS         REF BY
           =====                   =======         ======
           HCI_ReadLocalSupportedFeaturesCmd::?relay
                                   0000031A        hciReadLocalSupportedFeatures (hci_tl)
    -------------------------------------------------------------------------
BANK_RELAYS
  Relative segment, address: CODE 00000320 - 00000325 (0x6 bytes), align: 0
  Segment part 23.
           ENTRY                   ADDRESS         REF BY
           =====                   =======         ======
           HCI_ReadBDADDRCmd::?relay
                                   00000320        GAP_ParamsInit (gap_configmgr)
                                                   hciReadBDADDR (hci_tl)
    -------------------------------------------------------------------------
BANK_RELAYS
  Relative segment, address: CODE 00000326 - 0000032B (0x6 bytes), align: 0
  Segment part 25.
           ENTRY                   ADDRESS         REF BY
           =====                   =======         ======
           HCI_ReadRssiCmd::?relay
                                   00000326        hciReadRssi (hci_tl)
    -------------------------------------------------------------------------
BANK_RELAYS
  Relative segment, address: CODE 0000032C - 00000331 (0x6 bytes), align: 0
  Segment part 28.
           ENTRY                   ADDRESS         REF BY
           =====                   =======         ======
           HCI_LE_SetEventMaskCmd::?relay
                                   0000032C        hciLESetEventMask (hci_tl)
    -------------------------------------------------------------------------
BANK_RELAYS
  Relative segment, address: CODE 00000332 - 00000337 (0x6 bytes), align: 0
  Segment part 31.
           ENTRY                   ADDRESS         REF BY
           =====                   =======         ======
           HCI_LE_ReadLocalSupportedFeaturesCmd::?relay
                                   00000332        hciLEReadLocalSupportedFeatures (hci_tl)
    -------------------------------------------------------------------------
BANK_RELAYS
  Relative segment, address: CODE 00000338 - 0000033D (0x6 bytes), align: 0
  Segment part 34.
           ENTRY                   ADDRESS         REF BY
           =====                   =======         ======
           HCI_LE_SetRandomAddressCmd::?relay
                                   00000338        hciLESetRandomAddr (hci_tl)
    -------------------------------------------------------------------------
BANK_RELAYS
  Relative segment, address: CODE 0000033E - 00000343 (0x6 bytes), align: 0
  Segment part 36.
           ENTRY                   ADDRESS         REF BY
           =====                   =======         ======
           HCI_LE_SetAdvParamCmd::?relay
                                   0000033E        gapSetAdvParams (gap_peridevmgr)
                                                   hciLESetAdvParam (hci_tl)
    -------------------------------------------------------------------------
BANK_RELAYS
  Relative segment, address: CODE 00000344 - 00000349 (0x6 bytes), align: 0
  Segment part 39.
           ENTRY                   ADDRESS         REF BY
           =====                   =======         ======
           HCI_LE_SetAdvDataCmd::?relay
                                   00000344        GAP_UpdateAdvertisingData (gap_peridevmgr)
                                                   hciLESetAdvData (hci_tl)
    -------------------------------------------------------------------------
BANK_RELAYS
  Relative segment, address: CODE 0000034A - 0000034F (0x6 bytes), align: 0
  Segment part 41.
           ENTRY                   ADDRESS         REF BY
           =====                   =======         ======
           HCI_LE_SetScanRspDataCmd::?relay
                                   0000034A        GAP_UpdateAdvertisingData (gap_peridevmgr)
                                                   hciLESetScanRspData (hci_tl)
    -------------------------------------------------------------------------
BANK_RELAYS
  Relative segment, address: CODE 00000350 - 00000355 (0x6 bytes), align: 0
  Segment part 43.
           ENTRY                   ADDRESS         REF BY
           =====                   =======         ======
           HCI_LE_SetAdvEnableCmd::?relay
                                   00000350        GAP_EndDiscoverable (gap_peridevmgr)
                                                   gapSetAdvParamsStatus (gap_peridevmgr)
                                                   hciLESetAdvEnab (hci_tl)
    -------------------------------------------------------------------------
BANK_RELAYS
  Relative segment, address: CODE 00000356 - 0000035B (0x6 bytes), align: 0
  Segment part 45.
           ENTRY                   ADDRESS         REF BY
           =====                   =======         ======
           HCI_LE_ReadAdvChanTxPowerCmd::?relay
                                   00000356        hciLEReadAdvChanTxPower (hci_tl)
    -------------------------------------------------------------------------
BANK_RELAYS
  Relative segment, address: CODE 0000035C - 00000361 (0x6 bytes), align: 0
  Segment part 51.
           ENTRY                   ADDRESS         REF BY
           =====                   =======         ======
           HCI_LE_ReadWhiteListSizeCmd::?relay
                                   0000035C        hciLEReadWhiteListSize (hci_tl)
    -------------------------------------------------------------------------
BANK_RELAYS
  Relative segment, address: CODE 00000362 - 00000367 (0x6 bytes), align: 0
  Segment part 53.
           ENTRY                   ADDRESS         REF BY
           =====                   =======         ======
           HCI_LE_ClearWhiteListCmd::?relay
                                   00000362        hciLEClearWhiteList (hci_tl)
    -------------------------------------------------------------------------
BANK_RELAYS
  Relative segment, address: CODE 00000368 - 0000036D (0x6 bytes), align: 0
  Segment part 57.
           ENTRY                   ADDRESS         REF BY
           =====                   =======         ======
           HCI_LE_AddWhiteListCmd::?relay
                                   00000368        hciLEAddWhiteList (hci_tl)
    -------------------------------------------------------------------------
BANK_RELAYS
  Relative segment, address: CODE 0000036E - 00000373 (0x6 bytes), align: 0
  Segment part 59.
           ENTRY                   ADDRESS         REF BY
           =====                   =======         ======
           HCI_LE_RemoveWhiteListCmd::?relay
                                   0000036E        hciLERemoveWhiteList (hci_tl)
    -------------------------------------------------------------------------
BANK_RELAYS
  Relative segment, address: CODE 00000374 - 00000379 (0x6 bytes), align: 0
  Segment part 61.
           ENTRY                   ADDRESS         REF BY
           =====                   =======         ======
           HCI_LE_EncryptCmd::?relay
                                   00000374        hciLEEncrypt (hci_tl)
    -------------------------------------------------------------------------
BANK_RELAYS
  Relative segment, address: CODE 0000037A - 0000037F (0x6 bytes), align: 0
  Segment part 64.
           ENTRY                   ADDRESS         REF BY
           =====                   =======         ======
           HCI_LE_RandCmd::?relay
                                   0000037A        hciLERand (hci_tl)
    -------------------------------------------------------------------------
BANK_RELAYS
  Relative segment, address: CODE 00000380 - 00000385 (0x6 bytes), align: 0
  Segment part 66.
           ENTRY                   ADDRESS         REF BY
           =====                   =======         ======
           HCI_LE_ReadSupportedStatesCmd::?relay
                                   00000380        hciLEReadSupportedStates (hci_tl)
    -------------------------------------------------------------------------
BANK_RELAYS
  Relative segment, address: CODE 00000386 - 0000038B (0x6 bytes), align: 0
  Segment part 68.
           ENTRY                   ADDRESS         REF BY
           =====                   =======         ======
           HCI_LE_ReceiverTestCmd::?relay
                                   00000386        hciLEReceiverTest (hci_tl)
    -------------------------------------------------------------------------
BANK_RELAYS
  Relative segment, address: CODE 0000038C - 00000391 (0x6 bytes), align: 0
  Segment part 70.
           ENTRY                   ADDRESS         REF BY
           =====                   =======         ======
           HCI_LE_TransmitterTestCmd::?relay
                                   0000038C        hciLETransmitterTest (hci_tl)
    -------------------------------------------------------------------------
BANK_RELAYS
  Relative segment, address: CODE 00000392 - 00000397 (0x6 bytes), align: 0
  Segment part 72.
           ENTRY                   ADDRESS         REF BY
           =====                   =======         ======
           HCI_LE_TestEndCmd::?relay
                                   00000392        hciLETestEnd (hci_tl)
    -------------------------------------------------------------------------
BANK_RELAYS
  Relative segment, address: CODE 00000398 - 0000039D (0x6 bytes), align: 0
  Segment part 77.
           ENTRY                   ADDRESS         REF BY
           =====                   =======         ======
           HCI_EXT_SetRxGainCmd::?relay
                                   00000398        hciExtSetRxGain (hci_tl)
    -------------------------------------------------------------------------
BANK_RELAYS
  Relative segment, address: CODE 0000039E - 000003A3 (0x6 bytes), align: 0
  Segment part 79.
           ENTRY                   ADDRESS         REF BY
           =====                   =======         ======
           HCI_EXT_SetTxPowerCmd::?relay
                                   0000039E        hciExtSetTxPower (hci_tl)
    -------------------------------------------------------------------------
BANK_RELAYS
  Relative segment, address: CODE 000003A4 - 000003A9 (0x6 bytes), align: 0
  Segment part 86.
           ENTRY                   ADDRESS         REF BY
           =====                   =======         ======
           HCI_EXT_ClkDivOnHaltCmd::?relay
                                   000003A4        hciExtClkDivOnHalt (hci_tl)
    -------------------------------------------------------------------------
BANK_RELAYS
  Relative segment, address: CODE 000003AA - 000003AF (0x6 bytes), align: 0
  Segment part 88.
           ENTRY                   ADDRESS         REF BY
           =====                   =======         ======
           HCI_EXT_DeclareNvUsageCmd::?relay
                                   000003AA        hciExtDeclareNvUsage (hci_tl)
    -------------------------------------------------------------------------
BANK_RELAYS
  Relative segment, address: CODE 000003B0 - 000003B5 (0x6 bytes), align: 0
  Segment part 90.
           ENTRY                   ADDRESS         REF BY
           =====                   =======         ======
           HCI_EXT_DecryptCmd::?relay
                                   000003B0        hciExtDecrypt (hci_tl)
    -------------------------------------------------------------------------
BANK_RELAYS
  Relative segment, address: CODE 000003B6 - 000003BB (0x6 bytes), align: 0
  Segment part 92.
           ENTRY                   ADDRESS         REF BY
           =====                   =======         ======
           HCI_EXT_SetLocalSupportedFeaturesCmd::?relay
                                   000003B6        hciExtSetLocalSupportedFeatures (hci_tl)
    -------------------------------------------------------------------------
BANK_RELAYS
  Relative segment, address: CODE 000003BC - 000003C1 (0x6 bytes), align: 0
  Segment part 97.
           ENTRY                   ADDRESS         REF BY
           =====                   =======         ======
           HCI_EXT_ModemTestTxCmd::?relay
                                   000003BC        hciExtModemTestTx (hci_tl)
    -------------------------------------------------------------------------
BANK_RELAYS
  Relative segment, address: CODE 000003C2 - 000003C7 (0x6 bytes), align: 0
  Segment part 99.
           ENTRY                   ADDRESS         REF BY
           =====                   =======         ======
           HCI_EXT_ModemHopTestTxCmd::?relay
                                   000003C2        hciExtModemHopTestTx (hci_tl)
    -------------------------------------------------------------------------
BANK_RELAYS
  Relative segment, address: CODE 000003C8 - 000003CD (0x6 bytes), align: 0
  Segment part 103.
           ENTRY                   ADDRESS         REF BY
           =====                   =======         ======
           HCI_EXT_ModemTestRxCmd::?relay
                                   000003C8        hciExtModemtestRx (hci_tl)
    -------------------------------------------------------------------------
BANK_RELAYS
  Relative segment, address: CODE 000003CE - 000003D3 (0x6 bytes), align: 0
  Segment part 105.
           ENTRY                   ADDRESS         REF BY
           =====                   =======         ======
           HCI_EXT_EndModemTestCmd::?relay
                                   000003CE        hciExtEndModemTest (hci_tl)
    -------------------------------------------------------------------------
BANK_RELAYS
  Relative segment, address: CODE 000003D4 - 000003D9 (0x6 bytes), align: 0
  Segment part 107.
           ENTRY                   ADDRESS         REF BY
           =====                   =======         ======
           HCI_EXT_SetBDADDRCmd::?relay
                                   000003D4        hciExtSetBDADDR (hci_tl)
    -------------------------------------------------------------------------
BANK_RELAYS
  Relative segment, address: CODE 000003DA - 000003DF (0x6 bytes), align: 0
  Segment part 111.
           ENTRY                   ADDRESS         REF BY
           =====                   =======         ======
           HCI_EXT_SetFreqTuneCmd::?relay
                                   000003DA        hciExtSetFreqTune (hci_tl)
    -------------------------------------------------------------------------
BANK_RELAYS
  Relative segment, address: CODE 000003E0 - 000003E5 (0x6 bytes), align: 0
  Segment part 114.
           ENTRY                   ADDRESS         REF BY
           =====                   =======         ======
           HCI_EXT_SaveFreqTuneCmd::?relay
                                   000003E0        hciExtSaveFreqTune (hci_tl)
    -------------------------------------------------------------------------
BANK_RELAYS
  Relative segment, address: CODE 000003E6 - 000003EB (0x6 bytes), align: 0
  Segment part 116.
           ENTRY                   ADDRESS         REF BY
           =====                   =======         ======
           HCI_EXT_SetMaxDtmTxPowerCmd::?relay
                                   000003E6        hciExtSetMaxDtmTxPower (hci_tl)
    -------------------------------------------------------------------------
BANK_RELAYS
  Relative segment, address: CODE 000003EC - 000003F1 (0x6 bytes), align: 0
  Segment part 118.
           ENTRY                   ADDRESS         REF BY
           =====                   =======         ======
           HCI_EXT_MapPmIoPortCmd::?relay
                                   000003EC        hciExtMapPmIoPort (hci_tl)
    -------------------------------------------------------------------------
BANK_RELAYS
  Relative segment, address: CODE 000003F2 - 000003F7 (0x6 bytes), align: 0
  Segment part 120.
           ENTRY                   ADDRESS         REF BY
           =====                   =======         ======
           HCI_EXT_ExtendRfRangeCmd::?relay
                                   000003F2        hciExtExtendRfRange (hci_tl)
    -------------------------------------------------------------------------
BANK_RELAYS
  Relative segment, address: CODE 000003F8 - 000003FD (0x6 bytes), align: 0
  Segment part 122.
           ENTRY                   ADDRESS         REF BY
           =====                   =======         ======
           HCI_EXT_HaltDuringRfCmd::?relay
                                   000003F8        hciExtHaltDuringRf (hci_tl)
    -------------------------------------------------------------------------
BANK_RELAYS
  Relative segment, address: CODE 000003FE - 00000403 (0x6 bytes), align: 0
  Segment part 126.
           ENTRY                   ADDRESS         REF BY
           =====                   =======         ======
           HCI_EXT_BuildRevisionCmd::?relay
                                   000003FE        hciExtBuildRevision (hci_tl)
    -------------------------------------------------------------------------
BANK_RELAYS
  Relative segment, address: CODE 00000404 - 00000409 (0x6 bytes), align: 0
  Segment part 128.
           ENTRY                   ADDRESS         REF BY
           =====                   =======         ======
           LL_RandCback::?relay    00000404        llProcessPostRfOps (ll_common)
    -------------------------------------------------------------------------
BANK_RELAYS
  Relative segment, address: CODE 0000040A - 0000040F (0x6 bytes), align: 0
  Segment part 130.
           ENTRY                   ADDRESS         REF BY
           =====                   =======         ======
           LL_EXT_SetRxGainCback::?relay
                                   0000040A        llProcessPostRfOps (ll_common)
    -------------------------------------------------------------------------
BANK_RELAYS
  Relative segment, address: CODE 00000410 - 00000415 (0x6 bytes), align: 0
  Segment part 133.
           ENTRY                   ADDRESS         REF BY
           =====                   =======         ======
           LL_EXT_SetTxPowerCback::?relay
                                   00000410        llProcessPostRfOps (ll_common)
    -------------------------------------------------------------------------
BANK_RELAYS
  Relative segment, address: CODE 00000416 - 0000041B (0x6 bytes), align: 0
  Segment part 137.
           ENTRY                   ADDRESS         REF BY
           =====                   =======         ======
           LL_EXT_ExtendRfRangeCback::?relay
                                   00000416        llProcessPostRfOps (ll_common)
    -------------------------------------------------------------------------
<XDATA_ROM_C> 1 (was XDATA_ROM_C)
  Relative segment, address: CONST 00008F7C - 00008F84 (0x9 bytes), align: 0
  Segment part 6.             Intra module refs:   HCI_ReadLocalSupportedFeaturesCmd
    -------------------------------------------------------------------------
<XDATA_ROM_C> 1 (was XDATA_ROM_C)
  Relative segment, address: CONST 00008F85 - 00008F8D (0x9 bytes), align: 0
  Segment part 7.             Intra module refs:   HCI_LE_ReadSupportedStatesCmd
    -------------------------------------------------------------------------
<BANKED_CODE,XDATA_ROM_C_FLASH> 1 (was XDATA_ROM_C_FLASH)
  Relative segment, address: CODE 00008F7C - 00008F84 (0x9 bytes), align: 0
  Segment part 138.           Intra module refs:   Segment part 6
    -------------------------------------------------------------------------
<BANKED_CODE,XDATA_ROM_C_FLASH> 1 (was XDATA_ROM_C_FLASH)
  Relative segment, address: CODE 00008F85 - 00008F8D (0x9 bytes), align: 0
  Segment part 139.           Intra module refs:   Segment part 7

    -------------------------------------------------------------------------
  LIBRARY MODULE, NAME : hci_data

  SEGMENTS IN THE MODULE
  ======================
<BANKED_CODE,XDATA_ROM_C_FLASH> 1 (was BANKED_CODE)
  Relative segment, address: CODE 0000C596 - 0000C5E9 (0x54 bytes), align: 0
  Segment part 6.             Intra module refs:   HCI_ReverseBytes::?relay
           ENTRY                   ADDRESS         REF BY
           =====                   =======         ======
           HCI_ReverseBytes        0000C596 
               XSTACK = 00000000 ( 0000000C )
               ISTACK = 00000000 ( 00000001 )
    -------------------------------------------------------------------------
BANK_RELAYS
  Relative segment, address: CODE 0000041C - 00000421 (0x6 bytes), align: 0
  Segment part 7.
           ENTRY                   ADDRESS         REF BY
           =====                   =======         ======
           HCI_ReverseBytes::?relay
                                   0000041C        HCI_EXT_DecryptCmd (hci)
                                                   HCI_LE_EncryptCmd (hci)
                                                   hciExtDecrypt (hci_tl)
                                                   hciLEEncrypt (hci_tl)

    -------------------------------------------------------------------------
  LIBRARY MODULE, NAME : hci_event

  SEGMENTS IN THE MODULE
  ======================
XDATA_Z
  Relative segment, address: XDATA 000002E2 - 000002E2 (0x1 bytes), align: 0
  Segment part 6.
           ENTRY                   ADDRESS         REF BY
           =====                   =======         ======
           bleEvtMask              000002E2        HCI_LE_SetEventMaskCmd (hci)
                                                   hciInitEventMasks (hci_event_PATCH)
    -------------------------------------------------------------------------
XDATA_Z
  Relative segment, address: XDATA 000002E3 - 000002EA (0x8 bytes), align: 0
  Segment part 7.
           ENTRY                   ADDRESS         REF BY
           =====                   =======         ======
           pHciEvtMask             000002E3        HCI_SetEventMaskCmd (hci)
                                                   hciInitEventMasks (hci_event_PATCH)
    -------------------------------------------------------------------------
<BANKED_CODE,XDATA_ROM_C_FLASH> 1 (was BANKED_CODE)
  Relative segment, address: CODE 0000AE53 - 0000AF35 (0xe3 bytes), align: 0
  Segment part 8.             Intra module refs:   HCI_CommandCompleteEvent::?relay
           ENTRY                   ADDRESS         REF BY
           =====                   =======         ======
           HCI_CommandCompleteEvent
                                   0000AE53 
               calls direct
               XSTACK = 00000003 ( 00000014 )
    -------------------------------------------------------------------------
<BANKED_CODE,XDATA_ROM_C_FLASH> 1 (was BANKED_CODE)
  Relative segment, address: CODE 0000AF36 - 0000B050 (0x11b bytes), align: 0
  Segment part 16.            Intra module refs:   HCI_SendCommandCompleteEvent::?relay
           ENTRY                   ADDRESS         REF BY
           =====                   =======         ======
           HCI_SendCommandCompleteEvent
                                   0000AF36 
               calls direct
               XSTACK = 00000014 ( 00000010 )
               ISTACK = 00000000 ( 00000001 )
    -------------------------------------------------------------------------
<BANKED_CODE,XDATA_ROM_C_FLASH> 1 (was BANKED_CODE)
  Relative segment, address: CODE 0000B051 - 0000B055 (0x5 bytes), align: 0
  Segment part 18.            Intra module refs:   HCI_SendCommandCompleteEvent
    -------------------------------------------------------------------------
<BANKED_CODE,XDATA_ROM_C_FLASH> 1 (was BANKED_CODE)
  Relative segment, address: CODE 0000B056 - 0000B06C (0x17 bytes), align: 0
  Segment part 21.            Intra module refs:   HCI_SendCommandCompleteEvent
    -------------------------------------------------------------------------
<BANKED_CODE,XDATA_ROM_C_FLASH> 1 (was BANKED_CODE)
  Relative segment, address: CODE 0000B06D - 0000B071 (0x5 bytes), align: 0
  Segment part 22.            Intra module refs:   Segment part 21
    -------------------------------------------------------------------------
<BANKED_CODE,XDATA_ROM_C_FLASH> 1 (was BANKED_CODE)
  Relative segment, address: CODE 0000B072 - 0000B075 (0x4 bytes), align: 0
  Segment part 27.            Intra module refs:   HCI_SendCommandCompleteEvent
    -------------------------------------------------------------------------
<BANKED_CODE,XDATA_ROM_C_FLASH> 1 (was BANKED_CODE)
  Relative segment, address: CODE 0000B076 - 0000B079 (0x4 bytes), align: 0
  Segment part 28.            Intra module refs:   Segment part 27
                                                   Segment part 40
    -------------------------------------------------------------------------
<BANKED_CODE,XDATA_ROM_C_FLASH> 1 (was BANKED_CODE)
  Relative segment, address: CODE 0000B07A - 0000B080 (0x7 bytes), align: 0
  Segment part 29.            Intra module refs:   Segment part 28
                                                   Segment part 73
    -------------------------------------------------------------------------
<BANKED_CODE,XDATA_ROM_C_FLASH> 1 (was BANKED_CODE)
  Relative segment, address: CODE 0000B081 - 0000B086 (0x6 bytes), align: 0
  Segment part 38.            Intra module refs:   HCI_SendCommandCompleteEvent
    -------------------------------------------------------------------------
<BANKED_CODE,XDATA_ROM_C_FLASH> 1 (was BANKED_CODE)
  Relative segment, address: CODE 0000B087 - 0000B08D (0x7 bytes), align: 0
  Segment part 40.            Intra module refs:   HCI_SendCommandCompleteEvent
    -------------------------------------------------------------------------
<BANKED_CODE,XDATA_ROM_C_FLASH> 1 (was BANKED_CODE)
  Relative segment, address: CODE 0000B08E - 0000B094 (0x7 bytes), align: 0
  Segment part 42.            Intra module refs:   Segment part 21
    -------------------------------------------------------------------------
<BANKED_CODE,XDATA_ROM_C_FLASH> 1 (was BANKED_CODE)
  Relative segment, address: CODE 0000B095 - 0000B098 (0x4 bytes), align: 0
  Segment part 43.            Intra module refs:   Segment part 22
                                                   Segment part 42
    -------------------------------------------------------------------------
<BANKED_CODE,XDATA_ROM_C_FLASH> 1 (was BANKED_CODE)
  Relative segment, address: CODE 0000B099 - 0000B0A1 (0x9 bytes), align: 0
  Segment part 44.            Intra module refs:   Segment part 29
                                                   Segment part 43
    -------------------------------------------------------------------------
<BANKED_CODE,XDATA_ROM_C_FLASH> 1 (was BANKED_CODE)
  Relative segment, address: CODE 0000B0A2 - 0000B0AD (0xc bytes), align: 0
  Segment part 45.            Intra module refs:   HCI_SendCommandCompleteEvent
    -------------------------------------------------------------------------
<BANKED_CODE,XDATA_ROM_C_FLASH> 1 (was BANKED_CODE)
  Relative segment, address: CODE 0000B0AE - 0000B0B9 (0xc bytes), align: 0
  Segment part 46.            Intra module refs:   HCI_SendCommandCompleteEvent
    -------------------------------------------------------------------------
<BANKED_CODE,XDATA_ROM_C_FLASH> 1 (was BANKED_CODE)
  Relative segment, address: CODE 0000B0BA - 0000B0BB (0x2 bytes), align: 0
  Segment part 50.            Intra module refs:   HCI_SendCommandCompleteEvent
    -------------------------------------------------------------------------
<BANKED_CODE,XDATA_ROM_C_FLASH> 1 (was BANKED_CODE)
  Relative segment, address: CODE 0000B0BC - 0000B0BF (0x4 bytes), align: 0
  Segment part 51.            Intra module refs:   HCI_SendCommandCompleteEvent
                                                   Segment part 50
    -------------------------------------------------------------------------
<BANKED_CODE,XDATA_ROM_C_FLASH> 1 (was BANKED_CODE)
  Relative segment, address: CODE 0000B0C0 - 0000B0C5 (0x6 bytes), align: 0
  Segment part 52.            Intra module refs:   Segment part 21
                                                   Segment part 51
    -------------------------------------------------------------------------
<BANKED_CODE,XDATA_ROM_C_FLASH> 1 (was BANKED_CODE)
  Relative segment, address: CODE 0000B0C6 - 0000B0CB (0x6 bytes), align: 0
  Segment part 69.            Intra module refs:   Segment part 45
                                                   Segment part 46
    -------------------------------------------------------------------------
<BANKED_CODE,XDATA_ROM_C_FLASH> 1 (was BANKED_CODE)
  Relative segment, address: CODE 0000B0CC - 0000B0CF (0x4 bytes), align: 0
  Segment part 71.            Intra module refs:   HCI_SendCommandCompleteEvent
    -------------------------------------------------------------------------
<BANKED_CODE,XDATA_ROM_C_FLASH> 1 (was BANKED_CODE)
  Relative segment, address: CODE 0000B0D0 - 0000B0D3 (0x4 bytes), align: 0
  Segment part 72.            Intra module refs:   Segment part 71
    -------------------------------------------------------------------------
<BANKED_CODE,XDATA_ROM_C_FLASH> 1 (was BANKED_CODE)
  Relative segment, address: CODE 0000B0D4 - 0000B0D8 (0x5 bytes), align: 0
  Segment part 73.            Intra module refs:   Segment part 72
                                                   Segment part 75
    -------------------------------------------------------------------------
<BANKED_CODE,XDATA_ROM_C_FLASH> 1 (was BANKED_CODE)
  Relative segment, address: CODE 0000B0D9 - 0000B0DC (0x4 bytes), align: 0
  Segment part 74.            Intra module refs:   HCI_SendCommandCompleteEvent
    -------------------------------------------------------------------------
<BANKED_CODE,XDATA_ROM_C_FLASH> 1 (was BANKED_CODE)
  Relative segment, address: CODE 0000B0DD - 0000B0E1 (0x5 bytes), align: 0
  Segment part 75.            Intra module refs:   Segment part 74
    -------------------------------------------------------------------------
<BANKED_CODE,XDATA_ROM_C_FLASH> 1 (was BANKED_CODE)
  Relative segment, address: CODE 0000B0E2 - 0000B0E9 (0x8 bytes), align: 0
  Segment part 78.            Intra module refs:   HCI_CommandCompleteEvent
                                                   Segment part 79
    -------------------------------------------------------------------------
<BANKED_CODE,XDATA_ROM_C_FLASH> 1 (was BANKED_CODE)
  Relative segment, address: CODE 0000B0EA - 0000B0EE (0x5 bytes), align: 0
  Segment part 79.            Intra module refs:   HCI_CommandCompleteEvent
    -------------------------------------------------------------------------
<BANKED_CODE,XDATA_ROM_C_FLASH> 1 (was BANKED_CODE)
  Relative segment, address: CODE 0000B0EF - 0000B126 (0x38 bytes), align: 0
  Segment part 80.            Intra module refs:   LL_DirectTestEndDoneCback::?relay
           ENTRY                   ADDRESS         REF BY
           =====                   =======         ======
           LL_DirectTestEndDoneCback
                                   0000B0EF 
               calls direct
               XSTACK = 00000000 ( 00000003 )
               ISTACK = 00000000 ( 00000003 )
    -------------------------------------------------------------------------
BANK_RELAYS
  Relative segment, address: CODE 00000422 - 00000427 (0x6 bytes), align: 0
  Segment part 9.             Intra module refs:   LL_DirectTestEndDoneCback
           ENTRY                   ADDRESS         REF BY
           =====                   =======         ======
           HCI_CommandCompleteEvent::?relay
                                   00000422        HCI_LE_EncryptCmd (hci)
                                                   HCI_LE_RandCmd (hci)
                                                   HCI_LE_ReadBufSizeCmd (hci_PATCH)
                                                   HCI_LE_TestEndCmd (hci)
                                                   HCI_ReadBDADDRCmd (hci)
                                                   HCI_ReadLocalSupportedCommandsCmd (hci_PATCH)
                                                   HCI_ReadLocalVersionInfoCmd (hci)
                                                   HCI_ReadRssiCmd (hci)
                                                   HCI_ResetCmd (hci_PATCH)
                                                   HCI_SetEventMaskCmd (hci)
                                                   HCI_SetEventMaskPage2Cmd (hci_PATCH)
                                                   LL_RandCback (hci)
                                                   Segment part 20 (hci)
                                                   Segment part 46 (hci)
                                                   Segment part 82 (hci)
                                                   Segment part 93 (hci)
                                                   hciProcessHostToCtrlCmd (hci_tl)
    -------------------------------------------------------------------------
BANK_RELAYS
  Relative segment, address: CODE 00000428 - 0000042D (0x6 bytes), align: 0
  Segment part 17.            Intra module refs:   HCI_CommandCompleteEvent
           ENTRY                   ADDRESS         REF BY
           =====                   =======         ======
           HCI_SendCommandCompleteEvent::?relay
                                   00000428        HCI_VendorSpecifcCommandCompleteEvent (hci_event_PATCH)
    -------------------------------------------------------------------------
BANK_RELAYS
  Relative segment, address: CODE 0000042E - 00000433 (0x6 bytes), align: 0
  Segment part 81.
           ENTRY                   ADDRESS         REF BY
           =====                   =======         ======
           LL_DirectTestEndDoneCback::?relay
                                   0000042E        LL_DirectTestEnd (ll)

    -------------------------------------------------------------------------
  LIBRARY MODULE, NAME : hci_event_PATCH

  SEGMENTS IN THE MODULE
  ======================
XDATA_Z
  Relative segment, address: XDATA 000002EB - 000002F2 (0x8 bytes), align: 0
  Segment part 6.             Intra module refs:   hciInitEventMasks
           ENTRY                   ADDRESS         REF BY
           =====                   =======         ======
           pHciEvtMask2            000002EB        HCI_SetEventMaskPage2Cmd (hci_PATCH)
    -------------------------------------------------------------------------
<BANKED_CODE,XDATA_ROM_C_FLASH> 1 (was BANKED_CODE)
  Relative segment, address: CODE 0000BF16 - 0000BF58 (0x43 bytes), align: 0
  Segment part 7.             Intra module refs:   hciInitEventMasks::?relay
           ENTRY                   ADDRESS         REF BY
           =====                   =======         ======
           hciInitEventMasks       0000BF16 
               ISTACK = 00000000 ( 00000002 )
    -------------------------------------------------------------------------
<BANKED_CODE,XDATA_ROM_C_FLASH> 1 (was BANKED_CODE)
  Relative segment, address: CODE 0000BF59 - 0000C010 (0xb8 bytes), align: 0
  Segment part 21.            Intra module refs:   HCI_VendorSpecifcCommandCompleteEvent::?relay
           ENTRY                   ADDRESS         REF BY
           =====                   =======         ======
           HCI_VendorSpecifcCommandCompleteEvent
                                   0000BF59 
               calls direct
               XSTACK = 00000000 ( 00000014 )
               ISTACK = 00000000 ( 00000001 )
    -------------------------------------------------------------------------
BANK_RELAYS
  Relative segment, address: CODE 00000434 - 00000439 (0x6 bytes), align: 0
  Segment part 8.
           ENTRY                   ADDRESS         REF BY
           =====                   =======         ======
           hciInitEventMasks::?relay
                                   00000434        HCI_Init (hci_tl)
                                                   HCI_ResetCmd (hci_PATCH)
    -------------------------------------------------------------------------
BANK_RELAYS
  Relative segment, address: CODE 0000043A - 0000043F (0x6 bytes), align: 0
  Segment part 22.
           ENTRY                   ADDRESS         REF BY
           =====                   =======         ======
           HCI_VendorSpecifcCommandCompleteEvent::?relay
                                   0000043A        HCI_EXT_BuildRevisionCmd (hci)
                                                   HCI_EXT_DecryptCmd (hci)
                                                   HCI_EXT_DelaySleepCmd (hci_PATCH)
                                                   HCI_EXT_ExtendRfRangeCmd (hci)
                                                   HCI_EXT_ResetSystemCmd (hci_PATCH)
                                                   HCI_EXT_SetBDADDRCmd (hci)
                                                   HCI_EXT_SetRxGainCmd (hci)
                                                   HCI_EXT_SetTxPowerCmd (hci)
                                                   Segment part 112 (hci)
                                                   Segment part 131 (hci)
                                                   Segment part 73 (hci)

    -------------------------------------------------------------------------
  LIBRARY MODULE, NAME : hci_PATCH

  SEGMENTS IN THE MODULE
  ======================
<XDATA_ROM_C> 1 (was XDATA_ROM_C)
  Relative segment, address: CONST 00008EBE - 00008EFE (0x41 bytes), align: 0
  Segment part 6.             Intra module refs:   HCI_ReadLocalSupportedCommandsCmd
           ENTRY                   ADDRESS         REF BY
           =====                   =======         ======
           supportedCmdsTable      00008EBE 
    -------------------------------------------------------------------------
<BANKED_CODE,XDATA_ROM_C_FLASH> 1 (was BANKED_CODE)
  Relative segment, address: CODE 0000BB68 - 0000BB9B (0x34 bytes), align: 0
  Segment part 10.            Intra module refs:   HCI_ResetCmd::?relay
           ENTRY                   ADDRESS         REF BY
           =====                   =======         ======
           HCI_ResetCmd            0000BB68 
               calls direct
               XSTACK = 00000000 ( 00000001 )
               ISTACK = 00000000 ( 00000003 )
    -------------------------------------------------------------------------
<BANKED_CODE,XDATA_ROM_C_FLASH> 1 (was BANKED_CODE)
  Relative segment, address: CODE 0000BB9C - 0000BBB1 (0x16 bytes), align: 0
  Segment part 12.            Intra module refs:   HCI_ReadLocalSupportedCommandsCmd::?relay
           ENTRY                   ADDRESS         REF BY
           =====                   =======         ======
           HCI_ReadLocalSupportedCommandsCmd
                                   0000BB9C 
               calls direct
               ISTACK = 00000000 ( 00000002 )
    -------------------------------------------------------------------------
<BANKED_CODE,XDATA_ROM_C_FLASH> 1 (was BANKED_CODE)
  Relative segment, address: CODE 0000BBB2 - 0000BBE8 (0x37 bytes), align: 0
  Segment part 14.            Intra module refs:   HCI_LE_ReadBufSizeCmd::?relay
           ENTRY                   ADDRESS         REF BY
           =====                   =======         ======
           HCI_LE_ReadBufSizeCmd   0000BBB2 
               calls direct
               XSTACK = 00000000 ( 00000004 )
               ISTACK = 00000000 ( 00000002 )
    -------------------------------------------------------------------------
<BANKED_CODE,XDATA_ROM_C_FLASH> 1 (was BANKED_CODE)
  Relative segment, address: CODE 0000BBE9 - 0000BC3A (0x52 bytes), align: 0
  Segment part 16.            Intra module refs:   HCI_SetEventMaskPage2Cmd::?relay
           ENTRY                   ADDRESS         REF BY
           =====                   =======         ======
           HCI_SetEventMaskPage2Cmd
                                   0000BBE9 
               calls direct
               XSTACK = 00000000 ( 0000000D )
    -------------------------------------------------------------------------
<BANKED_CODE,XDATA_ROM_C_FLASH> 1 (was BANKED_CODE)
  Relative segment, address: CODE 0000BC3B - 0000BC76 (0x3c bytes), align: 0
  Segment part 18.            Intra module refs:   HCI_EXT_ResetSystemCmd::?relay
           ENTRY                   ADDRESS         REF BY
           =====                   =======         ======
           HCI_EXT_ResetSystemCmd
                                   0000BC3B 
               calls direct
               XSTACK = 00000000 ( 0000000C )
               ISTACK = 00000000 ( 00000001 )
    -------------------------------------------------------------------------
<BANKED_CODE,XDATA_ROM_C_FLASH> 1 (was BANKED_CODE)
  Relative segment, address: CODE 0000BC77 - 0000BC78 (0x2 bytes), align: 0
  Segment part 20.            Intra module refs:   HCI_EXT_DelaySleepCmd
                                                   HCI_LE_ReadBufSizeCmd
    -------------------------------------------------------------------------
<BANKED_CODE,XDATA_ROM_C_FLASH> 1 (was BANKED_CODE)
  Relative segment, address: CODE 0000BC79 - 0000BC7E (0x6 bytes), align: 0
  Segment part 21.            Intra module refs:   HCI_EXT_ResetSystemCmd
                                                   HCI_ResetCmd
                                                   HCI_SetEventMaskPage2Cmd
                                                   Segment part 20
    -------------------------------------------------------------------------
<BANKED_CODE,XDATA_ROM_C_FLASH> 1 (was BANKED_CODE)
  Relative segment, address: CODE 0000BC7F - 0000BCAD (0x2f bytes), align: 0
  Segment part 22.            Intra module refs:   HCI_EXT_DelaySleepCmd::?relay
           ENTRY                   ADDRESS         REF BY
           =====                   =======         ======
           HCI_EXT_DelaySleepCmd   0000BC7F 
               calls direct
               XSTACK = 00000000 ( 00000003 )
               ISTACK = 00000000 ( 00000002 )
    -------------------------------------------------------------------------
<BANKED_CODE,XDATA_ROM_C_FLASH> 1 (was BANKED_CODE)
  Relative segment, address: CODE 0000BCAE - 0000BCB0 (0x3 bytes), align: 0
  Segment part 24.            Intra module refs:   HCI_EXT_DelaySleepCmd
                                                   HCI_LE_ReadBufSizeCmd
                                                   HCI_ResetCmd
    -------------------------------------------------------------------------
<BANKED_CODE,XDATA_ROM_C_FLASH> 1 (was BANKED_CODE)
  Relative segment, address: CODE 0000BCB1 - 0000BCB7 (0x7 bytes), align: 0
  Segment part 25.            Intra module refs:   HCI_ReadLocalSupportedCommandsCmd
                                                   Segment part 24
    -------------------------------------------------------------------------
BANK_RELAYS
  Relative segment, address: CODE 00000440 - 00000445 (0x6 bytes), align: 0
  Segment part 11.
           ENTRY                   ADDRESS         REF BY
           =====                   =======         ======
           HCI_ResetCmd::?relay    00000440        hciReset (hci_tl)
    -------------------------------------------------------------------------
BANK_RELAYS
  Relative segment, address: CODE 00000446 - 0000044B (0x6 bytes), align: 0
  Segment part 13.
           ENTRY                   ADDRESS         REF BY
           =====                   =======         ======
           HCI_ReadLocalSupportedCommandsCmd::?relay
                                   00000446        hciReadLocalSupportedCommands (hci_tl)
    -------------------------------------------------------------------------
BANK_RELAYS
  Relative segment, address: CODE 0000044C - 00000451 (0x6 bytes), align: 0
  Segment part 15.
           ENTRY                   ADDRESS         REF BY
           =====                   =======         ======
           HCI_LE_ReadBufSizeCmd::?relay
                                   0000044C        gapReadBD_ADDRStatus (gap_configmgr)
                                                   hciLEReadBufSize (hci_tl)
    -------------------------------------------------------------------------
BANK_RELAYS
  Relative segment, address: CODE 00000452 - 00000457 (0x6 bytes), align: 0
  Segment part 17.
           ENTRY                   ADDRESS         REF BY
           =====                   =======         ======
           HCI_SetEventMaskPage2Cmd::?relay
                                   00000452        hciSetEventMaskPage2 (hci_tl)
    -------------------------------------------------------------------------
BANK_RELAYS
  Relative segment, address: CODE 00000458 - 0000045D (0x6 bytes), align: 0
  Segment part 19.
           ENTRY                   ADDRESS         REF BY
           =====                   =======         ======
           HCI_EXT_ResetSystemCmd::?relay
                                   00000458        hciExtResetSystem (hci_tl)
    -------------------------------------------------------------------------
BANK_RELAYS
  Relative segment, address: CODE 0000045E - 00000463 (0x6 bytes), align: 0
  Segment part 23.
           ENTRY                   ADDRESS         REF BY
           =====                   =======         ======
           HCI_EXT_DelaySleepCmd::?relay
                                   0000045E        hciExtDelaySleep (hci_tl)
    -------------------------------------------------------------------------
<BANKED_CODE,XDATA_ROM_C_FLASH> 1 (was XDATA_ROM_C_FLASH)
  Relative segment, address: CODE 00008EBE - 00008EFE (0x41 bytes), align: 0
  Segment part 26.            Intra module refs:   supportedCmdsTable

    -------------------------------------------------------------------------
  LIBRARY MODULE, NAME : ll

  SEGMENTS IN THE MODULE
  ======================
SFR_AN
  Relative segment, address: DATA 0000008D - 0000008D (0x1 bytes), align: 0
  Segment part 1. ROOT        Intra module refs:   LL_EXT_MapPmIoPort
           ENTRY                   ADDRESS         REF BY
           =====                   =======         ======
           P1IEN                   0000008D 
    -------------------------------------------------------------------------
SFR_AN
  Relative segment, address: DATA 000000AB - 000000AB (0x1 bytes), align: 0
  Segment part 4. ROOT        Intra module refs:   LL_EXT_MapPmIoPort
           ENTRY                   ADDRESS         REF BY
           =====                   =======         ======
           P0IEN                   000000AB 
    -------------------------------------------------------------------------
SFR_AN
  Relative segment, address: DATA 000000AE - 000000AE (0x1 bytes), align: 0
  Segment part 6. ROOT        Intra module refs:   LL_EXT_MapPmIoPort
           ENTRY                   ADDRESS         REF BY
           =====                   =======         ======
           PMUX                    000000AE 
    -------------------------------------------------------------------------
SFR_AN
  Relative segment, address: DATA 000000C9 - 000000C9 (0x1 bytes), align: 0
  Segment part 8. ROOT        Intra module refs:   LL_ProcessEvent
           ENTRY                   ADDRESS         REF BY
           =====                   =======         ======
           WDCTL                   000000C9 
    -------------------------------------------------------------------------
SFR_AN
  Relative segment, address: DATA 000000F2 - 000000F2 (0x1 bytes), align: 0
  Segment part 9. ROOT        Intra module refs:   LL_EXT_MapPmIoPort
           ENTRY                   ADDRESS         REF BY
           =====                   =======         ======
           APCFG                   000000F2 
    -------------------------------------------------------------------------
SFR_AN
  Relative segment, address: DATA 000000F3 - 000000F3 (0x1 bytes), align: 0
  Segment part 10. ROOT       Intra module refs:   LL_EXT_MapPmIoPort
           ENTRY                   ADDRESS         REF BY
           =====                   =======         ======
           P0SEL                   000000F3 
    -------------------------------------------------------------------------
SFR_AN
  Relative segment, address: DATA 000000F5 - 000000F5 (0x1 bytes), align: 0
  Segment part 12. ROOT       Intra module refs:   LL_EXT_MapPmIoPort
           ENTRY                   ADDRESS         REF BY
           =====                   =======         ======
           P2SEL                   000000F5 
    -------------------------------------------------------------------------
SFR_AN
  Relative segment, address: DATA 000000FF - 000000FF (0x1 bytes), align: 0
  Segment part 15. ROOT       Intra module refs:   LL_EXT_MapPmIoPort
           ENTRY                   ADDRESS         REF BY
           =====                   =======         ======
           P2DIR                   000000FF 
    -------------------------------------------------------------------------
SFR_AN
  Relative segment, address: DATA 000000D9 - 000000D9 (0x1 bytes), align: 0
  Segment part 17. ROOT       Intra module refs:   LL_DirectTestTxTest
                                                   LL_EXT_ModemHopTestTx
                                                   llDiscoverableAdvEvt_TaskEndOk (ll_advEndCauses)
                                                   llNonConnAdvEvt_TaskEndOk (ll_advEndCauses)
                                                   llSetupNonConnectableAdvEvt (ll_common)
                                                   llSetupScannableAdvEvt (ll_common)
           ENTRY                   ADDRESS         REF BY
           =====                   =======         ======
           RFD                     000000D9 
    -------------------------------------------------------------------------
SFR_AN
  Relative segment, address: DATA 000000E1 - 000000E1 (0x1 bytes), align: 0
  Segment part 18. ROOT       Intra module refs:   LL_DirectTestEnd
                                                   LL_DirectTestRxTest
                                                   LL_DirectTestTxTest
                                                   LL_ENC_GenerateTrueRandNum (ll_enc)
                                                   LL_EXT_ModemHopTestTx
                                                   LL_EXT_ModemTestRx
                                                   LL_EXT_ModemTestTx
                                                   LL_Reset
                                                   LL_SetAdvControl
                                                   PHY_Command (phy)
                                                   llAdvEvt_TaskAbort (ll_advEndCauses)
                                                   llDiscoverableAdvEvt_TaskEndOk (ll_advEndCauses)
                                                   llNonConnAdvEvt_TaskEndOk (ll_advEndCauses)
                                                   llScheduleTask (ll_scheduler)
                                                   llSetupAdv (ll_common)
                                                   llSetupNonConnectableAdvEvt (ll_common)
                                                   llSetupScannableAdvEvt (ll_common)
           ENTRY                   ADDRESS         REF BY
           =====                   =======         ======
           RFST                    000000E1 
    -------------------------------------------------------------------------
XDATA_Z
  Relative segment, address: XDATA 000002F3 - 000002F8 (0x6 bytes), align: 0
  Segment part 24.            Intra module refs:   LL_EXT_SetBDADDR
                                                   LL_Init
                                                   LL_ReadBDADDR
                                                   LL_SetAdvParam
                                                   Segment part 161
           ENTRY                   ADDRESS         REF BY
           =====                   =======         ======
           ownPublicAddr           000002F3 
    -------------------------------------------------------------------------
XDATA_Z
  Relative segment, address: XDATA 000002F9 - 000002FE (0x6 bytes), align: 0
  Segment part 25.            Intra module refs:   LL_Init
                                                   LL_SetAdvParam
                                                   LL_SetRandomAddress
           ENTRY                   ADDRESS         REF BY
           =====                   =======         ======
           ownRandomAddr           000002F9 
    -------------------------------------------------------------------------
XDATA_Z
  Relative segment, address: XDATA 000002FF - 00000304 (0x6 bytes), align: 0
  Segment part 26.            Intra module refs:   LL_EXT_SetBDADDR
                                                   Segment part 161
           ENTRY                   ADDRESS         REF BY
           =====                   =======         ======
           ownSavedPublicAddr      000002FF 
    -------------------------------------------------------------------------
XDATA_Z
  Relative segment, address: XDATA 00000305 - 00000305 (0x1 bytes), align: 0
  Segment part 27.            Intra module refs:   LL_EXT_ResetSystem
                                                   LL_Init
                                                   LL_ProcessEvent
                                                   LL_SetAdvControl
           ENTRY                   ADDRESS         REF BY
           =====                   =======         ======
           LL_TaskID               00000305        RF_NormalIsr (ll_isr)
                                                   llFreeTask (ll_scheduler)
                                                   llScheduleTask (ll_scheduler)
                                                   llT2OVFC1_ISR (ll_isr)
    -------------------------------------------------------------------------
XDATA_Z
  Relative segment, address: XDATA 00000306 - 00000306 (0x1 bytes), align: 0
  Segment part 28.            Intra module refs:   LL_DirectTestEnd
                                                   LL_DirectTestRxTest
                                                   LL_DirectTestTxTest
                                                   LL_EXT_DeclareNvUsage
                                                   LL_EXT_EndModemTest
                                                   LL_EXT_ModemHopTestTx
                                                   LL_EXT_ModemTestRx
                                                   LL_EXT_ModemTestTx
                                                   LL_EXT_SetBDADDR
                                                   LL_Rand
                                                   LL_ReadRssi
                                                   LL_Reset
                                                   LL_SetAdvControl
                                                   Segment part 114
           ENTRY                   ADDRESS         REF BY
           =====                   =======         ======
           llState                 00000306        RF_NormalIsr (ll_isr)
                                                   llFreeTask (ll_scheduler)
                                                   llScheduler (ll_scheduler)
                                                   llSetupNonConnectableAdvEvt (ll_common)
                                                   llSetupScannableAdvEvt (ll_common)
                                                   llT2OVFC1_ISR (ll_isr)
    -------------------------------------------------------------------------
XDATA_Z
  Relative segment, address: XDATA 00000307 - 00000307 (0x1 bytes), align: 0
  Segment part 29.            Intra module refs:   LL_ProcessEvent
           ENTRY                   ADDRESS         REF BY
           =====                   =======         ======
           taskEndCause            00000307        RF_NormalIsr (ll_isr)
    -------------------------------------------------------------------------
XDATA_Z
  Relative segment, address: XDATA 00000308 - 00000309 (0x2 bytes), align: 0
  Segment part 30.            Intra module refs:   LL_EXT_ExtendRfRange
                                                   LL_EXT_SetRxGain
                                                   LL_EXT_SetTxPower
                                                   LL_Rand
                                                   LL_Reset
           ENTRY                   ADDRESS         REF BY
           =====                   =======         ======
           postRfOperations        00000308        llProcessPostRfOps (ll_common)
    -------------------------------------------------------------------------
XDATA_Z
  Relative segment, address: XDATA 0000030A - 0000030A (0x1 bytes), align: 0
  Segment part 31.            Intra module refs:   LL_ReadRssi
           ENTRY                   ADDRESS         REF BY
           =====                   =======         ======
           rssiCorrection          0000030A        llSetRxGain (ll_common)
    -------------------------------------------------------------------------
XDATA_Z
  Relative segment, address: XDATA 0000030B - 0000030B (0x1 bytes), align: 0
  Segment part 32.            Intra module refs:   LL_EXT_ClkDivOnHalt
                                                   LL_Reset
           ENTRY                   ADDRESS         REF BY
           =====                   =======         ======
           clkDivOnHalt            0000030B        llT2OVFC1_ISR (ll_isr)
    -------------------------------------------------------------------------
XDATA_Z
  Relative segment, address: XDATA 0000030C - 0000030C (0x1 bytes), align: 0
  Segment part 33.            Intra module refs:   LL_EXT_DeclareNvUsage
                                                   LL_ProcessEvent
                                                   LL_Reset
                                                   LL_SetAdvControl
           ENTRY                   ADDRESS         REF BY
           =====                   =======         ======
           nvInUse                 0000030C        llScheduleTask (ll_scheduler)
                                                   llT2OVFC1_ISR (ll_isr)
    -------------------------------------------------------------------------
XDATA_Z
  Relative segment, address: XDATA 0000030D - 00000315 (0x9 bytes), align: 0
  Segment part 35.            Intra module refs:   LL_EXT_SetLocalSupportedFeatures
                                                   LL_ReadLocalSupportedFeatures
           ENTRY                   ADDRESS         REF BY
           =====                   =======         ======
           deviceFeatureSet        0000030D        llInitFeatureSet (ll_common)
    -------------------------------------------------------------------------
XDATA_Z
  Relative segment, address: XDATA 00000316 - 00000316 (0x1 bytes), align: 0
  Segment part 36.            Intra module refs:   LL_DirectTestTxTest
                                                   LL_EXT_SetMaxDtmTxPower
                                                   LL_Reset
           ENTRY                   ADDRESS         REF BY
           =====                   =======         ======
           maxTxPwrForDTM          00000316 
    -------------------------------------------------------------------------
XDATA_Z
  Relative segment, address: XDATA 00000317 - 0000031B (0x5 bytes), align: 0
  Segment part 37.            Intra module refs:   LL_Init
                                                   LL_ReadLocalVersionInfo
           ENTRY                   ADDRESS         REF BY
           =====                   =======         ======
           verInfo                 00000317 
    -------------------------------------------------------------------------
XDATA_Z
  Relative segment, address: XDATA 0000031C - 00000323 (0x8 bytes), align: 0
  Segment part 38.            Intra module refs:   LL_DirectTestEnd
                                                   LL_DirectTestRxTest
                                                   LL_DirectTestTxTest
                                                   LL_EXT_ModemHopTestTx
           ENTRY                   ADDRESS         REF BY
           =====                   =======         ======
           dtmInfo                 0000031C 
    -------------------------------------------------------------------------
XDATA_Z
  Relative segment, address: XDATA 00000324 - 00000325 (0x2 bytes), align: 0
  Segment part 39.            Intra module refs:   LL_EXT_BuildRevision
                                                   LL_Init
           ENTRY                   ADDRESS         REF BY
           =====                   =======         ======
           buildInfo               00000324 
    -------------------------------------------------------------------------
XDATA_Z
  Relative segment, address: XDATA 00000326 - 00000381 (0x5c bytes), align: 0
  Segment part 40.            Intra module refs:   LL_Init
                                                   LL_Reset
                                                   LL_SetAdvControl
                                                   LL_SetAdvData
                                                   LL_SetAdvParam
                                                   LL_SetScanRspData
           ENTRY                   ADDRESS         REF BY
           =====                   =======         ======
           advInfo                 00000326        Segment part 15 (ll_advEndCauses)
                                                   Segment part 16 (ll_advEndCauses)
                                                   Segment part 17 (ll_advEndCauses)
                                                   Segment part 186 (ll_common)
                                                   Segment part 19 (ll_advEndCauses)
                                                   Segment part 20 (ll_advEndCauses)
                                                   Segment part 21 (ll_advEndCauses)
                                                   Segment part 23 (ll_advEndCauses)
                                                   Segment part 77 (ll_common)
                                                   Segment part 83 (ll_common)
                                                   Segment part 85 (ll_common)
                                                   llAdvEvt_TaskAbort (ll_advEndCauses)
                                                   llCheckWhiteListUsage (ll_common)
                                                   llDiscoverableAdvEvt_TaskEndOk (ll_advEndCauses)
                                                   llNonConnAdvEvt_TaskEndOk (ll_advEndCauses)
                                                   llSetupAdv (ll_common)
                                                   llSetupNonConnectableAdvEvt (ll_common)
                                                   llSetupScannableAdvEvt (ll_common)
                                                   llStartAdvSetup (ll_common)
    -------------------------------------------------------------------------
XDATA_Z
  Relative segment, address: XDATA 00000382 - 00000383 (0x2 bytes), align: 0
  Segment part 41.            Intra module refs:   LL_EXT_MapPmIoPort
                                                   LL_Init
           ENTRY                   ADDRESS         REF BY
           =====                   =======         ======
           dcdcData                00000382 
    -------------------------------------------------------------------------
XDATA_Z
  Relative segment, address: XDATA 00000384 - 00000384 (0x1 bytes), align: 0
  Segment part 42.            Intra module refs:   LL_Init
           ENTRY                   ADDRESS         REF BY
           =====                   =======         ======
           extendRfRange           00000384        llExtendRfRange (ll_common)
                                                   llSetRxGain (ll_common)
                                                   llSetTxPower (ll_common)
    -------------------------------------------------------------------------
XDATA_Z
  Relative segment, address: XDATA 00000385 - 00000385 (0x1 bytes), align: 0
  Segment part 43.            Intra module refs:   LL_Reset
           ENTRY                   ADDRESS         REF BY
           =====                   =======         ======
           rxFifoFlowCtrl          00000385 
    -------------------------------------------------------------------------
XDATA_Z
  Relative segment, address: XDATA 00000386 - 00000386 (0x1 bytes), align: 0
  Segment part 44.            Intra module refs:   LL_EXT_ClkDivOnHalt
                                                   LL_EXT_HaltDuringRf
                                                   LL_Init
           ENTRY                   ADDRESS         REF BY
           =====                   =======         ======
           haltDuringRf            00000386        llScheduleTask (ll_scheduler)
                                                   llT2OVFC1_ISR (ll_isr)
    -------------------------------------------------------------------------
XDATA_Z
  Relative segment, address: XDATA 00000387 - 00000388 (0x2 bytes), align: 0
  Segment part 45.            Intra module refs:   LL_Init
                                                   LL_ProcessEvent
           ENTRY                   ADDRESS         REF BY
           =====                   =======         ======
           sleepDelay              00000387 
    -------------------------------------------------------------------------
XDATA_I
  Relative segment, address: XDATA 000010D5 - 000010E2 (0xe bytes), align: 0
  Segment part 46.            Intra module refs:   LL_ProcessEvent
           ENTRY                   ADDRESS         REF BY
           =====                   =======         ======
           taskEndCauses           000010D5        llSetupNonConnectableAdvEvt (ll_common)
                                                   llSetupScannableAdvEvt (ll_common)
    -------------------------------------------------------------------------
XDATA_I
  Relative segment, address: XDATA 000010E3 - 000010EE (0xc bytes), align: 0
  Segment part 48.            Intra module refs:   LL_ProcessEvent
           ENTRY                   ADDRESS         REF BY
           =====                   =======         ======
           taskErrorEndCauses      000010E3        Segment part 88 (ll_common)
    -------------------------------------------------------------------------
<XDATA_ROM_C> 1 (was XDATA_ROM_C)
  Relative segment, address: CONST 00008EFF - 00008F23 (0x25 bytes), align: 0
  Segment part 50.            Intra module refs:   Segment part 153
           ENTRY                   ADDRESS         REF BY
           =====                   =======         ======
           psbs9Data               00008EFF 
    -------------------------------------------------------------------------
XDATA_Z
  Relative segment, address: XDATA 00000389 - 00000389 (0x1 bytes), align: 0
  Segment part 51.            Intra module refs:   LL_Init
           ENTRY                   ADDRESS         REF BY
           =====                   =======         ======
           trngCounter             00000389        RF_NormalIsr (ll_isr)
    -------------------------------------------------------------------------
IDATA_Z
  Relative segment, address: IDATA 0000002A - 0000002B (0x2 bytes), align: 0
  Segment part 52. ROOT       Intra module refs:   LL_Init
           ENTRY                   ADDRESS         REF BY
           =====                   =======         ======
           myPC                    0000002A        RF_NormalIsr (ll_isr)
    -------------------------------------------------------------------------
<BANKED_CODE,CODE_C> 1 (was BANKED_CODE)
  Relative segment, address: CODE 000017B0 - 0000193C (0x18d bytes), align: 0
  Segment part 60.            Intra module refs:   LL_Init::?relay
           ENTRY                   ADDRESS         REF BY
           =====                   =======         ======
           LL_Init                 000017B0 
               calls direct
               XSTACK = 00000000 ( 0000000E )
               ISTACK = 00000000 ( 00000001 )
    -------------------------------------------------------------------------
<BANKED_CODE,CODE_C> 1 (was BANKED_CODE)
  Relative segment, address: CODE 0000193D - 00001945 (0x9 bytes), align: 0
  Segment part 62.            Intra module refs:   LL_Init
    -------------------------------------------------------------------------
<BANKED_CODE,CODE_C> 1 (was BANKED_CODE)
  Relative segment, address: CODE 00001946 - 00001A1B (0xd6 bytes), align: 0
  Segment part 63.            Intra module refs:   LL_ProcessEvent::?relay
           ENTRY                   ADDRESS         REF BY
           =====                   =======         ======
           LL_ProcessEvent         00001946 
               calls direct
               XSTACK = 00000000 ( 00000010 )
    -------------------------------------------------------------------------
<BANKED_CODE,CODE_C> 1 (was BANKED_CODE)
  Relative segment, address: CODE 00001A1C - 00001A6F (0x54 bytes), align: 0
  Segment part 65.            Intra module refs:   LL_TX_bm_alloc::?relay
           ENTRY                   ADDRESS         REF BY
           =====                   =======         ======
           LL_TX_bm_alloc          00001A1C 
               calls direct
               XSTACK = 00000000 ( 0000000A )
    -------------------------------------------------------------------------
<BANKED_CODE,CODE_C> 1 (was BANKED_CODE)
  Relative segment, address: CODE 00001A70 - 00001B11 (0xa2 bytes), align: 0
  Segment part 69.            Intra module refs:   LL_Reset::?relay
           ENTRY                   ADDRESS         REF BY
           =====                   =======         ======
           LL_Reset                00001A70 
               calls direct
               XSTACK = 0000000C ( 00000000 )
               ISTACK = 00000000 ( 00000002 )
    -------------------------------------------------------------------------
<BANKED_CODE,CODE_C> 1 (was BANKED_CODE)
  Relative segment, address: CODE 00001B12 - 00001B12 (0x1 bytes), align: 0
  Segment part 71.            Intra module refs:   LL_ReadBDADDR
                                                   LL_ReadLocalVersionInfo
                                                   LL_ReadRssi
                                                   LL_ReadSupportedStates
                                                   LL_SetRandomAddress
    -------------------------------------------------------------------------
<BANKED_CODE,CODE_C> 1 (was BANKED_CODE)
  Relative segment, address: CODE 00001B13 - 00001B14 (0x2 bytes), align: 0
  Segment part 72.            Intra module refs:   LL_ReadLocalSupportedFeatures
                                                   Segment part 71
    -------------------------------------------------------------------------
<BANKED_CODE,CODE_C> 1 (was BANKED_CODE)
  Relative segment, address: CODE 00001B15 - 00001B1B (0x7 bytes), align: 0
  Segment part 73.            Intra module refs:   LL_ClearWhiteList
                                                   LL_EXT_ClkDivOnHalt
                                                   LL_EXT_DeclareNvUsage
                                                   LL_EXT_EndModemTest
                                                   LL_EXT_HaltDuringRf
                                                   LL_EXT_ModemHopTestTx
                                                   LL_EXT_SetLocalSupportedFeatures
                                                   LL_EXT_SetMaxDtmTxPower
                                                   LL_Reset
                                                   Segment part 72
    -------------------------------------------------------------------------
<BANKED_CODE,CODE_C> 1 (was BANKED_CODE)
  Relative segment, address: CODE 00001B1C - 00001B4D (0x32 bytes), align: 0
  Segment part 74.            Intra module refs:   LL_ReadBDADDR::?relay
           ENTRY                   ADDRESS         REF BY
           =====                   =======         ======
           LL_ReadBDADDR           00001B1C 
               ISTACK = 00000000 ( 00000003 )
    -------------------------------------------------------------------------
<BANKED_CODE,CODE_C> 1 (was BANKED_CODE)
  Relative segment, address: CODE 00001B4E - 00001B54 (0x7 bytes), align: 0
  Segment part 76.            Intra module refs:   LL_ReadBDADDR
    -------------------------------------------------------------------------
<BANKED_CODE,CODE_C> 1 (was BANKED_CODE)
  Relative segment, address: CODE 00001B55 - 00001B5E (0xa bytes), align: 0
  Segment part 77.            Intra module refs:   LL_ReadBDADDR
    -------------------------------------------------------------------------
<BANKED_CODE,CODE_C> 1 (was BANKED_CODE)
  Relative segment, address: CODE 00001B5F - 00001B94 (0x36 bytes), align: 0
  Segment part 78.            Intra module refs:   LL_SetRandomAddress::?relay
           ENTRY                   ADDRESS         REF BY
           =====                   =======         ======
           LL_SetRandomAddress     00001B5F 
               ISTACK = 00000000 ( 00000002 )
    -------------------------------------------------------------------------
<BANKED_CODE,CODE_C> 1 (was BANKED_CODE)
  Relative segment, address: CODE 00001B95 - 00001B9B (0x7 bytes), align: 0
  Segment part 80.            Intra module refs:   LL_SetRandomAddress
    -------------------------------------------------------------------------
<BANKED_CODE,CODE_C> 1 (was BANKED_CODE)
  Relative segment, address: CODE 00001B9C - 00001BA5 (0xa bytes), align: 0
  Segment part 81.            Intra module refs:   LL_SetRandomAddress
    -------------------------------------------------------------------------
<BANKED_CODE,CODE_C> 1 (was BANKED_CODE)
  Relative segment, address: CODE 00001BA6 - 00001BB8 (0x13 bytes), align: 0
  Segment part 82.            Intra module refs:   LL_ClearWhiteList::?relay
           ENTRY                   ADDRESS         REF BY
           =====                   =======         ======
           LL_ClearWhiteList       00001BA6 
               calls direct
               ISTACK = 00000000 ( 00000002 )
    -------------------------------------------------------------------------
<BANKED_CODE,CODE_C> 1 (was BANKED_CODE)
  Relative segment, address: CODE 00001BB9 - 00001BF9 (0x41 bytes), align: 0
  Segment part 84.            Intra module refs:   LL_AddWhiteListDevice::?relay
           ENTRY                   ADDRESS         REF BY
           =====                   =======         ======
           LL_AddWhiteListDevice   00001BB9 
               calls direct
               XSTACK = 00000000 ( 00000009 )
    -------------------------------------------------------------------------
<BANKED_CODE,CODE_C> 1 (was BANKED_CODE)
  Relative segment, address: CODE 00001BFA - 00001C3B (0x42 bytes), align: 0
  Segment part 86.            Intra module refs:   LL_RemoveWhiteListDevice::?relay
           ENTRY                   ADDRESS         REF BY
           =====                   =======         ======
           LL_RemoveWhiteListDevice
                                   00001BFA 
               calls direct
               XSTACK = 00000000 ( 00000009 )
    -------------------------------------------------------------------------
<BANKED_CODE,CODE_C> 1 (was BANKED_CODE)
  Relative segment, address: CODE 00001C3C - 00001C4A (0xf bytes), align: 0
  Segment part 88.            Intra module refs:   LL_ReadWlSize::?relay
           ENTRY                   ADDRESS         REF BY
           =====                   =======         ======
           LL_ReadWlSize           00001C3C 
               calls direct
               XSTACK = 00000000 ( 00000009 )
               ISTACK = 00000000 ( 00000001 )
    -------------------------------------------------------------------------
<BANKED_CODE,CODE_C> 1 (was BANKED_CODE)
  Relative segment, address: CODE 00001C4B - 00001C77 (0x2d bytes), align: 0
  Segment part 92.            Intra module refs:   LL_Encrypt::?relay
           ENTRY                   ADDRESS         REF BY
           =====                   =======         ======
           LL_Encrypt              00001C4B 
               calls direct
               XSTACK = 00000002 ( 0000000C )
    -------------------------------------------------------------------------
<BANKED_CODE,CODE_C> 1 (was BANKED_CODE)
  Relative segment, address: CODE 00001C78 - 00001CC0 (0x49 bytes), align: 0
  Segment part 94.            Intra module refs:   LL_Rand::?relay
           ENTRY                   ADDRESS         REF BY
           =====                   =======         ======
           LL_Rand                 00001C78 
               calls direct
               XSTACK = 00000000 ( 0000000C )
    -------------------------------------------------------------------------
<BANKED_CODE,CODE_C> 1 (was BANKED_CODE)
  Relative segment, address: CODE 00001CC1 - 00001CC5 (0x5 bytes), align: 0
  Segment part 96.            Intra module refs:   LL_EXT_SaveFreqTune
                                                   LL_Init
                                                   LL_ProcessEvent
                                                   LL_Rand
                                                   LL_SetAdvControl
    -------------------------------------------------------------------------
<BANKED_CODE,CODE_C> 1 (was BANKED_CODE)
  Relative segment, address: CODE 00001CC6 - 00001CD3 (0xe bytes), align: 0
  Segment part 99.            Intra module refs:   LL_ReadSupportedStates::?relay
           ENTRY                   ADDRESS         REF BY
           =====                   =======         ======
           LL_ReadSupportedStates
                                   00001CC6 
               ISTACK = 00000000 ( 00000002 )
    -------------------------------------------------------------------------
<BANKED_CODE,CODE_C> 1 (was BANKED_CODE)
  Relative segment, address: CODE 00001CD4 - 00001CFD (0x2a bytes), align: 0
  Segment part 101.           Intra module refs:   LL_ReadLocalSupportedFeatures::?relay
           ENTRY                   ADDRESS         REF BY
           =====                   =======         ======
           LL_ReadLocalSupportedFeatures
                                   00001CD4 
               ISTACK = 00000000 ( 00000003 )
    -------------------------------------------------------------------------
<BANKED_CODE,CODE_C> 1 (was BANKED_CODE)
  Relative segment, address: CODE 00001CFE - 00001D31 (0x34 bytes), align: 0
  Segment part 103.           Intra module refs:   LL_ReadLocalVersionInfo::?relay
           ENTRY                   ADDRESS         REF BY
           =====                   =======         ======
           LL_ReadLocalVersionInfo
                                   00001CFE 
               XSTACK = 00000002 ( 00000000 )
               ISTACK = 00000000 ( 00000003 )
    -------------------------------------------------------------------------
<BANKED_CODE,CODE_C> 1 (was BANKED_CODE)
  Relative segment, address: CODE 00001D32 - 00001D38 (0x7 bytes), align: 0
  Segment part 105.           Intra module refs:   LL_ReadBDADDR
                                                   LL_ReadLocalVersionInfo
    -------------------------------------------------------------------------
<BANKED_CODE,CODE_C> 1 (was BANKED_CODE)
  Relative segment, address: CODE 00001D39 - 00001D3E (0x6 bytes), align: 0
  Segment part 106.           Intra module refs:   LL_ProcessEvent
                                                   LL_ReadLocalVersionInfo
                                                   LL_SetAdvParam
    -------------------------------------------------------------------------
<BANKED_CODE,CODE_C> 1 (was BANKED_CODE)
  Relative segment, address: CODE 00001D3F - 00001D6B (0x2d bytes), align: 0
  Segment part 107.           Intra module refs:   LL_ReadRssi::?relay
           ENTRY                   ADDRESS         REF BY
           =====                   =======         ======
           LL_ReadRssi             00001D3F 
               ISTACK = 00000000 ( 00000003 )
    -------------------------------------------------------------------------
<BANKED_CODE,CODE_C> 1 (was BANKED_CODE)
  Relative segment, address: CODE 00001D6C - 00001E98 (0x12d bytes), align: 0
  Segment part 109.           Intra module refs:   LL_DirectTestTxTest::?relay
           ENTRY                   ADDRESS         REF BY
           =====                   =======         ======
           LL_DirectTestTxTest     00001D6C 
               calls direct
               XSTACK = 00000000 ( 00000009 )
    -------------------------------------------------------------------------
<BANKED_CODE,CODE_C> 1 (was BANKED_CODE)
  Relative segment, address: CODE 00001E99 - 00001EF0 (0x58 bytes), align: 0
  Segment part 111.           Intra module refs:   LL_DirectTestRxTest::?relay
           ENTRY                   ADDRESS         REF BY
           =====                   =======         ======
           LL_DirectTestRxTest     00001E99 
               calls direct
               XSTACK = 00000000 ( 00000009 )
    -------------------------------------------------------------------------
<BANKED_CODE,CODE_C> 1 (was BANKED_CODE)
  Relative segment, address: CODE 00001EF1 - 00001EF6 (0x6 bytes), align: 0
  Segment part 113.           Intra module refs:   LL_DirectTestRxTest
                                                   LL_Init
    -------------------------------------------------------------------------
<BANKED_CODE,CODE_C> 1 (was BANKED_CODE)
  Relative segment, address: CODE 00001EF7 - 00001F03 (0xd bytes), align: 0
  Segment part 114.           Intra module refs:   LL_DirectTestRxTest
                                                   LL_DirectTestTxTest
    -------------------------------------------------------------------------
<BANKED_CODE,CODE_C> 1 (was BANKED_CODE)
  Relative segment, address: CODE 00001F04 - 00001F0C (0x9 bytes), align: 0
  Segment part 115.           Intra module refs:   Segment part 114
                                                   Segment part 62
    -------------------------------------------------------------------------
<BANKED_CODE,CODE_C> 1 (was BANKED_CODE)
  Relative segment, address: CODE 00001F0D - 00001F83 (0x77 bytes), align: 0
  Segment part 116.           Intra module refs:   LL_DirectTestEnd::?relay
           ENTRY                   ADDRESS         REF BY
           =====                   =======         ======
           LL_DirectTestEnd        00001F0D 
               calls direct
               XSTACK = 00000000 ( 0000000C )
    -------------------------------------------------------------------------
<BANKED_CODE,CODE_C> 1 (was BANKED_CODE)
  Relative segment, address: CODE 00001F84 - 00001F88 (0x5 bytes), align: 0
  Segment part 118.           Intra module refs:   LL_DirectTestEnd
                                                   LL_EXT_Decrypt
                                                   LL_EXT_MapPmIoPort
                                                   LL_Encrypt
                                                   LL_SetAdvData
                                                   LL_SetScanRspData
                                                   LL_TX_bm_alloc
    -------------------------------------------------------------------------
<BANKED_CODE,CODE_C> 1 (was BANKED_CODE)
  Relative segment, address: CODE 00001F89 - 0000210A (0x182 bytes), align: 0
  Segment part 119.           Intra module refs:   LL_SetAdvParam::?relay
           ENTRY                   ADDRESS         REF BY
           =====                   =======         ======
           LL_SetAdvParam          00001F89 
               calls direct
               XSTACK = 00000006 ( 00000009 )
    -------------------------------------------------------------------------
<BANKED_CODE,CODE_C> 1 (was BANKED_CODE)
  Relative segment, address: CODE 0000210B - 00002115 (0xb bytes), align: 0
  Segment part 121.           Intra module refs:   LL_SetAdvParam
    -------------------------------------------------------------------------
<BANKED_CODE,CODE_C> 1 (was BANKED_CODE)
  Relative segment, address: CODE 00002116 - 00002120 (0xb bytes), align: 0
  Segment part 122.           Intra module refs:   LL_SetAdvParam
    -------------------------------------------------------------------------
<BANKED_CODE,CODE_C> 1 (was BANKED_CODE)
  Relative segment, address: CODE 00002121 - 00002128 (0x8 bytes), align: 0
  Segment part 123.           Intra module refs:   LL_ReadWlSize
    -------------------------------------------------------------------------
<BANKED_CODE,CODE_C> 1 (was BANKED_CODE)
  Relative segment, address: CODE 00002129 - 0000212D (0x5 bytes), align: 0
  Segment part 124.           Intra module refs:   LL_AddWhiteListDevice
                                                   LL_DirectTestRxTest
                                                   LL_DirectTestTxTest
                                                   LL_EXT_BuildRevision
                                                   LL_EXT_ModemTestRx
                                                   LL_EXT_ModemTestTx
                                                   LL_EXT_ResetSystem
                                                   LL_EXT_SetFreqTune
                                                   LL_ReadAdvChanTxPower
                                                   LL_RemoveWhiteListDevice
                                                   LL_SetAdvParam
                                                   Segment part 123
    -------------------------------------------------------------------------
<BANKED_CODE,CODE_C> 1 (was BANKED_CODE)
  Relative segment, address: CODE 0000212E - 00002169 (0x3c bytes), align: 0
  Segment part 125.           Intra module refs:   LL_SetAdvData::?relay
           ENTRY                   ADDRESS         REF BY
           =====                   =======         ======
           LL_SetAdvData           0000212E 
               calls direct
               XSTACK = 00000000 ( 0000000C )
    -------------------------------------------------------------------------
<BANKED_CODE,CODE_C> 1 (was BANKED_CODE)
  Relative segment, address: CODE 0000216A - 000022E9 (0x180 bytes), align: 0
  Segment part 127.           Intra module refs:   LL_SetAdvControl::?relay
           ENTRY                   ADDRESS         REF BY
           =====                   =======         ======
           LL_SetAdvControl        0000216A 
               calls direct
               XSTACK = 00000000 ( 0000000C )
    -------------------------------------------------------------------------
<BANKED_CODE,CODE_C> 1 (was BANKED_CODE)
  Relative segment, address: CODE 000022EA - 000022F2 (0x9 bytes), align: 0
  Segment part 129.           Intra module refs:   LL_ProcessEvent
                                                   LL_SetAdvControl
    -------------------------------------------------------------------------
<BANKED_CODE,CODE_C> 1 (was BANKED_CODE)
  Relative segment, address: CODE 000022F3 - 00002313 (0x21 bytes), align: 0
  Segment part 130.           Intra module refs:   LL_ReadAdvChanTxPower::?relay
           ENTRY                   ADDRESS         REF BY
           =====                   =======         ======
           LL_ReadAdvChanTxPower   000022F3 
               calls direct
               XSTACK = 00000000 ( 00000009 )
               ISTACK = 00000000 ( 00000001 )
    -------------------------------------------------------------------------
<BANKED_CODE,CODE_C> 1 (was BANKED_CODE)
  Relative segment, address: CODE 00002314 - 0000234F (0x3c bytes), align: 0
  Segment part 132.           Intra module refs:   LL_SetScanRspData::?relay
           ENTRY                   ADDRESS         REF BY
           =====                   =======         ======
           LL_SetScanRspData       00002314 
               calls direct
               XSTACK = 00000000 ( 0000000C )
    -------------------------------------------------------------------------
<BANKED_CODE,CODE_C> 1 (was BANKED_CODE)
  Relative segment, address: CODE 00002350 - 00002358 (0x9 bytes), align: 0
  Segment part 134.           Intra module refs:   LL_SetAdvData
                                                   LL_SetScanRspData
    -------------------------------------------------------------------------
<BANKED_CODE,CODE_C> 1 (was BANKED_CODE)
  Relative segment, address: CODE 00002359 - 00002402 (0xaa bytes), align: 0
  Segment part 135.           Intra module refs:   LL_EXT_SetRxGain::?relay
           ENTRY                   ADDRESS         REF BY
           =====                   =======         ======
           LL_EXT_SetRxGain        00002359 
               calls direct
               XSTACK = 00000000 ( 00000014 )
               ISTACK = 00000000 ( 00000002 )
    -------------------------------------------------------------------------
<BANKED_CODE,CODE_C> 1 (was BANKED_CODE)
  Relative segment, address: CODE 00002403 - 00002407 (0x5 bytes), align: 0
  Segment part 137.           Intra module refs:   LL_EXT_ExtendRfRange
                                                   LL_EXT_SetRxGain
                                                   LL_EXT_SetTxPower
    -------------------------------------------------------------------------
<BANKED_CODE,CODE_C> 1 (was BANKED_CODE)
  Relative segment, address: CODE 00002408 - 000024DF (0xd8 bytes), align: 0
  Segment part 138.           Intra module refs:   LL_EXT_SetTxPower::?relay
           ENTRY                   ADDRESS         REF BY
           =====                   =======         ======
           LL_EXT_SetTxPower       00002408 
               calls direct
               XSTACK = 00000000 ( 00000014 )
               ISTACK = 00000000 ( 00000002 )
    -------------------------------------------------------------------------
<BANKED_CODE,CODE_C> 1 (was BANKED_CODE)
  Relative segment, address: CODE 000024E0 - 0000250A (0x2b bytes), align: 0
  Segment part 140.           Intra module refs:   LL_EXT_ClkDivOnHalt::?relay
           ENTRY                   ADDRESS         REF BY
           =====                   =======         ======
           LL_EXT_ClkDivOnHalt     000024E0 
               ISTACK = 00000000 ( 00000002 )
    -------------------------------------------------------------------------
<BANKED_CODE,CODE_C> 1 (was BANKED_CODE)
  Relative segment, address: CODE 0000250B - 00002535 (0x2b bytes), align: 0
  Segment part 142.           Intra module refs:   LL_EXT_DeclareNvUsage::?relay
           ENTRY                   ADDRESS         REF BY
           =====                   =======         ======
           LL_EXT_DeclareNvUsage   0000250B 
               ISTACK = 00000000 ( 00000002 )
    -------------------------------------------------------------------------
<BANKED_CODE,CODE_C> 1 (was BANKED_CODE)
  Relative segment, address: CODE 00002536 - 00002562 (0x2d bytes), align: 0
  Segment part 144.           Intra module refs:   LL_EXT_Decrypt::?relay
           ENTRY                   ADDRESS         REF BY
           =====                   =======         ======
           LL_EXT_Decrypt          00002536 
               calls direct
               XSTACK = 00000002 ( 0000000C )
    -------------------------------------------------------------------------
<BANKED_CODE,CODE_C> 1 (was BANKED_CODE)
  Relative segment, address: CODE 00002563 - 0000256E (0xc bytes), align: 0
  Segment part 146.           Intra module refs:   LL_EXT_Decrypt
                                                   LL_Encrypt
    -------------------------------------------------------------------------
<BANKED_CODE,CODE_C> 1 (was BANKED_CODE)
  Relative segment, address: CODE 0000256F - 00002593 (0x25 bytes), align: 0
  Segment part 147.           Intra module refs:   LL_EXT_SetLocalSupportedFeatures::?relay
           ENTRY                   ADDRESS         REF BY
           =====                   =======         ======
           LL_EXT_SetLocalSupportedFeatures
                                   0000256F 
               ISTACK = 00000000 ( 00000002 )
    -------------------------------------------------------------------------
<BANKED_CODE,CODE_C> 1 (was BANKED_CODE)
  Relative segment, address: CODE 00002594 - 00002609 (0x76 bytes), align: 0
  Segment part 149.           Intra module refs:   LL_EXT_ModemTestTx::?relay
           ENTRY                   ADDRESS         REF BY
           =====                   =======         ======
           LL_EXT_ModemTestTx      00002594 
               calls direct
               XSTACK = 00000000 ( 00000009 )
    -------------------------------------------------------------------------
<BANKED_CODE,CODE_C> 1 (was BANKED_CODE)
  Relative segment, address: CODE 0000260A - 0000266D (0x64 bytes), align: 0
  Segment part 151.           Intra module refs:   LL_EXT_ModemHopTestTx::?relay
           ENTRY                   ADDRESS         REF BY
           =====                   =======         ======
           LL_EXT_ModemHopTestTx   0000260A 
               calls direct
               ISTACK = 00000000 ( 00000002 )
    -------------------------------------------------------------------------
<BANKED_CODE,CODE_C> 1 (was BANKED_CODE)
  Relative segment, address: CODE 0000266E - 0000267E (0x11 bytes), align: 0
  Segment part 153.           Intra module refs:   LL_DirectTestTxTest
                                                   LL_EXT_ModemHopTestTx
    -------------------------------------------------------------------------
<BANKED_CODE,CODE_C> 1 (was BANKED_CODE)
  Relative segment, address: CODE 0000267F - 00002689 (0xb bytes), align: 0
  Segment part 154.           Intra module refs:   LL_DirectTestTxTest
                                                   LL_EXT_ModemHopTestTx
    -------------------------------------------------------------------------
<BANKED_CODE,CODE_C> 1 (was BANKED_CODE)
  Relative segment, address: CODE 0000268A - 000026D1 (0x48 bytes), align: 0
  Segment part 155.           Intra module refs:   LL_EXT_ModemTestRx::?relay
           ENTRY                   ADDRESS         REF BY
           =====                   =======         ======
           LL_EXT_ModemTestRx      0000268A 
               calls direct
               XSTACK = 00000000 ( 00000009 )
    -------------------------------------------------------------------------
<BANKED_CODE,CODE_C> 1 (was BANKED_CODE)
  Relative segment, address: CODE 000026D2 - 000026F3 (0x22 bytes), align: 0
  Segment part 157.           Intra module refs:   LL_EXT_EndModemTest::?relay
           ENTRY                   ADDRESS         REF BY
           =====                   =======         ======
           LL_EXT_EndModemTest     000026D2 
               calls direct
               ISTACK = 00000000 ( 00000002 )
    -------------------------------------------------------------------------
<BANKED_CODE,CODE_C> 1 (was BANKED_CODE)
  Relative segment, address: CODE 000026F4 - 000027DA (0xe7 bytes), align: 0
  Segment part 159.           Intra module refs:   LL_EXT_SetBDADDR::?relay
           ENTRY                   ADDRESS         REF BY
           =====                   =======         ======
           LL_EXT_SetBDADDR        000026F4 
               XSTACK = 00000000 ( 0000000D )
    -------------------------------------------------------------------------
<BANKED_CODE,CODE_C> 1 (was BANKED_CODE)
  Relative segment, address: CODE 000027DB - 0000280B (0x31 bytes), align: 0
  Segment part 161.           Intra module refs:   LL_EXT_SetBDADDR
                                                   LL_Init
    -------------------------------------------------------------------------
<BANKED_CODE,CODE_C> 1 (was BANKED_CODE)
  Relative segment, address: CODE 0000280C - 0000283C (0x31 bytes), align: 0
  Segment part 162.           Intra module refs:   LL_EXT_SetFreqTune::?relay
           ENTRY                   ADDRESS         REF BY
           =====                   =======         ======
           LL_EXT_SetFreqTune      0000280C 
               calls direct
               XSTACK = 00000000 ( 00000009 )
    -------------------------------------------------------------------------
<BANKED_CODE,CODE_C> 1 (was BANKED_CODE)
  Relative segment, address: CODE 0000283D - 0000289B (0x5f bytes), align: 0
  Segment part 164.           Intra module refs:   LL_EXT_SaveFreqTune::?relay
           ENTRY                   ADDRESS         REF BY
           =====                   =======         ======
           LL_EXT_SaveFreqTune     0000283D 
               calls direct
               XSTACK = 00000000 ( 00000012 )
               ISTACK = 00000000 ( 00000001 )
    -------------------------------------------------------------------------
<BANKED_CODE,CODE_C> 1 (was BANKED_CODE)
  Relative segment, address: CODE 0000289C - 000028C0 (0x25 bytes), align: 0
  Segment part 166.           Intra module refs:   LL_EXT_SetMaxDtmTxPower::?relay
           ENTRY                   ADDRESS         REF BY
           =====                   =======         ======
           LL_EXT_SetMaxDtmTxPower
                                   0000289C 
               ISTACK = 00000000 ( 00000002 )
    -------------------------------------------------------------------------
<BANKED_CODE,CODE_C> 1 (was BANKED_CODE)
  Relative segment, address: CODE 000028C1 - 000029B0 (0xf0 bytes), align: 0
  Segment part 168.           Intra module refs:   LL_EXT_MapPmIoPort::?relay
           ENTRY                   ADDRESS         REF BY
           =====                   =======         ======
           LL_EXT_MapPmIoPort      000028C1 
               XSTACK = 00000000 ( 0000000A )
    -------------------------------------------------------------------------
<BANKED_CODE,CODE_C> 1 (was BANKED_CODE)
  Relative segment, address: CODE 000029B1 - 00002A42 (0x92 bytes), align: 0
  Segment part 170.           Intra module refs:   LL_EXT_ExtendRfRange::?relay
           ENTRY                   ADDRESS         REF BY
           =====                   =======         ======
           LL_EXT_ExtendRfRange    000029B1 
               calls direct
               XSTACK = 00000000 ( 00000014 )
               ISTACK = 00000000 ( 00000002 )
    -------------------------------------------------------------------------
<BANKED_CODE,CODE_C> 1 (was BANKED_CODE)
  Relative segment, address: CODE 00002A43 - 00002A61 (0x1f bytes), align: 0
  Segment part 172.           Intra module refs:   LL_EXT_HaltDuringRf::?relay
           ENTRY                   ADDRESS         REF BY
           =====                   =======         ======
           LL_EXT_HaltDuringRf     00002A43 
               ISTACK = 00000000 ( 00000002 )
    -------------------------------------------------------------------------
<BANKED_CODE,CODE_C> 1 (was BANKED_CODE)
  Relative segment, address: CODE 00002A62 - 00002AA6 (0x45 bytes), align: 0
  Segment part 176.           Intra module refs:   LL_EXT_BuildRevision::?relay
           ENTRY                   ADDRESS         REF BY
           =====                   =======         ======
           LL_EXT_BuildRevision    00002A62 
               XSTACK = 00000000 ( 00000009 )
               ISTACK = 00000000 ( 00000001 )
    -------------------------------------------------------------------------
<BANKED_CODE,CODE_C> 1 (was BANKED_CODE)
  Relative segment, address: CODE 00002AA7 - 00002ADF (0x39 bytes), align: 0
  Segment part 180.           Intra module refs:   LL_EXT_ResetSystem::?relay
           ENTRY                   ADDRESS         REF BY
           =====                   =======         ======
           LL_EXT_ResetSystem      00002AA7 
               calls direct
               XSTACK = 00000000 ( 0000000D )
    -------------------------------------------------------------------------
XDATA_ID
  Relative segment, address: CODE 000001B1 - 000001BE (0xe bytes), align: 0
  Segment part 47.            Intra module refs:   taskEndCauses
    -------------------------------------------------------------------------
XDATA_ID
  Relative segment, address: CODE 000001BF - 000001CA (0xc bytes), align: 0
  Segment part 49.            Intra module refs:   taskErrorEndCauses
    -------------------------------------------------------------------------
<XDATA_ROM_C> 1 (was XDATA_ROM_C)
  Relative segment, address: CONST 00008FCC - 00008FCF (0x4 bytes), align: 0
  Segment part 53.            Intra module refs:   LL_Reset
                                                   llSetupAdv (ll_common)
           ENTRY                   ADDRESS         REF BY
           =====                   =======         ======
           __Constant_555555       00008FCC 
    -------------------------------------------------------------------------
<XDATA_ROM_C> 1 (was XDATA_ROM_C)
  Relative segment, address: CONST 00008FC4 - 00008FC7 (0x4 bytes), align: 0
  Segment part 54.            Intra module refs:   LL_DirectTestRxTest
                                                   LL_DirectTestTxTest
                                                   LL_EXT_ModemHopTestTx
                                                   LL_EXT_ModemTestRx
                                                   LL_EXT_ModemTestTx
           ENTRY                   ADDRESS         REF BY
           =====                   =======         ======
           __Constant_71764129     00008FC4 
    -------------------------------------------------------------------------
<XDATA_ROM_C> 1 (was XDATA_ROM_C)
  Relative segment, address: CONST 00008FC0 - 00008FC3 (0x4 bytes), align: 0
  Segment part 55.            Intra module refs:   LL_SetAdvControl
                                                   llScheduler (ll_scheduler)
           ENTRY                   ADDRESS         REF BY
           =====                   =======         ======
           __Constant_3            00008FC0 
    -------------------------------------------------------------------------
<XDATA_ROM_C> 1 (was XDATA_ROM_C)
  Relative segment, address: CONST 00008FAC - 00008FAF (0x4 bytes), align: 0
  Segment part 56.            Intra module refs:   LL_SetAdvControl
                                                   ll24BitTimeCompare (ll_timer2)
                                                   ll24BitTimeDelta (ll_timer2)
                                                   llDiscoverableAdvEvt_TaskEndOk (ll_advEndCauses)
                                                   llNonConnAdvEvt_TaskEndOk (ll_advEndCauses)
                                                   llScheduler (ll_scheduler)
           ENTRY                   ADDRESS         REF BY
           =====                   =======         ======
           __Constant_ffffff       00008FAC 
    -------------------------------------------------------------------------
<XDATA_ROM_C> 1 (was XDATA_ROM_C)
  Relative segment, address: CONST 00008FA4 - 00008FA7 (0x4 bytes), align: 0
  Segment part 57.            Intra module refs:   LL_EXT_ExtendRfRange
                                                   LL_EXT_SetRxGain
                                                   LL_EXT_SetTxPower
           ENTRY                   ADDRESS         REF BY
           =====                   =======         ======
           __Constant_b            00008FA4 
    -------------------------------------------------------------------------
<XDATA_ROM_C> 1 (was XDATA_ROM_C)
  Relative segment, address: CONST 00008F9C - 00008F9F (0x4 bytes), align: 0
  Segment part 58.            Intra module refs:   LL_EXT_SaveFreqTune
           ENTRY                   ADDRESS         REF BY
           =====                   =======         ======
           __Constant_ffffff00     00008F9C 
    -------------------------------------------------------------------------
BANK_RELAYS
  Relative segment, address: CODE 00000464 - 00000469 (0x6 bytes), align: 0
  Segment part 61.
           ENTRY                   ADDRESS         REF BY
           =====                   =======         ======
           LL_Init::?relay         00000464        osalInitTasks (OSAL_SimpleBLEBroadcaster)
    -------------------------------------------------------------------------
BANK_RELAYS
  Relative segment, address: CODE 0000046A - 0000046F (0x6 bytes), align: 0
  Segment part 64.
           ENTRY                   ADDRESS         REF BY
           =====                   =======         ======
           LL_ProcessEvent::?relay
                                   0000046A        tasksArr (OSAL_SimpleBLEBroadcaster)
    -------------------------------------------------------------------------
BANK_RELAYS
  Relative segment, address: CODE 00000470 - 00000475 (0x6 bytes), align: 0
  Segment part 66.
           ENTRY                   ADDRESS         REF BY
           =====                   =======         ======
           LL_TX_bm_alloc::?relay
                                   00000470        HCI_bm_alloc (hci)
    -------------------------------------------------------------------------
BANK_RELAYS
  Relative segment, address: CODE 00000476 - 0000047B (0x6 bytes), align: 0
  Segment part 70.            Intra module refs:   LL_EXT_EndModemTest
                                                   LL_Init
           ENTRY                   ADDRESS         REF BY
           =====                   =======         ======
           LL_Reset::?relay        00000476        HCI_ResetCmd (hci_PATCH)
    -------------------------------------------------------------------------
BANK_RELAYS
  Relative segment, address: CODE 0000047C - 00000481 (0x6 bytes), align: 0
  Segment part 75.
           ENTRY                   ADDRESS         REF BY
           =====                   =======         ======
           LL_ReadBDADDR::?relay   0000047C        HCI_ReadBDADDRCmd (hci)
    -------------------------------------------------------------------------
BANK_RELAYS
  Relative segment, address: CODE 00000482 - 00000487 (0x6 bytes), align: 0
  Segment part 79.
           ENTRY                   ADDRESS         REF BY
           =====                   =======         ======
           LL_SetRandomAddress::?relay
                                   00000482        HCI_LE_SetRandomAddressCmd (hci)
    -------------------------------------------------------------------------
BANK_RELAYS
  Relative segment, address: CODE 00000488 - 0000048D (0x6 bytes), align: 0
  Segment part 83.
           ENTRY                   ADDRESS         REF BY
           =====                   =======         ======
           LL_ClearWhiteList::?relay
                                   00000488        HCI_LE_ClearWhiteListCmd (hci)
    -------------------------------------------------------------------------
BANK_RELAYS
  Relative segment, address: CODE 0000048E - 00000493 (0x6 bytes), align: 0
  Segment part 85.
           ENTRY                   ADDRESS         REF BY
           =====                   =======         ======
           LL_AddWhiteListDevice::?relay
                                   0000048E        HCI_LE_AddWhiteListCmd (hci)
    -------------------------------------------------------------------------
BANK_RELAYS
  Relative segment, address: CODE 00000494 - 00000499 (0x6 bytes), align: 0
  Segment part 87.
           ENTRY                   ADDRESS         REF BY
           =====                   =======         ======
           LL_RemoveWhiteListDevice::?relay
                                   00000494        HCI_LE_RemoveWhiteListCmd (hci)
    -------------------------------------------------------------------------
BANK_RELAYS
  Relative segment, address: CODE 0000049A - 0000049F (0x6 bytes), align: 0
  Segment part 89.
           ENTRY                   ADDRESS         REF BY
           =====                   =======         ======
           LL_ReadWlSize::?relay   0000049A        HCI_LE_ReadWhiteListSizeCmd (hci)
    -------------------------------------------------------------------------
BANK_RELAYS
  Relative segment, address: CODE 000004A0 - 000004A5 (0x6 bytes), align: 0
  Segment part 93.
           ENTRY                   ADDRESS         REF BY
           =====                   =======         ======
           LL_Encrypt::?relay      000004A0        HCI_LE_EncryptCmd (hci)
    -------------------------------------------------------------------------
BANK_RELAYS
  Relative segment, address: CODE 000004A6 - 000004AB (0x6 bytes), align: 0
  Segment part 95.
           ENTRY                   ADDRESS         REF BY
           =====                   =======         ======
           LL_Rand::?relay         000004A6        HCI_LE_RandCmd (hci)
    -------------------------------------------------------------------------
BANK_RELAYS
  Relative segment, address: CODE 000004AC - 000004B1 (0x6 bytes), align: 0
  Segment part 100.
           ENTRY                   ADDRESS         REF BY
           =====                   =======         ======
           LL_ReadSupportedStates::?relay
                                   000004AC        HCI_LE_ReadSupportedStatesCmd (hci)
    -------------------------------------------------------------------------
BANK_RELAYS
  Relative segment, address: CODE 000004B2 - 000004B7 (0x6 bytes), align: 0
  Segment part 102.
           ENTRY                   ADDRESS         REF BY
           =====                   =======         ======
           LL_ReadLocalSupportedFeatures::?relay
                                   000004B2        HCI_LE_ReadLocalSupportedFeaturesCmd (hci)
    -------------------------------------------------------------------------
BANK_RELAYS
  Relative segment, address: CODE 000004B8 - 000004BD (0x6 bytes), align: 0
  Segment part 104.
           ENTRY                   ADDRESS         REF BY
           =====                   =======         ======
           LL_ReadLocalVersionInfo::?relay
                                   000004B8        HCI_ReadLocalVersionInfoCmd (hci)
    -------------------------------------------------------------------------
BANK_RELAYS
  Relative segment, address: CODE 000004BE - 000004C3 (0x6 bytes), align: 0
  Segment part 108.
           ENTRY                   ADDRESS         REF BY
           =====                   =======         ======
           LL_ReadRssi::?relay     000004BE        HCI_ReadRssiCmd (hci)
    -------------------------------------------------------------------------
BANK_RELAYS
  Relative segment, address: CODE 000004C4 - 000004C9 (0x6 bytes), align: 0
  Segment part 110.
           ENTRY                   ADDRESS         REF BY
           =====                   =======         ======
           LL_DirectTestTxTest::?relay
                                   000004C4        HCI_LE_TransmitterTestCmd (hci)
    -------------------------------------------------------------------------
BANK_RELAYS
  Relative segment, address: CODE 000004CA - 000004CF (0x6 bytes), align: 0
  Segment part 112.
           ENTRY                   ADDRESS         REF BY
           =====                   =======         ======
           LL_DirectTestRxTest::?relay
                                   000004CA        HCI_LE_ReceiverTestCmd (hci)
    -------------------------------------------------------------------------
BANK_RELAYS
  Relative segment, address: CODE 000004D0 - 000004D5 (0x6 bytes), align: 0
  Segment part 117.
           ENTRY                   ADDRESS         REF BY
           =====                   =======         ======
           LL_DirectTestEnd::?relay
                                   000004D0        HCI_LE_TestEndCmd (hci)
    -------------------------------------------------------------------------
BANK_RELAYS
  Relative segment, address: CODE 000004D6 - 000004DB (0x6 bytes), align: 0
  Segment part 120.
           ENTRY                   ADDRESS         REF BY
           =====                   =======         ======
           LL_SetAdvParam::?relay
                                   000004D6        HCI_LE_SetAdvParamCmd (hci)
    -------------------------------------------------------------------------
BANK_RELAYS
  Relative segment, address: CODE 000004DC - 000004E1 (0x6 bytes), align: 0
  Segment part 126.
           ENTRY                   ADDRESS         REF BY
           =====                   =======         ======
           LL_SetAdvData::?relay   000004DC        HCI_LE_SetAdvDataCmd (hci)
    -------------------------------------------------------------------------
BANK_RELAYS
  Relative segment, address: CODE 000004E2 - 000004E7 (0x6 bytes), align: 0
  Segment part 128.
           ENTRY                   ADDRESS         REF BY
           =====                   =======         ======
           LL_SetAdvControl::?relay
                                   000004E2        HCI_LE_SetAdvEnableCmd (hci)
    -------------------------------------------------------------------------
BANK_RELAYS
  Relative segment, address: CODE 000004E8 - 000004ED (0x6 bytes), align: 0
  Segment part 131.
           ENTRY                   ADDRESS         REF BY
           =====                   =======         ======
           LL_ReadAdvChanTxPower::?relay
                                   000004E8        HCI_LE_ReadAdvChanTxPowerCmd (hci)
    -------------------------------------------------------------------------
BANK_RELAYS
  Relative segment, address: CODE 000004EE - 000004F3 (0x6 bytes), align: 0
  Segment part 133.
           ENTRY                   ADDRESS         REF BY
           =====                   =======         ======
           LL_SetScanRspData::?relay
                                   000004EE        HCI_LE_SetScanRspDataCmd (hci)
    -------------------------------------------------------------------------
BANK_RELAYS
  Relative segment, address: CODE 000004F4 - 000004F9 (0x6 bytes), align: 0
  Segment part 136.
           ENTRY                   ADDRESS         REF BY
           =====                   =======         ======
           LL_EXT_SetRxGain::?relay
                                   000004F4        HCI_EXT_SetRxGainCmd (hci)
    -------------------------------------------------------------------------
BANK_RELAYS
  Relative segment, address: CODE 000004FA - 000004FF (0x6 bytes), align: 0
  Segment part 139.
           ENTRY                   ADDRESS         REF BY
           =====                   =======         ======
           LL_EXT_SetTxPower::?relay
                                   000004FA        HCI_EXT_SetTxPowerCmd (hci)
    -------------------------------------------------------------------------
BANK_RELAYS
  Relative segment, address: CODE 00000500 - 00000505 (0x6 bytes), align: 0
  Segment part 141.
           ENTRY                   ADDRESS         REF BY
           =====                   =======         ======
           LL_EXT_ClkDivOnHalt::?relay
                                   00000500        HCI_EXT_ClkDivOnHaltCmd (hci)
    -------------------------------------------------------------------------
BANK_RELAYS
  Relative segment, address: CODE 00000506 - 0000050B (0x6 bytes), align: 0
  Segment part 143.
           ENTRY                   ADDRESS         REF BY
           =====                   =======         ======
           LL_EXT_DeclareNvUsage::?relay
                                   00000506        HCI_EXT_DeclareNvUsageCmd (hci)
    -------------------------------------------------------------------------
BANK_RELAYS
  Relative segment, address: CODE 0000050C - 00000511 (0x6 bytes), align: 0
  Segment part 145.
           ENTRY                   ADDRESS         REF BY
           =====                   =======         ======
           LL_EXT_Decrypt::?relay
                                   0000050C        HCI_EXT_DecryptCmd (hci)
    -------------------------------------------------------------------------
BANK_RELAYS
  Relative segment, address: CODE 00000512 - 00000517 (0x6 bytes), align: 0
  Segment part 148.
           ENTRY                   ADDRESS         REF BY
           =====                   =======         ======
           LL_EXT_SetLocalSupportedFeatures::?relay
                                   00000512        HCI_EXT_SetLocalSupportedFeaturesCmd (hci)
    -------------------------------------------------------------------------
BANK_RELAYS
  Relative segment, address: CODE 00000518 - 0000051D (0x6 bytes), align: 0
  Segment part 150.
           ENTRY                   ADDRESS         REF BY
           =====                   =======         ======
           LL_EXT_ModemTestTx::?relay
                                   00000518        HCI_EXT_ModemTestTxCmd (hci)
    -------------------------------------------------------------------------
BANK_RELAYS
  Relative segment, address: CODE 0000051E - 00000523 (0x6 bytes), align: 0
  Segment part 152.
           ENTRY                   ADDRESS         REF BY
           =====                   =======         ======
           LL_EXT_ModemHopTestTx::?relay
                                   0000051E        HCI_EXT_ModemHopTestTxCmd (hci)
    -------------------------------------------------------------------------
BANK_RELAYS
  Relative segment, address: CODE 00000524 - 00000529 (0x6 bytes), align: 0
  Segment part 156.
           ENTRY                   ADDRESS         REF BY
           =====                   =======         ======
           LL_EXT_ModemTestRx::?relay
                                   00000524        HCI_EXT_ModemTestRxCmd (hci)
    -------------------------------------------------------------------------
BANK_RELAYS
  Relative segment, address: CODE 0000052A - 0000052F (0x6 bytes), align: 0
  Segment part 158.
           ENTRY                   ADDRESS         REF BY
           =====                   =======         ======
           LL_EXT_EndModemTest::?relay
                                   0000052A        HCI_EXT_EndModemTestCmd (hci)
    -------------------------------------------------------------------------
BANK_RELAYS
  Relative segment, address: CODE 00000530 - 00000535 (0x6 bytes), align: 0
  Segment part 160.
           ENTRY                   ADDRESS         REF BY
           =====                   =======         ======
           LL_EXT_SetBDADDR::?relay
                                   00000530        HCI_EXT_SetBDADDRCmd (hci)
    -------------------------------------------------------------------------
BANK_RELAYS
  Relative segment, address: CODE 00000536 - 0000053B (0x6 bytes), align: 0
  Segment part 163.
           ENTRY                   ADDRESS         REF BY
           =====                   =======         ======
           LL_EXT_SetFreqTune::?relay
                                   00000536        HCI_EXT_SetFreqTuneCmd (hci)
    -------------------------------------------------------------------------
BANK_RELAYS
  Relative segment, address: CODE 0000053C - 00000541 (0x6 bytes), align: 0
  Segment part 165.
           ENTRY                   ADDRESS         REF BY
           =====                   =======         ======
           LL_EXT_SaveFreqTune::?relay
                                   0000053C        HCI_EXT_SaveFreqTuneCmd (hci)
    -------------------------------------------------------------------------
BANK_RELAYS
  Relative segment, address: CODE 00000542 - 00000547 (0x6 bytes), align: 0
  Segment part 167.
           ENTRY                   ADDRESS         REF BY
           =====                   =======         ======
           LL_EXT_SetMaxDtmTxPower::?relay
                                   00000542        HCI_EXT_SetMaxDtmTxPowerCmd (hci)
    -------------------------------------------------------------------------
BANK_RELAYS
  Relative segment, address: CODE 00000548 - 0000054D (0x6 bytes), align: 0
  Segment part 169.
           ENTRY                   ADDRESS         REF BY
           =====                   =======         ======
           LL_EXT_MapPmIoPort::?relay
                                   00000548        HCI_EXT_MapPmIoPortCmd (hci)
    -------------------------------------------------------------------------
BANK_RELAYS
  Relative segment, address: CODE 0000054E - 00000553 (0x6 bytes), align: 0
  Segment part 171.
           ENTRY                   ADDRESS         REF BY
           =====                   =======         ======
           LL_EXT_ExtendRfRange::?relay
                                   0000054E        HCI_EXT_ExtendRfRangeCmd (hci)
    -------------------------------------------------------------------------
BANK_RELAYS
  Relative segment, address: CODE 00000554 - 00000559 (0x6 bytes), align: 0
  Segment part 173.
           ENTRY                   ADDRESS         REF BY
           =====                   =======         ======
           LL_EXT_HaltDuringRf::?relay
                                   00000554        HCI_EXT_HaltDuringRfCmd (hci)
    -------------------------------------------------------------------------
BANK_RELAYS
  Relative segment, address: CODE 0000055A - 0000055F (0x6 bytes), align: 0
  Segment part 177.
           ENTRY                   ADDRESS         REF BY
           =====                   =======         ======
           LL_EXT_BuildRevision::?relay
                                   0000055A        HCI_EXT_BuildRevisionCmd (hci)
    -------------------------------------------------------------------------
BANK_RELAYS
  Relative segment, address: CODE 00000560 - 00000565 (0x6 bytes), align: 0
  Segment part 181.
           ENTRY                   ADDRESS         REF BY
           =====                   =======         ======
           LL_EXT_ResetSystem::?relay
                                   00000560        HCI_EXT_ResetSystemCmd (hci_PATCH)
    -------------------------------------------------------------------------
<BANKED_CODE,XDATA_ROM_C_FLASH> 1 (was XDATA_ROM_C_FLASH)
  Relative segment, address: CODE 00008EFF - 00008F23 (0x25 bytes), align: 0
  Segment part 186.           Intra module refs:   psbs9Data
    -------------------------------------------------------------------------
<BANKED_CODE,XDATA_ROM_C_FLASH> 1 (was XDATA_ROM_C_FLASH)
  Relative segment, address: CODE 00008FCC - 00008FCF (0x4 bytes), align: 0
  Segment part 187.           Intra module refs:   __Constant_555555
    -------------------------------------------------------------------------
<BANKED_CODE,XDATA_ROM_C_FLASH> 1 (was XDATA_ROM_C_FLASH)
  Relative segment, address: CODE 00008FC4 - 00008FC7 (0x4 bytes), align: 0
  Segment part 188.           Intra module refs:   __Constant_71764129
    -------------------------------------------------------------------------
<BANKED_CODE,XDATA_ROM_C_FLASH> 1 (was XDATA_ROM_C_FLASH)
  Relative segment, address: CODE 00008FC0 - 00008FC3 (0x4 bytes), align: 0
  Segment part 189.           Intra module refs:   __Constant_3
    -------------------------------------------------------------------------
<BANKED_CODE,XDATA_ROM_C_FLASH> 1 (was XDATA_ROM_C_FLASH)
  Relative segment, address: CODE 00008FAC - 00008FAF (0x4 bytes), align: 0
  Segment part 190.           Intra module refs:   __Constant_ffffff
    -------------------------------------------------------------------------
<BANKED_CODE,XDATA_ROM_C_FLASH> 1 (was XDATA_ROM_C_FLASH)
  Relative segment, address: CODE 00008FA4 - 00008FA7 (0x4 bytes), align: 0
  Segment part 191.           Intra module refs:   __Constant_b
    -------------------------------------------------------------------------
<BANKED_CODE,XDATA_ROM_C_FLASH> 1 (was XDATA_ROM_C_FLASH)
  Relative segment, address: CODE 00008F9C - 00008F9F (0x4 bytes), align: 0
  Segment part 192.           Intra module refs:   __Constant_ffffff00

    -------------------------------------------------------------------------
  LIBRARY MODULE, NAME : ll_advEndCauses

  SEGMENTS IN THE MODULE
  ======================
<BANKED_CODE,XDATA_ROM_C_FLASH> 1 (was BANKED_CODE)
  Relative segment, address: CODE 0000B3C4 - 0000B47D (0xba bytes), align: 0
  Segment part 10.            Intra module refs:   llDiscoverableAdvEvt_TaskEndOk::?relay
           ENTRY                   ADDRESS         REF BY
           =====                   =======         ======
           llDiscoverableAdvEvt_TaskEndOk
                                   0000B3C4 
               calls direct
               XSTACK = 00000000 ( 00000010 )
    -------------------------------------------------------------------------
<BANKED_CODE,XDATA_ROM_C_FLASH> 1 (was BANKED_CODE)
  Relative segment, address: CODE 0000B47E - 0000B485 (0x8 bytes), align: 0
  Segment part 12.            Intra module refs:   llDiscoverableAdvEvt_TaskEndOk
                                                   llNonConnAdvEvt_TaskEndOk
    -------------------------------------------------------------------------
<BANKED_CODE,XDATA_ROM_C_FLASH> 1 (was BANKED_CODE)
  Relative segment, address: CODE 0000B486 - 0000B50E (0x89 bytes), align: 0
  Segment part 13.            Intra module refs:   llNonConnAdvEvt_TaskEndOk::?relay
           ENTRY                   ADDRESS         REF BY
           =====                   =======         ======
           llNonConnAdvEvt_TaskEndOk
                                   0000B486 
               calls direct
               XSTACK = 00000000 ( 00000010 )
    -------------------------------------------------------------------------
<BANKED_CODE,XDATA_ROM_C_FLASH> 1 (was BANKED_CODE)
  Relative segment, address: CODE 0000B50F - 0000B51F (0x11 bytes), align: 0
  Segment part 15.            Intra module refs:   llDiscoverableAdvEvt_TaskEndOk
                                                   llNonConnAdvEvt_TaskEndOk
    -------------------------------------------------------------------------
<BANKED_CODE,XDATA_ROM_C_FLASH> 1 (was BANKED_CODE)
  Relative segment, address: CODE 0000B520 - 0000B533 (0x14 bytes), align: 0
  Segment part 16.            Intra module refs:   llDiscoverableAdvEvt_TaskEndOk
                                                   llNonConnAdvEvt_TaskEndOk
    -------------------------------------------------------------------------
<BANKED_CODE,XDATA_ROM_C_FLASH> 1 (was BANKED_CODE)
  Relative segment, address: CODE 0000B534 - 0000B548 (0x15 bytes), align: 0
  Segment part 17.            Intra module refs:   llDiscoverableAdvEvt_TaskEndOk
                                                   llNonConnAdvEvt_TaskEndOk
    -------------------------------------------------------------------------
<BANKED_CODE,XDATA_ROM_C_FLASH> 1 (was BANKED_CODE)
  Relative segment, address: CODE 0000B549 - 0000B55B (0x13 bytes), align: 0
  Segment part 18.            Intra module refs:   llDiscoverableAdvEvt_TaskEndOk
                                                   llNonConnAdvEvt_TaskEndOk
    -------------------------------------------------------------------------
<BANKED_CODE,XDATA_ROM_C_FLASH> 1 (was BANKED_CODE)
  Relative segment, address: CODE 0000B55C - 0000B570 (0x15 bytes), align: 0
  Segment part 19.            Intra module refs:   llDiscoverableAdvEvt_TaskEndOk
                                                   llNonConnAdvEvt_TaskEndOk
    -------------------------------------------------------------------------
<BANKED_CODE,XDATA_ROM_C_FLASH> 1 (was BANKED_CODE)
  Relative segment, address: CODE 0000B571 - 0000B59B (0x2b bytes), align: 0
  Segment part 20.            Intra module refs:   llDiscoverableAdvEvt_TaskEndOk
                                                   llNonConnAdvEvt_TaskEndOk
    -------------------------------------------------------------------------
<BANKED_CODE,XDATA_ROM_C_FLASH> 1 (was BANKED_CODE)
  Relative segment, address: CODE 0000B59C - 0000B5C9 (0x2e bytes), align: 0
  Segment part 21.            Intra module refs:   llDiscoverableAdvEvt_TaskEndOk
                                                   llNonConnAdvEvt_TaskEndOk
    -------------------------------------------------------------------------
<BANKED_CODE,XDATA_ROM_C_FLASH> 1 (was BANKED_CODE)
  Relative segment, address: CODE 0000B5CA - 0000B5CB (0x2 bytes), align: 0
  Segment part 22.            Intra module refs:   Segment part 21
    -------------------------------------------------------------------------
<BANKED_CODE,XDATA_ROM_C_FLASH> 1 (was BANKED_CODE)
  Relative segment, address: CODE 0000B5CC - 0000B5D5 (0xa bytes), align: 0
  Segment part 23.            Intra module refs:   Segment part 18
                                                   Segment part 22
    -------------------------------------------------------------------------
<BANKED_CODE,XDATA_ROM_C_FLASH> 1 (was BANKED_CODE)
  Relative segment, address: CODE 0000B5D6 - 0000B5FF (0x2a bytes), align: 0
  Segment part 24.            Intra module refs:   llAdvEvt_TaskAbort::?relay
           ENTRY                   ADDRESS         REF BY
           =====                   =======         ======
           llAdvEvt_TaskAbort      0000B5D6 
               calls direct
               ISTACK = 00000000 ( 00000002 )
    -------------------------------------------------------------------------
BANK_RELAYS
  Relative segment, address: CODE 00000566 - 0000056B (0x6 bytes), align: 0
  Segment part 11.
           ENTRY                   ADDRESS         REF BY
           =====                   =======         ======
           llDiscoverableAdvEvt_TaskEndOk::?relay
                                   00000566        llSetupScannableAdvEvt (ll_common)
    -------------------------------------------------------------------------
BANK_RELAYS
  Relative segment, address: CODE 0000056C - 00000571 (0x6 bytes), align: 0
  Segment part 14.
           ENTRY                   ADDRESS         REF BY
           =====                   =======         ======
           llNonConnAdvEvt_TaskEndOk::?relay
                                   0000056C        Segment part 79 (ll_common)
                                                   Segment part 80 (ll_common)
    -------------------------------------------------------------------------
BANK_RELAYS
  Relative segment, address: CODE 00000572 - 00000577 (0x6 bytes), align: 0
  Segment part 25.
           ENTRY                   ADDRESS         REF BY
           =====                   =======         ======
           llAdvEvt_TaskAbort::?relay
                                   00000572        Segment part 84 (ll_common)

    -------------------------------------------------------------------------
  LIBRARY MODULE, NAME : ll_common

  SEGMENTS IN THE MODULE
  ======================
SFR_AN
  Relative segment, address: DATA 00000088 - 00000088 (0x1 bytes), align: 0
  Segment part 1. ROOT        Intra module refs:   llClearSetInts
           ENTRY                   ADDRESS         REF BY
           =====                   =======         ======
           _A_TCON                 00000088 
    -------------------------------------------------------------------------
SFR_AN
  Relative segment, address: DATA 000000A9 - 000000A9 (0x1 bytes), align: 0
  Segment part 7. ROOT        Intra module refs:   llClearSetInts
           ENTRY                   ADDRESS         REF BY
           =====                   =======         ======
           IP0                     000000A9 
    -------------------------------------------------------------------------
SFR_AN
  Relative segment, address: DATA 000000AF - 000000AF (0x1 bytes), align: 0
  Segment part 8. ROOT 
           ENTRY                   ADDRESS         REF BY
           =====                   =======         ======
           T1STAT                  000000AF 
    -------------------------------------------------------------------------
SFR_AN
  Relative segment, address: DATA 000000B9 - 000000B9 (0x1 bytes), align: 0
  Segment part 10. ROOT       Intra module refs:   llClearSetInts
           ENTRY                   ADDRESS         REF BY
           =====                   =======         ======
           IP1                     000000B9 
    -------------------------------------------------------------------------
SFR_AN
  Relative segment, address: DATA 000000DA - 000000DA (0x1 bytes), align: 0
  Segment part 13. ROOT 
           ENTRY                   ADDRESS         REF BY
           =====                   =======         ======
           T1CC0L                  000000DA 
    -------------------------------------------------------------------------
SFR_AN
  Relative segment, address: DATA 000000DB - 000000DB (0x1 bytes), align: 0
  Segment part 14. ROOT 
           ENTRY                   ADDRESS         REF BY
           =====                   =======         ======
           T1CC0H                  000000DB 
    -------------------------------------------------------------------------
SFR_AN
  Relative segment, address: DATA 000000E2 - 000000E2 (0x1 bytes), align: 0
  Segment part 15. ROOT 
           ENTRY                   ADDRESS         REF BY
           =====                   =======         ======
           T1CNTL                  000000E2 
    -------------------------------------------------------------------------
SFR_AN
  Relative segment, address: DATA 000000E3 - 000000E3 (0x1 bytes), align: 0
  Segment part 16. ROOT 
           ENTRY                   ADDRESS         REF BY
           =====                   =======         ======
           T1CNTH                  000000E3 
    -------------------------------------------------------------------------
SFR_AN
  Relative segment, address: DATA 000000E4 - 000000E4 (0x1 bytes), align: 0
  Segment part 17. ROOT 
           ENTRY                   ADDRESS         REF BY
           =====                   =======         ======
           T1CTL                   000000E4 
    -------------------------------------------------------------------------
SFR_AN
  Relative segment, address: DATA 000000E5 - 000000E5 (0x1 bytes), align: 0
  Segment part 18. ROOT 
           ENTRY                   ADDRESS         REF BY
           =====                   =======         ======
           T1CCTL0                 000000E5 
    -------------------------------------------------------------------------
<BANKED_CODE,CODE_C> 1 (was BANKED_CODE)
  Relative segment, address: CODE 0000663B - 00006683 (0x49 bytes), align: 0
  Segment part 40.            Intra module refs:   llRfInit::?relay
           ENTRY                   ADDRESS         REF BY
           =====                   =======         ======
           llRfInit                0000663B 
               calls direct
               ISTACK = 00000000 ( 00000002 )
    -------------------------------------------------------------------------
<BANKED_CODE,CODE_C> 1 (was BANKED_CODE)
  Relative segment, address: CODE 00006684 - 000066B0 (0x2d bytes), align: 0
  Segment part 42.            Intra module refs:   llSetFreqTune::?relay
           ENTRY                   ADDRESS         REF BY
           =====                   =======         ======
           llSetFreqTune           00006684 
               ISTACK = 00000000 ( 00000002 )
    -------------------------------------------------------------------------
<BANKED_CODE,CODE_C> 1 (was BANKED_CODE)
  Relative segment, address: CODE 000066B1 - 000066E2 (0x32 bytes), align: 0
  Segment part 44.            Intra module refs:   llClearSetInts::?relay
           ENTRY                   ADDRESS         REF BY
           =====                   =======         ======
           llClearSetInts          000066B1 
               calls direct
               XSTACK = 00000000 ( 00000009 )
    -------------------------------------------------------------------------
<BANKED_CODE,CODE_C> 1 (was BANKED_CODE)
  Relative segment, address: CODE 000066E3 - 000066EF (0xd bytes), align: 0
  Segment part 46.            Intra module refs:   llDisableRfInts::?relay
           ENTRY                   ADDRESS         REF BY
           =====                   =======         ======
           llDisableRfInts         000066E3 
               XSTACK = 00000009 ( 00000000 )
               ISTACK = 00000000 ( 00000002 )
    -------------------------------------------------------------------------
<BANKED_CODE,CODE_C> 1 (was BANKED_CODE)
  Relative segment, address: CODE 000066F0 - 000066FB (0xc bytes), align: 0
  Segment part 48.            Intra module refs:   llClearRfInts::?relay
           ENTRY                   ADDRESS         REF BY
           =====                   =======         ======
           llClearRfInts           000066F0 
               XSTACK = 00000009 ( 00000000 )
    -------------------------------------------------------------------------
<BANKED_CODE,CODE_C> 1 (was BANKED_CODE)
  Relative segment, address: CODE 000066FC - 0000670D (0x12 bytes), align: 0
  Segment part 50.            Intra module refs:   llEnableRfInts::?relay
           ENTRY                   ADDRESS         REF BY
           =====                   =======         ======
           llEnableRfInts          000066FC 
               XSTACK = 00000009 ( 00000000 )
               ISTACK = 00000000 ( 00000002 )
    -------------------------------------------------------------------------
<BANKED_CODE,CODE_C> 1 (was BANKED_CODE)
  Relative segment, address: CODE 0000670E - 000067D5 (0xc8 bytes), align: 0
  Segment part 52.            Intra module refs:   llProcessPostRfOps::?relay
           ENTRY                   ADDRESS         REF BY
           =====                   =======         ======
           llProcessPostRfOps      0000670E 
               calls direct
               XSTACK = 00000000 ( 00000008 )
               ISTACK = 00000000 ( 00000002 )
    -------------------------------------------------------------------------
<BANKED_CODE,CODE_C> 1 (was BANKED_CODE)
  Relative segment, address: CODE 000067D6 - 00006832 (0x5d bytes), align: 0
  Segment part 54.            Intra module refs:   llSetRxGain::?relay
           ENTRY                   ADDRESS         REF BY
           =====                   =======         ======
           llSetRxGain             000067D6 
               XSTACK = 00000008 ( 00000000 )
               ISTACK = 00000000 ( 00000002 )
    -------------------------------------------------------------------------
<BANKED_CODE,CODE_C> 1 (was BANKED_CODE)
  Relative segment, address: CODE 00006833 - 00006866 (0x34 bytes), align: 0
  Segment part 56.            Intra module refs:   llSetTxPower::?relay
           ENTRY                   ADDRESS         REF BY
           =====                   =======         ======
           llSetTxPower            00006833 
               XSTACK = 00000008 ( 00000000 )
               ISTACK = 00000000 ( 00000002 )
    -------------------------------------------------------------------------
<BANKED_CODE,CODE_C> 1 (was BANKED_CODE)
  Relative segment, address: CODE 00006867 - 00006868 (0x2 bytes), align: 0
  Segment part 58.            Intra module refs:   llDisableRfInts
                                                   llStartAdvSetup
    -------------------------------------------------------------------------
<BANKED_CODE,CODE_C> 1 (was BANKED_CODE)
  Relative segment, address: CODE 00006869 - 00006869 (0x1 bytes), align: 0
  Segment part 59.            Intra module refs:   Segment part 58
                                                   llEnableRfInts
                                                   llInitFeatureSet
    -------------------------------------------------------------------------
<BANKED_CODE,CODE_C> 1 (was BANKED_CODE)
  Relative segment, address: CODE 0000686A - 00006870 (0x7 bytes), align: 0
  Segment part 60.            Intra module refs:   Segment part 59
                                                   llCheckWhiteListUsage
                                                   llExtendRfRange
                                                   llGetTxPower
                                                   llProcessPostRfOps
                                                   llRfInit
                                                   llSetFreqTune
                                                   llSetRxGain
                                                   llSetTxPower
                                                   llSetupAdv
    -------------------------------------------------------------------------
<BANKED_CODE,CODE_C> 1 (was BANKED_CODE)
  Relative segment, address: CODE 00006871 - 000068A3 (0x33 bytes), align: 0
  Segment part 61.            Intra module refs:   llGetTxPower::?relay
           ENTRY                   ADDRESS         REF BY
           =====                   =======         ======
           llGetTxPower            00006871 
               ISTACK = 00000000 ( 00000002 )
    -------------------------------------------------------------------------
<BANKED_CODE,CODE_C> 1 (was BANKED_CODE)
  Relative segment, address: CODE 000068A4 - 000069C5 (0x122 bytes), align: 0
  Segment part 63.            Intra module refs:   llFindTxPowerSettings::?relay
           ENTRY                   ADDRESS         REF BY
           =====                   =======         ======
           llFindTxPowerSettings   000068A4 
               calls direct
               XSTACK = 00000000 ( 00000020 )
               ISTACK = 00000000 ( 00000001 )
    -------------------------------------------------------------------------
<BANKED_CODE,CODE_C> 1 (was BANKED_CODE)
  Relative segment, address: CODE 000069C6 - 000069D4 (0xf bytes), align: 0
  Segment part 65.            Intra module refs:   llFindTxPowerSettings
    -------------------------------------------------------------------------
<BANKED_CODE,CODE_C> 1 (was BANKED_CODE)
  Relative segment, address: CODE 000069D5 - 00006A21 (0x4d bytes), align: 0
  Segment part 66.            Intra module refs:   llExtendRfRange::?relay
           ENTRY                   ADDRESS         REF BY
           =====                   =======         ======
           llExtendRfRange         000069D5 
               calls direct
               XSTACK = 00000008 ( 00000000 )
               ISTACK = 00000000 ( 00000002 )
    -------------------------------------------------------------------------
<BANKED_CODE,CODE_C> 1 (was BANKED_CODE)
  Relative segment, address: CODE 00006A22 - 00006A3C (0x1b bytes), align: 0
  Segment part 71.            Intra module refs:   llCheckWhiteListUsage::?relay
           ENTRY                   ADDRESS         REF BY
           =====                   =======         ======
           llCheckWhiteListUsage   00006A22 
               ISTACK = 00000000 ( 00000002 )
    -------------------------------------------------------------------------
<BANKED_CODE,CODE_C> 1 (was BANKED_CODE)
  Relative segment, address: CODE 00006A3D - 00006AA1 (0x65 bytes), align: 0
  Segment part 73.            Intra module refs:   llSetupAdv::?relay
           ENTRY                   ADDRESS         REF BY
           =====                   =======         ======
           llSetupAdv              00006A3D 
               calls direct
               ISTACK = 00000000 ( 00000002 )
    -------------------------------------------------------------------------
<BANKED_CODE,CODE_C> 1 (was BANKED_CODE)
  Relative segment, address: CODE 00006AA2 - 00006AE2 (0x41 bytes), align: 0
  Segment part 75.            Intra module refs:   llSetupNonConnectableAdvEvt::?relay
           ENTRY                   ADDRESS         REF BY
           =====                   =======         ======
           llSetupNonConnectableAdvEvt
                                   00006AA2 
               XSTACK = 00000000 ( 00000009 )
    -------------------------------------------------------------------------
<BANKED_CODE,CODE_C> 1 (was BANKED_CODE)
  Relative segment, address: CODE 00006AE3 - 00006AEC (0xa bytes), align: 0
  Segment part 77.            Intra module refs:   llSetupNonConnectableAdvEvt
                                                   llSetupScannableAdvEvt
    -------------------------------------------------------------------------
<BANKED_CODE,CODE_C> 1 (was BANKED_CODE)
  Relative segment, address: CODE 00006AED - 00006AF2 (0x6 bytes), align: 0
  Segment part 78.            Intra module refs:   Segment part 77
    -------------------------------------------------------------------------
<BANKED_CODE,CODE_C> 1 (was BANKED_CODE)
  Relative segment, address: CODE 00006AF3 - 00006AFF (0xd bytes), align: 0
  Segment part 79.            Intra module refs:   llSetupNonConnectableAdvEvt
    -------------------------------------------------------------------------
<BANKED_CODE,CODE_C> 1 (was BANKED_CODE)
  Relative segment, address: CODE 00006B00 - 00006B08 (0x9 bytes), align: 0
  Segment part 80.            Intra module refs:   Segment part 79
    -------------------------------------------------------------------------
<BANKED_CODE,CODE_C> 1 (was BANKED_CODE)
  Relative segment, address: CODE 00006B09 - 00006B77 (0x6f bytes), align: 0
  Segment part 81.            Intra module refs:   llSetupScannableAdvEvt::?relay
           ENTRY                   ADDRESS         REF BY
           =====                   =======         ======
           llSetupScannableAdvEvt
                                   00006B09 
               XSTACK = 00000000 ( 00000009 )
    -------------------------------------------------------------------------
<BANKED_CODE,CODE_C> 1 (was BANKED_CODE)
  Relative segment, address: CODE 00006B78 - 00006B8B (0x14 bytes), align: 0
  Segment part 83.            Intra module refs:   llSetupNonConnectableAdvEvt
                                                   llSetupScannableAdvEvt
    -------------------------------------------------------------------------
<BANKED_CODE,CODE_C> 1 (was BANKED_CODE)
  Relative segment, address: CODE 00006B8C - 00006BB8 (0x2d bytes), align: 0
  Segment part 84.            Intra module refs:   llSetupNonConnectableAdvEvt
                                                   llSetupScannableAdvEvt
    -------------------------------------------------------------------------
<BANKED_CODE,CODE_C> 1 (was BANKED_CODE)
  Relative segment, address: CODE 00006BB9 - 00006BC2 (0xa bytes), align: 0
  Segment part 85.            Intra module refs:   Segment part 84
    -------------------------------------------------------------------------
<BANKED_CODE,CODE_C> 1 (was BANKED_CODE)
  Relative segment, address: CODE 00006BC3 - 00006BCD (0xb bytes), align: 0
  Segment part 88.            Intra module refs:   Segment part 84
    -------------------------------------------------------------------------
<BANKED_CODE,CODE_C> 1 (was BANKED_CODE)
  Relative segment, address: CODE 00006BCE - 00006BD1 (0x4 bytes), align: 0
  Segment part 93.            Intra module refs:   llSetupScannableAdvEvt
    -------------------------------------------------------------------------
<BANKED_CODE,CODE_C> 1 (was BANKED_CODE)
  Relative segment, address: CODE 00006BD2 - 00006BE0 (0xf bytes), align: 0
  Segment part 94.            Intra module refs:   Segment part 84
                                                   Segment part 93
    -------------------------------------------------------------------------
<BANKED_CODE,CODE_C> 1 (was BANKED_CODE)
  Relative segment, address: CODE 00006BE1 - 00006BE7 (0x7 bytes), align: 0
  Segment part 95.            Intra module refs:   Segment part 94
    -------------------------------------------------------------------------
<BANKED_CODE,CODE_C> 1 (was BANKED_CODE)
  Relative segment, address: CODE 00006BE8 - 00006BF0 (0x9 bytes), align: 0
  Segment part 96.            Intra module refs:   Segment part 95
    -------------------------------------------------------------------------
<BANKED_CODE,CODE_C> 1 (was BANKED_CODE)
  Relative segment, address: CODE 00006BF1 - 00006BF5 (0x5 bytes), align: 0
  Segment part 98.            Intra module refs:   llClearSetInts
                                                   llSetupNonConnectableAdvEvt
                                                   llSetupScannableAdvEvt
    -------------------------------------------------------------------------
<BANKED_CODE,CODE_C> 1 (was BANKED_CODE)
  Relative segment, address: CODE 00006BF6 - 00006C0D (0x18 bytes), align: 0
  Segment part 101.           Intra module refs:   llStartAdvSetup::?relay
           ENTRY                   ADDRESS         REF BY
           =====                   =======         ======
           llStartAdvSetup         00006BF6 
               is indirectly called
               ISTACK = 00000000 ( 00000002 )
    -------------------------------------------------------------------------
<BANKED_CODE,CODE_C> 1 (was BANKED_CODE)
  Relative segment, address: CODE 00006C0E - 00006C14 (0x7 bytes), align: 0
  Segment part 112.           Intra module refs:   llSetupNonConnectableAdvEvt
                                                   llSetupScannableAdvEvt
    -------------------------------------------------------------------------
<BANKED_CODE,CODE_C> 1 (was BANKED_CODE)
  Relative segment, address: CODE 00006C15 - 00006C1D (0x9 bytes), align: 0
  Segment part 122.           Intra module refs:   Segment part 78
    -------------------------------------------------------------------------
<BANKED_CODE,CODE_C> 1 (was BANKED_CODE)
  Relative segment, address: CODE 00006C1E - 00006C1F (0x2 bytes), align: 0
  Segment part 128.           Intra module refs:   llFindTxPowerSettings
    -------------------------------------------------------------------------
<BANKED_CODE,CODE_C> 1 (was BANKED_CODE)
  Relative segment, address: CODE 00006C20 - 00006C23 (0x4 bytes), align: 0
  Segment part 129.           Intra module refs:   Segment part 128
                                                   llProcessPostRfOps
    -------------------------------------------------------------------------
<BANKED_CODE,CODE_C> 1 (was BANKED_CODE)
  Relative segment, address: CODE 00006C24 - 00006C29 (0x6 bytes), align: 0
  Segment part 130.           Intra module refs:   Segment part 129
    -------------------------------------------------------------------------
<BANKED_CODE,CODE_C> 1 (was BANKED_CODE)
  Relative segment, address: CODE 00006C2A - 00006C2D (0x4 bytes), align: 0
  Segment part 186.           Intra module refs:   llSetupNonConnectableAdvEvt
                                                   llSetupScannableAdvEvt
    -------------------------------------------------------------------------
<BANKED_CODE,CODE_C> 1 (was BANKED_CODE)
  Relative segment, address: CODE 00006C2E - 00006C32 (0x5 bytes), align: 0
  Segment part 187.           Intra module refs:   Segment part 186
                                                   llGetTxPower
                                                   llSetupScannableAdvEvt
    -------------------------------------------------------------------------
<BANKED_CODE,CODE_C> 1 (was BANKED_CODE)
  Relative segment, address: CODE 00006C33 - 00006C47 (0x15 bytes), align: 0
  Segment part 188.           Intra module refs:   llInitFeatureSet::?relay
           ENTRY                   ADDRESS         REF BY
           =====                   =======         ======
           llInitFeatureSet        00006C33 
               ISTACK = 00000000 ( 00000002 )
    -------------------------------------------------------------------------
BANK_RELAYS
  Relative segment, address: CODE 00000578 - 0000057D (0x6 bytes), align: 0
  Segment part 41.
           ENTRY                   ADDRESS         REF BY
           =====                   =======         ======
           llRfInit::?relay        00000578        LL_DirectTestEnd (ll)
                                                   LL_ENC_GenerateTrueRandNum (ll_enc)
                                                   LL_Reset (ll)
    -------------------------------------------------------------------------
BANK_RELAYS
  Relative segment, address: CODE 0000057E - 00000583 (0x6 bytes), align: 0
  Segment part 43.            Intra module refs:   llRfInit
           ENTRY                   ADDRESS         REF BY
           =====                   =======         ======
           llSetFreqTune::?relay   0000057E        LL_EXT_SetFreqTune (ll)
    -------------------------------------------------------------------------
BANK_RELAYS
  Relative segment, address: CODE 00000584 - 00000589 (0x6 bytes), align: 0
  Segment part 45.
           ENTRY                   ADDRESS         REF BY
           =====                   =======         ======
           llClearSetInts::?relay
                                   00000584        LL_DirectTestEnd (ll)
                                                   LL_Reset (ll)
    -------------------------------------------------------------------------
BANK_RELAYS
  Relative segment, address: CODE 0000058A - 0000058F (0x6 bytes), align: 0
  Segment part 47.            Intra module refs:   llClearSetInts
           ENTRY                   ADDRESS         REF BY
           =====                   =======         ======
           llDisableRfInts::?relay
                                   0000058A        LL_DirectTestRxTest (ll)
                                                   LL_DirectTestTxTest (ll)
                                                   LL_EXT_ModemHopTestTx (ll)
                                                   LL_EXT_ModemTestRx (ll)
                                                   LL_EXT_ModemTestTx (ll)
    -------------------------------------------------------------------------
BANK_RELAYS
  Relative segment, address: CODE 00000590 - 00000595 (0x6 bytes), align: 0
  Segment part 49.            Intra module refs:   llClearSetInts
           ENTRY                   ADDRESS         REF BY
           =====                   =======         ======
           llClearRfInts::?relay   00000590 
    -------------------------------------------------------------------------
BANK_RELAYS
  Relative segment, address: CODE 00000596 - 0000059B (0x6 bytes), align: 0
  Segment part 51.            Intra module refs:   llClearSetInts
           ENTRY                   ADDRESS         REF BY
           =====                   =======         ======
           llEnableRfInts::?relay
                                   00000596 
    -------------------------------------------------------------------------
BANK_RELAYS
  Relative segment, address: CODE 0000059C - 000005A1 (0x6 bytes), align: 0
  Segment part 53.
           ENTRY                   ADDRESS         REF BY
           =====                   =======         ======
           llProcessPostRfOps::?relay
                                   0000059C        RF_NormalIsr (ll_isr)
                                                   llScheduler (ll_scheduler)
    -------------------------------------------------------------------------
BANK_RELAYS
  Relative segment, address: CODE 000005A2 - 000005A7 (0x6 bytes), align: 0
  Segment part 55.            Intra module refs:   llExtendRfRange
                                                   llProcessPostRfOps
                                                   llRfInit
           ENTRY                   ADDRESS         REF BY
           =====                   =======         ======
           llSetRxGain::?relay     000005A2        LL_ENC_GenerateTrueRandNum (ll_enc)
                                                   LL_EXT_SetRxGain (ll)
    -------------------------------------------------------------------------
BANK_RELAYS
  Relative segment, address: CODE 000005A8 - 000005AD (0x6 bytes), align: 0
  Segment part 57.            Intra module refs:   llProcessPostRfOps
                                                   llRfInit
           ENTRY                   ADDRESS         REF BY
           =====                   =======         ======
           llSetTxPower::?relay    000005A8        LL_DirectTestTxTest (ll)
                                                   LL_EXT_SetTxPower (ll)
    -------------------------------------------------------------------------
BANK_RELAYS
  Relative segment, address: CODE 000005AE - 000005B3 (0x6 bytes), align: 0
  Segment part 62.
           ENTRY                   ADDRESS         REF BY
           =====                   =======         ======
           llGetTxPower::?relay    000005AE        LL_ReadAdvChanTxPower (ll)
    -------------------------------------------------------------------------
BANK_RELAYS
  Relative segment, address: CODE 000005B4 - 000005B9 (0x6 bytes), align: 0
  Segment part 64.
           ENTRY                   ADDRESS         REF BY
           =====                   =======         ======
           llFindTxPowerSettings::?relay
                                   000005B4        LL_Init (ll)
    -------------------------------------------------------------------------
BANK_RELAYS
  Relative segment, address: CODE 000005BA - 000005BF (0x6 bytes), align: 0
  Segment part 67.            Intra module refs:   llProcessPostRfOps
           ENTRY                   ADDRESS         REF BY
           =====                   =======         ======
           llExtendRfRange::?relay
                                   000005BA        LL_EXT_ExtendRfRange (ll)
    -------------------------------------------------------------------------
BANK_RELAYS
  Relative segment, address: CODE 000005C0 - 000005C5 (0x6 bytes), align: 0
  Segment part 72.
           ENTRY                   ADDRESS         REF BY
           =====                   =======         ======
           llCheckWhiteListUsage::?relay
                                   000005C0        LL_AddWhiteListDevice (ll)
                                                   LL_ClearWhiteList (ll)
                                                   LL_RemoveWhiteListDevice (ll)
    -------------------------------------------------------------------------
BANK_RELAYS
  Relative segment, address: CODE 000005C6 - 000005CB (0x6 bytes), align: 0
  Segment part 74.
           ENTRY                   ADDRESS         REF BY
           =====                   =======         ======
           llSetupAdv::?relay      000005C6        LL_SetAdvControl (ll)
                                                   llScheduler (ll_scheduler)
    -------------------------------------------------------------------------
BANK_RELAYS
  Relative segment, address: CODE 000005CC - 000005D1 (0x6 bytes), align: 0
  Segment part 76.            Intra module refs:   llSetupAdv
           ENTRY                   ADDRESS         REF BY
           =====                   =======         ======
           llSetupNonConnectableAdvEvt::?relay
                                   000005CC 
    -------------------------------------------------------------------------
BANK_RELAYS
  Relative segment, address: CODE 000005D2 - 000005D7 (0x6 bytes), align: 0
  Segment part 82.            Intra module refs:   llSetupAdv
           ENTRY                   ADDRESS         REF BY
           =====                   =======         ======
           llSetupScannableAdvEvt::?relay
                                   000005D2 
    -------------------------------------------------------------------------
BANK_RELAYS
  Relative segment, address: CODE 000005D8 - 000005DD (0x6 bytes), align: 0
  Segment part 102.           Intra module refs:   llSetupAdv
           ENTRY                   ADDRESS         REF BY
           =====                   =======         ======
           llStartAdvSetup::?relay
                                   000005D8        Segment part 18 (ll_advEndCauses)
    -------------------------------------------------------------------------
BANK_RELAYS
  Relative segment, address: CODE 000005DE - 000005E3 (0x6 bytes), align: 0
  Segment part 189.
           ENTRY                   ADDRESS         REF BY
           =====                   =======         ======
           llInitFeatureSet::?relay
                                   000005DE        LL_Reset (ll)
    -------------------------------------------------------------------------
<XDATA_ROM_C> 1 (was XDATA_ROM_C)
  Relative segment, address: CONST 00008FA0 - 00008FA3 (0x4 bytes), align: 0
  Segment part 31.            Intra module refs:   llFindTxPowerSettings
    -------------------------------------------------------------------------
<XDATA_ROM_C> 1 (was XDATA_ROM_C)
  Relative segment, address: CONST 00008F8E - 00008F95 (0x8 bytes), align: 0
  Segment part 32.            Intra module refs:   llFindTxPowerSettings
    -------------------------------------------------------------------------
<XDATA_ROM_C> 1 (was XDATA_ROM_C)
  Relative segment, address: CONST 00008FA8 - 00008FAB (0x4 bytes), align: 0
  Segment part 35.            Intra module refs:   llSetupAdv
           ENTRY                   ADDRESS         REF BY
           =====                   =======         ======
           __Constant_8e89bed6     00008FA8 
    -------------------------------------------------------------------------
<BANKED_CODE,XDATA_ROM_C_FLASH> 1 (was XDATA_ROM_C_FLASH)
  Relative segment, address: CODE 00008FA0 - 00008FA3 (0x4 bytes), align: 0
  Segment part 216.           Intra module refs:   Segment part 31
    -------------------------------------------------------------------------
<BANKED_CODE,XDATA_ROM_C_FLASH> 1 (was XDATA_ROM_C_FLASH)
  Relative segment, address: CODE 00008F8E - 00008F95 (0x8 bytes), align: 0
  Segment part 217.           Intra module refs:   Segment part 32
    -------------------------------------------------------------------------
<BANKED_CODE,XDATA_ROM_C_FLASH> 1 (was XDATA_ROM_C_FLASH)
  Relative segment, address: CODE 00008FA8 - 00008FAB (0x4 bytes), align: 0
  Segment part 220.           Intra module refs:   __Constant_8e89bed6

    -------------------------------------------------------------------------
  LIBRARY MODULE, NAME : ll_constData

  SEGMENTS IN THE MODULE
  ======================
<BANKED_CODE,CODE_C> 1 (was CODE_C)
  Relative segment, address: CODE 000017AC - 000017AF (0x4 bytes), align: 2
  Segment part 6.
           ENTRY                   ADDRESS         REF BY
           =====                   =======         ======
           savedTxPowerSetting     000017AC        llExtendRfRange (ll_common)
                                                   llFindTxPowerSettings (ll_common)
                                                   llGetTxPower (ll_common)
                                                   llSetTxPower (ll_common)
    -------------------------------------------------------------------------
<XDATA_ROM_C> 1 (was XDATA_ROM_C)
  Relative segment, address: CONST 00008F98 - 00008F9B (0x4 bytes), align: 2
  Segment part 7.
           ENTRY                   ADDRESS         REF BY
           =====                   =======         ======
           txOutputPower           00008F98        llGetTxPower (ll_common)
    -------------------------------------------------------------------------
<BANKED_CODE,CODE_C> 1 (was CODE_C)
  Relative segment, address: CODE 000017A8 - 000017AB (0x4 bytes), align: 2
  Segment part 8.
           ENTRY                   ADDRESS         REF BY
           =====                   =======         ======
           ptmFreqTune             000017A8        LL_EXT_SaveFreqTune (ll)
                                                   llRfInit (ll_common)
    -------------------------------------------------------------------------
<BANKED_CODE,XDATA_ROM_C_FLASH> 1 (was XDATA_ROM_C_FLASH)
  Relative segment, address: CODE 00008F98 - 00008F9B (0x4 bytes), align: 2
  Segment part 10.            Intra module refs:   txOutputPower

    -------------------------------------------------------------------------
  LIBRARY MODULE, NAME : ll_enc

  SEGMENTS IN THE MODULE
  ======================
SFR_AN
  Relative segment, address: DATA 000000BC - 000000BC (0x1 bytes), align: 0
  Segment part 3. ROOT        Intra module refs:   LL_ENC_GenerateTrueRandNum
           ENTRY                   ADDRESS         REF BY
           =====                   =======         ======
           RNDL                    000000BC 
    -------------------------------------------------------------------------
SFR_AN
  Relative segment, address: DATA 000000BD - 000000BD (0x1 bytes), align: 0
  Segment part 4. ROOT        Intra module refs:   LL_ENC_GenerateTrueRandNum
           ENTRY                   ADDRESS         REF BY
           =====                   =======         ======
           RNDH                    000000BD 
    -------------------------------------------------------------------------
SFR_AN
  Relative segment, address: DATA 000000D7 - 000000D7 (0x1 bytes), align: 0
  Segment part 7. ROOT 
           ENTRY                   ADDRESS         REF BY
           =====                   =======         ======
           DMAREQ                  000000D7 
    -------------------------------------------------------------------------
<BANKED_CODE,XDATA_ROM_C_FLASH> 1 (was BANKED_CODE)
  Relative segment, address: CODE 0000B600 - 0000B604 (0x5 bytes), align: 0
  Segment part 17.            Intra module refs:   LL_ENC_GenerateTrueRandNum
    -------------------------------------------------------------------------
<BANKED_CODE,XDATA_ROM_C_FLASH> 1 (was BANKED_CODE)
  Relative segment, address: CODE 0000B605 - 0000B610 (0xc bytes), align: 0
  Segment part 18.            Intra module refs:   LL_ENC_GeneratePseudoRandNum::?relay
           ENTRY                   ADDRESS         REF BY
           =====                   =======         ======
           LL_ENC_GeneratePseudoRandNum
                                   0000B605 
               ISTACK = 00000000 ( 00000002 )
    -------------------------------------------------------------------------
<BANKED_CODE,XDATA_ROM_C_FLASH> 1 (was BANKED_CODE)
  Relative segment, address: CODE 0000B611 - 0000B6D2 (0xc2 bytes), align: 0
  Segment part 20.            Intra module refs:   LL_ENC_GenerateTrueRandNum::?relay
           ENTRY                   ADDRESS         REF BY
           =====                   =======         ======
           LL_ENC_GenerateTrueRandNum
                                   0000B611 
               calls direct
               XSTACK = 00000000 ( 0000000C )
               ISTACK = 00000000 ( 00000001 )
    -------------------------------------------------------------------------
<BANKED_CODE,XDATA_ROM_C_FLASH> 1 (was BANKED_CODE)
  Relative segment, address: CODE 0000B6D3 - 0000B6DF (0xd bytes), align: 0
  Segment part 22.            Intra module refs:   LL_ENC_GenerateTrueRandNum
    -------------------------------------------------------------------------
<BANKED_CODE,XDATA_ROM_C_FLASH> 1 (was BANKED_CODE)
  Relative segment, address: CODE 0000B6E0 - 0000B70D (0x2e bytes), align: 0
  Segment part 23.            Intra module refs:   LL_ENC_AES128_Encrypt::?relay
           ENTRY                   ADDRESS         REF BY
           =====                   =======         ======
           LL_ENC_AES128_Encrypt   0000B6E0 
               calls direct
               XSTACK = 00000002 ( 0000000A )
    -------------------------------------------------------------------------
<BANKED_CODE,XDATA_ROM_C_FLASH> 1 (was BANKED_CODE)
  Relative segment, address: CODE 0000B70E - 0000B710 (0x3 bytes), align: 0
  Segment part 25.            Intra module refs:   LL_ENC_AES128_Decrypt
                                                   LL_ENC_AES128_Encrypt
    -------------------------------------------------------------------------
<BANKED_CODE,XDATA_ROM_C_FLASH> 1 (was BANKED_CODE)
  Relative segment, address: CODE 0000B711 - 0000B715 (0x5 bytes), align: 0
  Segment part 26.            Intra module refs:   LL_ENC_SetupCryptoDMA
                                                   Segment part 25
    -------------------------------------------------------------------------
<BANKED_CODE,XDATA_ROM_C_FLASH> 1 (was BANKED_CODE)
  Relative segment, address: CODE 0000B716 - 0000B745 (0x30 bytes), align: 0
  Segment part 27.            Intra module refs:   LL_ENC_AES128_Decrypt::?relay
           ENTRY                   ADDRESS         REF BY
           =====                   =======         ======
           LL_ENC_AES128_Decrypt   0000B716 
               calls direct
               XSTACK = 00000002 ( 0000000A )
    -------------------------------------------------------------------------
<BANKED_CODE,XDATA_ROM_C_FLASH> 1 (was BANKED_CODE)
  Relative segment, address: CODE 0000B746 - 0000B77D (0x38 bytes), align: 0
  Segment part 29.            Intra module refs:   LL_ENC_InitAesDMA::?relay
           ENTRY                   ADDRESS         REF BY
           =====                   =======         ======
           LL_ENC_InitAesDMA       0000B746 
               ISTACK = 00000000 ( 00000002 )
    -------------------------------------------------------------------------
<BANKED_CODE,XDATA_ROM_C_FLASH> 1 (was BANKED_CODE)
  Relative segment, address: CODE 0000B77E - 0000B780 (0x3 bytes), align: 0
  Segment part 31.            Intra module refs:   LL_ENC_LoadKey
    -------------------------------------------------------------------------
<BANKED_CODE,XDATA_ROM_C_FLASH> 1 (was BANKED_CODE)
  Relative segment, address: CODE 0000B781 - 0000B787 (0x7 bytes), align: 0
  Segment part 32.            Intra module refs:   LL_ENC_GeneratePseudoRandNum
                                                   LL_ENC_InitAesDMA
                                                   LL_ENC_SetupLoadDMA
                                                   Segment part 31
    -------------------------------------------------------------------------
<BANKED_CODE,XDATA_ROM_C_FLASH> 1 (was BANKED_CODE)
  Relative segment, address: CODE 0000B788 - 0000B7A0 (0x19 bytes), align: 0
  Segment part 37.            Intra module refs:   LL_ENC_SetupLoadDMA::?relay
           ENTRY                   ADDRESS         REF BY
           =====                   =======         ======
           LL_ENC_SetupLoadDMA     0000B788 
               ISTACK = 00000000 ( 00000002 )
    -------------------------------------------------------------------------
<BANKED_CODE,XDATA_ROM_C_FLASH> 1 (was BANKED_CODE)
  Relative segment, address: CODE 0000B7A1 - 0000B7D9 (0x39 bytes), align: 0
  Segment part 39.            Intra module refs:   LL_ENC_SetupCryptoDMA::?relay
           ENTRY                   ADDRESS         REF BY
           =====                   =======         ======
           LL_ENC_SetupCryptoDMA   0000B7A1 
               XSTACK = 0000000A ( 00000009 )
    -------------------------------------------------------------------------
<BANKED_CODE,XDATA_ROM_C_FLASH> 1 (was BANKED_CODE)
  Relative segment, address: CODE 0000B7DA - 0000B7E5 (0xc bytes), align: 0
  Segment part 41.            Intra module refs:   LL_ENC_SetupCryptoDMA
                                                   LL_ENC_SetupLoadDMA
    -------------------------------------------------------------------------
<BANKED_CODE,XDATA_ROM_C_FLASH> 1 (was BANKED_CODE)
  Relative segment, address: CODE 0000B7E6 - 0000B7F8 (0x13 bytes), align: 0
  Segment part 42.            Intra module refs:   LL_ENC_StartAES::?relay
           ENTRY                   ADDRESS         REF BY
           =====                   =======         ======
           LL_ENC_StartAES         0000B7E6 
               XSTACK = 00000009 ( 00000000 )
    -------------------------------------------------------------------------
<BANKED_CODE,XDATA_ROM_C_FLASH> 1 (was BANKED_CODE)
  Relative segment, address: CODE 0000B7F9 - 0000B80E (0x16 bytes), align: 0
  Segment part 46.            Intra module refs:   LL_ENC_LoadKey::?relay
           ENTRY                   ADDRESS         REF BY
           =====                   =======         ======
           LL_ENC_LoadKey          0000B7F9 
               calls direct
               XSTACK = 00000009 ( 00000000 )
               ISTACK = 00000000 ( 00000002 )
    -------------------------------------------------------------------------
BANK_RELAYS
  Relative segment, address: CODE 000005E4 - 000005E9 (0x6 bytes), align: 0
  Segment part 19.
           ENTRY                   ADDRESS         REF BY
           =====                   =======         ======
           LL_ENC_GeneratePseudoRandNum::?relay
                                   000005E4        llDiscoverableAdvEvt_TaskEndOk (ll_advEndCauses)
                                                   llNonConnAdvEvt_TaskEndOk (ll_advEndCauses)
    -------------------------------------------------------------------------
BANK_RELAYS
  Relative segment, address: CODE 000005EA - 000005EF (0x6 bytes), align: 0
  Segment part 21.
           ENTRY                   ADDRESS         REF BY
           =====                   =======         ======
           LL_ENC_GenerateTrueRandNum::?relay
                                   000005EA        LL_Init (ll)
                                                   LL_Rand (ll)
                                                   llProcessPostRfOps (ll_common)
    -------------------------------------------------------------------------
BANK_RELAYS
  Relative segment, address: CODE 000005F0 - 000005F5 (0x6 bytes), align: 0
  Segment part 24.
           ENTRY                   ADDRESS         REF BY
           =====                   =======         ======
           LL_ENC_AES128_Encrypt::?relay
                                   000005F0        LL_Encrypt (ll)
    -------------------------------------------------------------------------
BANK_RELAYS
  Relative segment, address: CODE 000005F6 - 000005FB (0x6 bytes), align: 0
  Segment part 28.
           ENTRY                   ADDRESS         REF BY
           =====                   =======         ======
           LL_ENC_AES128_Decrypt::?relay
                                   000005F6        LL_EXT_Decrypt (ll)
    -------------------------------------------------------------------------
BANK_RELAYS
  Relative segment, address: CODE 000005FC - 00000601 (0x6 bytes), align: 0
  Segment part 30.
           ENTRY                   ADDRESS         REF BY
           =====                   =======         ======
           LL_ENC_InitAesDMA::?relay
                                   000005FC        LL_Init (ll)
    -------------------------------------------------------------------------
BANK_RELAYS
  Relative segment, address: CODE 00000602 - 00000607 (0x6 bytes), align: 0
  Segment part 38.            Intra module refs:   LL_ENC_LoadKey
           ENTRY                   ADDRESS         REF BY
           =====                   =======         ======
           LL_ENC_SetupLoadDMA::?relay
                                   00000602 
    -------------------------------------------------------------------------
BANK_RELAYS
  Relative segment, address: CODE 00000608 - 0000060D (0x6 bytes), align: 0
  Segment part 40.            Intra module refs:   LL_ENC_AES128_Decrypt
                                                   LL_ENC_AES128_Encrypt
           ENTRY                   ADDRESS         REF BY
           =====                   =======         ======
           LL_ENC_SetupCryptoDMA::?relay
                                   00000608 
    -------------------------------------------------------------------------
BANK_RELAYS
  Relative segment, address: CODE 0000060E - 00000613 (0x6 bytes), align: 0
  Segment part 43.            Intra module refs:   Segment part 25
                                                   Segment part 31
           ENTRY                   ADDRESS         REF BY
           =====                   =======         ======
           LL_ENC_StartAES::?relay
                                   0000060E 
    -------------------------------------------------------------------------
BANK_RELAYS
  Relative segment, address: CODE 00000614 - 00000619 (0x6 bytes), align: 0
  Segment part 47.            Intra module refs:   LL_ENC_AES128_Decrypt
                                                   LL_ENC_AES128_Encrypt
           ENTRY                   ADDRESS         REF BY
           =====                   =======         ======
           LL_ENC_LoadKey::?relay
                                   00000614 

    -------------------------------------------------------------------------
  LIBRARY MODULE, NAME : ll_errorEndCauses

  SEGMENTS IN THE MODULE
  ======================
<BANKED_CODE,CODE_C> 1 (was BANKED_CODE)
  Relative segment, address: CODE 00007FFB - 00007FFD (0x3 bytes), align: 0
  Segment part 6.             Intra module refs:   llUnexpectedEndCauseHandler::?relay
           ENTRY                   ADDRESS         REF BY
           =====                   =======         ======
           llUnexpectedEndCauseHandler
                                   00007FFB 
    -------------------------------------------------------------------------
BANK_RELAYS
  Relative segment, address: CODE 0000061A - 0000061F (0x6 bytes), align: 0
  Segment part 7.
           ENTRY                   ADDRESS         REF BY
           =====                   =======         ======
           llUnexpectedEndCauseHandler::?relay
                                   0000061A        Segment part 47 (ll)
                                                   Segment part 49 (ll)
                                                   Segment part 88 (ll_common)
                                                   Segment part 94 (ll_common)
                                                   Segment part 96 (ll_common)

    -------------------------------------------------------------------------
  PROGRAM MODULE, NAME : ll_halt

  SEGMENTS IN THE MODULE
  ======================
NEAR_CODE
  Relative segment, address: CODE 000013B4 - 000013BA (0x7 bytes), align: 2
  Segment part 0.
           ENTRY                   ADDRESS         REF BY
           =====                   =======         ======
           HaltMcuUsingPhyFlag     000013B4        llT2OVFC1_ISR (ll_isr)
    -------------------------------------------------------------------------
DATA_Z
  Relative segment, address: DATA 00000021 - 00000022 (0x2 bytes), align: 0
  Segment part 1.             Intra module refs:   HaltMcuUsingPhyFlag
           ENTRY                   ADDRESS         REF BY
           =====                   =======         ======
           phyState                00000021        LL_Reset (ll)
                                                   RF_NormalIsr (ll_isr)
                                                   llT2OVFC1_ISR (ll_isr)
           clkState                00000022        llT2OVFC1_ISR (ll_isr)

    -------------------------------------------------------------------------
  PROGRAM MODULE, NAME : ll_isr

  SEGMENTS IN THE MODULE
  ======================
SFR_AN
  Relative segment, address: DATA 0000009B - 0000009B (0x1 bytes), align: 0
  Segment part 1. ROOT        Intra module refs:   RF_NormalIsr
                                                   llClearSetInts (ll_common)
           ENTRY                   ADDRESS         REF BY
           =====                   =======         ======
           S1CON                   0000009B 
    -------------------------------------------------------------------------
SFR_AN
  Relative segment, address: DATA 0000009F - 0000009F (0x1 bytes), align: 0
  Segment part 2. ROOT        Intra module refs:   LL_Init (ll)
                                                   RF_NormalIsr
           ENTRY                   ADDRESS         REF BY
           =====                   =======         ======
           FMAP                    0000009F 
    -------------------------------------------------------------------------
SFR_AN
  Relative segment, address: DATA 000000A1 - 000000A1 (0x1 bytes), align: 0
  Segment part 3. ROOT        Intra module refs:   T2_Isr
                                                   llDisableT2Ints (ll_timer2)
                                                   llDisableT2IntsEvts (ll_timer2)
                                                   llInitTimer2 (ll_timer2)
                                                   llSetT2C1Event1 (ll_timer2)
                                                   llSetT2OVFC1Event1 (ll_timer2)
                                                   llSetT2OVFC1Timeout (ll_timer2)
                                                   llSetT2OVFC2Event2 (ll_timer2)
           ENTRY                   ADDRESS         REF BY
           =====                   =======         ======
           T2IRQF                  000000A1 
    -------------------------------------------------------------------------
SFR_AN
  Relative segment, address: DATA 000000A7 - 000000A7 (0x1 bytes), align: 0
  Segment part 4. ROOT        Intra module refs:   T2_Isr
                                                   llDisableT2Ints (ll_timer2)
                                                   llDisableT2IntsEvts (ll_timer2)
                                                   llInitTimer2 (ll_timer2)
                                                   llSetT2C1Event1 (ll_timer2)
                                                   llSetT2OVFC1Event1 (ll_timer2)
                                                   llSetT2OVFC1Timeout (ll_timer2)
                                                   llSetT2OVFC2Event2 (ll_timer2)
           ENTRY                   ADDRESS         REF BY
           =====                   =======         ======
           T2IRQM                  000000A7 
    -------------------------------------------------------------------------
SFR_AN
  Relative segment, address: DATA 000000A8 - 000000A8 (0x1 bytes), align: 0
  Segment part 5. ROOT        Intra module refs:   HalFlashRead (hal_flash)
                                                   LL_Init (ll)
                                                   LL_ProcessEvent (ll)
                                                   LL_Reset (ll)
                                                   LL_SetAdvControl (ll)
                                                   Onboard_soft_reset (OnBoard)
                                                   RF_NormalIsr
                                                   halSleepTimerIsr (hal_sleep)
                                                   halUartPollRx (hal_uart)
                                                   llClearSetInts (ll_common)
                                                   llDisableT2E1 (ll_timer2)
                                                   llDisableT2Ints (ll_timer2)
                                                   llDisableT2IntsEvts (ll_timer2)
                                                   llGetCurrentTime (ll_timer2)
                                                   llSetT2C1Event1 (ll_timer2)
                                                   llSetT2Delta (ll_timer2)
                                                   llSetT2OVFC1Event1 (ll_timer2)
                                                   llSetT2OVFC1Timeout (ll_timer2)
                                                   llSetT2OVFC2Event2 (ll_timer2)
                                                   llStartTimer2 (ll_timer2)
                                                   llStopTimer2 (ll_timer2)
                                                   llT2OVFC1_ISR
                                                   ll_McuPrecisionCount (ll_timer2)
                                                   main (SimpleBLEBroadcaster_Main)
                                                   osalTimerUpdate (OSAL_Timers)
                                                   osal_CbTimerProcessEvent (osal_cbtimer)
                                                   osal_bm_alloc (osal_bufmgr)
                                                   osal_bm_free (osal_bufmgr)
                                                   osal_clear_event (OSAL)
                                                   osal_get_timeoutEx (OSAL_Timers)
                                                   osal_int_disable (OSAL)
                                                   osal_mem_alloc (OSAL_Memory)
                                                   osal_mem_free (OSAL_Memory)
                                                   osal_mem_kick (OSAL_Memory)
                                                   osal_msg_enqueue (OSAL)
                                                   osal_msg_extract (OSAL)
                                                   osal_msg_push (OSAL)
                                                   osal_msg_receive (OSAL)
                                                   osal_pwrmgr_task_state (OSAL_PwrMgr)
                                                   osal_run_system (OSAL)
                                                   osal_set_event (OSAL)
                                                   osal_start_reload_timer (OSAL_Timers)
                                                   osal_start_timerEx (OSAL_Timers)
                                                   osal_stop_timerEx (OSAL_Timers)
           ENTRY                   ADDRESS         REF BY
           =====                   =======         ======
           _A_IEN0                 000000A8 
    -------------------------------------------------------------------------
SFR_AN
  Relative segment, address: DATA 000000BE - 000000BE (0x1 bytes), align: 0
  Segment part 6. ROOT        Intra module refs:   llT2OVFC1_ISR
                                                   main (SimpleBLEBroadcaster_Main)
           ENTRY                   ADDRESS         REF BY
           =====                   =======         ======
           SLEEPCMD                000000BE 
    -------------------------------------------------------------------------
SFR_AN
  Relative segment, address: DATA 000000C6 - 000000C6 (0x1 bytes), align: 0
  Segment part 7. ROOT        Intra module refs:   LL_EXT_MapPmIoPort (ll)
                                                   llSetFreqTune (ll_common)
                                                   llT2OVFC1_ISR
                                                   main (SimpleBLEBroadcaster_Main)
           ENTRY                   ADDRESS         REF BY
           =====                   =======         ======
           CLKCONCMD               000000C6 
    -------------------------------------------------------------------------
SFR_AN
  Relative segment, address: DATA 00000091 - 00000091 (0x1 bytes), align: 0
  Segment part 8. ROOT        Intra module refs:   LL_SetAdvControl (ll)
                                                   RF_NormalIsr
                                                   llClearRfInts (ll_common)
                                                   llScheduleTask (ll_scheduler)
           ENTRY                   ADDRESS         REF BY
           =====                   =======         ======
           RFIRQF1                 00000091 
    -------------------------------------------------------------------------
SFR_AN
  Relative segment, address: DATA 000000BF - 000000BF (0x1 bytes), align: 0
  Segment part 9. ROOT        Intra module refs:   RF_ErrorIsr
                                                   llAdvEvt_TaskAbort (ll_advEndCauses)
                                                   llClearRfInts (ll_common)
           ENTRY                   ADDRESS         REF BY
           =====                   =======         ======
           RFERRF                  000000BF 
    -------------------------------------------------------------------------
SFR_AN
  Relative segment, address: DATA 000000E9 - 000000E9 (0x1 bytes), align: 0
  Segment part 10. ROOT       Intra module refs:   RF_NormalIsr
                                                   llClearRfInts (ll_common)
           ENTRY                   ADDRESS         REF BY
           =====                   =======         ======
           RFIRQF0                 000000E9 
    -------------------------------------------------------------------------
NEAR_CODE
  Relative segment, address: CODE 000013BB - 000014B8 (0xfe bytes), align: 0
  Segment part 19.            Intra module refs:   RF_NormalIsr::??INTVEC 131
           ENTRY                   ADDRESS         REF BY
           =====                   =======         ======
           RF_NormalIsr            000013BB 
               interrupt function
               calls direct
               XSTACK = 00000000 ( 00000011 )
               ISTACK = 00000000 ( 00000001 )
    -------------------------------------------------------------------------
NEAR_CODE
  Relative segment, address: CODE 000014B9 - 0000152E (0x76 bytes), align: 0
  Segment part 20.            Intra module refs:   RF_ErrorIsr::??INTVEC 3
           ENTRY                   ADDRESS         REF BY
           =====                   =======         ======
           RF_ErrorIsr             000014B9 
               interrupt function
               ISTACK = 00000000 ( 00000004 )
    -------------------------------------------------------------------------
NEAR_CODE
  Relative segment, address: CODE 0000152F - 00001582 (0x54 bytes), align: 0
  Segment part 21.            Intra module refs:   T2_Isr::??INTVEC 83
           ENTRY                   ADDRESS         REF BY
           =====                   =======         ======
           T2_Isr                  0000152F 
               interrupt function
               calls direct
               XSTACK = 00000000 ( 0000000E )
    -------------------------------------------------------------------------
NEAR_CODE
  Relative segment, address: CODE 00001583 - 000015F8 (0x76 bytes), align: 0
  Segment part 22.            Intra module refs:   T2_Isr
           ENTRY                   ADDRESS         REF BY
           =====                   =======         ======
           llT2OVFC1_ISR           00001583 
               calls direct
               XSTACK = 0000000E ( 00000008 )
    -------------------------------------------------------------------------
INTVEC
  Common segment, address: CODE 00000000 - 00000005 (0x6 bytes), align: 0
  Segment part 11. ROOT 
           ENTRY                   ADDRESS         REF BY
           =====                   =======         ======
           RF_ErrorIsr::??INTVEC 3
                                   00000003 
    -------------------------------------------------------------------------
INTVEC
  Common segment, address: CODE 00000000 - 00000055 (0x56 bytes), align: 0
  Segment part 12. ROOT 
           ENTRY                   ADDRESS         REF BY
           =====                   =======         ======
           T2_Isr::??INTVEC 83     00000053 
    -------------------------------------------------------------------------
INTVEC
  Common segment, address: CODE 00000000 - 00000085 (0x86 bytes), align: 0
  Segment part 13. ROOT 
           ENTRY                   ADDRESS         REF BY
           =====                   =======         ======
           RF_NormalIsr::??INTVEC 131
                                   00000083 

    -------------------------------------------------------------------------
  LIBRARY MODULE, NAME : ll_scheduler

  SEGMENTS IN THE MODULE
  ======================
XDATA_Z
  Relative segment, address: XDATA 0000038A - 000003AA (0x21 bytes), align: 0
  Segment part 8.             Intra module refs:   llAllocTask
                                                   llFindNextSecTask
                                                   llFreeTask
                                                   llGetCurrentTask
                                                   llGetNumTasks
                                                   llGetTask
                                                   llGetTaskState
                                                   llScheduleTask
                                                   llScheduler
                                                   llSchedulerInit
    -------------------------------------------------------------------------
<BANKED_CODE,CODE_C> 1 (was BANKED_CODE)
  Relative segment, address: CODE 0000777A - 0000779D (0x24 bytes), align: 0
  Segment part 19.            Intra module refs:   llSchedulerInit::?relay
           ENTRY                   ADDRESS         REF BY
           =====                   =======         ======
           llSchedulerInit         0000777A 
               ISTACK = 00000000 ( 00000002 )
    -------------------------------------------------------------------------
<BANKED_CODE,CODE_C> 1 (was BANKED_CODE)
  Relative segment, address: CODE 0000779E - 0000789A (0xfd bytes), align: 0
  Segment part 21.            Intra module refs:   llScheduler::?relay
           ENTRY                   ADDRESS         REF BY
           =====                   =======         ======
           llScheduler             0000779E 
               calls direct
               XSTACK = 00000000 ( 00000014 )
    -------------------------------------------------------------------------
<BANKED_CODE,CODE_C> 1 (was BANKED_CODE)
  Relative segment, address: CODE 0000789B - 0000789F (0x5 bytes), align: 0
  Segment part 23.            Intra module refs:   llScheduleTask
                                                   llScheduler
    -------------------------------------------------------------------------
<BANKED_CODE,CODE_C> 1 (was BANKED_CODE)
  Relative segment, address: CODE 000078A0 - 000079EE (0x14f bytes), align: 0
  Segment part 24.            Intra module refs:   llScheduleTask::?relay
           ENTRY                   ADDRESS         REF BY
           =====                   =======         ======
           llScheduleTask          000078A0 
               calls direct
               XSTACK = 00000010 ( 00000014 )
    -------------------------------------------------------------------------
<BANKED_CODE,CODE_C> 1 (was BANKED_CODE)
  Relative segment, address: CODE 000079EF - 000079FA (0xc bytes), align: 0
  Segment part 26.            Intra module refs:   llScheduleTask
                                                   llScheduler
    -------------------------------------------------------------------------
<BANKED_CODE,CODE_C> 1 (was BANKED_CODE)
  Relative segment, address: CODE 000079FB - 00007A06 (0xc bytes), align: 0
  Segment part 27.            Intra module refs:   llScheduleTask
    -------------------------------------------------------------------------
<BANKED_CODE,CODE_C> 1 (was BANKED_CODE)
  Relative segment, address: CODE 00007A07 - 00007B85 (0x17f bytes), align: 0
  Segment part 30.            Intra module refs:   llFindNextSecTask::?relay
           ENTRY                   ADDRESS         REF BY
           =====                   =======         ======
           llFindNextSecTask       00007A07 
               calls direct
               XSTACK = 00000010 ( 00000016 )
    -------------------------------------------------------------------------
<BANKED_CODE,CODE_C> 1 (was BANKED_CODE)
  Relative segment, address: CODE 00007B86 - 00007C00 (0x7b bytes), align: 0
  Segment part 32.            Intra module refs:   llAllocTask::?relay
           ENTRY                   ADDRESS         REF BY
           =====                   =======         ======
           llAllocTask             00007B86 
               calls direct
               XSTACK = 00000000 ( 00000009 )
    -------------------------------------------------------------------------
<BANKED_CODE,CODE_C> 1 (was BANKED_CODE)
  Relative segment, address: CODE 00007C01 - 00007C46 (0x46 bytes), align: 0
  Segment part 34.            Intra module refs:   llFreeTask::?relay
           ENTRY                   ADDRESS         REF BY
           =====                   =======         ======
           llFreeTask              00007C01 
               calls direct
               ISTACK = 00000000 ( 00000002 )
    -------------------------------------------------------------------------
<BANKED_CODE,CODE_C> 1 (was BANKED_CODE)
  Relative segment, address: CODE 00007C47 - 00007C47 (0x1 bytes), align: 0
  Segment part 37.            Intra module refs:   llSchedulerInit
    -------------------------------------------------------------------------
<BANKED_CODE,CODE_C> 1 (was BANKED_CODE)
  Relative segment, address: CODE 00007C48 - 00007C4E (0x7 bytes), align: 0
  Segment part 38.            Intra module refs:   Segment part 37
                                                   Segment part 45
                                                   llFreeTask
                                                   llGetCurrentTask
                                                   llGetTask
                                                   llGetTaskState
    -------------------------------------------------------------------------
<BANKED_CODE,CODE_C> 1 (was BANKED_CODE)
  Relative segment, address: CODE 00007C4F - 00007C68 (0x1a bytes), align: 0
  Segment part 39.            Intra module refs:   llGetCurrentTask::?relay
           ENTRY                   ADDRESS         REF BY
           =====                   =======         ======
           llGetCurrentTask        00007C4F 
               ISTACK = 00000000 ( 00000002 )
    -------------------------------------------------------------------------
<BANKED_CODE,CODE_C> 1 (was BANKED_CODE)
  Relative segment, address: CODE 00007C69 - 00007C7E (0x16 bytes), align: 0
  Segment part 41.            Intra module refs:   llGetTaskState::?relay
           ENTRY                   ADDRESS         REF BY
           =====                   =======         ======
           llGetTaskState          00007C69 
               XSTACK = 00000012 ( 00000000 )
               ISTACK = 00000000 ( 00000002 )
    -------------------------------------------------------------------------
<BANKED_CODE,CODE_C> 1 (was BANKED_CODE)
  Relative segment, address: CODE 00007C7F - 00007C82 (0x4 bytes), align: 0
  Segment part 45.            Intra module refs:   llGetNumTasks
    -------------------------------------------------------------------------
<BANKED_CODE,CODE_C> 1 (was BANKED_CODE)
  Relative segment, address: CODE 00007C83 - 00007C9F (0x1d bytes), align: 0
  Segment part 46.            Intra module refs:   llGetTask::?relay
           ENTRY                   ADDRESS         REF BY
           =====                   =======         ======
           llGetTask               00007C83 
               XSTACK = 00000012 ( 00000000 )
               ISTACK = 00000000 ( 00000002 )
    -------------------------------------------------------------------------
<BANKED_CODE,CODE_C> 1 (was BANKED_CODE)
  Relative segment, address: CODE 00007CA0 - 00007CA8 (0x9 bytes), align: 0
  Segment part 48.            Intra module refs:   llGetNumTasks::?relay
           ENTRY                   ADDRESS         REF BY
           =====                   =======         ======
           llGetNumTasks           00007CA0 
               ISTACK = 00000000 ( 00000002 )
    -------------------------------------------------------------------------
<XDATA_ROM_C> 1 (was XDATA_ROM_C)
  Relative segment, address: CONST 00008FB0 - 00008FB3 (0x4 bytes), align: 0
  Segment part 9.             Intra module refs:   llScheduler
           ENTRY                   ADDRESS         REF BY
           =====                   =======         ======
           __Constant_a            00008FB0 
    -------------------------------------------------------------------------
<XDATA_ROM_C> 1 (was XDATA_ROM_C)
  Relative segment, address: CONST 00008FB4 - 00008FB7 (0x4 bytes), align: 0
  Segment part 13.            Intra module refs:   llScheduleTask
           ENTRY                   ADDRESS         REF BY
           =====                   =======         ======
           __Constant_5            00008FB4 
    -------------------------------------------------------------------------
<XDATA_ROM_C> 1 (was XDATA_ROM_C)
  Relative segment, address: CONST 00008FB8 - 00008FBB (0x4 bytes), align: 0
  Segment part 18.            Intra module refs:   llFindNextSecTask
           ENTRY                   ADDRESS         REF BY
           =====                   =======         ======
           __Constant_fffffff6     00008FB8 
    -------------------------------------------------------------------------
BANK_RELAYS
  Relative segment, address: CODE 00000620 - 00000625 (0x6 bytes), align: 0
  Segment part 20.
           ENTRY                   ADDRESS         REF BY
           =====                   =======         ======
           llSchedulerInit::?relay
                                   00000620        LL_Reset (ll)
    -------------------------------------------------------------------------
BANK_RELAYS
  Relative segment, address: CODE 00000626 - 0000062B (0x6 bytes), align: 0
  Segment part 22.
           ENTRY                   ADDRESS         REF BY
           =====                   =======         ======
           llScheduler::?relay     00000626        LL_SetAdvControl (ll)
                                                   Segment part 12 (ll_advEndCauses)
                                                   llAdvEvt_TaskAbort (ll_advEndCauses)
    -------------------------------------------------------------------------
BANK_RELAYS
  Relative segment, address: CODE 0000062C - 00000631 (0x6 bytes), align: 0
  Segment part 25.            Intra module refs:   llScheduler
           ENTRY                   ADDRESS         REF BY
           =====                   =======         ======
           llScheduleTask::?relay
                                   0000062C 
    -------------------------------------------------------------------------
BANK_RELAYS
  Relative segment, address: CODE 00000632 - 00000637 (0x6 bytes), align: 0
  Segment part 31.            Intra module refs:   llScheduler
           ENTRY                   ADDRESS         REF BY
           =====                   =======         ======
           llFindNextSecTask::?relay
                                   00000632 
    -------------------------------------------------------------------------
BANK_RELAYS
  Relative segment, address: CODE 00000638 - 0000063D (0x6 bytes), align: 0
  Segment part 33.
           ENTRY                   ADDRESS         REF BY
           =====                   =======         ======
           llAllocTask::?relay     00000638        LL_SetAdvControl (ll)
    -------------------------------------------------------------------------
BANK_RELAYS
  Relative segment, address: CODE 0000063E - 00000643 (0x6 bytes), align: 0
  Segment part 35.
           ENTRY                   ADDRESS         REF BY
           =====                   =======         ======
           llFreeTask::?relay      0000063E        LL_SetAdvControl (ll)
                                                   llAdvEvt_TaskAbort (ll_advEndCauses)
    -------------------------------------------------------------------------
BANK_RELAYS
  Relative segment, address: CODE 00000644 - 00000649 (0x6 bytes), align: 0
  Segment part 40.
           ENTRY                   ADDRESS         REF BY
           =====                   =======         ======
           llGetCurrentTask::?relay
                                   00000644        LL_EXT_ExtendRfRange (ll)
                                                   LL_EXT_SetRxGain (ll)
                                                   LL_EXT_SetTxPower (ll)
                                                   LL_Rand (ll)
    -------------------------------------------------------------------------
BANK_RELAYS
  Relative segment, address: CODE 0000064A - 0000064F (0x6 bytes), align: 0
  Segment part 42.            Intra module refs:   llFindNextSecTask
           ENTRY                   ADDRESS         REF BY
           =====                   =======         ======
           llGetTaskState::?relay
                                   0000064A        llAdvEvt_TaskAbort (ll_advEndCauses)
                                                   llDiscoverableAdvEvt_TaskEndOk (ll_advEndCauses)
                                                   llNonConnAdvEvt_TaskEndOk (ll_advEndCauses)
    -------------------------------------------------------------------------
BANK_RELAYS
  Relative segment, address: CODE 00000650 - 00000655 (0x6 bytes), align: 0
  Segment part 47.            Intra module refs:   llFindNextSecTask
           ENTRY                   ADDRESS         REF BY
           =====                   =======         ======
           llGetTask::?relay       00000650 
    -------------------------------------------------------------------------
BANK_RELAYS
  Relative segment, address: CODE 00000656 - 0000065B (0x6 bytes), align: 0
  Segment part 49.
           ENTRY                   ADDRESS         REF BY
           =====                   =======         ======
           llGetNumTasks::?relay   00000656        LL_SetAdvControl (ll)
    -------------------------------------------------------------------------
<BANKED_CODE,XDATA_ROM_C_FLASH> 1 (was XDATA_ROM_C_FLASH)
  Relative segment, address: CODE 00008FB0 - 00008FB3 (0x4 bytes), align: 0
  Segment part 70.            Intra module refs:   __Constant_a
    -------------------------------------------------------------------------
<BANKED_CODE,XDATA_ROM_C_FLASH> 1 (was XDATA_ROM_C_FLASH)
  Relative segment, address: CODE 00008FB4 - 00008FB7 (0x4 bytes), align: 0
  Segment part 74.            Intra module refs:   __Constant_5
    -------------------------------------------------------------------------
<BANKED_CODE,XDATA_ROM_C_FLASH> 1 (was XDATA_ROM_C_FLASH)
  Relative segment, address: CODE 00008FB8 - 00008FBB (0x4 bytes), align: 0
  Segment part 79.            Intra module refs:   __Constant_fffffff6

    -------------------------------------------------------------------------
  LIBRARY MODULE, NAME : ll_sleep

  SEGMENTS IN THE MODULE
  ======================
SFR_AN
  Relative segment, address: DATA 000000A0 - 000000A0 (0x1 bytes), align: 0
  Segment part 4. ROOT 
           ENTRY                   ADDRESS         REF BY
           =====                   =======         ======
           _A_P2                   000000A0 
    -------------------------------------------------------------------------
<XDATA_ROM_C> 1 (was XDATA_ROM_C)
  Relative segment, address: CONST 00008FBC - 00008FBF (0x4 bytes), align: 0
  Segment part 15.            Intra module refs:   ll24BitTimeCompare (ll_timer2)
           ENTRY                   ADDRESS         REF BY
           =====                   =======         ======
           __Constant_c801         00008FBC 
    -------------------------------------------------------------------------
<BANKED_CODE,XDATA_ROM_C_FLASH> 1 (was XDATA_ROM_C_FLASH)
  Relative segment, address: CODE 00008FBC - 00008FBF (0x4 bytes), align: 0
  Segment part 24.            Intra module refs:   __Constant_c801

    -------------------------------------------------------------------------
  LIBRARY MODULE, NAME : ll_timer2

  SEGMENTS IN THE MODULE
  ======================
SFR_AN
  Relative segment, address: DATA 00000094 - 00000094 (0x1 bytes), align: 0
  Segment part 1. ROOT        Intra module refs:   llInitTimer2
                                                   llStartTimer2
                                                   llStopTimer2
           ENTRY                   ADDRESS         REF BY
           =====                   =======         ======
           T2CTRL                  00000094 
    -------------------------------------------------------------------------
SFR_AN
  Relative segment, address: DATA 0000009C - 0000009C (0x1 bytes), align: 0
  Segment part 5. ROOT        Intra module refs:   llDisableT2E1
                                                   llDisableT2IntsEvts
                                                   llInitTimer2
                                                   llSetT2C1Event1
                                                   llSetT2OVFC1Event1
                                                   llSetT2OVFC2Event2
           ENTRY                   ADDRESS         REF BY
           =====                   =======         ======
           T2CSPCFG                0000009C 
    -------------------------------------------------------------------------
SFR_AN
  Relative segment, address: DATA 000000A2 - 000000A2 (0x1 bytes), align: 0
  Segment part 7. ROOT        Intra module refs:   llGetCurrentTime
                                                   llInitTimer2
                                                   llSetT2C1Event1
                                                   llSetT2Delta
                                                   ll_McuPrecisionCount
           ENTRY                   ADDRESS         REF BY
           =====                   =======         ======
           T2M0                    000000A2 
    -------------------------------------------------------------------------
SFR_AN
  Relative segment, address: DATA 000000A3 - 000000A3 (0x1 bytes), align: 0
  Segment part 8. ROOT        Intra module refs:   llInitTimer2
                                                   llSetT2C1Event1
                                                   llSetT2Delta
           ENTRY                   ADDRESS         REF BY
           =====                   =======         ======
           T2M1                    000000A3 
    -------------------------------------------------------------------------
SFR_AN
  Relative segment, address: DATA 000000A4 - 000000A4 (0x1 bytes), align: 0
  Segment part 9. ROOT        Intra module refs:   llGetCurrentTime
                                                   llInitTimer2
                                                   llSetT2OVFC1Event1
                                                   llSetT2OVFC1Timeout
                                                   llSetT2OVFC2Event2
                                                   ll_McuPrecisionCount
           ENTRY                   ADDRESS         REF BY
           =====                   =======         ======
           T2MOVF0                 000000A4 
    -------------------------------------------------------------------------
SFR_AN
  Relative segment, address: DATA 000000A5 - 000000A5 (0x1 bytes), align: 0
  Segment part 10. ROOT       Intra module refs:   llGetCurrentTime
                                                   llInitTimer2
                                                   llSetT2OVFC1Event1
                                                   llSetT2OVFC1Timeout
                                                   llSetT2OVFC2Event2
                                                   ll_McuPrecisionCount
           ENTRY                   ADDRESS         REF BY
           =====                   =======         ======
           T2MOVF1                 000000A5 
    -------------------------------------------------------------------------
SFR_AN
  Relative segment, address: DATA 000000A6 - 000000A6 (0x1 bytes), align: 0
  Segment part 11. ROOT       Intra module refs:   llGetCurrentTime
                                                   llInitTimer2
                                                   llSetT2OVFC1Event1
                                                   llSetT2OVFC1Timeout
                                                   llSetT2OVFC2Event2
           ENTRY                   ADDRESS         REF BY
           =====                   =======         ======
           T2MOVF2                 000000A6 
    -------------------------------------------------------------------------
SFR_AN
  Relative segment, address: DATA 000000C3 - 000000C3 (0x1 bytes), align: 0
  Segment part 14. ROOT       Intra module refs:   llGetCurrentTime
                                                   llInitTimer2
                                                   llSetT2C1Event1
                                                   llSetT2Delta
                                                   llSetT2OVFC1Event1
                                                   llSetT2OVFC1Timeout
                                                   llSetT2OVFC2Event2
                                                   ll_McuPrecisionCount
           ENTRY                   ADDRESS         REF BY
           =====                   =======         ======
           T2MSEL                  000000C3 
    -------------------------------------------------------------------------
<BANKED_CODE,XDATA_ROM_C_FLASH> 1 (was BANKED_CODE)
  Relative segment, address: CODE 0000A5A8 - 0000A61D (0x76 bytes), align: 0
  Segment part 24.            Intra module refs:   llInitTimer2::?relay
           ENTRY                   ADDRESS         REF BY
           =====                   =======         ======
           llInitTimer2            0000A5A8 
               calls direct
               ISTACK = 00000000 ( 00000002 )
    -------------------------------------------------------------------------
<BANKED_CODE,XDATA_ROM_C_FLASH> 1 (was BANKED_CODE)
  Relative segment, address: CODE 0000A61E - 0000A62D (0x10 bytes), align: 0
  Segment part 26.            Intra module refs:   llStopTimer2::?relay
           ENTRY                   ADDRESS         REF BY
           =====                   =======         ======
           llStopTimer2            0000A61E 
    -------------------------------------------------------------------------
<BANKED_CODE,XDATA_ROM_C_FLASH> 1 (was BANKED_CODE)
  Relative segment, address: CODE 0000A62E - 0000A633 (0x6 bytes), align: 0
  Segment part 28.            Intra module refs:   llStartTimer2
                                                   llStopTimer2
    -------------------------------------------------------------------------
<BANKED_CODE,XDATA_ROM_C_FLASH> 1 (was BANKED_CODE)
  Relative segment, address: CODE 0000A634 - 0000A645 (0x12 bytes), align: 0
  Segment part 29.            Intra module refs:   llStartTimer2::?relay
           ENTRY                   ADDRESS         REF BY
           =====                   =======         ======
           llStartTimer2           0000A634 
    -------------------------------------------------------------------------
<BANKED_CODE,XDATA_ROM_C_FLASH> 1 (was BANKED_CODE)
  Relative segment, address: CODE 0000A646 - 0000A652 (0xd bytes), align: 0
  Segment part 33.            Intra module refs:   llSetT2C1Event1
    -------------------------------------------------------------------------
<BANKED_CODE,XDATA_ROM_C_FLASH> 1 (was BANKED_CODE)
  Relative segment, address: CODE 0000A653 - 0000A655 (0x3 bytes), align: 0
  Segment part 34.            Intra module refs:   llSetT2C1Event1
    -------------------------------------------------------------------------
<BANKED_CODE,XDATA_ROM_C_FLASH> 1 (was BANKED_CODE)
  Relative segment, address: CODE 0000A656 - 0000A661 (0xc bytes), align: 0
  Segment part 35.            Intra module refs:   Segment part 34
                                                   llSetT2Delta
    -------------------------------------------------------------------------
<BANKED_CODE,XDATA_ROM_C_FLASH> 1 (was BANKED_CODE)
  Relative segment, address: CODE 0000A662 - 0000A677 (0x16 bytes), align: 0
  Segment part 38.            Intra module refs:   ll_McuPrecisionCount
    -------------------------------------------------------------------------
<BANKED_CODE,XDATA_ROM_C_FLASH> 1 (was BANKED_CODE)
  Relative segment, address: CODE 0000A678 - 0000A67B (0x4 bytes), align: 0
  Segment part 39.            Intra module refs:   Segment part 33
                                                   Segment part 38
                                                   llSetT2Delta
    -------------------------------------------------------------------------
<BANKED_CODE,XDATA_ROM_C_FLASH> 1 (was BANKED_CODE)
  Relative segment, address: CODE 0000A67C - 0000A692 (0x17 bytes), align: 0
  Segment part 40.            Intra module refs:   llGetCurrentTime
    -------------------------------------------------------------------------
<BANKED_CODE,XDATA_ROM_C_FLASH> 1 (was BANKED_CODE)
  Relative segment, address: CODE 0000A693 - 0000A6B7 (0x25 bytes), align: 0
  Segment part 41.            Intra module refs:   Segment part 40
    -------------------------------------------------------------------------
<BANKED_CODE,XDATA_ROM_C_FLASH> 1 (was BANKED_CODE)
  Relative segment, address: CODE 0000A6B8 - 0000A6B9 (0x2 bytes), align: 0
  Segment part 42.            Intra module refs:   Segment part 41
                                                   Segment part 47
    -------------------------------------------------------------------------
<BANKED_CODE,XDATA_ROM_C_FLASH> 1 (was BANKED_CODE)
  Relative segment, address: CODE 0000A6BA - 0000A6BC (0x3 bytes), align: 0
  Segment part 43.            Intra module refs:   Segment part 39
                                                   Segment part 42
    -------------------------------------------------------------------------
<BANKED_CODE,XDATA_ROM_C_FLASH> 1 (was BANKED_CODE)
  Relative segment, address: CODE 0000A6BD - 0000A6C3 (0x7 bytes), align: 0
  Segment part 44.            Intra module refs:   Segment part 43
                                                   llInitTimer2
    -------------------------------------------------------------------------
<BANKED_CODE,XDATA_ROM_C_FLASH> 1 (was BANKED_CODE)
  Relative segment, address: CODE 0000A6C4 - 0000A6E4 (0x21 bytes), align: 0
  Segment part 45.            Intra module refs:   llSetT2OVFC1Timeout::?relay
           ENTRY                   ADDRESS         REF BY
           =====                   =======         ======
           llSetT2OVFC1Timeout     0000A6C4 
               XSTACK = 00000000 ( 00000004 )
               ISTACK = 00000000 ( 00000002 )
    -------------------------------------------------------------------------
<BANKED_CODE,XDATA_ROM_C_FLASH> 1 (was BANKED_CODE)
  Relative segment, address: CODE 0000A6E5 - 0000A6F1 (0xd bytes), align: 0
  Segment part 47.            Intra module refs:   llSetT2OVFC1Event1
                                                   llSetT2OVFC1Timeout
    -------------------------------------------------------------------------
<BANKED_CODE,XDATA_ROM_C_FLASH> 1 (was BANKED_CODE)
  Relative segment, address: CODE 0000A6F2 - 0000A6F4 (0x3 bytes), align: 0
  Segment part 48.            Intra module refs:   llSetT2OVFC1Event1
                                                   llSetT2OVFC1Timeout
    -------------------------------------------------------------------------
<BANKED_CODE,XDATA_ROM_C_FLASH> 1 (was BANKED_CODE)
  Relative segment, address: CODE 0000A6F5 - 0000A700 (0xc bytes), align: 0
  Segment part 49.            Intra module refs:   Segment part 48
                                                   llSetT2OVFC2Event2
    -------------------------------------------------------------------------
<BANKED_CODE,XDATA_ROM_C_FLASH> 1 (was BANKED_CODE)
  Relative segment, address: CODE 0000A701 - 0000A723 (0x23 bytes), align: 0
  Segment part 52.            Intra module refs:   llSetT2C1Event1::?relay
           ENTRY                   ADDRESS         REF BY
           =====                   =======         ======
           llSetT2C1Event1         0000A701 
               XSTACK = 00000000 ( 00000002 )
               ISTACK = 00000000 ( 00000002 )
    -------------------------------------------------------------------------
<BANKED_CODE,XDATA_ROM_C_FLASH> 1 (was BANKED_CODE)
  Relative segment, address: CODE 0000A724 - 0000A72A (0x7 bytes), align: 0
  Segment part 54.            Intra module refs:   llSetT2C1Event1
    -------------------------------------------------------------------------
<BANKED_CODE,XDATA_ROM_C_FLASH> 1 (was BANKED_CODE)
  Relative segment, address: CODE 0000A72B - 0000A73A (0x10 bytes), align: 0
  Segment part 55.            Intra module refs:   Segment part 54
    -------------------------------------------------------------------------
<BANKED_CODE,XDATA_ROM_C_FLASH> 1 (was BANKED_CODE)
  Relative segment, address: CODE 0000A73B - 0000A763 (0x29 bytes), align: 0
  Segment part 56.            Intra module refs:   llSetT2OVFC1Event1::?relay
           ENTRY                   ADDRESS         REF BY
           =====                   =======         ======
           llSetT2OVFC1Event1      0000A73B 
               XSTACK = 00000000 ( 00000004 )
               ISTACK = 00000000 ( 00000002 )
    -------------------------------------------------------------------------
<BANKED_CODE,XDATA_ROM_C_FLASH> 1 (was BANKED_CODE)
  Relative segment, address: CODE 0000A764 - 0000A769 (0x6 bytes), align: 0
  Segment part 58.            Intra module refs:   llSetT2OVFC1Event1
                                                   llSetT2OVFC1Timeout
                                                   llSetT2OVFC2Event2
    -------------------------------------------------------------------------
<BANKED_CODE,XDATA_ROM_C_FLASH> 1 (was BANKED_CODE)
  Relative segment, address: CODE 0000A76A - 0000A774 (0xb bytes), align: 0
  Segment part 59.            Intra module refs:   llSetT2OVFC1Event1
                                                   llSetT2OVFC1Timeout
    -------------------------------------------------------------------------
<BANKED_CODE,XDATA_ROM_C_FLASH> 1 (was BANKED_CODE)
  Relative segment, address: CODE 0000A775 - 0000A7D1 (0x5d bytes), align: 0
  Segment part 60.            Intra module refs:   llSetT2OVFC2Event2::?relay
           ENTRY                   ADDRESS         REF BY
           =====                   =======         ======
           llSetT2OVFC2Event2      0000A775 
               XSTACK = 00000000 ( 00000010 )
    -------------------------------------------------------------------------
<BANKED_CODE,XDATA_ROM_C_FLASH> 1 (was BANKED_CODE)
  Relative segment, address: CODE 0000A7D2 - 0000A7D5 (0x4 bytes), align: 0
  Segment part 62.            Intra module refs:   llSetT2OVFC2Event2
    -------------------------------------------------------------------------
<BANKED_CODE,XDATA_ROM_C_FLASH> 1 (was BANKED_CODE)
  Relative segment, address: CODE 0000A7D6 - 0000A7E7 (0x12 bytes), align: 0
  Segment part 63.            Intra module refs:   Segment part 59
                                                   Segment part 62
    -------------------------------------------------------------------------
<BANKED_CODE,XDATA_ROM_C_FLASH> 1 (was BANKED_CODE)
  Relative segment, address: CODE 0000A7E8 - 0000A828 (0x41 bytes), align: 0
  Segment part 64.            Intra module refs:   llSetT2Delta::?relay
           ENTRY                   ADDRESS         REF BY
           =====                   =======         ======
           llSetT2Delta            0000A7E8 
               XSTACK = 00000000 ( 00000002 )
               ISTACK = 00000000 ( 00000002 )
    -------------------------------------------------------------------------
<BANKED_CODE,XDATA_ROM_C_FLASH> 1 (was BANKED_CODE)
  Relative segment, address: CODE 0000A829 - 0000A831 (0x9 bytes), align: 0
  Segment part 66.            Intra module refs:   llDisableT2Ints::?relay
           ENTRY                   ADDRESS         REF BY
           =====                   =======         ======
           llDisableT2Ints         0000A829 
    -------------------------------------------------------------------------
<BANKED_CODE,XDATA_ROM_C_FLASH> 1 (was BANKED_CODE)
  Relative segment, address: CODE 0000A832 - 0000A83D (0xc bytes), align: 0
  Segment part 68.            Intra module refs:   llDisableT2IntsEvts::?relay
           ENTRY                   ADDRESS         REF BY
           =====                   =======         ======
           llDisableT2IntsEvts     0000A832 
    -------------------------------------------------------------------------
<BANKED_CODE,XDATA_ROM_C_FLASH> 1 (was BANKED_CODE)
  Relative segment, address: CODE 0000A83E - 0000A84B (0xe bytes), align: 0
  Segment part 70.            Intra module refs:   llDisableT2E1::?relay
           ENTRY                   ADDRESS         REF BY
           =====                   =======         ======
           llDisableT2E1           0000A83E 
    -------------------------------------------------------------------------
<BANKED_CODE,XDATA_ROM_C_FLASH> 1 (was BANKED_CODE)
  Relative segment, address: CODE 0000A84C - 0000A84E (0x3 bytes), align: 0
  Segment part 72.            Intra module refs:   llDisableT2Ints
                                                   llDisableT2IntsEvts
    -------------------------------------------------------------------------
<BANKED_CODE,XDATA_ROM_C_FLASH> 1 (was BANKED_CODE)
  Relative segment, address: CODE 0000A84F - 0000A857 (0x9 bytes), align: 0
  Segment part 73.            Intra module refs:   Segment part 72
                                                   llDisableT2E1
    -------------------------------------------------------------------------
<BANKED_CODE,XDATA_ROM_C_FLASH> 1 (was BANKED_CODE)
  Relative segment, address: CODE 0000A858 - 0000A85C (0x5 bytes), align: 0
  Segment part 74.            Intra module refs:   Segment part 28
                                                   Segment part 73
    -------------------------------------------------------------------------
<BANKED_CODE,XDATA_ROM_C_FLASH> 1 (was BANKED_CODE)
  Relative segment, address: CODE 0000A85D - 0000A871 (0x15 bytes), align: 0
  Segment part 79.            Intra module refs:   llGetCurrentTime::?relay
           ENTRY                   ADDRESS         REF BY
           =====                   =======         ======
           llGetCurrentTime        0000A85D 
               XSTACK = 00000000 ( 00000004 )
               ISTACK = 00000000 ( 00000003 )
    -------------------------------------------------------------------------
NEAR_CODE
  Relative segment, address: CODE 000015F9 - 0000164F (0x57 bytes), align: 0
  Segment part 96.
           ENTRY                   ADDRESS         REF BY
           =====                   =======         ======
           ll24BitTimeCompare      000015F9        LL_EXT_ExtendRfRange (ll)
                                                   LL_EXT_SetRxGain (ll)
                                                   LL_EXT_SetTxPower (ll)
                                                   llFindNextSecTask (ll_scheduler)
                                                   llScheduler (ll_scheduler)
               XSTACK = 00000004 ( 0000000F )
    -------------------------------------------------------------------------
NEAR_CODE
  Relative segment, address: CODE 00001650 - 00001654 (0x5 bytes), align: 0
  Segment part 97.            Intra module refs:   ll24BitTimeCompare
    -------------------------------------------------------------------------
NEAR_CODE
  Relative segment, address: CODE 00001655 - 000016BC (0x68 bytes), align: 0
  Segment part 98.
           ENTRY                   ADDRESS         REF BY
           =====                   =======         ======
           ll24BitTimeDelta        00001655        LL_EXT_ExtendRfRange (ll)
                                                   LL_EXT_SetRxGain (ll)
                                                   LL_EXT_SetTxPower (ll)
                                                   llScheduleTask (ll_scheduler)
               XSTACK = 00000004 ( 00000013 )
    -------------------------------------------------------------------------
<BANKED_CODE,XDATA_ROM_C_FLASH> 1 (was BANKED_CODE)
  Relative segment, address: CODE 0000A872 - 0000A89F (0x2e bytes), align: 0
  Segment part 94.            Intra module refs:   ll_McuPrecisionCount::?relay
           ENTRY                   ADDRESS         REF BY
           =====                   =======         ======
           ll_McuPrecisionCount    0000A872 
               XSTACK = 00000000 ( 00000002 )
               ISTACK = 00000000 ( 00000003 )
    -------------------------------------------------------------------------
BANK_RELAYS
  Relative segment, address: CODE 0000065C - 00000661 (0x6 bytes), align: 0
  Segment part 25.
           ENTRY                   ADDRESS         REF BY
           =====                   =======         ======
           llInitTimer2::?relay    0000065C        LL_Init (ll)
    -------------------------------------------------------------------------
BANK_RELAYS
  Relative segment, address: CODE 00000662 - 00000667 (0x6 bytes), align: 0
  Segment part 27.            Intra module refs:   llInitTimer2
           ENTRY                   ADDRESS         REF BY
           =====                   =======         ======
           llStopTimer2::?relay    00000662 
    -------------------------------------------------------------------------
BANK_RELAYS
  Relative segment, address: CODE 00000668 - 0000066D (0x6 bytes), align: 0
  Segment part 30.            Intra module refs:   llInitTimer2
           ENTRY                   ADDRESS         REF BY
           =====                   =======         ======
           llStartTimer2::?relay   00000668 
    -------------------------------------------------------------------------
BANK_RELAYS
  Relative segment, address: CODE 0000066E - 00000673 (0x6 bytes), align: 0
  Segment part 46.
           ENTRY                   ADDRESS         REF BY
           =====                   =======         ======
           llSetT2OVFC1Timeout::?relay
                                   0000066E        llScheduleTask (ll_scheduler)
    -------------------------------------------------------------------------
BANK_RELAYS
  Relative segment, address: CODE 00000674 - 00000679 (0x6 bytes), align: 0
  Segment part 53.
           ENTRY                   ADDRESS         REF BY
           =====                   =======         ======
           llSetT2C1Event1::?relay
                                   00000674        LL_DirectTestTxTest (ll)
                                                   LL_EXT_ModemHopTestTx (ll)
                                                   llT2OVFC1_ISR (ll_isr)
    -------------------------------------------------------------------------
BANK_RELAYS
  Relative segment, address: CODE 0000067A - 0000067F (0x6 bytes), align: 0
  Segment part 57.
           ENTRY                   ADDRESS         REF BY
           =====                   =======         ======
           llSetT2OVFC1Event1::?relay
                                   0000067A        llScheduleTask (ll_scheduler)
    -------------------------------------------------------------------------
BANK_RELAYS
  Relative segment, address: CODE 00000680 - 00000685 (0x6 bytes), align: 0
  Segment part 61.
           ENTRY                   ADDRESS         REF BY
           =====                   =======         ======
           llSetT2OVFC2Event2::?relay
                                   00000680        llScheduleTask (ll_scheduler)
    -------------------------------------------------------------------------
BANK_RELAYS
  Relative segment, address: CODE 00000686 - 0000068B (0x6 bytes), align: 0
  Segment part 65.
           ENTRY                   ADDRESS         REF BY
           =====                   =======         ======
           llSetT2Delta::?relay    00000686        llScheduleTask (ll_scheduler)
    -------------------------------------------------------------------------
BANK_RELAYS
  Relative segment, address: CODE 0000068C - 00000691 (0x6 bytes), align: 0
  Segment part 67.
           ENTRY                   ADDRESS         REF BY
           =====                   =======         ======
           llDisableT2Ints::?relay
                                   0000068C        RF_NormalIsr (ll_isr)
    -------------------------------------------------------------------------
BANK_RELAYS
  Relative segment, address: CODE 00000692 - 00000697 (0x6 bytes), align: 0
  Segment part 69.
           ENTRY                   ADDRESS         REF BY
           =====                   =======         ======
           llDisableT2IntsEvts::?relay
                                   00000692        LL_DirectTestRxTest (ll)
                                                   LL_DirectTestTxTest (ll)
                                                   LL_EXT_ModemHopTestTx (ll)
                                                   LL_EXT_ModemTestRx (ll)
                                                   LL_EXT_ModemTestTx (ll)
                                                   LL_Reset (ll)
                                                   LL_SetAdvControl (ll)
                                                   RF_NormalIsr (ll_isr)
    -------------------------------------------------------------------------
BANK_RELAYS
  Relative segment, address: CODE 00000698 - 0000069D (0x6 bytes), align: 0
  Segment part 71.
           ENTRY                   ADDRESS         REF BY
           =====                   =======         ======
           llDisableT2E1::?relay   00000698        RF_NormalIsr (ll_isr)
    -------------------------------------------------------------------------
BANK_RELAYS
  Relative segment, address: CODE 0000069E - 000006A3 (0x6 bytes), align: 0
  Segment part 80.
           ENTRY                   ADDRESS         REF BY
           =====                   =======         ======
           llGetCurrentTime::?relay
                                   0000069E        LL_EXT_ExtendRfRange (ll)
                                                   LL_EXT_SetRxGain (ll)
                                                   LL_EXT_SetTxPower (ll)
                                                   LL_SetAdvControl (ll)
                                                   llAllocTask (ll_scheduler)
                                                   llScheduleTask (ll_scheduler)
                                                   llScheduler (ll_scheduler)
    -------------------------------------------------------------------------
BANK_RELAYS
  Relative segment, address: CODE 000006A4 - 000006A9 (0x6 bytes), align: 0
  Segment part 95.
           ENTRY                   ADDRESS         REF BY
           =====                   =======         ======
           ll_McuPrecisionCount::?relay
                                   000006A4        osalTimeUpdate (OSAL_ClockBLE)

    -------------------------------------------------------------------------
  LIBRARY MODULE, NAME : phy

  SEGMENTS IN THE MODULE
  ======================
XDATA_Z
  Relative segment, address: XDATA 000003AB - 000003AB (0x1 bytes), align: 0
  Segment part 11.            Intra module refs:   PHY_AddWlEntry
                                                   PHY_ClearWhitelist
                                                   PHY_RemoveWlEntry
                                                   Segment part 92
           ENTRY                   ADDRESS         REF BY
           =====                   =======         ======
           numWLEntries            000003AB 
    -------------------------------------------------------------------------
<BANKED_CODE,CODE_C> 1 (was BANKED_CODE)
  Relative segment, address: CODE 00007201 - 00007213 (0x13 bytes), align: 0
  Segment part 12.            Intra module refs:   PHY_Init::?relay
           ENTRY                   ADDRESS         REF BY
           =====                   =======         ======
           PHY_Init                00007201 
               calls direct
               ISTACK = 00000000 ( 00000002 )
    -------------------------------------------------------------------------
<BANKED_CODE,CODE_C> 1 (was BANKED_CODE)
  Relative segment, address: CODE 00007214 - 0000722D (0x1a bytes), align: 0
  Segment part 18.            Intra module refs:   PHY_Reset::?relay
           ENTRY                   ADDRESS         REF BY
           =====                   =======         ======
           PHY_Reset               00007214 
               ISTACK = 00000000 ( 00000002 )
    -------------------------------------------------------------------------
<BANKED_CODE,CODE_C> 1 (was BANKED_CODE)
  Relative segment, address: CODE 0000722E - 0000725A (0x2d bytes), align: 0
  Segment part 20.            Intra module refs:   PHY_LoadNR::?relay
           ENTRY                   ADDRESS         REF BY
           =====                   =======         ======
           PHY_LoadNR              0000722E 
               ISTACK = 00000000 ( 00000002 )
    -------------------------------------------------------------------------
<BANKED_CODE,CODE_C> 1 (was BANKED_CODE)
  Relative segment, address: CODE 0000725B - 00007294 (0x3a bytes), align: 0
  Segment part 22.            Intra module refs:   PHY_VerifyNR::?relay
           ENTRY                   ADDRESS         REF BY
           =====                   =======         ======
           PHY_VerifyNR            0000725B 
               ISTACK = 00000000 ( 00000002 )
    -------------------------------------------------------------------------
<BANKED_CODE,CODE_C> 1 (was BANKED_CODE)
  Relative segment, address: CODE 00007295 - 000072A0 (0xc bytes), align: 0
  Segment part 24.            Intra module refs:   PHY_LoadNR
                                                   PHY_VerifyNR
    -------------------------------------------------------------------------
<BANKED_CODE,CODE_C> 1 (was BANKED_CODE)
  Relative segment, address: CODE 000072A1 - 000072D3 (0x33 bytes), align: 0
  Segment part 25.            Intra module refs:   PHY_ClearAllRegsAndFifos::?relay
           ENTRY                   ADDRESS         REF BY
           =====                   =======         ======
           PHY_ClearAllRegsAndFifos
                                   000072A1 
               ISTACK = 00000000 ( 00000002 )
    -------------------------------------------------------------------------
<BANKED_CODE,CODE_C> 1 (was BANKED_CODE)
  Relative segment, address: CODE 000072D4 - 00007311 (0x3e bytes), align: 0
  Segment part 31.            Intra module refs:   PHY_SetOwnAddr::?relay
           ENTRY                   ADDRESS         REF BY
           =====                   =======         ======
           PHY_SetOwnAddr          000072D4 
               ISTACK = 00000000 ( 00000002 )
    -------------------------------------------------------------------------
<BANKED_CODE,CODE_C> 1 (was BANKED_CODE)
  Relative segment, address: CODE 00007312 - 0000731A (0x9 bytes), align: 0
  Segment part 35.            Intra module refs:   PHY_SetOwnAddr
    -------------------------------------------------------------------------
<BANKED_CODE,CODE_C> 1 (was BANKED_CODE)
  Relative segment, address: CODE 0000731B - 0000731F (0x5 bytes), align: 0
  Segment part 36.            Intra module refs:   PHY_SetOwnAddr
    -------------------------------------------------------------------------
<BANKED_CODE,CODE_C> 1 (was BANKED_CODE)
  Relative segment, address: CODE 00007320 - 00007324 (0x5 bytes), align: 0
  Segment part 37.            Intra module refs:   PHY_SetOwnAddr
    -------------------------------------------------------------------------
<BANKED_CODE,CODE_C> 1 (was BANKED_CODE)
  Relative segment, address: CODE 00007325 - 0000732A (0x6 bytes), align: 0
  Segment part 38.            Intra module refs:   PHY_SetOwnAddr
    -------------------------------------------------------------------------
<BANKED_CODE,CODE_C> 1 (was BANKED_CODE)
  Relative segment, address: CODE 0000732B - 0000732F (0x5 bytes), align: 0
  Segment part 39.            Intra module refs:   Segment part 37
                                                   Segment part 38
    -------------------------------------------------------------------------
<BANKED_CODE,CODE_C> 1 (was BANKED_CODE)
  Relative segment, address: CODE 00007330 - 00007338 (0x9 bytes), align: 0
  Segment part 40.            Intra module refs:   Segment part 36
                                                   Segment part 39
    -------------------------------------------------------------------------
<BANKED_CODE,CODE_C> 1 (was BANKED_CODE)
  Relative segment, address: CODE 00007339 - 00007346 (0xe bytes), align: 0
  Segment part 41.            Intra module refs:   PHY_SetCRCInit::?relay
           ENTRY                   ADDRESS         REF BY
           =====                   =======         ======
           PHY_SetCRCInit          00007339 
               XSTACK = 00000000 ( 00000010 )
    -------------------------------------------------------------------------
<BANKED_CODE,CODE_C> 1 (was BANKED_CODE)
  Relative segment, address: CODE 00007347 - 0000734D (0x7 bytes), align: 0
  Segment part 43.            Intra module refs:   PHY_SetCRCInit
                                                   PHY_SetSyncWord
    -------------------------------------------------------------------------
<BANKED_CODE,CODE_C> 1 (was BANKED_CODE)
  Relative segment, address: CODE 0000734E - 00007358 (0xb bytes), align: 0
  Segment part 44.            Intra module refs:   PHY_GetAdvChans::?relay
           ENTRY                   ADDRESS         REF BY
           =====                   =======         ======
           PHY_GetAdvChans         0000734E 
               ISTACK = 00000000 ( 00000002 )
    -------------------------------------------------------------------------
<BANKED_CODE,CODE_C> 1 (was BANKED_CODE)
  Relative segment, address: CODE 00007359 - 00007365 (0xd bytes), align: 0
  Segment part 46.            Intra module refs:   PHY_SetAdvChans::?relay
           ENTRY                   ADDRESS         REF BY
           =====                   =======         ======
           PHY_SetAdvChans         00007359 
               ISTACK = 00000000 ( 00000002 )
    -------------------------------------------------------------------------
<BANKED_CODE,CODE_C> 1 (was BANKED_CODE)
  Relative segment, address: CODE 00007366 - 0000737C (0x17 bytes), align: 0
  Segment part 48.            Intra module refs:   PHY_SetEndConnection::?relay
           ENTRY                   ADDRESS         REF BY
           =====                   =======         ======
           PHY_SetEndConnection    00007366 
               ISTACK = 00000000 ( 00000002 )
    -------------------------------------------------------------------------
<BANKED_CODE,CODE_C> 1 (was BANKED_CODE)
  Relative segment, address: CODE 0000737D - 0000738A (0xe bytes), align: 0
  Segment part 50.            Intra module refs:   PHY_ConfigureMD::?relay
           ENTRY                   ADDRESS         REF BY
           =====                   =======         ======
           PHY_ConfigureMD         0000737D 
               ISTACK = 00000000 ( 00000002 )
    -------------------------------------------------------------------------
<BANKED_CODE,CODE_C> 1 (was BANKED_CODE)
  Relative segment, address: CODE 0000738B - 00007395 (0xb bytes), align: 0
  Segment part 58.            Intra module refs:   PHY_GetEndCause::?relay
           ENTRY                   ADDRESS         REF BY
           =====                   =======         ======
           PHY_GetEndCause         0000738B 
               ISTACK = 00000000 ( 00000002 )
    -------------------------------------------------------------------------
<BANKED_CODE,CODE_C> 1 (was BANKED_CODE)
  Relative segment, address: CODE 00007396 - 000073A8 (0x13 bytes), align: 0
  Segment part 68.            Intra module refs:   PHY_SetSyncWord::?relay
           ENTRY                   ADDRESS         REF BY
           =====                   =======         ======
           PHY_SetSyncWord         00007396 
               XSTACK = 00000000 ( 00000010 )
    -------------------------------------------------------------------------
<BANKED_CODE,CODE_C> 1 (was BANKED_CODE)
  Relative segment, address: CODE 000073A9 - 000073C1 (0x19 bytes), align: 0
  Segment part 72.            Intra module refs:   PHY_ClearWhitelist::?relay
           ENTRY                   ADDRESS         REF BY
           =====                   =======         ======
           PHY_ClearWhitelist      000073A9 
               ISTACK = 00000000 ( 00000002 )
    -------------------------------------------------------------------------
<BANKED_CODE,CODE_C> 1 (was BANKED_CODE)
  Relative segment, address: CODE 000073C2 - 000073C2 (0x1 bytes), align: 0
  Segment part 78.            Intra module refs:   PHY_ClearBlacklistIndex
                                                   PHY_SetBlacklistIndex
    -------------------------------------------------------------------------
<BANKED_CODE,CODE_C> 1 (was BANKED_CODE)
  Relative segment, address: CODE 000073C3 - 000073C7 (0x5 bytes), align: 0
  Segment part 79.            Intra module refs:   PHY_RemoveWlEntry
                                                   Segment part 78
    -------------------------------------------------------------------------
<BANKED_CODE,CODE_C> 1 (was BANKED_CODE)
  Relative segment, address: CODE 000073C8 - 000073CB (0x4 bytes), align: 0
  Segment part 84.            Intra module refs:   PHY_GetAdvChans
                                                   PHY_GetEndCause
    -------------------------------------------------------------------------
<BANKED_CODE,CODE_C> 1 (was BANKED_CODE)
  Relative segment, address: CODE 000073CC - 000073D0 (0x5 bytes), align: 0
  Segment part 85.            Intra module refs:   PHY_GetWlSize::?relay
           ENTRY                   ADDRESS         REF BY
           =====                   =======         ======
           PHY_GetWlSize           000073CC 
    -------------------------------------------------------------------------
<BANKED_CODE,CODE_C> 1 (was BANKED_CODE)
  Relative segment, address: CODE 000073D1 - 00007467 (0x97 bytes), align: 0
  Segment part 87.            Intra module refs:   PHY_AddWlEntry::?relay
           ENTRY                   ADDRESS         REF BY
           =====                   =======         ======
           PHY_AddWlEntry          000073D1 
               calls direct
               XSTACK = 00000000 ( 0000000C )
               ISTACK = 00000000 ( 00000001 )
    -------------------------------------------------------------------------
<BANKED_CODE,CODE_C> 1 (was BANKED_CODE)
  Relative segment, address: CODE 00007468 - 000074B8 (0x51 bytes), align: 0
  Segment part 89.            Intra module refs:   PHY_RemoveWlEntry::?relay
           ENTRY                   ADDRESS         REF BY
           =====                   =======         ======
           PHY_RemoveWlEntry       00007468 
               calls direct
               XSTACK = 00000000 ( 0000000A )
               ISTACK = 00000000 ( 00000001 )
    -------------------------------------------------------------------------
<BANKED_CODE,CODE_C> 1 (was BANKED_CODE)
  Relative segment, address: CODE 000074B9 - 000074C5 (0xd bytes), align: 0
  Segment part 91.            Intra module refs:   PHY_AddWlEntry
                                                   PHY_RemoveWlEntry
    -------------------------------------------------------------------------
<BANKED_CODE,CODE_C> 1 (was BANKED_CODE)
  Relative segment, address: CODE 000074C6 - 000074CF (0xa bytes), align: 0
  Segment part 92.            Intra module refs:   PHY_RemoveWlEntry
    -------------------------------------------------------------------------
<BANKED_CODE,CODE_C> 1 (was BANKED_CODE)
  Relative segment, address: CODE 000074D0 - 000074DF (0x10 bytes), align: 0
  Segment part 93.            Intra module refs:   PHY_SetAdvWlPolicy::?relay
           ENTRY                   ADDRESS         REF BY
           =====                   =======         ======
           PHY_SetAdvWlPolicy      000074D0 
               ISTACK = 00000000 ( 00000002 )
    -------------------------------------------------------------------------
<BANKED_CODE,CODE_C> 1 (was BANKED_CODE)
  Relative segment, address: CODE 000074E0 - 000074F9 (0x1a bytes), align: 0
  Segment part 99.            Intra module refs:   PHY_SetBlacklistIndex::?relay
           ENTRY                   ADDRESS         REF BY
           =====                   =======         ======
           PHY_SetBlacklistIndex   000074E0 
               XSTACK = 0000000C ( 0000000A )
    -------------------------------------------------------------------------
<BANKED_CODE,CODE_C> 1 (was BANKED_CODE)
  Relative segment, address: CODE 000074FA - 00007516 (0x1d bytes), align: 0
  Segment part 104.           Intra module refs:   PHY_ClearBlacklistIndex::?relay
           ENTRY                   ADDRESS         REF BY
           =====                   =======         ======
           PHY_ClearBlacklistIndex
                                   000074FA 
               XSTACK = 0000000C ( 0000000A )
    -------------------------------------------------------------------------
<BANKED_CODE,CODE_C> 1 (was BANKED_CODE)
  Relative segment, address: CODE 00007517 - 00007521 (0xb bytes), align: 0
  Segment part 106.           Intra module refs:   PHY_ClearBlacklist::?relay
           ENTRY                   ADDRESS         REF BY
           =====                   =======         ======
           PHY_ClearBlacklist      00007517 
               ISTACK = 00000000 ( 00000002 )
    -------------------------------------------------------------------------
<BANKED_CODE,CODE_C> 1 (was BANKED_CODE)
  Relative segment, address: CODE 00007522 - 00007526 (0x5 bytes), align: 0
  Segment part 111.           Intra module refs:   PHY_AddWlEntry
    -------------------------------------------------------------------------
<BANKED_CODE,CODE_C> 1 (was BANKED_CODE)
  Relative segment, address: CODE 00007527 - 0000752B (0x5 bytes), align: 0
  Segment part 118.           Intra module refs:   PHY_ClearSavedWhiteList
    -------------------------------------------------------------------------
<BANKED_CODE,CODE_C> 1 (was BANKED_CODE)
  Relative segment, address: CODE 0000752C - 00007531 (0x6 bytes), align: 0
  Segment part 119.           Intra module refs:   PHY_SetOwnAddr
                                                   Segment part 118
    -------------------------------------------------------------------------
<BANKED_CODE,CODE_C> 1 (was BANKED_CODE)
  Relative segment, address: CODE 00007532 - 00007547 (0x16 bytes), align: 0
  Segment part 121.           Intra module refs:   PHY_ClearSavedWhiteList::?relay
           ENTRY                   ADDRESS         REF BY
           =====                   =======         ======
           PHY_ClearSavedWhiteList
                                   00007532 
               ISTACK = 00000000 ( 00000002 )
    -------------------------------------------------------------------------
<BANKED_CODE,CODE_C> 1 (was BANKED_CODE)
  Relative segment, address: CODE 00007548 - 0000754D (0x6 bytes), align: 0
  Segment part 123.           Intra module refs:   PHY_ClearSavedWhiteList
    -------------------------------------------------------------------------
<BANKED_CODE,CODE_C> 1 (was BANKED_CODE)
  Relative segment, address: CODE 0000754E - 0000755B (0xe bytes), align: 0
  Segment part 124.           Intra module refs:   PHY_Command::?relay
           ENTRY                   ADDRESS         REF BY
           =====                   =======         ======
           PHY_Command             0000754E 
    -------------------------------------------------------------------------
<BANKED_CODE,CODE_C> 1 (was BANKED_CODE)
  Relative segment, address: CODE 0000755C - 0000755F (0x4 bytes), align: 0
  Segment part 131.           Intra module refs:   PHY_AddWlEntry
                                                   PHY_RawGetNumTxPkts
    -------------------------------------------------------------------------
<BANKED_CODE,CODE_C> 1 (was BANKED_CODE)
  Relative segment, address: CODE 00007560 - 00007564 (0x5 bytes), align: 0
  Segment part 132.           Intra module refs:   Segment part 131
                                                   Segment part 217
    -------------------------------------------------------------------------
<BANKED_CODE,CODE_C> 1 (was BANKED_CODE)
  Relative segment, address: CODE 00007565 - 0000756F (0xb bytes), align: 0
  Segment part 134.           Intra module refs:   PHY_ConfigureFifoDataProcessing::?relay
           ENTRY                   ADDRESS         REF BY
           =====                   =======         ======
           PHY_ConfigureFifoDataProcessing
                                   00007565 
               ISTACK = 00000000 ( 00000002 )
    -------------------------------------------------------------------------
<BANKED_CODE,CODE_C> 1 (was BANKED_CODE)
  Relative segment, address: CODE 00007570 - 00007584 (0x15 bytes), align: 0
  Segment part 136.           Intra module refs:   PHY_ConfigureAppendRfStatus::?relay
           ENTRY                   ADDRESS         REF BY
           =====                   =======         ======
           PHY_ConfigureAppendRfStatus
                                   00007570 
               ISTACK = 00000000 ( 00000002 )
    -------------------------------------------------------------------------
<BANKED_CODE,CODE_C> 1 (was BANKED_CODE)
  Relative segment, address: CODE 00007585 - 0000758F (0xb bytes), align: 0
  Segment part 138.           Intra module refs:   PHY_SetFifoConfig::?relay
           ENTRY                   ADDRESS         REF BY
           =====                   =======         ======
           PHY_SetFifoConfig       00007585 
               ISTACK = 00000000 ( 00000002 )
    -------------------------------------------------------------------------
<BANKED_CODE,CODE_C> 1 (was BANKED_CODE)
  Relative segment, address: CODE 00007590 - 00007598 (0x9 bytes), align: 0
  Segment part 150.           Intra module refs:   PHY_SetSyncWord
    -------------------------------------------------------------------------
<BANKED_CODE,CODE_C> 1 (was BANKED_CODE)
  Relative segment, address: CODE 00007599 - 000075F9 (0x61 bytes), align: 0
  Segment part 151.           Intra module refs:   PHY_ConfigWhitener::?relay
           ENTRY                   ADDRESS         REF BY
           =====                   =======         ======
           PHY_ConfigWhitener      00007599 
               ISTACK = 00000000 ( 00000002 )
    -------------------------------------------------------------------------
<BANKED_CODE,CODE_C> 1 (was BANKED_CODE)
  Relative segment, address: CODE 000075FA - 000075FB (0x2 bytes), align: 0
  Segment part 179.           Intra module refs:   PHY_RawRxInit
    -------------------------------------------------------------------------
<BANKED_CODE,CODE_C> 1 (was BANKED_CODE)
  Relative segment, address: CODE 000075FC - 000075FD (0x2 bytes), align: 0
  Segment part 180.           Intra module refs:   PHY_ClearAllRegsAndFifos
                                                   Segment part 179
    -------------------------------------------------------------------------
<BANKED_CODE,CODE_C> 1 (was BANKED_CODE)
  Relative segment, address: CODE 000075FE - 000075FE (0x1 bytes), align: 0
  Segment part 181.           Intra module refs:   PHY_RawTxInit
                                                   Segment part 180
    -------------------------------------------------------------------------
<BANKED_CODE,CODE_C> 1 (was BANKED_CODE)
  Relative segment, address: CODE 000075FF - 000075FF (0x1 bytes), align: 0
  Segment part 182.           Intra module refs:   Segment part 181
                                                   Segment part 211
    -------------------------------------------------------------------------
<BANKED_CODE,CODE_C> 1 (was BANKED_CODE)
  Relative segment, address: CODE 00007600 - 00007600 (0x1 bytes), align: 0
  Segment part 183.           Intra module refs:   PHY_ClearBlacklist
                                                   PHY_ConfigureAppendRfStatus
                                                   PHY_ConfigureFifoDataProcessing
                                                   PHY_ConfigureMD
                                                   PHY_RawGetRxData
                                                   PHY_SetAdvChans
                                                   PHY_SetAdvWlPolicy
                                                   PHY_SetEndConnection
                                                   PHY_SetFifoConfig
                                                   PHY_SetOwnAddr
                                                   PHY_SetRfFreq
                                                   Segment part 123
                                                   Segment part 182
    -------------------------------------------------------------------------
<BANKED_CODE,CODE_C> 1 (was BANKED_CODE)
  Relative segment, address: CODE 00007601 - 00007607 (0x7 bytes), align: 0
  Segment part 184.           Intra module refs:   PHY_ClearWhitelist
                                                   PHY_ConfigWhitener
                                                   PHY_Init
                                                   PHY_LoadNR
                                                   PHY_Reset
                                                   PHY_VerifyNR
                                                   Segment part 183
                                                   Segment part 84
    -------------------------------------------------------------------------
<BANKED_CODE,CODE_C> 1 (was BANKED_CODE)
  Relative segment, address: CODE 00007608 - 0000762E (0x27 bytes), align: 0
  Segment part 204.           Intra module refs:   PHY_RawTxInit::?relay
           ENTRY                   ADDRESS         REF BY
           =====                   =======         ======
           PHY_RawTxInit           00007608 
               ISTACK = 00000000 ( 00000002 )
    -------------------------------------------------------------------------
<BANKED_CODE,CODE_C> 1 (was BANKED_CODE)
  Relative segment, address: CODE 0000762F - 0000765A (0x2c bytes), align: 0
  Segment part 206.           Intra module refs:   PHY_RawRxInit::?relay
           ENTRY                   ADDRESS         REF BY
           =====                   =======         ======
           PHY_RawRxInit           0000762F 
               ISTACK = 00000000 ( 00000002 )
    -------------------------------------------------------------------------
<BANKED_CODE,CODE_C> 1 (was BANKED_CODE)
  Relative segment, address: CODE 0000765B - 00007669 (0xf bytes), align: 0
  Segment part 208.           Intra module refs:   PHY_RawRxInit
                                                   PHY_RawTxInit
    -------------------------------------------------------------------------
<BANKED_CODE,CODE_C> 1 (was BANKED_CODE)
  Relative segment, address: CODE 0000766A - 00007676 (0xd bytes), align: 0
  Segment part 209.           Intra module refs:   PHY_RawGetNumTxPkts::?relay
           ENTRY                   ADDRESS         REF BY
           =====                   =======         ======
           PHY_RawGetNumTxPkts     0000766A 
               ISTACK = 00000000 ( 00000003 )
    -------------------------------------------------------------------------
<BANKED_CODE,CODE_C> 1 (was BANKED_CODE)
  Relative segment, address: CODE 00007677 - 0000767C (0x6 bytes), align: 0
  Segment part 211.           Intra module refs:   PHY_RawGetNumTxPkts
    -------------------------------------------------------------------------
<BANKED_CODE,CODE_C> 1 (was BANKED_CODE)
  Relative segment, address: CODE 0000767D - 00007682 (0x6 bytes), align: 0
  Segment part 212.           Intra module refs:   PHY_RawGetRxData
                                                   Segment part 132
                                                   Segment part 211
    -------------------------------------------------------------------------
<BANKED_CODE,CODE_C> 1 (was BANKED_CODE)
  Relative segment, address: CODE 00007683 - 000076BA (0x38 bytes), align: 0
  Segment part 215.           Intra module refs:   PHY_RawGetRxData::?relay
           ENTRY                   ADDRESS         REF BY
           =====                   =======         ======
           PHY_RawGetRxData        00007683 
               XSTACK = 00000002 ( 00000000 )
               ISTACK = 00000000 ( 00000003 )
    -------------------------------------------------------------------------
<BANKED_CODE,CODE_C> 1 (was BANKED_CODE)
  Relative segment, address: CODE 000076BB - 000076C4 (0xa bytes), align: 0
  Segment part 217.           Intra module refs:   PHY_RawGetRxData
    -------------------------------------------------------------------------
<BANKED_CODE,CODE_C> 1 (was BANKED_CODE)
  Relative segment, address: CODE 000076C5 - 000076F7 (0x33 bytes), align: 0
  Segment part 218.           Intra module refs:   PHY_SetRfFreq::?relay
           ENTRY                   ADDRESS         REF BY
           =====                   =======         ======
           PHY_SetRfFreq           000076C5 
               ISTACK = 00000000 ( 00000002 )
    -------------------------------------------------------------------------
<BANKED_CODE,CODE_C> 1 (was BANKED_CODE)
  Relative segment, address: CODE 000076F8 - 00007774 (0x7d bytes), align: 0
  Segment part 220.           Intra module refs:   phyFindWlEntry::?relay
           LOCAL                   ADDRESS         
           =====                   =======         
           phyFindWlEntry          000076F8 
               XSTACK = 0000000C ( 0000000B )
    -------------------------------------------------------------------------
<BANKED_CODE,CODE_C> 1 (was BANKED_CODE)
  Relative segment, address: CODE 00007775 - 00007779 (0x5 bytes), align: 0
  Segment part 222.           Intra module refs:   phyFindWlEntry
    -------------------------------------------------------------------------
BANK_RELAYS
  Relative segment, address: CODE 000006AA - 000006AF (0x6 bytes), align: 0
  Segment part 13.
           ENTRY                   ADDRESS         REF BY
           =====                   =======         ======
           PHY_Init::?relay        000006AA        LL_Init (ll)
    -------------------------------------------------------------------------
BANK_RELAYS
  Relative segment, address: CODE 000006B0 - 000006B5 (0x6 bytes), align: 0
  Segment part 19.            Intra module refs:   PHY_Init
           ENTRY                   ADDRESS         REF BY
           =====                   =======         ======
           PHY_Reset::?relay       000006B0        llScheduleTask (ll_scheduler)
    -------------------------------------------------------------------------
BANK_RELAYS
  Relative segment, address: CODE 000006B6 - 000006BB (0x6 bytes), align: 0
  Segment part 21.            Intra module refs:   PHY_Init
           ENTRY                   ADDRESS         REF BY
           =====                   =======         ======
           PHY_LoadNR::?relay      000006B6 
    -------------------------------------------------------------------------
BANK_RELAYS
  Relative segment, address: CODE 000006BC - 000006C1 (0x6 bytes), align: 0
  Segment part 23.            Intra module refs:   PHY_Init
           ENTRY                   ADDRESS         REF BY
           =====                   =======         ======
           PHY_VerifyNR::?relay    000006BC 
    -------------------------------------------------------------------------
BANK_RELAYS
  Relative segment, address: CODE 000006C2 - 000006C7 (0x6 bytes), align: 0
  Segment part 26.            Intra module refs:   PHY_Init
           ENTRY                   ADDRESS         REF BY
           =====                   =======         ======
           PHY_ClearAllRegsAndFifos::?relay
                                   000006C2        LL_Reset (ll)
    -------------------------------------------------------------------------
BANK_RELAYS
  Relative segment, address: CODE 000006C8 - 000006CD (0x6 bytes), align: 0
  Segment part 32.
           ENTRY                   ADDRESS         REF BY
           =====                   =======         ======
           PHY_SetOwnAddr::?relay
                                   000006C8        llSetupAdv (ll_common)
    -------------------------------------------------------------------------
BANK_RELAYS
  Relative segment, address: CODE 000006CE - 000006D3 (0x6 bytes), align: 0
  Segment part 42.
           ENTRY                   ADDRESS         REF BY
           =====                   =======         ======
           PHY_SetCRCInit::?relay
                                   000006CE        LL_Reset (ll)
                                                   llSetupAdv (ll_common)
    -------------------------------------------------------------------------
BANK_RELAYS
  Relative segment, address: CODE 000006D4 - 000006D9 (0x6 bytes), align: 0
  Segment part 45.
           ENTRY                   ADDRESS         REF BY
           =====                   =======         ======
           PHY_GetAdvChans::?relay
                                   000006D4        llDiscoverableAdvEvt_TaskEndOk (ll_advEndCauses)
                                                   llNonConnAdvEvt_TaskEndOk (ll_advEndCauses)
    -------------------------------------------------------------------------
BANK_RELAYS
  Relative segment, address: CODE 000006DA - 000006DF (0x6 bytes), align: 0
  Segment part 47.
           ENTRY                   ADDRESS         REF BY
           =====                   =======         ======
           PHY_SetAdvChans::?relay
                                   000006DA        llDiscoverableAdvEvt_TaskEndOk (ll_advEndCauses)
                                                   llNonConnAdvEvt_TaskEndOk (ll_advEndCauses)
                                                   llSetupAdv (ll_common)
    -------------------------------------------------------------------------
BANK_RELAYS
  Relative segment, address: CODE 000006E0 - 000006E5 (0x6 bytes), align: 0
  Segment part 49.
           ENTRY                   ADDRESS         REF BY
           =====                   =======         ======
           PHY_SetEndConnection::?relay
                                   000006E0        RF_NormalIsr (ll_isr)
    -------------------------------------------------------------------------
BANK_RELAYS
  Relative segment, address: CODE 000006E6 - 000006EB (0x6 bytes), align: 0
  Segment part 51.
           ENTRY                   ADDRESS         REF BY
           =====                   =======         ======
           PHY_ConfigureMD::?relay
                                   000006E6        LL_Reset (ll)
    -------------------------------------------------------------------------
BANK_RELAYS
  Relative segment, address: CODE 000006EC - 000006F1 (0x6 bytes), align: 0
  Segment part 59.
           ENTRY                   ADDRESS         REF BY
           =====                   =======         ======
           PHY_GetEndCause::?relay
                                   000006EC        RF_NormalIsr (ll_isr)
    -------------------------------------------------------------------------
BANK_RELAYS
  Relative segment, address: CODE 000006F2 - 000006F7 (0x6 bytes), align: 0
  Segment part 69.
           ENTRY                   ADDRESS         REF BY
           =====                   =======         ======
           PHY_SetSyncWord::?relay
                                   000006F2        LL_DirectTestRxTest (ll)
                                                   LL_DirectTestTxTest (ll)
                                                   LL_EXT_ModemHopTestTx (ll)
                                                   LL_EXT_ModemTestRx (ll)
                                                   LL_EXT_ModemTestTx (ll)
                                                   llSetupAdv (ll_common)
    -------------------------------------------------------------------------
BANK_RELAYS
  Relative segment, address: CODE 000006F8 - 000006FD (0x6 bytes), align: 0
  Segment part 73.
           ENTRY                   ADDRESS         REF BY
           =====                   =======         ======
           PHY_ClearWhitelist::?relay
                                   000006F8        LL_ClearWhiteList (ll)
                                                   LL_Reset (ll)
    -------------------------------------------------------------------------
BANK_RELAYS
  Relative segment, address: CODE 000006FE - 00000703 (0x6 bytes), align: 0
  Segment part 86.
           ENTRY                   ADDRESS         REF BY
           =====                   =======         ======
           PHY_GetWlSize::?relay   000006FE        LL_ReadWlSize (ll)
    -------------------------------------------------------------------------
BANK_RELAYS
  Relative segment, address: CODE 00000704 - 00000709 (0x6 bytes), align: 0
  Segment part 88.
           ENTRY                   ADDRESS         REF BY
           =====                   =======         ======
           PHY_AddWlEntry::?relay
                                   00000704        LL_AddWhiteListDevice (ll)
    -------------------------------------------------------------------------
BANK_RELAYS
  Relative segment, address: CODE 0000070A - 0000070F (0x6 bytes), align: 0
  Segment part 90.
           ENTRY                   ADDRESS         REF BY
           =====                   =======         ======
           PHY_RemoveWlEntry::?relay
                                   0000070A        LL_RemoveWhiteListDevice (ll)
    -------------------------------------------------------------------------
BANK_RELAYS
  Relative segment, address: CODE 00000710 - 00000715 (0x6 bytes), align: 0
  Segment part 94.
           ENTRY                   ADDRESS         REF BY
           =====                   =======         ======
           PHY_SetAdvWlPolicy::?relay
                                   00000710        LL_SetAdvParam (ll)
    -------------------------------------------------------------------------
BANK_RELAYS
  Relative segment, address: CODE 00000716 - 0000071B (0x6 bytes), align: 0
  Segment part 100.           Intra module refs:   PHY_AddWlEntry
           ENTRY                   ADDRESS         REF BY
           =====                   =======         ======
           PHY_SetBlacklistIndex::?relay
                                   00000716 
    -------------------------------------------------------------------------
BANK_RELAYS
  Relative segment, address: CODE 0000071C - 00000721 (0x6 bytes), align: 0
  Segment part 105.           Intra module refs:   PHY_AddWlEntry
                                                   PHY_RemoveWlEntry
           ENTRY                   ADDRESS         REF BY
           =====                   =======         ======
           PHY_ClearBlacklistIndex::?relay
                                   0000071C 
    -------------------------------------------------------------------------
BANK_RELAYS
  Relative segment, address: CODE 00000722 - 00000727 (0x6 bytes), align: 0
  Segment part 107.
           ENTRY                   ADDRESS         REF BY
           =====                   =======         ======
           PHY_ClearBlacklist::?relay
                                   00000722        LL_Reset (ll)
    -------------------------------------------------------------------------
BANK_RELAYS
  Relative segment, address: CODE 00000728 - 0000072D (0x6 bytes), align: 0
  Segment part 122.
           ENTRY                   ADDRESS         REF BY
           =====                   =======         ======
           PHY_ClearSavedWhiteList::?relay
                                   00000728        LL_Reset (ll)
    -------------------------------------------------------------------------
BANK_RELAYS
  Relative segment, address: CODE 0000072E - 00000733 (0x6 bytes), align: 0
  Segment part 125.
           ENTRY                   ADDRESS         REF BY
           =====                   =======         ======
           PHY_Command::?relay     0000072E        LL_DirectTestRxTest (ll)
                                                   LL_DirectTestTxTest (ll)
                                                   LL_EXT_ModemHopTestTx (ll)
                                                   LL_EXT_ModemTestRx (ll)
                                                   LL_EXT_ModemTestTx (ll)
    -------------------------------------------------------------------------
BANK_RELAYS
  Relative segment, address: CODE 00000734 - 00000739 (0x6 bytes), align: 0
  Segment part 135.
           ENTRY                   ADDRESS         REF BY
           =====                   =======         ======
           PHY_ConfigureFifoDataProcessing::?relay
                                   00000734        LL_Reset (ll)
    -------------------------------------------------------------------------
BANK_RELAYS
  Relative segment, address: CODE 0000073A - 0000073F (0x6 bytes), align: 0
  Segment part 137.
           ENTRY                   ADDRESS         REF BY
           =====                   =======         ======
           PHY_ConfigureAppendRfStatus::?relay
                                   0000073A        LL_Reset (ll)
                                                   llSetupAdv (ll_common)
    -------------------------------------------------------------------------
BANK_RELAYS
  Relative segment, address: CODE 00000740 - 00000745 (0x6 bytes), align: 0
  Segment part 139.
           ENTRY                   ADDRESS         REF BY
           =====                   =======         ======
           PHY_SetFifoConfig::?relay
                                   00000740        LL_Reset (ll)
    -------------------------------------------------------------------------
BANK_RELAYS
  Relative segment, address: CODE 00000746 - 0000074B (0x6 bytes), align: 0
  Segment part 152.
           ENTRY                   ADDRESS         REF BY
           =====                   =======         ======
           PHY_ConfigWhitener::?relay
                                   00000746        LL_DirectTestEnd (ll)
                                                   LL_DirectTestRxTest (ll)
                                                   LL_DirectTestTxTest (ll)
                                                   LL_EXT_ModemHopTestTx (ll)
                                                   LL_EXT_ModemTestRx (ll)
                                                   LL_EXT_ModemTestTx (ll)
                                                   llRfInit (ll_common)
    -------------------------------------------------------------------------
BANK_RELAYS
  Relative segment, address: CODE 0000074C - 00000751 (0x6 bytes), align: 0
  Segment part 205.
           ENTRY                   ADDRESS         REF BY
           =====                   =======         ======
           PHY_RawTxInit::?relay   0000074C        LL_DirectTestTxTest (ll)
                                                   LL_EXT_ModemHopTestTx (ll)
    -------------------------------------------------------------------------
BANK_RELAYS
  Relative segment, address: CODE 00000752 - 00000757 (0x6 bytes), align: 0
  Segment part 207.
           ENTRY                   ADDRESS         REF BY
           =====                   =======         ======
           PHY_RawRxInit::?relay   00000752        LL_DirectTestRxTest (ll)
    -------------------------------------------------------------------------
BANK_RELAYS
  Relative segment, address: CODE 00000758 - 0000075D (0x6 bytes), align: 0
  Segment part 210.
           ENTRY                   ADDRESS         REF BY
           =====                   =======         ======
           PHY_RawGetNumTxPkts::?relay
                                   00000758        LL_DirectTestEnd (ll)
    -------------------------------------------------------------------------
BANK_RELAYS
  Relative segment, address: CODE 0000075E - 00000763 (0x6 bytes), align: 0
  Segment part 216.
           ENTRY                   ADDRESS         REF BY
           =====                   =======         ======
           PHY_RawGetRxData::?relay
                                   0000075E        LL_DirectTestEnd (ll)
    -------------------------------------------------------------------------
BANK_RELAYS
  Relative segment, address: CODE 00000764 - 00000769 (0x6 bytes), align: 0
  Segment part 219.
           ENTRY                   ADDRESS         REF BY
           =====                   =======         ======
           PHY_SetRfFreq::?relay   00000764        LL_DirectTestRxTest (ll)
                                                   LL_DirectTestTxTest (ll)
                                                   LL_EXT_ModemHopTestTx (ll)
                                                   LL_EXT_ModemTestRx (ll)
                                                   LL_EXT_ModemTestTx (ll)
    -------------------------------------------------------------------------
BANK_RELAYS
  Relative segment, address: CODE 0000076A - 0000076F (0x6 bytes), align: 0
  Segment part 221.           Intra module refs:   PHY_AddWlEntry
                                                   PHY_RemoveWlEntry
           LOCAL                   ADDRESS         
           =====                   =======         
           phyFindWlEntry::?relay
                                   0000076A 

    -------------------------------------------------------------------------
  LIBRARY MODULE, NAME : phy_image

  SEGMENTS IN THE MODULE
  ======================
<XDATA_ROM_C> 1 (was XDATA_ROM_C)
  Relative segment, address: CONST 00008000 - 00008DFD (0xdfe bytes), align: 0
  Segment part 6.
           ENTRY                   ADDRESS         REF BY
           =====                   =======         ======
           NanoRiscImage           00008000        Segment part 24 (phy)
    -------------------------------------------------------------------------
<BANKED_CODE,XDATA_ROM_C_FLASH> 1 (was XDATA_ROM_C_FLASH)
  Relative segment, address: CODE 00008000 - 00008DFD (0xdfe bytes), align: 0
  Segment part 7.             Intra module refs:   NanoRiscImage

    *************************************************************************

  FILE NAME : C:\ble\BLE-CC254x-1.4.1.43908\Projects\ble\Libraries\Common\bin\CC254x_BLE_HCI_TL_bcast.lib
  LIBRARY MODULE, NAME : hci_tl

  SEGMENTS IN THE MODULE
  ======================
XDATA_Z
  Relative segment, address: XDATA 000003AC - 000003AC (0x1 bytes), align: 0
  Segment part 6.             Intra module refs:   HCI_Init
                                                   HCI_ProcessEvent
                                                   hciProcessCtrlToHost
                                                   hciSerialPacketParser
           ENTRY                   ADDRESS         REF BY
           =====                   =======         ======
           hciTaskID               000003AC        HCI_SendCommandCompleteEvent (hci_event)
    -------------------------------------------------------------------------
XDATA_Z
  Relative segment, address: XDATA 000003AD - 000003AD (0x1 bytes), align: 0
  Segment part 7.             Intra module refs:   HCI_Init
           ENTRY                   ADDRESS         REF BY
           =====                   =======         ======
           hciTestTaskID           000003AD        HCI_EXT_SetBDADDRCmd (hci)
    -------------------------------------------------------------------------
XDATA_Z
  Relative segment, address: XDATA 000003AE - 000003AE (0x1 bytes), align: 0
  Segment part 8.             Intra module refs:   HCI_GAPTaskRegister
                                                   HCI_Init
           ENTRY                   ADDRESS         REF BY
           =====                   =======         ======
           hciGapTaskID            000003AE        HCI_CommandCompleteEvent (hci_event)
                                                   HCI_VendorSpecifcCommandCompleteEvent (hci_event_PATCH)
    -------------------------------------------------------------------------
XDATA_Z
  Relative segment, address: XDATA 000003AF - 000003AF (0x1 bytes), align: 0
  Segment part 9.             Intra module refs:   HCI_Init
           ENTRY                   ADDRESS         REF BY
           =====                   =======         ======
           hciL2capTaskID          000003AF 
    -------------------------------------------------------------------------
XDATA_Z
  Relative segment, address: XDATA 000003B0 - 000003B0 (0x1 bytes), align: 0
  Segment part 10.            Intra module refs:   HCI_Init
           ENTRY                   ADDRESS         REF BY
           =====                   =======         ======
           hciSmpTaskID            000003B0        HCI_CommandCompleteEvent (hci_event)
    -------------------------------------------------------------------------
XDATA_Z
  Relative segment, address: XDATA 000003B1 - 000003B1 (0x1 bytes), align: 0
  Segment part 11.            Intra module refs:   HCI_Init
                                                   hciSerialPacketParser
           ENTRY                   ADDRESS         REF BY
           =====                   =======         ======
           hciExtTaskID            000003B1 
    -------------------------------------------------------------------------
<XDATA_ROM_C> 1 (was XDATA_ROM_C)
  Relative segment, address: CONST 00008DFE - 00008EBD (0xc0 bytes), align: 0
  Segment part 12.            Intra module refs:   hciProcessHostToCtrlCmd
           ENTRY                   ADDRESS         REF BY
           =====                   =======         ======
           hciCmdTable             00008DFE 
    -------------------------------------------------------------------------
<BANKED_CODE,CODE_C> 1 (was BANKED_CODE)
  Relative segment, address: CODE 00004817 - 00004846 (0x30 bytes), align: 0
  Segment part 17.            Intra module refs:   HCI_Init::?relay
           ENTRY                   ADDRESS         REF BY
           =====                   =======         ======
           HCI_Init                00004817 
               calls direct
               XSTACK = 00000000 ( 00000009 )
    -------------------------------------------------------------------------
<BANKED_CODE,CODE_C> 1 (was BANKED_CODE)
  Relative segment, address: CODE 00004847 - 0000484B (0x5 bytes), align: 0
  Segment part 19.            Intra module refs:   HCI_Init
                                                   hciProcessHostToCtrlData
    -------------------------------------------------------------------------
<BANKED_CODE,CODE_C> 1 (was BANKED_CODE)
  Relative segment, address: CODE 0000484C - 0000488E (0x43 bytes), align: 0
  Segment part 20.            Intra module refs:   HCI_ProcessEvent::?relay
           ENTRY                   ADDRESS         REF BY
           =====                   =======         ======
           HCI_ProcessEvent        0000484C 
               calls direct
               XSTACK = 00000000 ( 0000000A )
    -------------------------------------------------------------------------
<BANKED_CODE,CODE_C> 1 (was BANKED_CODE)
  Relative segment, address: CODE 0000488F - 00004899 (0xb bytes), align: 0
  Segment part 24.            Intra module refs:   HCI_GAPTaskRegister::?relay
           ENTRY                   ADDRESS         REF BY
           =====                   =======         ======
           HCI_GAPTaskRegister     0000488F 
               ISTACK = 00000000 ( 00000002 )
    -------------------------------------------------------------------------
<BANKED_CODE,CODE_C> 1 (was BANKED_CODE)
  Relative segment, address: CODE 0000489A - 00004BA0 (0x307 bytes), align: 0
  Segment part 32.            Intra module refs:   hciSerialPacketParser::?relay
           ENTRY                   ADDRESS         REF BY
           =====                   =======         ======
           hciSerialPacketParser   0000489A 
               calls direct, is indirectly called
               XSTACK = 00000000 ( 0000000E )
               ISTACK = 00000000 ( 00000001 )
    -------------------------------------------------------------------------
<BANKED_CODE,CODE_C> 1 (was BANKED_CODE)
  Relative segment, address: CODE 00004BA1 - 00004BAA (0xa bytes), align: 0
  Segment part 34.            Intra module refs:   hciSerialPacketParser
    -------------------------------------------------------------------------
<BANKED_CODE,CODE_C> 1 (was BANKED_CODE)
  Relative segment, address: CODE 00004BAB - 00004BBA (0x10 bytes), align: 0
  Segment part 35.            Intra module refs:   hciSerialPacketParser
    -------------------------------------------------------------------------
<BANKED_CODE,CODE_C> 1 (was BANKED_CODE)
  Relative segment, address: CODE 00004BBB - 00004BCA (0x10 bytes), align: 0
  Segment part 36.            Intra module refs:   hciSerialPacketParser
    -------------------------------------------------------------------------
<BANKED_CODE,CODE_C> 1 (was BANKED_CODE)
  Relative segment, address: CODE 00004BCB - 00004BD9 (0xf bytes), align: 0
  Segment part 37.            Intra module refs:   hciSerialPacketParser
    -------------------------------------------------------------------------
<BANKED_CODE,CODE_C> 1 (was BANKED_CODE)
  Relative segment, address: CODE 00004BDA - 00004BE0 (0x7 bytes), align: 0
  Segment part 38.            Intra module refs:   hciSerialPacketParser
    -------------------------------------------------------------------------
<BANKED_CODE,CODE_C> 1 (was BANKED_CODE)
  Relative segment, address: CODE 00004BE1 - 00004BEA (0xa bytes), align: 0
  Segment part 39.            Intra module refs:   Segment part 38
                                                   hciSerialPacketParser
    -------------------------------------------------------------------------
<BANKED_CODE,CODE_C> 1 (was BANKED_CODE)
  Relative segment, address: CODE 00004BEB - 00004BF1 (0x7 bytes), align: 0
  Segment part 40.            Intra module refs:   hciSerialPacketParser
    -------------------------------------------------------------------------
<BANKED_CODE,CODE_C> 1 (was BANKED_CODE)
  Relative segment, address: CODE 00004BF2 - 00004BFC (0xb bytes), align: 0
  Segment part 41.            Intra module refs:   hciSerialPacketParser
    -------------------------------------------------------------------------
<BANKED_CODE,CODE_C> 1 (was BANKED_CODE)
  Relative segment, address: CODE 00004BFD - 00004C09 (0xd bytes), align: 0
  Segment part 42.            Intra module refs:   Segment part 40
                                                   Segment part 41
    -------------------------------------------------------------------------
<BANKED_CODE,CODE_C> 1 (was BANKED_CODE)
  Relative segment, address: CODE 00004C0A - 00004C12 (0x9 bytes), align: 0
  Segment part 43.            Intra module refs:   hciSerialPacketParser
    -------------------------------------------------------------------------
XDATA_Z
  Relative segment, address: XDATA 000003B2 - 000003B2 (0x1 bytes), align: 0
  Segment part 13.            Intra module refs:   Segment part 36
                                                   hciSerialPacketParser
    -------------------------------------------------------------------------
XDATA_Z
  Relative segment, address: XDATA 000003B3 - 000003B3 (0x1 bytes), align: 0
  Segment part 14.            Intra module refs:   hciSerialPacketParser
    -------------------------------------------------------------------------
XDATA_Z
  Relative segment, address: XDATA 000003B4 - 000003B5 (0x2 bytes), align: 0
  Segment part 15.            Intra module refs:   hciSerialPacketParser
    -------------------------------------------------------------------------
XDATA_Z
  Relative segment, address: XDATA 000003B6 - 000003B7 (0x2 bytes), align: 0
  Segment part 16.            Intra module refs:   Segment part 35
                                                   Segment part 42
                                                   hciSerialPacketParser
    -------------------------------------------------------------------------
<BANKED_CODE,CODE_C> 1 (was BANKED_CODE)
  Relative segment, address: CODE 00004C13 - 00004CDE (0xcc bytes), align: 0
  Segment part 44.            Intra module refs:   hciProcessHostToCtrlCmd::?relay
           ENTRY                   ADDRESS         REF BY
           =====                   =======         ======
           hciProcessHostToCtrlCmd
                                   00004C13 
               calls direct
               XSTACK = 0000000A ( 00000010 )
    -------------------------------------------------------------------------
<BANKED_CODE,CODE_C> 1 (was BANKED_CODE)
  Relative segment, address: CODE 00004CDF - 00004CE4 (0x6 bytes), align: 0
  Segment part 46.            Intra module refs:   hciProcessHostToCtrlCmd
    -------------------------------------------------------------------------
<BANKED_CODE,CODE_C> 1 (was BANKED_CODE)
  Relative segment, address: CODE 00004CE5 - 00004CEB (0x7 bytes), align: 0
  Segment part 47.            Intra module refs:   Segment part 46
                                                   hciProcessHostToCtrlCmd
    -------------------------------------------------------------------------
<BANKED_CODE,CODE_C> 1 (was BANKED_CODE)
  Relative segment, address: CODE 00004CEC - 00004D1B (0x30 bytes), align: 0
  Segment part 48.            Intra module refs:   hciProcessHostToCtrlData::?relay
           ENTRY                   ADDRESS         REF BY
           =====                   =======         ======
           hciProcessHostToCtrlData
                                   00004CEC 
               calls direct
               XSTACK = 0000000A ( 00000009 )
    -------------------------------------------------------------------------
<BANKED_CODE,CODE_C> 1 (was BANKED_CODE)
  Relative segment, address: CODE 00004D1C - 00004D21 (0x6 bytes), align: 0
  Segment part 50.            Intra module refs:   hciProcessCtrlToHost
                                                   hciProcessHostToCtrlData
                                                   hciSerialPacketParser
    -------------------------------------------------------------------------
<BANKED_CODE,CODE_C> 1 (was BANKED_CODE)
  Relative segment, address: CODE 00004D22 - 00004DA3 (0x82 bytes), align: 0
  Segment part 51.            Intra module refs:   hciProcessCtrlToHost::?relay
           ENTRY                   ADDRESS         REF BY
           =====                   =======         ======
           hciProcessCtrlToHost    00004D22 
               calls direct
               XSTACK = 0000000A ( 0000000C )
    -------------------------------------------------------------------------
<BANKED_CODE,CODE_C> 1 (was BANKED_CODE)
  Relative segment, address: CODE 00004DA4 - 00004DAD (0xa bytes), align: 0
  Segment part 53.            Intra module refs:   hciProcessCtrlToHost
                                                   hciProcessHostToCtrlCmd
    -------------------------------------------------------------------------
<BANKED_CODE,CODE_C> 1 (was BANKED_CODE)
  Relative segment, address: CODE 00004DAE - 00004DB7 (0xa bytes), align: 0
  Segment part 54.            Intra module refs:   hciSetEventMask::?relay
           ENTRY                   ADDRESS         REF BY
           =====                   =======         ======
           hciSetEventMask         00004DAE 
               calls direct, is indirectly called
               ISTACK = 00000000 ( 00000002 )
    -------------------------------------------------------------------------
<BANKED_CODE,CODE_C> 1 (was BANKED_CODE)
  Relative segment, address: CODE 00004DB8 - 00004DC1 (0xa bytes), align: 0
  Segment part 56.            Intra module refs:   hciSetEventMaskPage2::?relay
           ENTRY                   ADDRESS         REF BY
           =====                   =======         ======
           hciSetEventMaskPage2    00004DB8 
               calls direct, is indirectly called
               ISTACK = 00000000 ( 00000002 )
    -------------------------------------------------------------------------
<BANKED_CODE,CODE_C> 1 (was BANKED_CODE)
  Relative segment, address: CODE 00004DC2 - 00004DCB (0xa bytes), align: 0
  Segment part 58.            Intra module refs:   hciReset::?relay
           ENTRY                   ADDRESS         REF BY
           =====                   =======         ======
           hciReset                00004DC2 
               calls direct, is indirectly called
               ISTACK = 00000000 ( 00000002 )
    -------------------------------------------------------------------------
<BANKED_CODE,CODE_C> 1 (was BANKED_CODE)
  Relative segment, address: CODE 00004DCC - 00004DD5 (0xa bytes), align: 0
  Segment part 60.            Intra module refs:   hciReadLocalVersionInfo::?relay
           ENTRY                   ADDRESS         REF BY
           =====                   =======         ======
           hciReadLocalVersionInfo
                                   00004DCC 
               calls direct, is indirectly called
               ISTACK = 00000000 ( 00000002 )
    -------------------------------------------------------------------------
<BANKED_CODE,CODE_C> 1 (was BANKED_CODE)
  Relative segment, address: CODE 00004DD6 - 00004DDF (0xa bytes), align: 0
  Segment part 62.            Intra module refs:   hciReadLocalSupportedCommands::?relay
           ENTRY                   ADDRESS         REF BY
           =====                   =======         ======
           hciReadLocalSupportedCommands
                                   00004DD6 
               calls direct, is indirectly called
               ISTACK = 00000000 ( 00000002 )
    -------------------------------------------------------------------------
<BANKED_CODE,CODE_C> 1 (was BANKED_CODE)
  Relative segment, address: CODE 00004DE0 - 00004DE9 (0xa bytes), align: 0
  Segment part 64.            Intra module refs:   hciReadLocalSupportedFeatures::?relay
           ENTRY                   ADDRESS         REF BY
           =====                   =======         ======
           hciReadLocalSupportedFeatures
                                   00004DE0 
               calls direct, is indirectly called
               ISTACK = 00000000 ( 00000002 )
    -------------------------------------------------------------------------
<BANKED_CODE,CODE_C> 1 (was BANKED_CODE)
  Relative segment, address: CODE 00004DEA - 00004DF6 (0xd bytes), align: 0
  Segment part 66.            Intra module refs:   hciReadRssi::?relay
           ENTRY                   ADDRESS         REF BY
           =====                   =======         ======
           hciReadRssi             00004DEA 
               calls direct, is indirectly called
               ISTACK = 00000000 ( 00000002 )
    -------------------------------------------------------------------------
<BANKED_CODE,CODE_C> 1 (was BANKED_CODE)
  Relative segment, address: CODE 00004DF7 - 00004E00 (0xa bytes), align: 0
  Segment part 68.            Intra module refs:   hciLESetEventMask::?relay
           ENTRY                   ADDRESS         REF BY
           =====                   =======         ======
           hciLESetEventMask       00004DF7 
               calls direct, is indirectly called
               ISTACK = 00000000 ( 00000002 )
    -------------------------------------------------------------------------
<BANKED_CODE,CODE_C> 1 (was BANKED_CODE)
  Relative segment, address: CODE 00004E01 - 00004E0A (0xa bytes), align: 0
  Segment part 70.            Intra module refs:   hciLEReadBufSize::?relay
           ENTRY                   ADDRESS         REF BY
           =====                   =======         ======
           hciLEReadBufSize        00004E01 
               calls direct, is indirectly called
               ISTACK = 00000000 ( 00000002 )
    -------------------------------------------------------------------------
<BANKED_CODE,CODE_C> 1 (was BANKED_CODE)
  Relative segment, address: CODE 00004E0B - 00004E14 (0xa bytes), align: 0
  Segment part 72.            Intra module refs:   hciLEReadLocalSupportedFeatures::?relay
           ENTRY                   ADDRESS         REF BY
           =====                   =======         ======
           hciLEReadLocalSupportedFeatures
                                   00004E0B 
               calls direct, is indirectly called
               ISTACK = 00000000 ( 00000002 )
    -------------------------------------------------------------------------
<BANKED_CODE,CODE_C> 1 (was BANKED_CODE)
  Relative segment, address: CODE 00004E15 - 00004E1E (0xa bytes), align: 0
  Segment part 74.            Intra module refs:   hciLESetRandomAddr::?relay
           ENTRY                   ADDRESS         REF BY
           =====                   =======         ======
           hciLESetRandomAddr      00004E15 
               calls direct, is indirectly called
               ISTACK = 00000000 ( 00000002 )
    -------------------------------------------------------------------------
<BANKED_CODE,CODE_C> 1 (was BANKED_CODE)
  Relative segment, address: CODE 00004E1F - 00004E95 (0x77 bytes), align: 0
  Segment part 76.            Intra module refs:   hciLESetAdvParam::?relay
           ENTRY                   ADDRESS         REF BY
           =====                   =======         ======
           hciLESetAdvParam        00004E1F 
               calls direct, is indirectly called
               XSTACK = 00000000 ( 00000010 )
    -------------------------------------------------------------------------
<BANKED_CODE,CODE_C> 1 (was BANKED_CODE)
  Relative segment, address: CODE 00004E96 - 00004E9B (0x6 bytes), align: 0
  Segment part 78.            Intra module refs:   hciLESetAdvParam
    -------------------------------------------------------------------------
<BANKED_CODE,CODE_C> 1 (was BANKED_CODE)
  Relative segment, address: CODE 00004E9C - 00004EA1 (0x6 bytes), align: 0
  Segment part 79.            Intra module refs:   Segment part 78
                                                   hciLESetAdvParam
    -------------------------------------------------------------------------
<BANKED_CODE,CODE_C> 1 (was BANKED_CODE)
  Relative segment, address: CODE 00004EA2 - 00004EBE (0x1d bytes), align: 0
  Segment part 80.            Intra module refs:   hciLESetAdvData::?relay
           ENTRY                   ADDRESS         REF BY
           =====                   =======         ======
           hciLESetAdvData         00004EA2 
               calls direct, is indirectly called
               ISTACK = 00000000 ( 00000002 )
    -------------------------------------------------------------------------
<BANKED_CODE,CODE_C> 1 (was BANKED_CODE)
  Relative segment, address: CODE 00004EBF - 00004EDB (0x1d bytes), align: 0
  Segment part 82.            Intra module refs:   hciLESetScanRspData::?relay
           ENTRY                   ADDRESS         REF BY
           =====                   =======         ======
           hciLESetScanRspData     00004EBF 
               calls direct, is indirectly called
               ISTACK = 00000000 ( 00000002 )
    -------------------------------------------------------------------------
<BANKED_CODE,CODE_C> 1 (was BANKED_CODE)
  Relative segment, address: CODE 00004EDC - 00004EEB (0x10 bytes), align: 0
  Segment part 84.            Intra module refs:   hciLESetAdvEnab::?relay
           ENTRY                   ADDRESS         REF BY
           =====                   =======         ======
           hciLESetAdvEnab         00004EDC 
               calls direct, is indirectly called
               ISTACK = 00000000 ( 00000002 )
    -------------------------------------------------------------------------
<BANKED_CODE,CODE_C> 1 (was BANKED_CODE)
  Relative segment, address: CODE 00004EEC - 00004EF5 (0xa bytes), align: 0
  Segment part 86.            Intra module refs:   hciLEReadAdvChanTxPower::?relay
           ENTRY                   ADDRESS         REF BY
           =====                   =======         ======
           hciLEReadAdvChanTxPower
                                   00004EEC 
               calls direct, is indirectly called
               ISTACK = 00000000 ( 00000002 )
    -------------------------------------------------------------------------
<BANKED_CODE,CODE_C> 1 (was BANKED_CODE)
  Relative segment, address: CODE 00004EF6 - 00004EFE (0x9 bytes), align: 0
  Segment part 88.            Intra module refs:   hciLEReadWhiteListSize::?relay
           ENTRY                   ADDRESS         REF BY
           =====                   =======         ======
           hciLEReadWhiteListSize
                                   00004EF6 
               calls direct, is indirectly called
               ISTACK = 00000000 ( 00000002 )
    -------------------------------------------------------------------------
<BANKED_CODE,CODE_C> 1 (was BANKED_CODE)
  Relative segment, address: CODE 00004EFF - 00004F07 (0x9 bytes), align: 0
  Segment part 90.            Intra module refs:   hciLEClearWhiteList::?relay
           ENTRY                   ADDRESS         REF BY
           =====                   =======         ======
           hciLEClearWhiteList     00004EFF 
               calls direct, is indirectly called
               ISTACK = 00000000 ( 00000002 )
    -------------------------------------------------------------------------
<BANKED_CODE,CODE_C> 1 (was BANKED_CODE)
  Relative segment, address: CODE 00004F08 - 00004F23 (0x1c bytes), align: 0
  Segment part 92.            Intra module refs:   hciLEAddWhiteList::?relay
           ENTRY                   ADDRESS         REF BY
           =====                   =======         ======
           hciLEAddWhiteList       00004F08 
               calls direct, is indirectly called
               ISTACK = 00000000 ( 00000002 )
    -------------------------------------------------------------------------
<BANKED_CODE,CODE_C> 1 (was BANKED_CODE)
  Relative segment, address: CODE 00004F24 - 00004F3F (0x1c bytes), align: 0
  Segment part 94.            Intra module refs:   hciLERemoveWhiteList::?relay
           ENTRY                   ADDRESS         REF BY
           =====                   =======         ======
           hciLERemoveWhiteList    00004F24 
               calls direct, is indirectly called
               ISTACK = 00000000 ( 00000002 )
    -------------------------------------------------------------------------
<BANKED_CODE,CODE_C> 1 (was BANKED_CODE)
  Relative segment, address: CODE 00004F40 - 00004F5E (0x1f bytes), align: 0
  Segment part 96.            Intra module refs:   hciLEEncrypt::?relay
           ENTRY                   ADDRESS         REF BY
           =====                   =======         ======
           hciLEEncrypt            00004F40 
               calls direct, is indirectly called
               XSTACK = 00000000 ( 0000000A )
    -------------------------------------------------------------------------
<BANKED_CODE,CODE_C> 1 (was BANKED_CODE)
  Relative segment, address: CODE 00004F5F - 00004F63 (0x5 bytes), align: 0
  Segment part 98.            Intra module refs:   HCI_ProcessEvent
                                                   hciExtDecrypt
                                                   hciLEEncrypt
                                                   hciLESetAdvParam
    -------------------------------------------------------------------------
<BANKED_CODE,CODE_C> 1 (was BANKED_CODE)
  Relative segment, address: CODE 00004F64 - 00004F6C (0x9 bytes), align: 0
  Segment part 99.            Intra module refs:   hciLERand::?relay
           ENTRY                   ADDRESS         REF BY
           =====                   =======         ======
           hciLERand               00004F64 
               calls direct, is indirectly called
               ISTACK = 00000000 ( 00000002 )
    -------------------------------------------------------------------------
<BANKED_CODE,CODE_C> 1 (was BANKED_CODE)
  Relative segment, address: CODE 00004F6D - 00004F75 (0x9 bytes), align: 0
  Segment part 101.           Intra module refs:   hciLEReadSupportedStates::?relay
           ENTRY                   ADDRESS         REF BY
           =====                   =======         ======
           hciLEReadSupportedStates
                                   00004F6D 
               calls direct, is indirectly called
               ISTACK = 00000000 ( 00000002 )
    -------------------------------------------------------------------------
<BANKED_CODE,CODE_C> 1 (was BANKED_CODE)
  Relative segment, address: CODE 00004F76 - 00004F76 (0x1 bytes), align: 0
  Segment part 103.           Intra module refs:   HCI_GAPTaskRegister
    -------------------------------------------------------------------------
<BANKED_CODE,CODE_C> 1 (was BANKED_CODE)
  Relative segment, address: CODE 00004F77 - 00004F7D (0x7 bytes), align: 0
  Segment part 104.           Intra module refs:   Segment part 103
                                                   hciExtBuildRevision
                                                   hciExtClkDivOnHalt
                                                   hciExtDeclareNvUsage
                                                   hciExtDelaySleep
                                                   hciExtEndModemTest
                                                   hciExtExtendRfRange
                                                   hciExtHaltDuringRf
                                                   hciExtMapPmIoPort
                                                   hciExtModemHopTestTx
                                                   hciExtModemTestTx
                                                   hciExtModemtestRx
                                                   hciExtResetSystem
                                                   hciExtSaveFreqTune
                                                   hciExtSetBDADDR
                                                   hciExtSetFreqTune
                                                   hciExtSetLocalSupportedFeatures
                                                   hciExtSetMaxDtmTxPower
                                                   hciExtSetRxGain
                                                   hciExtSetTxPower
                                                   hciLEAddWhiteList
                                                   hciLEClearWhiteList
                                                   hciLERand
                                                   hciLEReadAdvChanTxPower
                                                   hciLEReadBufSize
                                                   hciLEReadLocalSupportedFeatures
                                                   hciLEReadSupportedStates
                                                   hciLEReadWhiteListSize
                                                   hciLEReceiverTest
                                                   hciLERemoveWhiteList
                                                   hciLESetAdvData
                                                   hciLESetAdvEnab
                                                   hciLESetEventMask
                                                   hciLESetRandomAddr
                                                   hciLESetScanRspData
                                                   hciLETestEnd
                                                   hciLETransmitterTest
                                                   hciReadBDADDR
                                                   hciReadLocalSupportedCommands
                                                   hciReadLocalSupportedFeatures
                                                   hciReadLocalVersionInfo
                                                   hciReadRssi
                                                   hciReset
                                                   hciSetEventMask
                                                   hciSetEventMaskPage2
    -------------------------------------------------------------------------
<BANKED_CODE,CODE_C> 1 (was BANKED_CODE)
  Relative segment, address: CODE 00004F7E - 00004F8C (0xf bytes), align: 0
  Segment part 105.           Intra module refs:   hciLEReceiverTest::?relay
           ENTRY                   ADDRESS         REF BY
           =====                   =======         ======
           hciLEReceiverTest       00004F7E 
               calls direct, is indirectly called
               ISTACK = 00000000 ( 00000002 )
    -------------------------------------------------------------------------
<BANKED_CODE,CODE_C> 1 (was BANKED_CODE)
  Relative segment, address: CODE 00004F8D - 00004FA4 (0x18 bytes), align: 0
  Segment part 107.           Intra module refs:   hciLETransmitterTest::?relay
           ENTRY                   ADDRESS         REF BY
           =====                   =======         ======
           hciLETransmitterTest    00004F8D 
               calls direct, is indirectly called
               ISTACK = 00000000 ( 00000002 )
    -------------------------------------------------------------------------
<BANKED_CODE,CODE_C> 1 (was BANKED_CODE)
  Relative segment, address: CODE 00004FA5 - 00004FAD (0x9 bytes), align: 0
  Segment part 109.           Intra module refs:   hciLETestEnd::?relay
           ENTRY                   ADDRESS         REF BY
           =====                   =======         ======
           hciLETestEnd            00004FA5 
               calls direct, is indirectly called
               ISTACK = 00000000 ( 00000002 )
    -------------------------------------------------------------------------
<BANKED_CODE,CODE_C> 1 (was BANKED_CODE)
  Relative segment, address: CODE 00004FAE - 00004FBC (0xf bytes), align: 0
  Segment part 111.           Intra module refs:   hciExtSetRxGain::?relay
           ENTRY                   ADDRESS         REF BY
           =====                   =======         ======
           hciExtSetRxGain         00004FAE 
               calls direct, is indirectly called
               ISTACK = 00000000 ( 00000002 )
    -------------------------------------------------------------------------
<BANKED_CODE,CODE_C> 1 (was BANKED_CODE)
  Relative segment, address: CODE 00004FBD - 00004FCB (0xf bytes), align: 0
  Segment part 113.           Intra module refs:   hciExtSetTxPower::?relay
           ENTRY                   ADDRESS         REF BY
           =====                   =======         ======
           hciExtSetTxPower        00004FBD 
               calls direct, is indirectly called
               ISTACK = 00000000 ( 00000002 )
    -------------------------------------------------------------------------
<BANKED_CODE,CODE_C> 1 (was BANKED_CODE)
  Relative segment, address: CODE 00004FCC - 00004FD4 (0x9 bytes), align: 0
  Segment part 115.           Intra module refs:   hciExtExtendRfRange::?relay
           ENTRY                   ADDRESS         REF BY
           =====                   =======         ======
           hciExtExtendRfRange     00004FCC 
               calls direct, is indirectly called
               ISTACK = 00000000 ( 00000002 )
    -------------------------------------------------------------------------
<BANKED_CODE,CODE_C> 1 (was BANKED_CODE)
  Relative segment, address: CODE 00004FD5 - 00004FE3 (0xf bytes), align: 0
  Segment part 117.           Intra module refs:   hciExtHaltDuringRf::?relay
           ENTRY                   ADDRESS         REF BY
           =====                   =======         ======
           hciExtHaltDuringRf      00004FD5 
               calls direct, is indirectly called
               ISTACK = 00000000 ( 00000002 )
    -------------------------------------------------------------------------
<BANKED_CODE,CODE_C> 1 (was BANKED_CODE)
  Relative segment, address: CODE 00004FE4 - 00004FF2 (0xf bytes), align: 0
  Segment part 119.           Intra module refs:   hciExtSetMaxDtmTxPower::?relay
           ENTRY                   ADDRESS         REF BY
           =====                   =======         ======
           hciExtSetMaxDtmTxPower
                                   00004FE4 
               calls direct, is indirectly called
               ISTACK = 00000000 ( 00000002 )
    -------------------------------------------------------------------------
<BANKED_CODE,CODE_C> 1 (was BANKED_CODE)
  Relative segment, address: CODE 00004FF3 - 00004FFF (0xd bytes), align: 0
  Segment part 121.           Intra module refs:   hciExtMapPmIoPort::?relay
           ENTRY                   ADDRESS         REF BY
           =====                   =======         ======
           hciExtMapPmIoPort       00004FF3 
               calls direct, is indirectly called
               ISTACK = 00000000 ( 00000002 )
    -------------------------------------------------------------------------
<BANKED_CODE,CODE_C> 1 (was BANKED_CODE)
  Relative segment, address: CODE 00005000 - 00005003 (0x4 bytes), align: 0
  Segment part 123.           Intra module refs:   hciExtMapPmIoPort
                                                   hciExtModemTestTx
    -------------------------------------------------------------------------
<BANKED_CODE,CODE_C> 1 (was BANKED_CODE)
  Relative segment, address: CODE 00005004 - 00005011 (0xe bytes), align: 0
  Segment part 124.           Intra module refs:   Segment part 123
                                                   hciLETransmitterTest
    -------------------------------------------------------------------------
<BANKED_CODE,CODE_C> 1 (was BANKED_CODE)
  Relative segment, address: CODE 00005012 - 00005021 (0x10 bytes), align: 0
  Segment part 125.           Intra module refs:   hciExtClkDivOnHalt::?relay
           ENTRY                   ADDRESS         REF BY
           =====                   =======         ======
           hciExtClkDivOnHalt      00005012 
               calls direct, is indirectly called
               ISTACK = 00000000 ( 00000002 )
    -------------------------------------------------------------------------
<BANKED_CODE,CODE_C> 1 (was BANKED_CODE)
  Relative segment, address: CODE 00005022 - 00005031 (0x10 bytes), align: 0
  Segment part 127.           Intra module refs:   hciExtDeclareNvUsage::?relay
           ENTRY                   ADDRESS         REF BY
           =====                   =======         ======
           hciExtDeclareNvUsage    00005022 
               calls direct, is indirectly called
               ISTACK = 00000000 ( 00000002 )
    -------------------------------------------------------------------------
<BANKED_CODE,CODE_C> 1 (was BANKED_CODE)
  Relative segment, address: CODE 00005032 - 00005053 (0x22 bytes), align: 0
  Segment part 129.           Intra module refs:   hciExtDecrypt::?relay
           ENTRY                   ADDRESS         REF BY
           =====                   =======         ======
           hciExtDecrypt           00005032 
               calls direct, is indirectly called
               XSTACK = 00000000 ( 0000000A )
    -------------------------------------------------------------------------
<BANKED_CODE,CODE_C> 1 (was BANKED_CODE)
  Relative segment, address: CODE 00005054 - 00005062 (0xf bytes), align: 0
  Segment part 131.           Intra module refs:   hciExtDecrypt
                                                   hciLEEncrypt
    -------------------------------------------------------------------------
<BANKED_CODE,CODE_C> 1 (was BANKED_CODE)
  Relative segment, address: CODE 00005063 - 0000506C (0xa bytes), align: 0
  Segment part 132.           Intra module refs:   hciExtSetLocalSupportedFeatures::?relay
           ENTRY                   ADDRESS         REF BY
           =====                   =======         ======
           hciExtSetLocalSupportedFeatures
                                   00005063 
               calls direct, is indirectly called
               ISTACK = 00000000 ( 00000002 )
    -------------------------------------------------------------------------
<BANKED_CODE,CODE_C> 1 (was BANKED_CODE)
  Relative segment, address: CODE 0000506D - 00005091 (0x25 bytes), align: 0
  Segment part 134.           Intra module refs:   hciExtBuildRevision::?relay
           ENTRY                   ADDRESS         REF BY
           =====                   =======         ======
           hciExtBuildRevision     0000506D 
               calls direct, is indirectly called
               ISTACK = 00000000 ( 00000002 )
    -------------------------------------------------------------------------
<BANKED_CODE,CODE_C> 1 (was BANKED_CODE)
  Relative segment, address: CODE 00005092 - 0000509E (0xd bytes), align: 0
  Segment part 136.           Intra module refs:   hciExtDelaySleep::?relay
           ENTRY                   ADDRESS         REF BY
           =====                   =======         ======
           hciExtDelaySleep        00005092 
               calls direct, is indirectly called
               ISTACK = 00000000 ( 00000002 )
    -------------------------------------------------------------------------
<BANKED_CODE,CODE_C> 1 (was BANKED_CODE)
  Relative segment, address: CODE 0000509F - 000050B1 (0x13 bytes), align: 0
  Segment part 138.           Intra module refs:   hciExtDelaySleep
                                                   hciReadRssi
    -------------------------------------------------------------------------
<BANKED_CODE,CODE_C> 1 (was BANKED_CODE)
  Relative segment, address: CODE 000050B2 - 000050C1 (0x10 bytes), align: 0
  Segment part 139.           Intra module refs:   hciExtResetSystem::?relay
           ENTRY                   ADDRESS         REF BY
           =====                   =======         ======
           hciExtResetSystem       000050B2 
               calls direct, is indirectly called
               ISTACK = 00000000 ( 00000002 )
    -------------------------------------------------------------------------
<BANKED_CODE,CODE_C> 1 (was BANKED_CODE)
  Relative segment, address: CODE 000050C2 - 000050CB (0xa bytes), align: 0
  Segment part 141.           Intra module refs:   hciReadBDADDR::?relay
           ENTRY                   ADDRESS         REF BY
           =====                   =======         ======
           hciReadBDADDR           000050C2 
               calls direct, is indirectly called
               ISTACK = 00000000 ( 00000002 )
    -------------------------------------------------------------------------
<BANKED_CODE,CODE_C> 1 (was BANKED_CODE)
  Relative segment, address: CODE 000050CC - 000050D8 (0xd bytes), align: 0
  Segment part 143.           Intra module refs:   hciExtModemTestTx::?relay
           ENTRY                   ADDRESS         REF BY
           =====                   =======         ======
           hciExtModemTestTx       000050CC 
               calls direct, is indirectly called
               ISTACK = 00000000 ( 00000002 )
    -------------------------------------------------------------------------
<BANKED_CODE,CODE_C> 1 (was BANKED_CODE)
  Relative segment, address: CODE 000050D9 - 000050E2 (0xa bytes), align: 0
  Segment part 145.           Intra module refs:   hciExtModemHopTestTx::?relay
           ENTRY                   ADDRESS         REF BY
           =====                   =======         ======
           hciExtModemHopTestTx    000050D9 
               calls direct, is indirectly called
               ISTACK = 00000000 ( 00000002 )
    -------------------------------------------------------------------------
<BANKED_CODE,CODE_C> 1 (was BANKED_CODE)
  Relative segment, address: CODE 000050E3 - 000050F2 (0x10 bytes), align: 0
  Segment part 147.           Intra module refs:   hciExtModemtestRx::?relay
           ENTRY                   ADDRESS         REF BY
           =====                   =======         ======
           hciExtModemtestRx       000050E3 
               calls direct, is indirectly called
               ISTACK = 00000000 ( 00000002 )
    -------------------------------------------------------------------------
<BANKED_CODE,CODE_C> 1 (was BANKED_CODE)
  Relative segment, address: CODE 000050F3 - 000050FC (0xa bytes), align: 0
  Segment part 149.           Intra module refs:   hciExtEndModemTest::?relay
           ENTRY                   ADDRESS         REF BY
           =====                   =======         ======
           hciExtEndModemTest      000050F3 
               calls direct, is indirectly called
               ISTACK = 00000000 ( 00000002 )
    -------------------------------------------------------------------------
<BANKED_CODE,CODE_C> 1 (was BANKED_CODE)
  Relative segment, address: CODE 000050FD - 00005106 (0xa bytes), align: 0
  Segment part 151.           Intra module refs:   hciExtSetBDADDR::?relay
           ENTRY                   ADDRESS         REF BY
           =====                   =======         ======
           hciExtSetBDADDR         000050FD 
               calls direct, is indirectly called
               ISTACK = 00000000 ( 00000002 )
    -------------------------------------------------------------------------
<BANKED_CODE,CODE_C> 1 (was BANKED_CODE)
  Relative segment, address: CODE 00005107 - 00005116 (0x10 bytes), align: 0
  Segment part 155.           Intra module refs:   hciExtSetFreqTune::?relay
           ENTRY                   ADDRESS         REF BY
           =====                   =======         ======
           hciExtSetFreqTune       00005107 
               calls direct, is indirectly called
               ISTACK = 00000000 ( 00000002 )
    -------------------------------------------------------------------------
<BANKED_CODE,CODE_C> 1 (was BANKED_CODE)
  Relative segment, address: CODE 00005117 - 00005120 (0xa bytes), align: 0
  Segment part 157.           Intra module refs:   hciExtSaveFreqTune::?relay
           ENTRY                   ADDRESS         REF BY
           =====                   =======         ======
           hciExtSaveFreqTune      00005117 
               calls direct, is indirectly called
               ISTACK = 00000000 ( 00000002 )
    -------------------------------------------------------------------------
BANK_RELAYS
  Relative segment, address: CODE 00000770 - 00000775 (0x6 bytes), align: 0
  Segment part 18.
           ENTRY                   ADDRESS         REF BY
           =====                   =======         ======
           HCI_Init::?relay        00000770        osalInitTasks (OSAL_SimpleBLEBroadcaster)
    -------------------------------------------------------------------------
BANK_RELAYS
  Relative segment, address: CODE 00000776 - 0000077B (0x6 bytes), align: 0
  Segment part 21.
           ENTRY                   ADDRESS         REF BY
           =====                   =======         ======
           HCI_ProcessEvent::?relay
                                   00000776        tasksArr (OSAL_SimpleBLEBroadcaster)
    -------------------------------------------------------------------------
BANK_RELAYS
  Relative segment, address: CODE 0000077C - 00000781 (0x6 bytes), align: 0
  Segment part 25.
           ENTRY                   ADDRESS         REF BY
           =====                   =======         ======
           HCI_GAPTaskRegister::?relay
                                   0000077C        GAP_Init (gap_simpletask)
    -------------------------------------------------------------------------
BANK_RELAYS
  Relative segment, address: CODE 00000782 - 00000787 (0x6 bytes), align: 0
  Segment part 33.            Intra module refs:   HCI_Init
           ENTRY                   ADDRESS         REF BY
           =====                   =======         ======
           hciSerialPacketParser::?relay
                                   00000782 
    -------------------------------------------------------------------------
BANK_RELAYS
  Relative segment, address: CODE 00000788 - 0000078D (0x6 bytes), align: 0
  Segment part 45.            Intra module refs:   HCI_ProcessEvent
           ENTRY                   ADDRESS         REF BY
           =====                   =======         ======
           hciProcessHostToCtrlCmd::?relay
                                   00000788 
    -------------------------------------------------------------------------
BANK_RELAYS
  Relative segment, address: CODE 0000078E - 00000793 (0x6 bytes), align: 0
  Segment part 49.            Intra module refs:   HCI_ProcessEvent
           ENTRY                   ADDRESS         REF BY
           =====                   =======         ======
           hciProcessHostToCtrlData::?relay
                                   0000078E 
    -------------------------------------------------------------------------
BANK_RELAYS
  Relative segment, address: CODE 00000794 - 00000799 (0x6 bytes), align: 0
  Segment part 52.            Intra module refs:   HCI_ProcessEvent
           ENTRY                   ADDRESS         REF BY
           =====                   =======         ======
           hciProcessCtrlToHost::?relay
                                   00000794 
    -------------------------------------------------------------------------
BANK_RELAYS
  Relative segment, address: CODE 0000079A - 0000079F (0x6 bytes), align: 0
  Segment part 55.            Intra module refs:   hciCmdTable
           ENTRY                   ADDRESS         REF BY
           =====                   =======         ======
           hciSetEventMask::?relay
                                   0000079A 
    -------------------------------------------------------------------------
BANK_RELAYS
  Relative segment, address: CODE 000007A0 - 000007A5 (0x6 bytes), align: 0
  Segment part 57.            Intra module refs:   hciCmdTable
           ENTRY                   ADDRESS         REF BY
           =====                   =======         ======
           hciSetEventMaskPage2::?relay
                                   000007A0 
    -------------------------------------------------------------------------
BANK_RELAYS
  Relative segment, address: CODE 000007A6 - 000007AB (0x6 bytes), align: 0
  Segment part 59.            Intra module refs:   hciCmdTable
           ENTRY                   ADDRESS         REF BY
           =====                   =======         ======
           hciReset::?relay        000007A6 
    -------------------------------------------------------------------------
BANK_RELAYS
  Relative segment, address: CODE 000007AC - 000007B1 (0x6 bytes), align: 0
  Segment part 61.            Intra module refs:   hciCmdTable
           ENTRY                   ADDRESS         REF BY
           =====                   =======         ======
           hciReadLocalVersionInfo::?relay
                                   000007AC 
    -------------------------------------------------------------------------
BANK_RELAYS
  Relative segment, address: CODE 000007B2 - 000007B7 (0x6 bytes), align: 0
  Segment part 63.            Intra module refs:   hciCmdTable
           ENTRY                   ADDRESS         REF BY
           =====                   =======         ======
           hciReadLocalSupportedCommands::?relay
                                   000007B2 
    -------------------------------------------------------------------------
BANK_RELAYS
  Relative segment, address: CODE 000007B8 - 000007BD (0x6 bytes), align: 0
  Segment part 65.            Intra module refs:   hciCmdTable
           ENTRY                   ADDRESS         REF BY
           =====                   =======         ======
           hciReadLocalSupportedFeatures::?relay
                                   000007B8 
    -------------------------------------------------------------------------
BANK_RELAYS
  Relative segment, address: CODE 000007BE - 000007C3 (0x6 bytes), align: 0
  Segment part 67.            Intra module refs:   hciCmdTable
           ENTRY                   ADDRESS         REF BY
           =====                   =======         ======
           hciReadRssi::?relay     000007BE 
    -------------------------------------------------------------------------
BANK_RELAYS
  Relative segment, address: CODE 000007C4 - 000007C9 (0x6 bytes), align: 0
  Segment part 69.            Intra module refs:   hciCmdTable
           ENTRY                   ADDRESS         REF BY
           =====                   =======         ======
           hciLESetEventMask::?relay
                                   000007C4 
    -------------------------------------------------------------------------
BANK_RELAYS
  Relative segment, address: CODE 000007CA - 000007CF (0x6 bytes), align: 0
  Segment part 71.            Intra module refs:   hciCmdTable
           ENTRY                   ADDRESS         REF BY
           =====                   =======         ======
           hciLEReadBufSize::?relay
                                   000007CA 
    -------------------------------------------------------------------------
BANK_RELAYS
  Relative segment, address: CODE 000007D0 - 000007D5 (0x6 bytes), align: 0
  Segment part 73.            Intra module refs:   hciCmdTable
           ENTRY                   ADDRESS         REF BY
           =====                   =======         ======
           hciLEReadLocalSupportedFeatures::?relay
                                   000007D0 
    -------------------------------------------------------------------------
BANK_RELAYS
  Relative segment, address: CODE 000007D6 - 000007DB (0x6 bytes), align: 0
  Segment part 75.            Intra module refs:   hciCmdTable
           ENTRY                   ADDRESS         REF BY
           =====                   =======         ======
           hciLESetRandomAddr::?relay
                                   000007D6 
    -------------------------------------------------------------------------
BANK_RELAYS
  Relative segment, address: CODE 000007DC - 000007E1 (0x6 bytes), align: 0
  Segment part 77.            Intra module refs:   hciCmdTable
           ENTRY                   ADDRESS         REF BY
           =====                   =======         ======
           hciLESetAdvParam::?relay
                                   000007DC 
    -------------------------------------------------------------------------
BANK_RELAYS
  Relative segment, address: CODE 000007E2 - 000007E7 (0x6 bytes), align: 0
  Segment part 81.            Intra module refs:   hciCmdTable
           ENTRY                   ADDRESS         REF BY
           =====                   =======         ======
           hciLESetAdvData::?relay
                                   000007E2 
    -------------------------------------------------------------------------
BANK_RELAYS
  Relative segment, address: CODE 000007E8 - 000007ED (0x6 bytes), align: 0
  Segment part 83.            Intra module refs:   hciCmdTable
           ENTRY                   ADDRESS         REF BY
           =====                   =======         ======
           hciLESetScanRspData::?relay
                                   000007E8 
    -------------------------------------------------------------------------
BANK_RELAYS
  Relative segment, address: CODE 000007EE - 000007F3 (0x6 bytes), align: 0
  Segment part 85.            Intra module refs:   hciCmdTable
           ENTRY                   ADDRESS         REF BY
           =====                   =======         ======
           hciLESetAdvEnab::?relay
                                   000007EE 
    -------------------------------------------------------------------------
BANK_RELAYS
  Relative segment, address: CODE 000007F4 - 000007F9 (0x6 bytes), align: 0
  Segment part 87.            Intra module refs:   hciCmdTable
           ENTRY                   ADDRESS         REF BY
           =====                   =======         ======
           hciLEReadAdvChanTxPower::?relay
                                   000007F4 
    -------------------------------------------------------------------------
BANK_RELAYS
  Relative segment, address: CODE 000007FA - 000007FF (0x6 bytes), align: 0
  Segment part 89.            Intra module refs:   hciCmdTable
           ENTRY                   ADDRESS         REF BY
           =====                   =======         ======
           hciLEReadWhiteListSize::?relay
                                   000007FA 
    -------------------------------------------------------------------------
BANK_RELAYS
  Relative segment, address: CODE 00000800 - 00000805 (0x6 bytes), align: 0
  Segment part 91.            Intra module refs:   hciCmdTable
           ENTRY                   ADDRESS         REF BY
           =====                   =======         ======
           hciLEClearWhiteList::?relay
                                   00000800 
    -------------------------------------------------------------------------
BANK_RELAYS
  Relative segment, address: CODE 00000806 - 0000080B (0x6 bytes), align: 0
  Segment part 93.            Intra module refs:   hciCmdTable
           ENTRY                   ADDRESS         REF BY
           =====                   =======         ======
           hciLEAddWhiteList::?relay
                                   00000806 
    -------------------------------------------------------------------------
BANK_RELAYS
  Relative segment, address: CODE 0000080C - 00000811 (0x6 bytes), align: 0
  Segment part 95.            Intra module refs:   hciCmdTable
           ENTRY                   ADDRESS         REF BY
           =====                   =======         ======
           hciLERemoveWhiteList::?relay
                                   0000080C 
    -------------------------------------------------------------------------
BANK_RELAYS
  Relative segment, address: CODE 00000812 - 00000817 (0x6 bytes), align: 0
  Segment part 97.            Intra module refs:   hciCmdTable
           ENTRY                   ADDRESS         REF BY
           =====                   =======         ======
           hciLEEncrypt::?relay    00000812 
    -------------------------------------------------------------------------
BANK_RELAYS
  Relative segment, address: CODE 00000818 - 0000081D (0x6 bytes), align: 0
  Segment part 100.           Intra module refs:   hciCmdTable
           ENTRY                   ADDRESS         REF BY
           =====                   =======         ======
           hciLERand::?relay       00000818 
    -------------------------------------------------------------------------
BANK_RELAYS
  Relative segment, address: CODE 0000081E - 00000823 (0x6 bytes), align: 0
  Segment part 102.           Intra module refs:   hciCmdTable
           ENTRY                   ADDRESS         REF BY
           =====                   =======         ======
           hciLEReadSupportedStates::?relay
                                   0000081E 
    -------------------------------------------------------------------------
BANK_RELAYS
  Relative segment, address: CODE 00000824 - 00000829 (0x6 bytes), align: 0
  Segment part 106.           Intra module refs:   hciCmdTable
           ENTRY                   ADDRESS         REF BY
           =====                   =======         ======
           hciLEReceiverTest::?relay
                                   00000824 
    -------------------------------------------------------------------------
BANK_RELAYS
  Relative segment, address: CODE 0000082A - 0000082F (0x6 bytes), align: 0
  Segment part 108.           Intra module refs:   hciCmdTable
           ENTRY                   ADDRESS         REF BY
           =====                   =======         ======
           hciLETransmitterTest::?relay
                                   0000082A 
    -------------------------------------------------------------------------
BANK_RELAYS
  Relative segment, address: CODE 00000830 - 00000835 (0x6 bytes), align: 0
  Segment part 110.           Intra module refs:   hciCmdTable
           ENTRY                   ADDRESS         REF BY
           =====                   =======         ======
           hciLETestEnd::?relay    00000830 
    -------------------------------------------------------------------------
BANK_RELAYS
  Relative segment, address: CODE 00000836 - 0000083B (0x6 bytes), align: 0
  Segment part 112.           Intra module refs:   hciCmdTable
           ENTRY                   ADDRESS         REF BY
           =====                   =======         ======
           hciExtSetRxGain::?relay
                                   00000836 
    -------------------------------------------------------------------------
BANK_RELAYS
  Relative segment, address: CODE 0000083C - 00000841 (0x6 bytes), align: 0
  Segment part 114.           Intra module refs:   hciCmdTable
           ENTRY                   ADDRESS         REF BY
           =====                   =======         ======
           hciExtSetTxPower::?relay
                                   0000083C 
    -------------------------------------------------------------------------
BANK_RELAYS
  Relative segment, address: CODE 00000842 - 00000847 (0x6 bytes), align: 0
  Segment part 116.           Intra module refs:   hciCmdTable
           ENTRY                   ADDRESS         REF BY
           =====                   =======         ======
           hciExtExtendRfRange::?relay
                                   00000842 
    -------------------------------------------------------------------------
BANK_RELAYS
  Relative segment, address: CODE 00000848 - 0000084D (0x6 bytes), align: 0
  Segment part 118.           Intra module refs:   hciCmdTable
           ENTRY                   ADDRESS         REF BY
           =====                   =======         ======
           hciExtHaltDuringRf::?relay
                                   00000848 
    -------------------------------------------------------------------------
BANK_RELAYS
  Relative segment, address: CODE 0000084E - 00000853 (0x6 bytes), align: 0
  Segment part 120.           Intra module refs:   hciCmdTable
           ENTRY                   ADDRESS         REF BY
           =====                   =======         ======
           hciExtSetMaxDtmTxPower::?relay
                                   0000084E 
    -------------------------------------------------------------------------
BANK_RELAYS
  Relative segment, address: CODE 00000854 - 00000859 (0x6 bytes), align: 0
  Segment part 122.           Intra module refs:   hciCmdTable
           ENTRY                   ADDRESS         REF BY
           =====                   =======         ======
           hciExtMapPmIoPort::?relay
                                   00000854 
    -------------------------------------------------------------------------
BANK_RELAYS
  Relative segment, address: CODE 0000085A - 0000085F (0x6 bytes), align: 0
  Segment part 126.           Intra module refs:   hciCmdTable
           ENTRY                   ADDRESS         REF BY
           =====                   =======         ======
           hciExtClkDivOnHalt::?relay
                                   0000085A 
    -------------------------------------------------------------------------
BANK_RELAYS
  Relative segment, address: CODE 00000860 - 00000865 (0x6 bytes), align: 0
  Segment part 128.           Intra module refs:   hciCmdTable
           ENTRY                   ADDRESS         REF BY
           =====                   =======         ======
           hciExtDeclareNvUsage::?relay
                                   00000860 
    -------------------------------------------------------------------------
BANK_RELAYS
  Relative segment, address: CODE 00000866 - 0000086B (0x6 bytes), align: 0
  Segment part 130.           Intra module refs:   hciCmdTable
           ENTRY                   ADDRESS         REF BY
           =====                   =======         ======
           hciExtDecrypt::?relay   00000866 
    -------------------------------------------------------------------------
BANK_RELAYS
  Relative segment, address: CODE 0000086C - 00000871 (0x6 bytes), align: 0
  Segment part 133.           Intra module refs:   hciCmdTable
           ENTRY                   ADDRESS         REF BY
           =====                   =======         ======
           hciExtSetLocalSupportedFeatures::?relay
                                   0000086C 
    -------------------------------------------------------------------------
BANK_RELAYS
  Relative segment, address: CODE 00000872 - 00000877 (0x6 bytes), align: 0
  Segment part 135.           Intra module refs:   hciCmdTable
           ENTRY                   ADDRESS         REF BY
           =====                   =======         ======
           hciExtBuildRevision::?relay
                                   00000872 
    -------------------------------------------------------------------------
BANK_RELAYS
  Relative segment, address: CODE 00000878 - 0000087D (0x6 bytes), align: 0
  Segment part 137.           Intra module refs:   hciCmdTable
           ENTRY                   ADDRESS         REF BY
           =====                   =======         ======
           hciExtDelaySleep::?relay
                                   00000878 
    -------------------------------------------------------------------------
BANK_RELAYS
  Relative segment, address: CODE 0000087E - 00000883 (0x6 bytes), align: 0
  Segment part 140.           Intra module refs:   hciCmdTable
           ENTRY                   ADDRESS         REF BY
           =====                   =======         ======
           hciExtResetSystem::?relay
                                   0000087E 
    -------------------------------------------------------------------------
BANK_RELAYS
  Relative segment, address: CODE 00000884 - 00000889 (0x6 bytes), align: 0
  Segment part 142.           Intra module refs:   hciCmdTable
           ENTRY                   ADDRESS         REF BY
           =====                   =======         ======
           hciReadBDADDR::?relay   00000884 
    -------------------------------------------------------------------------
BANK_RELAYS
  Relative segment, address: CODE 0000088A - 0000088F (0x6 bytes), align: 0
  Segment part 144.           Intra module refs:   hciCmdTable
           ENTRY                   ADDRESS         REF BY
           =====                   =======         ======
           hciExtModemTestTx::?relay
                                   0000088A 
    -------------------------------------------------------------------------
BANK_RELAYS
  Relative segment, address: CODE 00000890 - 00000895 (0x6 bytes), align: 0
  Segment part 146.           Intra module refs:   hciCmdTable
           ENTRY                   ADDRESS         REF BY
           =====                   =======         ======
           hciExtModemHopTestTx::?relay
                                   00000890 
    -------------------------------------------------------------------------
BANK_RELAYS
  Relative segment, address: CODE 00000896 - 0000089B (0x6 bytes), align: 0
  Segment part 148.           Intra module refs:   hciCmdTable
           ENTRY                   ADDRESS         REF BY
           =====                   =======         ======
           hciExtModemtestRx::?relay
                                   00000896 
    -------------------------------------------------------------------------
BANK_RELAYS
  Relative segment, address: CODE 0000089C - 000008A1 (0x6 bytes), align: 0
  Segment part 150.           Intra module refs:   hciCmdTable
           ENTRY                   ADDRESS         REF BY
           =====                   =======         ======
           hciExtEndModemTest::?relay
                                   0000089C 
    -------------------------------------------------------------------------
BANK_RELAYS
  Relative segment, address: CODE 000008A2 - 000008A7 (0x6 bytes), align: 0
  Segment part 152.           Intra module refs:   hciCmdTable
           ENTRY                   ADDRESS         REF BY
           =====                   =======         ======
           hciExtSetBDADDR::?relay
                                   000008A2 
    -------------------------------------------------------------------------
BANK_RELAYS
  Relative segment, address: CODE 000008A8 - 000008AD (0x6 bytes), align: 0
  Segment part 156.           Intra module refs:   hciCmdTable
           ENTRY                   ADDRESS         REF BY
           =====                   =======         ======
           hciExtSetFreqTune::?relay
                                   000008A8 
    -------------------------------------------------------------------------
BANK_RELAYS
  Relative segment, address: CODE 000008AE - 000008B3 (0x6 bytes), align: 0
  Segment part 158.           Intra module refs:   hciCmdTable
           ENTRY                   ADDRESS         REF BY
           =====                   =======         ======
           hciExtSaveFreqTune::?relay
                                   000008AE 
    -------------------------------------------------------------------------
<BANKED_CODE,XDATA_ROM_C_FLASH> 1 (was XDATA_ROM_C_FLASH)
  Relative segment, address: CODE 00008DFE - 00008EBD (0xc0 bytes), align: 0
  Segment part 159.           Intra module refs:   hciCmdTable

    *************************************************************************

  FILE NAME : C:\ble\BLE-CC254x-1.4.1.43908\Projects\ble\SimpleBLEBroadcaster-usb\CC2540\CC2540USB\Obj\gap.r51
  PROGRAM MODULE, NAME : gap

  SEGMENTS IN THE MODULE
  ======================
<BANKED_CODE,XDATA_ROM_C_FLASH> 1 (was BANKED_CODE)
  Relative segment, address: CODE 0000C635 - 0000C67F (0x4b bytes), align: 0
  Segment part 6.             Intra module refs:   GAP_DeviceInit::?relay
           ENTRY                   ADDRESS         REF BY
           =====                   =======         ======
           GAP_DeviceInit          0000C635 
               calls direct
               XSTACK = 00000004 ( 0000000C )
    -------------------------------------------------------------------------
BANK_RELAYS
  Relative segment, address: CODE 000008B4 - 000008B9 (0x6 bytes), align: 0
  Segment part 7.
           ENTRY                   ADDRESS         REF BY
           =====                   =======         ======
           GAP_DeviceInit::?relay
                                   000008B4        gapRole_SetupGAP (broadcaster)

    *************************************************************************

  FILE NAME : C:\ble\BLE-CC254x-1.4.1.43908\Projects\ble\SimpleBLEBroadcaster-usb\CC2540\CC2540USB\Obj\gattservapp_util.r51
    *************************************************************************

  FILE NAME : C:\ble\BLE-CC254x-1.4.1.43908\Projects\ble\SimpleBLEBroadcaster-usb\CC2540\CC2540USB\Obj\hal_adc.r51
  PROGRAM MODULE, NAME : hal_adc

  SEGMENTS IN THE MODULE
  ======================
SFR_AN
  Relative segment, address: DATA 000000B4 - 000000B4 (0x1 bytes), align: 0
  Segment part 1. ROOT        Intra module refs:   LL_ENC_GenerateTrueRandNum (ll_enc)
           ENTRY                   ADDRESS         REF BY
           =====                   =======         ======
           ADCCON1                 000000B4 
    -------------------------------------------------------------------------
SFR_AN
  Relative segment, address: DATA 000000B6 - 000000B6 (0x1 bytes), align: 0
  Segment part 2. ROOT 
           ENTRY                   ADDRESS         REF BY
           =====                   =======         ======
           ADCCON3                 000000B6 
    -------------------------------------------------------------------------
SFR_AN
  Relative segment, address: DATA 000000BA - 000000BA (0x1 bytes), align: 0
  Segment part 3. ROOT 
           ENTRY                   ADDRESS         REF BY
           =====                   =======         ======
           ADCL                    000000BA 
    -------------------------------------------------------------------------
SFR_AN
  Relative segment, address: DATA 000000BB - 000000BB (0x1 bytes), align: 0
  Segment part 4. ROOT 
           ENTRY                   ADDRESS         REF BY
           =====                   =======         ======
           ADCH                    000000BB 
    -------------------------------------------------------------------------
SFR_AN
  Relative segment, address: DATA 000000F2 - 000000F2 (0x1 bytes), align: 0
  Segment part 5. ROOT 
           ENTRY                   ADDRESS         REF BY
           =====                   =======         ======
           ADCCFG                  000000F2 
    -------------------------------------------------------------------------
XDATA_Z
  Relative segment, address: XDATA 000003B8 - 000003B8 (0x1 bytes), align: 0
  Segment part 11.            Intra module refs:   HalAdcInit
           LOCAL                   ADDRESS         
           =====                   =======         
           adcRef                  000003B8 
    -------------------------------------------------------------------------
<BANKED_CODE,XDATA_ROM_C_FLASH> 1 (was BANKED_CODE)
  Relative segment, address: CODE 0000C6F2 - 0000C702 (0x11 bytes), align: 0
  Segment part 12.            Intra module refs:   HalAdcInit::?relay
           ENTRY                   ADDRESS         REF BY
           =====                   =======         ======
           HalAdcInit              0000C6F2 
               ISTACK = 00000000 ( 00000002 )
    -------------------------------------------------------------------------
BANK_RELAYS
  Relative segment, address: CODE 000008BA - 000008BF (0x6 bytes), align: 0
  Segment part 13.
           ENTRY                   ADDRESS         REF BY
           =====                   =======         ======
           HalAdcInit::?relay      000008BA        HalDriverInit (hal_drivers)

    *************************************************************************

  FILE NAME : C:\ble\BLE-CC254x-1.4.1.43908\Projects\ble\SimpleBLEBroadcaster-usb\CC2540\CC2540USB\Obj\hal_aes.r51
  PROGRAM MODULE, NAME : hal_aes

  SEGMENTS IN THE MODULE
  ======================
SFR_AN
  Relative segment, address: DATA 000000B3 - 000000B3 (0x1 bytes), align: 0
  Segment part 1. ROOT        Intra module refs:   LL_ENC_LoadKey (ll_enc)
                                                   LL_ENC_StartAES (ll_enc)
           ENTRY                   ADDRESS         REF BY
           =====                   =======         ======
           ENCCS                   000000B3 
    -------------------------------------------------------------------------
SFR_AN
  Relative segment, address: DATA 000000D1 - 000000D1 (0x1 bytes), align: 0
  Segment part 2. ROOT        Intra module refs:   HalFlashWrite (hal_flash)
                                                   LL_ENC_SetupCryptoDMA (ll_enc)
                                                   LL_ENC_SetupLoadDMA (ll_enc)
           ENTRY                   ADDRESS         REF BY
           =====                   =======         ======
           DMAIRQ                  000000D1 
    -------------------------------------------------------------------------
SFR_AN
  Relative segment, address: DATA 000000D6 - 000000D6 (0x1 bytes), align: 0
  Segment part 3. ROOT        Intra module refs:   HalFlashWrite (hal_flash)
                                                   LL_ENC_SetupCryptoDMA (ll_enc)
                                                   LL_ENC_SetupLoadDMA (ll_enc)
           ENTRY                   ADDRESS         REF BY
           =====                   =======         ======
           DMAARM                  000000D6 
    -------------------------------------------------------------------------
<BANKED_CODE,XDATA_ROM_C_FLASH> 1 (was BANKED_CODE)
  Relative segment, address: CODE 0000AB7A - 0000AE44 (0x2cb bytes), align: 0
  Segment part 10.            Intra module refs:   aesDmaInit::?relay
           ENTRY                   ADDRESS         REF BY
           =====                   =======         ======
           aesDmaInit              0000AB7A 
               ISTACK = 00000000 ( 00000003 )
    -------------------------------------------------------------------------
<BANKED_CODE,XDATA_ROM_C_FLASH> 1 (was BANKED_CODE)
  Relative segment, address: CODE 0000AE45 - 0000AE52 (0xe bytes), align: 0
  Segment part 18.            Intra module refs:   HalAesInit::?relay
           ENTRY                   ADDRESS         REF BY
           =====                   =======         ======
           HalAesInit              0000AE45 
               calls direct
               ISTACK = 00000000 ( 00000002 )
    -------------------------------------------------------------------------
BANK_RELAYS
  Relative segment, address: CODE 000008C0 - 000008C5 (0x6 bytes), align: 0
  Segment part 11.            Intra module refs:   HalAesInit
           ENTRY                   ADDRESS         REF BY
           =====                   =======         ======
           aesDmaInit::?relay      000008C0 
    -------------------------------------------------------------------------
BANK_RELAYS
  Relative segment, address: CODE 000008C6 - 000008CB (0x6 bytes), align: 0
  Segment part 19.
           ENTRY                   ADDRESS         REF BY
           =====                   =======         ======
           HalAesInit::?relay      000008C6        HalDriverInit (hal_drivers)

    *************************************************************************

  FILE NAME : C:\ble\BLE-CC254x-1.4.1.43908\Projects\ble\SimpleBLEBroadcaster-usb\CC2540\CC2540USB\Obj\hal_assert.r51
  PROGRAM MODULE, NAME : hal_assert

  SEGMENTS IN THE MODULE
  ======================
SFR_AN
  Relative segment, address: DATA 00000080 - 00000080 (0x1 bytes), align: 0
  Segment part 1. ROOT        Intra module refs:   HalLedOnOff (hal_led)
           ENTRY                   ADDRESS         REF BY
           =====                   =======         ======
           _A_P0                   00000080 
           LOCAL                   ADDRESS         
           =====                   =======         
           P0                      00000080 
    -------------------------------------------------------------------------
SFR_AN
  Relative segment, address: DATA 00000090 - 00000090 (0x1 bytes), align: 0
  Segment part 2. ROOT        Intra module refs:   HalLedOnOff (hal_led)
                                                   HalUARTOpenUSB (hal_uart)
                                                   llSetRxGain (ll_common)
           ENTRY                   ADDRESS         REF BY
           =====                   =======         ======
           _A_P1                   00000090 
           LOCAL                   ADDRESS         
           =====                   =======         
           P1                      00000090 
    -------------------------------------------------------------------------
SFR_AN
  Relative segment, address: DATA 0000009D - 0000009D (0x1 bytes), align: 0
  Segment part 3. ROOT        Intra module refs:   main (SimpleBLEBroadcaster_Main)
                                                   usbirqHandler (usb_interrupt)
           ENTRY                   ADDRESS         REF BY
           =====                   =======         ======
           SLEEPSTA                0000009D 
    -------------------------------------------------------------------------
SFR_AN
  Relative segment, address: DATA 0000009E - 0000009E (0x1 bytes), align: 0
  Segment part 4. ROOT        Intra module refs:   llSetFreqTune (ll_common)
                                                   main (SimpleBLEBroadcaster_Main)
           ENTRY                   ADDRESS         REF BY
           =====                   =======         ======
           CLKCONSTA               0000009E 
    -------------------------------------------------------------------------
<BANKED_CODE,CODE_C> 1 (was BANKED_CODE)
  Relative segment, address: CODE 00007FF5 - 00007FF7 (0x3 bytes), align: 0
  Segment part 16.            Intra module refs:   halAssertHandler::?relay
           ENTRY                   ADDRESS         REF BY
           =====                   =======         ======
           halAssertHandler        00007FF5 
    -------------------------------------------------------------------------
BANK_RELAYS
  Relative segment, address: CODE 000008CC - 000008D1 (0x6 bytes), align: 0
  Segment part 17.
           ENTRY                   ADDRESS         REF BY
           =====                   =======         ======
           halAssertHandler::?relay
                                   000008CC        SimpleBLEBroadcaster_Init (simpleBLEBroadcaster)
                                                   compactPage (osal_snv)
                                                   findItem (osal_snv)
                                                   osal_mem_free (OSAL_Memory)
                                                   osal_mem_kick (OSAL_Memory)
                                                   osal_snv_init (osal_snv)

    *************************************************************************

  FILE NAME : C:\ble\BLE-CC254x-1.4.1.43908\Projects\ble\SimpleBLEBroadcaster-usb\CC2540\CC2540USB\Obj\hal_dma.r51
  PROGRAM MODULE, NAME : hal_dma

  SEGMENTS IN THE MODULE
  ======================
SFR_AN
  Relative segment, address: DATA 000000D2 - 000000D2 (0x1 bytes), align: 0
  Segment part 1. ROOT        Intra module refs:   HalDmaInit
           ENTRY                   ADDRESS         REF BY
           =====                   =======         ======
           DMA1CFGL                000000D2 
    -------------------------------------------------------------------------
SFR_AN
  Relative segment, address: DATA 000000D3 - 000000D3 (0x1 bytes), align: 0
  Segment part 2. ROOT        Intra module refs:   HalDmaInit
           ENTRY                   ADDRESS         REF BY
           =====                   =======         ======
           DMA1CFGH                000000D3 
    -------------------------------------------------------------------------
SFR_AN
  Relative segment, address: DATA 000000D4 - 000000D4 (0x1 bytes), align: 0
  Segment part 3. ROOT        Intra module refs:   HalDmaInit
           ENTRY                   ADDRESS         REF BY
           =====                   =======         ======
           DMA0CFGL                000000D4 
    -------------------------------------------------------------------------
SFR_AN
  Relative segment, address: DATA 000000D5 - 000000D5 (0x1 bytes), align: 0
  Segment part 4. ROOT        Intra module refs:   HalDmaInit
           ENTRY                   ADDRESS         REF BY
           =====                   =======         ======
           DMA0CFGH                000000D5 
    -------------------------------------------------------------------------
XDATA_Z
  Relative segment, address: XDATA 000003B9 - 000003C0 (0x8 bytes), align: 0
  Segment part 10.            Intra module refs:   HalDmaInit
           ENTRY                   ADDRESS         REF BY
           =====                   =======         ======
           dmaCh0                  000003B9        HalFlashWrite (hal_flash)
    -------------------------------------------------------------------------
XDATA_Z
  Relative segment, address: XDATA 000003C1 - 000003E0 (0x20 bytes), align: 0
  Segment part 11.            Intra module refs:   HalDmaInit
           ENTRY                   ADDRESS         REF BY
           =====                   =======         ======
           dmaCh1234               000003C1        LL_ENC_InitAesDMA (ll_enc)
                                                   LL_ENC_SetupCryptoDMA (ll_enc)
                                                   LL_ENC_SetupLoadDMA (ll_enc)
                                                   Segment part 41 (ll_enc)
                                                   aesDmaInit (hal_aes)
    -------------------------------------------------------------------------
<BANKED_CODE,CODE_C> 1 (was BANKED_CODE)
  Relative segment, address: CODE 00007FD8 - 00007FF4 (0x1d bytes), align: 0
  Segment part 12.            Intra module refs:   HalDmaInit::?relay
           ENTRY                   ADDRESS         REF BY
           =====                   =======         ======
           HalDmaInit              00007FD8 
    -------------------------------------------------------------------------
BANK_RELAYS
  Relative segment, address: CODE 000008D2 - 000008D7 (0x6 bytes), align: 0
  Segment part 13.
           ENTRY                   ADDRESS         REF BY
           =====                   =======         ======
           HalDmaInit::?relay      000008D2        HalDriverInit (hal_drivers)

    *************************************************************************

  FILE NAME : C:\ble\BLE-CC254x-1.4.1.43908\Projects\ble\SimpleBLEBroadcaster-usb\CC2540\CC2540USB\Obj\hal_drivers.r51
  PROGRAM MODULE, NAME : hal_drivers

  SEGMENTS IN THE MODULE
  ======================
XDATA_Z
  Relative segment, address: XDATA 000003E1 - 000003E1 (0x1 bytes), align: 0
  Segment part 6.             Intra module refs:   Hal_Init
                                                   Hal_ProcessEvent
           ENTRY                   ADDRESS         REF BY
           =====                   =======         ======
           Hal_TaskID              000003E1        HalLedBlink (hal_led)
                                                   HalLedUpdate (hal_led)
    -------------------------------------------------------------------------
<BANKED_CODE,XDATA_ROM_C_FLASH> 1 (was BANKED_CODE)
  Relative segment, address: CODE 0000C2C8 - 0000C2D7 (0x10 bytes), align: 0
  Segment part 7.             Intra module refs:   Hal_Init::?relay
           ENTRY                   ADDRESS         REF BY
           =====                   =======         ======
           Hal_Init                0000C2C8 
               ISTACK = 00000000 ( 00000002 )
    -------------------------------------------------------------------------
<BANKED_CODE,XDATA_ROM_C_FLASH> 1 (was BANKED_CODE)
  Relative segment, address: CODE 0000C2D8 - 0000C2F1 (0x1a bytes), align: 0
  Segment part 9.             Intra module refs:   HalDriverInit::?relay
           ENTRY                   ADDRESS         REF BY
           =====                   =======         ======
           HalDriverInit           0000C2D8 
               calls direct
               ISTACK = 00000000 ( 00000002 )
    -------------------------------------------------------------------------
<BANKED_CODE,XDATA_ROM_C_FLASH> 1 (was BANKED_CODE)
  Relative segment, address: CODE 0000C2F2 - 0000C370 (0x7f bytes), align: 0
  Segment part 11.            Intra module refs:   Hal_ProcessEvent::?relay
           ENTRY                   ADDRESS         REF BY
           =====                   =======         ======
           Hal_ProcessEvent        0000C2F2 
               calls direct
               XSTACK = 00000000 ( 0000000E )
    -------------------------------------------------------------------------
<BANKED_CODE,XDATA_ROM_C_FLASH> 1 (was BANKED_CODE)
  Relative segment, address: CODE 0000C371 - 0000C37E (0xe bytes), align: 0
  Segment part 13.            Intra module refs:   Hal_ProcessPoll::?relay
           ENTRY                   ADDRESS         REF BY
           =====                   =======         ======
           Hal_ProcessPoll         0000C371 
               calls direct
               ISTACK = 00000000 ( 00000002 )
    -------------------------------------------------------------------------
BANK_RELAYS
  Relative segment, address: CODE 000008D8 - 000008DD (0x6 bytes), align: 0
  Segment part 8.
           ENTRY                   ADDRESS         REF BY
           =====                   =======         ======
           Hal_Init::?relay        000008D8        osalInitTasks (OSAL_SimpleBLEBroadcaster)
    -------------------------------------------------------------------------
BANK_RELAYS
  Relative segment, address: CODE 000008DE - 000008E3 (0x6 bytes), align: 0
  Segment part 10.
           ENTRY                   ADDRESS         REF BY
           =====                   =======         ======
           HalDriverInit::?relay   000008DE        main (SimpleBLEBroadcaster_Main)
    -------------------------------------------------------------------------
BANK_RELAYS
  Relative segment, address: CODE 000008E4 - 000008E9 (0x6 bytes), align: 0
  Segment part 12.
           ENTRY                   ADDRESS         REF BY
           =====                   =======         ======
           Hal_ProcessEvent::?relay
                                   000008E4        tasksArr (OSAL_SimpleBLEBroadcaster)
    -------------------------------------------------------------------------
BANK_RELAYS
  Relative segment, address: CODE 000008EA - 000008EF (0x6 bytes), align: 0
  Segment part 14.
           ENTRY                   ADDRESS         REF BY
           =====                   =======         ======
           Hal_ProcessPoll::?relay
                                   000008EA        osal_run_system (OSAL)

    *************************************************************************

  FILE NAME : C:\ble\BLE-CC254x-1.4.1.43908\Projects\ble\SimpleBLEBroadcaster-usb\CC2540\CC2540USB\Obj\hal_flash.r51
  PROGRAM MODULE, NAME : hal_flash

  SEGMENTS IN THE MODULE
  ======================
SFR_AN
  Relative segment, address: DATA 000000C7 - 000000C7 (0x1 bytes), align: 0
  Segment part 2. ROOT        Intra module refs:   HalFlashRead
                                                   __low_level_init (hal_startup)
           ENTRY                   ADDRESS         REF BY
           =====                   =======         ======
           MEMCTR                  000000C7 
    -------------------------------------------------------------------------
<BANKED_CODE,XDATA_ROM_C_FLASH> 1 (was BANKED_CODE)
  Relative segment, address: CODE 0000A2A3 - 0000A34A (0xa8 bytes), align: 0
  Segment part 10.            Intra module refs:   HalFlashRead::?relay
           ENTRY                   ADDRESS         REF BY
           =====                   =======         ======
           HalFlashRead            0000A2A3 
               XSTACK = 00000002 ( 0000000D )
               ISTACK = 00000000 ( 00000001 )
    -------------------------------------------------------------------------
<BANKED_CODE,XDATA_ROM_C_FLASH> 1 (was BANKED_CODE)
  Relative segment, address: CODE 0000A34B - 0000A58C (0x242 bytes), align: 0
  Segment part 12.            Intra module refs:   HalFlashWrite::?relay
           ENTRY                   ADDRESS         REF BY
           =====                   =======         ======
           HalFlashWrite           0000A34B 
               XSTACK = 00000002 ( 0000000C )
               ISTACK = 00000000 ( 00000001 )
    -------------------------------------------------------------------------
<BANKED_CODE,XDATA_ROM_C_FLASH> 1 (was BANKED_CODE)
  Relative segment, address: CODE 0000A58D - 0000A5A7 (0x1b bytes), align: 0
  Segment part 14.            Intra module refs:   HalFlashErase::?relay
           ENTRY                   ADDRESS         REF BY
           =====                   =======         ======
           HalFlashErase           0000A58D 
               ISTACK = 00000000 ( 00000002 )
    -------------------------------------------------------------------------
BANK_RELAYS
  Relative segment, address: CODE 000008F0 - 000008F5 (0x6 bytes), align: 0
  Segment part 11.
           ENTRY                   ADDRESS         REF BY
           =====                   =======         ======
           HalFlashRead::?relay    000008F0        LL_Init (ll)
                                                   cleanErasedPage (osal_snv)
                                                   compactPage (osal_snv)
                                                   erasePage (osal_snv)
                                                   findItem (osal_snv)
                                                   findOffset (osal_snv)
                                                   initNV (osal_snv)
                                                   osal_snv_read (osal_snv)
                                                   osal_snv_write (osal_snv)
                                                   verifyWordM (osal_snv)
                                                   xferItem (osal_snv)
    -------------------------------------------------------------------------
BANK_RELAYS
  Relative segment, address: CODE 000008F6 - 000008FB (0x6 bytes), align: 0
  Segment part 13.
           ENTRY                   ADDRESS         REF BY
           =====                   =======         ======
           HalFlashWrite::?relay   000008F6        LL_EXT_SaveFreqTune (ll)
                                                   llFindTxPowerSettings (ll_common)
                                                   writeWord (osal_snv)
                                                   writeWordM (osal_snv)
    -------------------------------------------------------------------------
BANK_RELAYS
  Relative segment, address: CODE 000008FC - 00000901 (0x6 bytes), align: 0
  Segment part 15.
           ENTRY                   ADDRESS         REF BY
           =====                   =======         ======
           HalFlashErase::?relay   000008FC        erasePage (osal_snv)

    *************************************************************************

  FILE NAME : C:\ble\BLE-CC254x-1.4.1.43908\Projects\ble\SimpleBLEBroadcaster-usb\CC2540\CC2540USB\Obj\hal_key.r51
  PROGRAM MODULE, NAME : hal_key

  SEGMENTS IN THE MODULE
  ======================
<BANKED_CODE,CODE_C> 1 (was BANKED_CODE)
  Relative segment, address: CODE 00007FF8 - 00007FFA (0x3 bytes), align: 0
  Segment part 8.             Intra module refs:   HalKeyConfig::?relay
           ENTRY                   ADDRESS         REF BY
           =====                   =======         ======
           HalKeyConfig            00007FF8 
    -------------------------------------------------------------------------
BANK_RELAYS
  Relative segment, address: CODE 00000902 - 00000907 (0x6 bytes), align: 0
  Segment part 9.
           ENTRY                   ADDRESS         REF BY
           =====                   =======         ======
           HalKeyConfig::?relay    00000902        InitBoard (OnBoard)
                                                   OnBoard_KeyCallback (OnBoard)

    *************************************************************************

  FILE NAME : C:\ble\BLE-CC254x-1.4.1.43908\Projects\ble\SimpleBLEBroadcaster-usb\CC2540\CC2540USB\Obj\hal_lcd.r51
    *************************************************************************

  FILE NAME : C:\ble\BLE-CC254x-1.4.1.43908\Projects\ble\SimpleBLEBroadcaster-usb\CC2540\CC2540USB\Obj\hal_led.r51
  PROGRAM MODULE, NAME : hal_led

  SEGMENTS IN THE MODULE
  ======================
SFR_AN
  Relative segment, address: DATA 000000FD - 000000FD (0x1 bytes), align: 0
  Segment part 3. ROOT        Intra module refs:   HalLedInit
                                                   LL_EXT_MapPmIoPort (ll)
           ENTRY                   ADDRESS         REF BY
           =====                   =======         ======
           P0DIR                   000000FD 
    -------------------------------------------------------------------------
SFR_AN
  Relative segment, address: DATA 000000FE - 000000FE (0x1 bytes), align: 0
  Segment part 4. ROOT        Intra module refs:   HalLedInit
                                                   HalUARTOpenUSB (hal_uart)
                                                   LL_EXT_MapPmIoPort (ll)
                                                   llExtendRfRange (ll_common)
           ENTRY                   ADDRESS         REF BY
           =====                   =======         ======
           P1DIR                   000000FE 
    -------------------------------------------------------------------------
XDATA_Z
  Relative segment, address: XDATA 000003E2 - 000003E2 (0x1 bytes), align: 0
  Segment part 10.            Intra module refs:   HalLedBlink
                                                   HalLedOnOff
                                                   HalLedSet
           LOCAL                   ADDRESS         
           =====                   =======         
           HalLedState             000003E2 
    -------------------------------------------------------------------------
XDATA_Z
  Relative segment, address: XDATA 000003E3 - 000003E3 (0x1 bytes), align: 0
  Segment part 12.            Intra module refs:   HalLedBlink
                                                   HalLedUpdate
           LOCAL                   ADDRESS         
           =====                   =======         
           preBlinkState           000003E3 
    -------------------------------------------------------------------------
XDATA_Z
  Relative segment, address: XDATA 000003E4 - 00000408 (0x25 bytes), align: 0
  Segment part 13.            Intra module refs:   HalLedBlink
                                                   HalLedInit
                                                   HalLedSet
                                                   HalLedUpdate
           LOCAL                   ADDRESS         
           =====                   =======         
           HalLedStatusControl     000003E4 
    -------------------------------------------------------------------------
<BANKED_CODE,XDATA_ROM_C_FLASH> 1 (was BANKED_CODE)
  Relative segment, address: CODE 00008FE8 - 00009006 (0x1f bytes), align: 0
  Segment part 15.            Intra module refs:   HalLedInit::?relay
           ENTRY                   ADDRESS         REF BY
           =====                   =======         ======
           HalLedInit              00008FE8 
               calls direct
               ISTACK = 00000000 ( 00000002 )
    -------------------------------------------------------------------------
<BANKED_CODE,XDATA_ROM_C_FLASH> 1 (was BANKED_CODE)
  Relative segment, address: CODE 00009007 - 0000909C (0x96 bytes), align: 0
  Segment part 17.            Intra module refs:   HalLedSet::?relay
           ENTRY                   ADDRESS         REF BY
           =====                   =======         ======
           HalLedSet               00009007 
               calls direct, is recursive
               XSTACK = 0000001B ( 0000000B )
               ISTACK = 00000000 ( 00000001 )
    -------------------------------------------------------------------------
<BANKED_CODE,XDATA_ROM_C_FLASH> 1 (was BANKED_CODE)
  Relative segment, address: CODE 0000909D - 0000919A (0xfe bytes), align: 0
  Segment part 19.            Intra module refs:   HalLedBlink::?relay
           ENTRY                   ADDRESS         REF BY
           =====                   =======         ======
           HalLedBlink             0000909D 
               calls direct, is recursive
               XSTACK = 0000000B ( 0000000E )
               ISTACK = 00000000 ( 00000001 )
    -------------------------------------------------------------------------
<BANKED_CODE,XDATA_ROM_C_FLASH> 1 (was BANKED_CODE)
  Relative segment, address: CODE 0000919B - 000093FA (0x260 bytes), align: 0
  Segment part 21.            Intra module refs:   HalLedUpdate::?relay
           ENTRY                   ADDRESS         REF BY
           =====                   =======         ======
           HalLedUpdate            0000919B 
               calls direct
               XSTACK = 00000000 ( 0000001F )
               ISTACK = 00000000 ( 00000001 )
    -------------------------------------------------------------------------
<BANKED_CODE,XDATA_ROM_C_FLASH> 1 (was BANKED_CODE)
  Relative segment, address: CODE 000093FB - 0000945A (0x60 bytes), align: 0
  Segment part 23.            Intra module refs:   HalLedOnOff::?relay
           ENTRY                   ADDRESS         REF BY
           =====                   =======         ======
           HalLedOnOff             000093FB 
               XSTACK = 0000001B ( 00000000 )
               ISTACK = 00000000 ( 00000002 )
    -------------------------------------------------------------------------
<XDATA_ROM_C> 1 (was XDATA_ROM_C)
  Relative segment, address: CONST 00008FC8 - 00008FCB (0x4 bytes), align: 0
  Segment part 14.            Intra module refs:   HalLedUpdate
                                                   LL_EXT_ResetSystem (ll)
           ENTRY                   ADDRESS         REF BY
           =====                   =======         ======
           __Constant_64           00008FC8 
    -------------------------------------------------------------------------
BANK_RELAYS
  Relative segment, address: CODE 00000908 - 0000090D (0x6 bytes), align: 0
  Segment part 16.
           ENTRY                   ADDRESS         REF BY
           =====                   =======         ======
           HalLedInit::?relay      00000908        HalDriverInit (hal_drivers)
    -------------------------------------------------------------------------
BANK_RELAYS
  Relative segment, address: CODE 0000090E - 00000913 (0x6 bytes), align: 0
  Segment part 18.            Intra module refs:   HalLedBlink
                                                   HalLedInit
                                                   HalLedUpdate
           ENTRY                   ADDRESS         REF BY
           =====                   =======         ======
           HalLedSet::?relay       0000090E        InitBoard (OnBoard)
                                                   peripheralStateNotificationCB (simpleBLEBroadcaster)
    -------------------------------------------------------------------------
BANK_RELAYS
  Relative segment, address: CODE 00000914 - 00000919 (0x6 bytes), align: 0
  Segment part 20.            Intra module refs:   HalLedSet
           ENTRY                   ADDRESS         REF BY
           =====                   =======         ======
           HalLedBlink::?relay     00000914 
    -------------------------------------------------------------------------
BANK_RELAYS
  Relative segment, address: CODE 0000091A - 0000091F (0x6 bytes), align: 0
  Segment part 22.
           ENTRY                   ADDRESS         REF BY
           =====                   =======         ======
           HalLedUpdate::?relay    0000091A        Hal_ProcessEvent (hal_drivers)
    -------------------------------------------------------------------------
BANK_RELAYS
  Relative segment, address: CODE 00000920 - 00000925 (0x6 bytes), align: 0
  Segment part 24.            Intra module refs:   HalLedSet
                                                   HalLedUpdate
           ENTRY                   ADDRESS         REF BY
           =====                   =======         ======
           HalLedOnOff::?relay     00000920 
    -------------------------------------------------------------------------
<BANKED_CODE,XDATA_ROM_C_FLASH> 1 (was XDATA_ROM_C_FLASH)
  Relative segment, address: CODE 00008FC8 - 00008FCB (0x4 bytes), align: 0
  Segment part 31.            Intra module refs:   __Constant_64

    *************************************************************************

  FILE NAME : C:\ble\BLE-CC254x-1.4.1.43908\Projects\ble\SimpleBLEBroadcaster-usb\CC2540\CC2540USB\Obj\hal_sleep.r51
  PROGRAM MODULE, NAME : hal_sleep

  SEGMENTS IN THE MODULE
  ======================
SFR_AN
  Relative segment, address: DATA 00000087 - 00000087 (0x1 bytes), align: 0
  Segment part 1. ROOT 
           ENTRY                   ADDRESS         REF BY
           =====                   =======         ======
           PCON                    00000087 
    -------------------------------------------------------------------------
SFR_AN
  Relative segment, address: DATA 00000095 - 00000095 (0x1 bytes), align: 0
  Segment part 2. ROOT        Intra module refs:   halUartPollRx (hal_uart)
           ENTRY                   ADDRESS         REF BY
           =====                   =======         ======
           ST0                     00000095 
    -------------------------------------------------------------------------
SFR_AN
  Relative segment, address: DATA 00000096 - 00000096 (0x1 bytes), align: 0
  Segment part 3. ROOT 
           ENTRY                   ADDRESS         REF BY
           =====                   =======         ======
           ST1                     00000096 
    -------------------------------------------------------------------------
SFR_AN
  Relative segment, address: DATA 00000097 - 00000097 (0x1 bytes), align: 0
  Segment part 4. ROOT 
           ENTRY                   ADDRESS         REF BY
           =====                   =======         ======
           ST2                     00000097 
    -------------------------------------------------------------------------
SFR_AN
  Relative segment, address: DATA 0000009A - 0000009A (0x1 bytes), align: 0
  Segment part 5. ROOT        Intra module refs:   llClearSetInts (ll_common)
                                                   usbirqInit (usb_interrupt)
           ENTRY                   ADDRESS         REF BY
           =====                   =======         ======
           IEN2                    0000009A 
    -------------------------------------------------------------------------
SFR_AN
  Relative segment, address: DATA 000000AD - 000000AD (0x1 bytes), align: 0
  Segment part 7. ROOT 
           ENTRY                   ADDRESS         REF BY
           =====                   =======         ======
           STLOAD                  000000AD 
    -------------------------------------------------------------------------
SFR_AN
  Relative segment, address: DATA 000000B8 - 000000B8 (0x1 bytes), align: 0
  Segment part 8. ROOT        Intra module refs:   llClearSetInts (ll_common)
           ENTRY                   ADDRESS         REF BY
           =====                   =======         ======
           _A_IEN1                 000000B8 
           LOCAL                   ADDRESS         
           =====                   =======         
           IEN1                    000000B8 
    -------------------------------------------------------------------------
SFR_AN
  Relative segment, address: DATA 000000C0 - 000000C0 (0x1 bytes), align: 0
  Segment part 10. ROOT       Intra module refs:   halSleepTimerIsr
                                                   llClearSetInts (ll_common)
           ENTRY                   ADDRESS         REF BY
           =====                   =======         ======
           _A_IRCON                000000C0 
           LOCAL                   ADDRESS         
           =====                   =======         
           IRCON                   000000C0 
    -------------------------------------------------------------------------
NEAR_CODE
  Relative segment, address: CODE 000016BD - 000016E1 (0x25 bytes), align: 0
  Segment part 40.            Intra module refs:   halSleepTimerIsr::??INTVEC 43
           ENTRY                   ADDRESS         REF BY
           =====                   =======         ======
           halSleepTimerIsr        000016BD 
               interrupt function
               ISTACK = 00000000 ( 00000004 )
    -------------------------------------------------------------------------
INTVEC
  Common segment, address: CODE 00000000 - 0000002D (0x2e bytes), align: 0
  Segment part 11. ROOT 
           ENTRY                   ADDRESS         REF BY
           =====                   =======         ======
           halSleepTimerIsr::??INTVEC 43
                                   0000002B 

    *************************************************************************

  FILE NAME : C:\ble\BLE-CC254x-1.4.1.43908\Projects\ble\SimpleBLEBroadcaster-usb\CC2540\CC2540USB\Obj\hal_startup.r51
  PROGRAM MODULE, NAME : hal_startup

  SEGMENTS IN THE MODULE
  ======================
CSTART
  Relative segment, address: CODE 00000086 - 00000090 (0xb bytes), align: 0
  Segment part 7. ROOT 
           ENTRY                   ADDRESS         REF BY
           =====                   =======         ======
           __low_level_init        00000086        __low_level_init_call (?cmain)

    *************************************************************************

  FILE NAME : C:\ble\BLE-CC254x-1.4.1.43908\Projects\ble\SimpleBLEBroadcaster-usb\CC2540\CC2540USB\Obj\hal_timer.r51
    *************************************************************************

  FILE NAME : C:\ble\BLE-CC254x-1.4.1.43908\Projects\ble\SimpleBLEBroadcaster-usb\CC2540\CC2540USB\Obj\hal_uart.r51
  PROGRAM MODULE, NAME : hal_uart

  SEGMENTS IN THE MODULE
  ======================
SFR_AN
  Relative segment, address: DATA 000000F4 - 000000F4 (0x1 bytes), align: 0
  Segment part 4. ROOT        Intra module refs:   HalUARTOpenUSB
                                                   LL_EXT_MapPmIoPort (ll)
                                                   llExtendRfRange (ll_common)
           ENTRY                   ADDRESS         REF BY
           =====                   =======         ======
           P1SEL                   000000F4 
    -------------------------------------------------------------------------
<XDATA_N> 1 (was XDATA_N)
  Relative segment, address: XDATA 0000124E - 0000134D (0x100 bytes), align: 0
  Segment part 11.            Intra module refs:   HalUARTRx
                                                   halUartPollRx
           LOCAL                   ADDRESS         
           =====                   =======         
           halUartRxQ              0000124E 
    -------------------------------------------------------------------------
<XDATA_N> 1 (was XDATA_N)
  Relative segment, address: XDATA 0000114E - 0000124D (0x100 bytes), align: 0
  Segment part 12.            Intra module refs:   HalUARTTx
                                                   halUartPollTx
           LOCAL                   ADDRESS         
           =====                   =======         
           halUartTxQ              0000114E 
    -------------------------------------------------------------------------
XDATA_Z
  Relative segment, address: XDATA 00000409 - 00000409 (0x1 bytes), align: 0
  Segment part 13.            Intra module refs:   HalUARTRx
                                                   HalUARTRxAvailUSB
                                                   halUartPollRx
           LOCAL                   ADDRESS         
           =====                   =======         
           halUartRxH              00000409 
    -------------------------------------------------------------------------
XDATA_Z
  Relative segment, address: XDATA 0000040A - 0000040A (0x1 bytes), align: 0
  Segment part 14.            Intra module refs:   HalUARTRx
                                                   HalUARTRxAvailUSB
                                                   halUartPollRx
           LOCAL                   ADDRESS         
           =====                   =======         
           halUartRxT              0000040A 
    -------------------------------------------------------------------------
XDATA_Z
  Relative segment, address: XDATA 0000040B - 0000040B (0x1 bytes), align: 0
  Segment part 15.            Intra module refs:   halUartPollTx
           LOCAL                   ADDRESS         
           =====                   =======         
           halUartTxH              0000040B 
    -------------------------------------------------------------------------
XDATA_Z
  Relative segment, address: XDATA 0000040C - 0000040C (0x1 bytes), align: 0
  Segment part 16.            Intra module refs:   HalUARTTx
                                                   halUartPollTx
           LOCAL                   ADDRESS         
           =====                   =======         
           halUartTxT              0000040C 
    -------------------------------------------------------------------------
XDATA_Z
  Relative segment, address: XDATA 0000040D - 0000040D (0x1 bytes), align: 0
  Segment part 17.            Intra module refs:   halUartPollRx
           LOCAL                   ADDRESS         
           =====                   =======         
           rxTick                  0000040D 
    -------------------------------------------------------------------------
XDATA_Z
  Relative segment, address: XDATA 0000040E - 0000040E (0x1 bytes), align: 0
  Segment part 18.            Intra module refs:   halUartPollRx
           LOCAL                   ADDRESS         
           =====                   =======         
           rxShdw                  0000040E 
    -------------------------------------------------------------------------
XDATA_Z
  Relative segment, address: XDATA 0000040F - 0000040F (0x1 bytes), align: 0
  Segment part 19.            Intra module refs:   HalUARTTx
                                                   halUartPollTx
           LOCAL                   ADDRESS         
           =====                   =======         
           usbTxMT                 0000040F 
    -------------------------------------------------------------------------
XDATA_Z
  Relative segment, address: XDATA 00000410 - 00000411 (0x2 bytes), align: 0
  Segment part 20.            Intra module refs:   HalUARTOpenUSB
                                                   halUartPollRx
                                                   halUartPollTx
           LOCAL                   ADDRESS         
           =====                   =======         
           usbCB                   00000410 
    -------------------------------------------------------------------------
<BANKED_CODE,XDATA_ROM_C_FLASH> 1 (was BANKED_CODE)
  Relative segment, address: CODE 0000984F - 0000988A (0x3c bytes), align: 0
  Segment part 21.            Intra module refs:   HalUARTInitUSB::?relay
           LOCAL                   ADDRESS         
           =====                   =======         
           HalUARTInitUSB          0000984F 
               calls direct
               XSTACK = 00000000 ( 00000009 )
    -------------------------------------------------------------------------
<BANKED_CODE,XDATA_ROM_C_FLASH> 1 (was BANKED_CODE)
  Relative segment, address: CODE 0000988B - 000098B3 (0x29 bytes), align: 0
  Segment part 23.            Intra module refs:   HalUARTOpenUSB::?relay
           LOCAL                   ADDRESS         
           =====                   =======         
           HalUARTOpenUSB          0000988B 
               XSTACK = 00000009 ( 00000000 )
               ISTACK = 00000000 ( 00000002 )
    -------------------------------------------------------------------------
<BANKED_CODE,XDATA_ROM_C_FLASH> 1 (was BANKED_CODE)
  Relative segment, address: CODE 000098B4 - 000098C7 (0x14 bytes), align: 0
  Segment part 25.            Intra module refs:   HalUARTPollUSB::?relay
           LOCAL                   ADDRESS         
           =====                   =======         
           HalUARTPollUSB          000098B4 
               calls direct
               ISTACK = 00000000 ( 00000002 )
    -------------------------------------------------------------------------
<BANKED_CODE,XDATA_ROM_C_FLASH> 1 (was BANKED_CODE)
  Relative segment, address: CODE 000098C8 - 00009914 (0x4d bytes), align: 0
  Segment part 27.            Intra module refs:   HalUARTRx::?relay
           ENTRY                   ADDRESS         REF BY
           =====                   =======         ======
           HalUARTRx               000098C8 
               XSTACK = 0000000B ( 00000009 )
               ISTACK = 00000000 ( 00000001 )
    -------------------------------------------------------------------------
<BANKED_CODE,XDATA_ROM_C_FLASH> 1 (was BANKED_CODE)
  Relative segment, address: CODE 00009915 - 0000995F (0x4b bytes), align: 0
  Segment part 29.            Intra module refs:   HalUARTTx::?relay
           ENTRY                   ADDRESS         REF BY
           =====                   =======         ======
           HalUARTTx               00009915 
               XSTACK = 0000000B ( 00000000 )
               ISTACK = 00000000 ( 00000003 )
    -------------------------------------------------------------------------
<BANKED_CODE,XDATA_ROM_C_FLASH> 1 (was BANKED_CODE)
  Relative segment, address: CODE 00009960 - 000099AB (0x4c bytes), align: 0
  Segment part 31.            Intra module refs:   HalUARTRxAvailUSB::?relay
           LOCAL                   ADDRESS         
           =====                   =======         
           HalUARTRxAvailUSB       00009960 
               XSTACK = 00000009 ( 00000000 )
               ISTACK = 00000000 ( 00000002 )
    -------------------------------------------------------------------------
<BANKED_CODE,XDATA_ROM_C_FLASH> 1 (was BANKED_CODE)
  Relative segment, address: CODE 000099AC - 00009A07 (0x5c bytes), align: 0
  Segment part 33.            Intra module refs:   halUartPollEvt::?relay
           LOCAL                   ADDRESS         
           =====                   =======         
           halUartPollEvt          000099AC 
               calls direct
               ISTACK = 00000000 ( 00000002 )
    -------------------------------------------------------------------------
<BANKED_CODE,XDATA_ROM_C_FLASH> 1 (was BANKED_CODE)
  Relative segment, address: CODE 00009A08 - 00009AFE (0xf7 bytes), align: 0
  Segment part 35.            Intra module refs:   halUartPollRx::?relay
           LOCAL                   ADDRESS         
           =====                   =======         
           halUartPollRx           00009A08 
               XSTACK = 00000000 ( 0000000B )
               ISTACK = 00000000 ( 00000001 )
    -------------------------------------------------------------------------
<BANKED_CODE,XDATA_ROM_C_FLASH> 1 (was BANKED_CODE)
  Relative segment, address: CODE 00009AFF - 00009B8D (0x8f bytes), align: 0
  Segment part 37.            Intra module refs:   halUartPollTx::?relay
           LOCAL                   ADDRESS         
           =====                   =======         
           halUartPollTx           00009AFF 
               XSTACK = 00000000 ( 00000009 )
    -------------------------------------------------------------------------
<BANKED_CODE,XDATA_ROM_C_FLASH> 1 (was BANKED_CODE)
  Relative segment, address: CODE 00009B8E - 00009B9B (0xe bytes), align: 0
  Segment part 39.            Intra module refs:   HalUARTInit::?relay
           ENTRY                   ADDRESS         REF BY
           =====                   =======         ======
           HalUARTInit             00009B8E 
               calls direct
               ISTACK = 00000000 ( 00000002 )
    -------------------------------------------------------------------------
<BANKED_CODE,XDATA_ROM_C_FLASH> 1 (was BANKED_CODE)
  Relative segment, address: CODE 00009B9C - 00009BB4 (0x19 bytes), align: 0
  Segment part 41.            Intra module refs:   HalUARTOpen::?relay
           ENTRY                   ADDRESS         REF BY
           =====                   =======         ======
           HalUARTOpen             00009B9C 
               calls direct
               XSTACK = 00000000 ( 00000009 )
    -------------------------------------------------------------------------
<BANKED_CODE,XDATA_ROM_C_FLASH> 1 (was BANKED_CODE)
  Relative segment, address: CODE 00009BB5 - 00009BD5 (0x21 bytes), align: 0
  Segment part 43.            Intra module refs:   HalUARTRead::?relay
           ENTRY                   ADDRESS         REF BY
           =====                   =======         ======
           HalUARTRead             00009BB5 
               calls direct
               XSTACK = 00000000 ( 0000000B )
    -------------------------------------------------------------------------
<BANKED_CODE,XDATA_ROM_C_FLASH> 1 (was BANKED_CODE)
  Relative segment, address: CODE 00009BD6 - 00009BF7 (0x22 bytes), align: 0
  Segment part 45.            Intra module refs:   HalUARTWrite::?relay
           ENTRY                   ADDRESS         REF BY
           =====                   =======         ======
           HalUARTWrite            00009BD6 
               calls direct
               XSTACK = 00000000 ( 0000000B )
    -------------------------------------------------------------------------
<BANKED_CODE,XDATA_ROM_C_FLASH> 1 (was BANKED_CODE)
  Relative segment, address: CODE 00009BF8 - 00009C05 (0xe bytes), align: 0
  Segment part 51.            Intra module refs:   HalUARTPoll::?relay
           ENTRY                   ADDRESS         REF BY
           =====                   =======         ======
           HalUARTPoll             00009BF8 
               calls direct
               ISTACK = 00000000 ( 00000002 )
    -------------------------------------------------------------------------
<BANKED_CODE,XDATA_ROM_C_FLASH> 1 (was BANKED_CODE)
  Relative segment, address: CODE 00009C06 - 00009C14 (0xf bytes), align: 0
  Segment part 53.            Intra module refs:   Hal_UART_RxBufLen::?relay
           ENTRY                   ADDRESS         REF BY
           =====                   =======         ======
           Hal_UART_RxBufLen       00009C06 
               calls direct
               XSTACK = 00000000 ( 00000009 )
    -------------------------------------------------------------------------
BANK_RELAYS
  Relative segment, address: CODE 00000926 - 0000092B (0x6 bytes), align: 0
  Segment part 22.            Intra module refs:   HalUARTInit
           LOCAL                   ADDRESS         
           =====                   =======         
           HalUARTInitUSB::?relay
                                   00000926 
    -------------------------------------------------------------------------
BANK_RELAYS
  Relative segment, address: CODE 0000092C - 00000931 (0x6 bytes), align: 0
  Segment part 24.            Intra module refs:   HalUARTOpen
           LOCAL                   ADDRESS         
           =====                   =======         
           HalUARTOpenUSB::?relay
                                   0000092C 
    -------------------------------------------------------------------------
BANK_RELAYS
  Relative segment, address: CODE 00000932 - 00000937 (0x6 bytes), align: 0
  Segment part 26.            Intra module refs:   HalUARTPoll
           LOCAL                   ADDRESS         
           =====                   =======         
           HalUARTPollUSB::?relay
                                   00000932 
    -------------------------------------------------------------------------
BANK_RELAYS
  Relative segment, address: CODE 00000938 - 0000093D (0x6 bytes), align: 0
  Segment part 28.            Intra module refs:   HalUARTRead
           ENTRY                   ADDRESS         REF BY
           =====                   =======         ======
           HalUARTRx::?relay       00000938 
    -------------------------------------------------------------------------
BANK_RELAYS
  Relative segment, address: CODE 0000093E - 00000943 (0x6 bytes), align: 0
  Segment part 30.            Intra module refs:   HalUARTWrite
           ENTRY                   ADDRESS         REF BY
           =====                   =======         ======
           HalUARTTx::?relay       0000093E 
    -------------------------------------------------------------------------
BANK_RELAYS
  Relative segment, address: CODE 00000944 - 00000949 (0x6 bytes), align: 0
  Segment part 32.            Intra module refs:   Hal_UART_RxBufLen
           LOCAL                   ADDRESS         
           =====                   =======         
           HalUARTRxAvailUSB::?relay
                                   00000944 
    -------------------------------------------------------------------------
BANK_RELAYS
  Relative segment, address: CODE 0000094A - 0000094F (0x6 bytes), align: 0
  Segment part 34.            Intra module refs:   HalUARTPollUSB
           LOCAL                   ADDRESS         
           =====                   =======         
           halUartPollEvt::?relay
                                   0000094A 
    -------------------------------------------------------------------------
BANK_RELAYS
  Relative segment, address: CODE 00000950 - 00000955 (0x6 bytes), align: 0
  Segment part 36.            Intra module refs:   HalUARTPollUSB
           LOCAL                   ADDRESS         
           =====                   =======         
           halUartPollRx::?relay   00000950 
    -------------------------------------------------------------------------
BANK_RELAYS
  Relative segment, address: CODE 00000956 - 0000095B (0x6 bytes), align: 0
  Segment part 38.            Intra module refs:   HalUARTPollUSB
           LOCAL                   ADDRESS         
           =====                   =======         
           halUartPollTx::?relay   00000956 
    -------------------------------------------------------------------------
BANK_RELAYS
  Relative segment, address: CODE 0000095C - 00000961 (0x6 bytes), align: 0
  Segment part 40.
           ENTRY                   ADDRESS         REF BY
           =====                   =======         ======
           HalUARTInit::?relay     0000095C        HalDriverInit (hal_drivers)
    -------------------------------------------------------------------------
BANK_RELAYS
  Relative segment, address: CODE 00000962 - 00000967 (0x6 bytes), align: 0
  Segment part 42.
           ENTRY                   ADDRESS         REF BY
           =====                   =======         ======
           HalUARTOpen::?relay     00000962        NPI_InitTransport (npi)
    -------------------------------------------------------------------------
BANK_RELAYS
  Relative segment, address: CODE 00000968 - 0000096D (0x6 bytes), align: 0
  Segment part 44.
           ENTRY                   ADDRESS         REF BY
           =====                   =======         ======
           HalUARTRead::?relay     00000968        NPI_ReadTransport (npi)
    -------------------------------------------------------------------------
BANK_RELAYS
  Relative segment, address: CODE 0000096E - 00000973 (0x6 bytes), align: 0
  Segment part 46.
           ENTRY                   ADDRESS         REF BY
           =====                   =======         ======
           HalUARTWrite::?relay    0000096E        NPI_WriteTransport (npi)
                                                   SerialDebug_process (serialInterface)
                                                   sendSerialEvt (serialInterface)
    -------------------------------------------------------------------------
BANK_RELAYS
  Relative segment, address: CODE 00000974 - 00000979 (0x6 bytes), align: 0
  Segment part 52.
           ENTRY                   ADDRESS         REF BY
           =====                   =======         ======
           HalUARTPoll::?relay     00000974        Hal_ProcessPoll (hal_drivers)
    -------------------------------------------------------------------------
BANK_RELAYS
  Relative segment, address: CODE 0000097A - 0000097F (0x6 bytes), align: 0
  Segment part 54.
           ENTRY                   ADDRESS         REF BY
           =====                   =======         ======
           Hal_UART_RxBufLen::?relay
                                   0000097A        NPI_RxBufLen (npi)

    *************************************************************************

  FILE NAME : C:\ble\BLE-CC254x-1.4.1.43908\Projects\ble\SimpleBLEBroadcaster-usb\CC2540\CC2540USB\Obj\npi.r51
  PROGRAM MODULE, NAME : npi

  SEGMENTS IN THE MODULE
  ======================
<BANKED_CODE,XDATA_ROM_C_FLASH> 1 (was BANKED_CODE)
  Relative segment, address: CODE 0000C1FA - 0000C272 (0x79 bytes), align: 0
  Segment part 6.             Intra module refs:   NPI_InitTransport::?relay
           ENTRY                   ADDRESS         REF BY
           =====                   =======         ======
           NPI_InitTransport       0000C1FA 
               calls direct
               XSTACK = 00000000 ( 00000026 )
    -------------------------------------------------------------------------
<BANKED_CODE,XDATA_ROM_C_FLASH> 1 (was BANKED_CODE)
  Relative segment, address: CODE 0000C273 - 0000C291 (0x1f bytes), align: 0
  Segment part 8.             Intra module refs:   NPI_ReadTransport::?relay
           ENTRY                   ADDRESS         REF BY
           =====                   =======         ======
           NPI_ReadTransport       0000C273 
               calls direct
               XSTACK = 00000000 ( 0000000A )
    -------------------------------------------------------------------------
<BANKED_CODE,XDATA_ROM_C_FLASH> 1 (was BANKED_CODE)
  Relative segment, address: CODE 0000C292 - 0000C2B0 (0x1f bytes), align: 0
  Segment part 10.            Intra module refs:   NPI_WriteTransport::?relay
           ENTRY                   ADDRESS         REF BY
           =====                   =======         ======
           NPI_WriteTransport      0000C292 
               calls direct
               XSTACK = 00000000 ( 0000000A )
    -------------------------------------------------------------------------
<BANKED_CODE,XDATA_ROM_C_FLASH> 1 (was BANKED_CODE)
  Relative segment, address: CODE 0000C2B1 - 0000C2C0 (0x10 bytes), align: 0
  Segment part 12.            Intra module refs:   NPI_RxBufLen::?relay
           ENTRY                   ADDRESS         REF BY
           =====                   =======         ======
           NPI_RxBufLen            0000C2B1 
               calls direct
               ISTACK = 00000000 ( 00000002 )
    -------------------------------------------------------------------------
<BANKED_CODE,XDATA_ROM_C_FLASH> 1 (was BANKED_CODE)
  Relative segment, address: CODE 0000C2C1 - 0000C2C7 (0x7 bytes), align: 0
  Segment part 14.            Intra module refs:   NPI_GetMaxRxBufSize::?relay
           ENTRY                   ADDRESS         REF BY
           =====                   =======         ======
           NPI_GetMaxRxBufSize     0000C2C1 
    -------------------------------------------------------------------------
BANK_RELAYS
  Relative segment, address: CODE 00000980 - 00000985 (0x6 bytes), align: 0
  Segment part 7.
           ENTRY                   ADDRESS         REF BY
           =====                   =======         ======
           NPI_InitTransport::?relay
                                   00000980        HCI_Init (hci_tl)
                                                   SerialInterface_Init (serialInterface)
    -------------------------------------------------------------------------
BANK_RELAYS
  Relative segment, address: CODE 00000986 - 0000098B (0x6 bytes), align: 0
  Segment part 9.
           ENTRY                   ADDRESS         REF BY
           =====                   =======         ======
           NPI_ReadTransport::?relay
                                   00000986        cSerialPacketParser (serialInterface)
                                                   hciSerialPacketParser (hci_tl)
    -------------------------------------------------------------------------
BANK_RELAYS
  Relative segment, address: CODE 0000098C - 00000991 (0x6 bytes), align: 0
  Segment part 11.
           ENTRY                   ADDRESS         REF BY
           =====                   =======         ======
           NPI_WriteTransport::?relay
                                   0000098C        hciProcessCtrlToHost (hci_tl)
    -------------------------------------------------------------------------
BANK_RELAYS
  Relative segment, address: CODE 00000992 - 00000997 (0x6 bytes), align: 0
  Segment part 13.
           ENTRY                   ADDRESS         REF BY
           =====                   =======         ======
           NPI_RxBufLen::?relay    00000992        cSerialPacketParser (serialInterface)
                                                   hciSerialPacketParser (hci_tl)
    -------------------------------------------------------------------------
BANK_RELAYS
  Relative segment, address: CODE 00000998 - 0000099D (0x6 bytes), align: 0
  Segment part 15.
           ENTRY                   ADDRESS         REF BY
           =====                   =======         ======
           NPI_GetMaxRxBufSize::?relay
                                   00000998        hciSerialPacketParser (hci_tl)

    *************************************************************************

  FILE NAME : C:\ble\BLE-CC254x-1.4.1.43908\Projects\ble\SimpleBLEBroadcaster-usb\CC2540\CC2540USB\Obj\OnBoard.r51
  PROGRAM MODULE, NAME : OnBoard

  SEGMENTS IN THE MODULE
  ======================
XDATA_Z
  Relative segment, address: XDATA 00000412 - 00000412 (0x1 bytes), align: 0
  Segment part 7.             Intra module refs:   InitBoard
                                                   OnBoard_KeyCallback
           ENTRY                   ADDRESS         REF BY
           =====                   =======         ======
           OnboardKeyIntEnable     00000412 
    -------------------------------------------------------------------------
XDATA_I
  Relative segment, address: XDATA 000010EF - 000010EF (0x1 bytes), align: 0
  Segment part 8.             Intra module refs:   OnBoard_SendKeys
           LOCAL                   ADDRESS         
           =====                   =======         
           registeredKeysTaskID    000010EF 
    -------------------------------------------------------------------------
<BANKED_CODE,XDATA_ROM_C_FLASH> 1 (was BANKED_CODE)
  Relative segment, address: CODE 0000C011 - 0000C041 (0x31 bytes), align: 0
  Segment part 10.            Intra module refs:   InitBoard::?relay
           ENTRY                   ADDRESS         REF BY
           =====                   =======         ======
           InitBoard               0000C011 
               calls direct
               XSTACK = 00000000 ( 00000009 )
    -------------------------------------------------------------------------
<BANKED_CODE,XDATA_ROM_C_FLASH> 1 (was BANKED_CODE)
  Relative segment, address: CODE 0000C042 - 0000C09F (0x5e bytes), align: 0
  Segment part 18.            Intra module refs:   OnBoard_SendKeys::?relay
           ENTRY                   ADDRESS         REF BY
           =====                   =======         ======
           OnBoard_SendKeys        0000C042 
               calls direct
               XSTACK = 00000009 ( 0000000C )
               ISTACK = 00000000 ( 00000001 )
    -------------------------------------------------------------------------
<BANKED_CODE,XDATA_ROM_C_FLASH> 1 (was BANKED_CODE)
  Relative segment, address: CODE 0000C0A0 - 0000C108 (0x69 bytes), align: 0
  Segment part 20.            Intra module refs:   OnBoard_KeyCallback::?relay
           ENTRY                   ADDRESS         REF BY
           =====                   =======         ======
           OnBoard_KeyCallback     0000C0A0 
               calls direct, is indirectly called
               XSTACK = 00000000 ( 00000009 )
    -------------------------------------------------------------------------
NEAR_CODE
  Relative segment, address: CODE 000016E2 - 000016E7 (0x6 bytes), align: 0
  Segment part 24.
           ENTRY                   ADDRESS         REF BY
           =====                   =======         ======
           Onboard_soft_reset      000016E2        LL_ProcessEvent (ll)
    -------------------------------------------------------------------------
XDATA_ID
  Relative segment, address: CODE 000001CB - 000001CB (0x1 bytes), align: 0
  Segment part 9.             Intra module refs:   registeredKeysTaskID
    -------------------------------------------------------------------------
BANK_RELAYS
  Relative segment, address: CODE 0000099E - 000009A3 (0x6 bytes), align: 0
  Segment part 11.
           ENTRY                   ADDRESS         REF BY
           =====                   =======         ======
           InitBoard::?relay       0000099E        main (SimpleBLEBroadcaster_Main)
    -------------------------------------------------------------------------
BANK_RELAYS
  Relative segment, address: CODE 000009A4 - 000009A9 (0x6 bytes), align: 0
  Segment part 19.            Intra module refs:   OnBoard_KeyCallback
           ENTRY                   ADDRESS         REF BY
           =====                   =======         ======
           OnBoard_SendKeys::?relay
                                   000009A4 
    -------------------------------------------------------------------------
BANK_RELAYS
  Relative segment, address: CODE 000009AA - 000009AF (0x6 bytes), align: 0
  Segment part 21.            Intra module refs:   InitBoard
                                                   OnBoard_KeyCallback
           ENTRY                   ADDRESS         REF BY
           =====                   =======         ======
           OnBoard_KeyCallback::?relay
                                   000009AA 

    *************************************************************************

  FILE NAME : C:\ble\BLE-CC254x-1.4.1.43908\Projects\ble\SimpleBLEBroadcaster-usb\CC2540\CC2540USB\Obj\OSAL.r51
  PROGRAM MODULE, NAME : OSAL

  SEGMENTS IN THE MODULE
  ======================
XDATA_Z
  Relative segment, address: XDATA 00000413 - 00000414 (0x2 bytes), align: 0
  Segment part 11.            Intra module refs:   osal_init_system
                                                   osal_msg_enqueue_push
                                                   osal_msg_receive
           ENTRY                   ADDRESS         REF BY
           =====                   =======         ======
           osal_qHead              00000413 
    -------------------------------------------------------------------------
XDATA_I
  Relative segment, address: XDATA 000010F0 - 000010F0 (0x1 bytes), align: 0
  Segment part 12.            Intra module refs:   osal_run_system
           LOCAL                   ADDRESS         
           =====                   =======         
           activeTaskID            000010F0 
    -------------------------------------------------------------------------
<BANKED_CODE,CODE_C> 1 (was BANKED_CODE)
  Relative segment, address: CODE 00005F9C - 00005FF7 (0x5c bytes), align: 0
  Segment part 18.            Intra module refs:   osal_memcpy::?relay
           ENTRY                   ADDRESS         REF BY
           =====                   =======         ======
           osal_memcpy             00005F9C 
               XSTACK = 00000010 ( 0000000C )
               ISTACK = 00000000 ( 00000001 )
    -------------------------------------------------------------------------
<BANKED_CODE,CODE_C> 1 (was BANKED_CODE)
  Relative segment, address: CODE 00005FF8 - 00006069 (0x72 bytes), align: 0
  Segment part 24.            Intra module refs:   osal_memcmp::?relay
           ENTRY                   ADDRESS         REF BY
           =====                   =======         ======
           osal_memcmp             00005FF8 
               XSTACK = 00000002 ( 0000000F )
    -------------------------------------------------------------------------
<BANKED_CODE,CODE_C> 1 (was BANKED_CODE)
  Relative segment, address: CODE 0000606A - 00006092 (0x29 bytes), align: 0
  Segment part 26.            Intra module refs:   osal_memset::?relay
           ENTRY                   ADDRESS         REF BY
           =====                   =======         ======
           osal_memset             0000606A 
               calls direct
               XSTACK = 00000000 ( 0000000D )
    -------------------------------------------------------------------------
<BANKED_CODE,CODE_C> 1 (was BANKED_CODE)
  Relative segment, address: CODE 00006093 - 000060F4 (0x62 bytes), align: 0
  Segment part 36.            Intra module refs:   osal_msg_allocate::?relay
           ENTRY                   ADDRESS         REF BY
           =====                   =======         ======
           osal_msg_allocate       00006093 
               calls direct
               XSTACK = 00000000 ( 0000000C )
    -------------------------------------------------------------------------
<BANKED_CODE,CODE_C> 1 (was BANKED_CODE)
  Relative segment, address: CODE 000060F5 - 00006132 (0x3e bytes), align: 0
  Segment part 38.            Intra module refs:   osal_msg_deallocate::?relay
           ENTRY                   ADDRESS         REF BY
           =====                   =======         ======
           osal_msg_deallocate     000060F5 
               calls direct
               XSTACK = 0000000A ( 0000000A )
    -------------------------------------------------------------------------
<BANKED_CODE,CODE_C> 1 (was BANKED_CODE)
  Relative segment, address: CODE 00006133 - 0000614D (0x1b bytes), align: 0
  Segment part 40.            Intra module refs:   osal_msg_send::?relay
           ENTRY                   ADDRESS         REF BY
           =====                   =======         ======
           osal_msg_send           00006133 
               calls direct
               XSTACK = 00000000 ( 00000009 )
    -------------------------------------------------------------------------
<BANKED_CODE,CODE_C> 1 (was BANKED_CODE)
  Relative segment, address: CODE 0000614E - 00006168 (0x1b bytes), align: 0
  Segment part 42.            Intra module refs:   osal_msg_push_front::?relay
           ENTRY                   ADDRESS         REF BY
           =====                   =======         ======
           osal_msg_push_front     0000614E 
               calls direct
               XSTACK = 00000000 ( 00000009 )
    -------------------------------------------------------------------------
<BANKED_CODE,CODE_C> 1 (was BANKED_CODE)
  Relative segment, address: CODE 00006169 - 00006203 (0x9b bytes), align: 0
  Segment part 44.            Intra module refs:   osal_msg_enqueue_push::?relay
           LOCAL                   ADDRESS         
           =====                   =======         
           osal_msg_enqueue_push   00006169 
               calls direct
               XSTACK = 00000009 ( 0000000A )
               ISTACK = 00000000 ( 00000001 )
    -------------------------------------------------------------------------
<BANKED_CODE,CODE_C> 1 (was BANKED_CODE)
  Relative segment, address: CODE 00006204 - 000062AC (0xa9 bytes), align: 0
  Segment part 46.            Intra module refs:   osal_msg_receive::?relay
           ENTRY                   ADDRESS         REF BY
           =====                   =======         ======
           osal_msg_receive        00006204 
               calls direct
               XSTACK = 00000000 ( 00000010 )
    -------------------------------------------------------------------------
<BANKED_CODE,CODE_C> 1 (was BANKED_CODE)
  Relative segment, address: CODE 000062AD - 0000632F (0x83 bytes), align: 0
  Segment part 52.            Intra module refs:   osal_msg_enqueue::?relay
           ENTRY                   ADDRESS         REF BY
           =====                   =======         ======
           osal_msg_enqueue        000062AD 
               XSTACK = 0000000A ( 00000009 )
    -------------------------------------------------------------------------
<BANKED_CODE,CODE_C> 1 (was BANKED_CODE)
  Relative segment, address: CODE 00006330 - 00006368 (0x39 bytes), align: 0
  Segment part 56.            Intra module refs:   osal_msg_push::?relay
           ENTRY                   ADDRESS         REF BY
           =====                   =======         ======
           osal_msg_push           00006330 
               XSTACK = 0000000A ( 00000009 )
    -------------------------------------------------------------------------
<BANKED_CODE,CODE_C> 1 (was BANKED_CODE)
  Relative segment, address: CODE 00006369 - 000063F3 (0x8b bytes), align: 0
  Segment part 58.            Intra module refs:   osal_msg_extract::?relay
           ENTRY                   ADDRESS         REF BY
           =====                   =======         ======
           osal_msg_extract        00006369 
               XSTACK = 00000010 ( 0000000A )
    -------------------------------------------------------------------------
<BANKED_CODE,CODE_C> 1 (was BANKED_CODE)
  Relative segment, address: CODE 000063F4 - 0000644A (0x57 bytes), align: 0
  Segment part 62.            Intra module refs:   osal_set_event::?relay
           ENTRY                   ADDRESS         REF BY
           =====                   =======         ======
           osal_set_event          000063F4 
               XSTACK = 0000000E ( 00000009 )
    -------------------------------------------------------------------------
<BANKED_CODE,CODE_C> 1 (was BANKED_CODE)
  Relative segment, address: CODE 0000644B - 000064A8 (0x5e bytes), align: 0
  Segment part 64.            Intra module refs:   osal_clear_event::?relay
           ENTRY                   ADDRESS         REF BY
           =====                   =======         ======
           osal_clear_event        0000644B 
               XSTACK = 0000000E ( 00000009 )
    -------------------------------------------------------------------------
<BANKED_CODE,CODE_C> 1 (was BANKED_CODE)
  Relative segment, address: CODE 000064A9 - 000064BA (0x12 bytes), align: 0
  Segment part 70.            Intra module refs:   osal_int_disable::?relay
           ENTRY                   ADDRESS         REF BY
           =====                   =======         ======
           osal_int_disable        000064A9 
    -------------------------------------------------------------------------
<BANKED_CODE,CODE_C> 1 (was BANKED_CODE)
  Relative segment, address: CODE 000064BB - 000064E0 (0x26 bytes), align: 0
  Segment part 72.            Intra module refs:   osal_init_system::?relay
           ENTRY                   ADDRESS         REF BY
           =====                   =======         ======
           osal_init_system        000064BB 
               calls direct
               ISTACK = 00000000 ( 00000002 )
    -------------------------------------------------------------------------
<BANKED_CODE,CODE_C> 1 (was BANKED_CODE)
  Relative segment, address: CODE 000064E1 - 000064E9 (0x9 bytes), align: 0
  Segment part 74.            Intra module refs:   osal_start_system::?relay
           ENTRY                   ADDRESS         REF BY
           =====                   =======         ======
           osal_start_system       000064E1 
               calls direct
               ISTACK = 00000000 ( 00000002 )
    -------------------------------------------------------------------------
<BANKED_CODE,CODE_C> 1 (was BANKED_CODE)
  Relative segment, address: CODE 000064EA - 0000663A (0x151 bytes), align: 0
  Segment part 76.            Intra module refs:   osal_run_system::?relay
           ENTRY                   ADDRESS         REF BY
           =====                   =======         ======
           osal_run_system         000064EA 
               calls direct
               XSTACK = 00000000 ( 0000000E )
    -------------------------------------------------------------------------
XDATA_ID
  Relative segment, address: CODE 000001CC - 000001CC (0x1 bytes), align: 0
  Segment part 13.            Intra module refs:   activeTaskID
    -------------------------------------------------------------------------
BANK_RELAYS
  Relative segment, address: CODE 000009B0 - 000009B5 (0x6 bytes), align: 0
  Segment part 19.
           ENTRY                   ADDRESS         REF BY
           =====                   =======         ======
           osal_memcpy::?relay     000009B0        GAPRole_GetParameter (broadcaster)
                                                   GAPRole_ProcessEvent (broadcaster)
                                                   GAPRole_SetParameter (broadcaster)
                                                   GAP_MakeDiscoverable (gap_peridevmgr)
                                                   GAP_UpdateAdvertisingData (gap_peridevmgr)
                                                   HCI_CommandCompleteEvent (hci_event)
                                                   HCI_SendCommandCompleteEvent (hci_event)
                                                   HCI_SetEventMaskCmd (hci)
                                                   HCI_SetEventMaskPage2Cmd (hci_PATCH)
                                                   HCI_VendorSpecifcCommandCompleteEvent (hci_event_PATCH)
                                                   LL_RandCback (hci)
                                                   LL_SetAdvData (ll)
                                                   LL_SetScanRspData (ll)
                                                   gapProcessRandomAddrComplete (gap_configmgr)
                                                   gapReadBD_ADDRStatus (gap_configmgr)
                                                   gapRole_ProcessGAPMsg (broadcaster)
                                                   gapSendDeviceInitDoneEvent (gap_configmgr)
    -------------------------------------------------------------------------
BANK_RELAYS
  Relative segment, address: CODE 000009B6 - 000009BB (0x6 bytes), align: 0
  Segment part 25.
           ENTRY                   ADDRESS         REF BY
           =====                   =======         ======
           osal_memcmp::?relay     000009B6        verifyWordM (osal_snv)
    -------------------------------------------------------------------------
BANK_RELAYS
  Relative segment, address: CODE 000009BC - 000009C1 (0x6 bytes), align: 0
  Segment part 27.
           ENTRY                   ADDRESS         REF BY
           =====                   =======         ======
           osal_memset::?relay     000009BC        GAPRole_SetParameter (broadcaster)
                                                   GAP_ParamsInit (gap_configmgr)
                                                   GAP_PeriDevMgrInit (gap_peridevmgr)
                                                   GAP_UpdateAdvertisingData (gap_peridevmgr)
                                                   osalInitTasks (OSAL_SimpleBLEBroadcaster)
                                                   osal_CbTimerInit (osal_cbtimer)
    -------------------------------------------------------------------------
BANK_RELAYS
  Relative segment, address: CODE 000009C2 - 000009C7 (0x6 bytes), align: 0
  Segment part 37.
           ENTRY                   ADDRESS         REF BY
           =====                   =======         ======
           osal_msg_allocate::?relay
                                   000009C2        HCI_CommandCompleteEvent (hci_event)
                                                   HCI_SendCommandCompleteEvent (hci_event)
                                                   HCI_VendorSpecifcCommandCompleteEvent (hci_event_PATCH)
                                                   OnBoard_SendKeys (OnBoard)
                                                   gapProcessRandomAddrComplete (gap_configmgr)
                                                   gapSendDeviceInitDoneEvent (gap_configmgr)
                                                   gapSendMakeDiscEvent (gap_peridevmgr)
                                                   gapWriteAdvDataStatus (gap_peridevmgr)
                                                   gapWriteAdvEnableStatus (gap_peridevmgr)
                                                   hciSerialPacketParser (hci_tl)
    -------------------------------------------------------------------------
BANK_RELAYS
  Relative segment, address: CODE 000009C8 - 000009CD (0x6 bytes), align: 0
  Segment part 39.            Intra module refs:   osal_msg_enqueue_push
           ENTRY                   ADDRESS         REF BY
           =====                   =======         ======
           osal_msg_deallocate::?relay
                                   000009C8        GAPRole_ProcessEvent (broadcaster)
                                                   GAP_ProcessEvent (gap_simpletask)
                                                   Hal_ProcessEvent (hal_drivers)
                                                   SerialInterface_ProcessEvent (serialInterface)
                                                   SimpleBLEBroadcaster_ProcessEvent (simpleBLEBroadcaster)
                                                   hciProcessCtrlToHost (hci_tl)
                                                   hciProcessHostToCtrlCmd (hci_tl)
                                                   hciProcessHostToCtrlData (hci_tl)
                                                   hciSerialPacketParser (hci_tl)
    -------------------------------------------------------------------------
BANK_RELAYS
  Relative segment, address: CODE 000009CE - 000009D3 (0x6 bytes), align: 0
  Segment part 41.
           ENTRY                   ADDRESS         REF BY
           =====                   =======         ======
           osal_msg_send::?relay   000009CE        GAP_ProcessEvent (gap_simpletask)
                                                   HCI_CommandCompleteEvent (hci_event)
                                                   HCI_SendCommandCompleteEvent (hci_event)
                                                   HCI_VendorSpecifcCommandCompleteEvent (hci_event_PATCH)
                                                   OnBoard_SendKeys (OnBoard)
                                                   gapProcessRandomAddrComplete (gap_configmgr)
                                                   gapSendDeviceInitDoneEvent (gap_configmgr)
                                                   gapSendMakeDiscEvent (gap_peridevmgr)
                                                   gapWriteAdvDataStatus (gap_peridevmgr)
                                                   gapWriteAdvEnableStatus (gap_peridevmgr)
                                                   hciSerialPacketParser (hci_tl)
    -------------------------------------------------------------------------
BANK_RELAYS
  Relative segment, address: CODE 000009D4 - 000009D9 (0x6 bytes), align: 0
  Segment part 43.
           ENTRY                   ADDRESS         REF BY
           =====                   =======         ======
           osal_msg_push_front::?relay
                                   000009D4        hciProcessCtrlToHost (hci_tl)
    -------------------------------------------------------------------------
BANK_RELAYS
  Relative segment, address: CODE 000009DA - 000009DF (0x6 bytes), align: 0
  Segment part 45.            Intra module refs:   osal_msg_push_front
                                                   osal_msg_send
           LOCAL                   ADDRESS         
           =====                   =======         
           osal_msg_enqueue_push::?relay
                                   000009DA 
    -------------------------------------------------------------------------
BANK_RELAYS
  Relative segment, address: CODE 000009E0 - 000009E5 (0x6 bytes), align: 0
  Segment part 47.
           ENTRY                   ADDRESS         REF BY
           =====                   =======         ======
           osal_msg_receive::?relay
                                   000009E0        GAPRole_ProcessEvent (broadcaster)
                                                   GAP_ProcessEvent (gap_simpletask)
                                                   HCI_ProcessEvent (hci_tl)
                                                   Hal_ProcessEvent (hal_drivers)
                                                   SerialInterface_ProcessEvent (serialInterface)
                                                   SimpleBLEBroadcaster_ProcessEvent (simpleBLEBroadcaster)
    -------------------------------------------------------------------------
BANK_RELAYS
  Relative segment, address: CODE 000009E6 - 000009EB (0x6 bytes), align: 0
  Segment part 53.            Intra module refs:   osal_msg_enqueue_push
           ENTRY                   ADDRESS         REF BY
           =====                   =======         ======
           osal_msg_enqueue::?relay
                                   000009E6 
    -------------------------------------------------------------------------
BANK_RELAYS
  Relative segment, address: CODE 000009EC - 000009F1 (0x6 bytes), align: 0
  Segment part 57.            Intra module refs:   osal_msg_enqueue_push
           ENTRY                   ADDRESS         REF BY
           =====                   =======         ======
           osal_msg_push::?relay   000009EC 
    -------------------------------------------------------------------------
BANK_RELAYS
  Relative segment, address: CODE 000009F2 - 000009F7 (0x6 bytes), align: 0
  Segment part 59.            Intra module refs:   osal_msg_receive
           ENTRY                   ADDRESS         REF BY
           =====                   =======         ======
           osal_msg_extract::?relay
                                   000009F2 
    -------------------------------------------------------------------------
BANK_RELAYS
  Relative segment, address: CODE 000009F8 - 000009FD (0x6 bytes), align: 0
  Segment part 63.            Intra module refs:   osal_msg_enqueue_push
                                                   osal_msg_receive
           ENTRY                   ADDRESS         REF BY
           =====                   =======         ======
           osal_set_event::?relay
                                   000009F8        GAPRole_SetParameter (broadcaster)
                                                   HCI_EXT_SetBDADDRCmd (hci)
                                                   HalLedBlink (hal_led)
                                                   LL_Init (ll)
                                                   RF_NormalIsr (ll_isr)
                                                   SimpleBLEBroadcaster_Init (simpleBLEBroadcaster)
                                                   cSerialPacketParser (serialInterface)
                                                   gapRole_ProcessGAPMsg (broadcaster)
                                                   llDiscoverableAdvEvt_TaskEndOk (ll_advEndCauses)
                                                   llNonConnAdvEvt_TaskEndOk (ll_advEndCauses)
                                                   osalTimerUpdate (OSAL_Timers)
                                                   parseCmd (serialInterface)
    -------------------------------------------------------------------------
BANK_RELAYS
  Relative segment, address: CODE 000009FE - 00000A03 (0x6 bytes), align: 0
  Segment part 65.            Intra module refs:   osal_msg_receive
           ENTRY                   ADDRESS         REF BY
           =====                   =======         ======
           osal_clear_event::?relay
                                   000009FE        LL_SetAdvControl (ll)
                                                   llT2OVFC1_ISR (ll_isr)
    -------------------------------------------------------------------------
BANK_RELAYS
  Relative segment, address: CODE 00000A04 - 00000A09 (0x6 bytes), align: 0
  Segment part 71.
           ENTRY                   ADDRESS         REF BY
           =====                   =======         ======
           osal_int_disable::?relay
                                   00000A04        InitBoard (OnBoard)
    -------------------------------------------------------------------------
BANK_RELAYS
  Relative segment, address: CODE 00000A0A - 00000A0F (0x6 bytes), align: 0
  Segment part 73.
           ENTRY                   ADDRESS         REF BY
           =====                   =======         ======
           osal_init_system::?relay
                                   00000A0A        main (SimpleBLEBroadcaster_Main)
    -------------------------------------------------------------------------
BANK_RELAYS
  Relative segment, address: CODE 00000A10 - 00000A15 (0x6 bytes), align: 0
  Segment part 75.
           ENTRY                   ADDRESS         REF BY
           =====                   =======         ======
           osal_start_system::?relay
                                   00000A10        main (SimpleBLEBroadcaster_Main)
    -------------------------------------------------------------------------
BANK_RELAYS
  Relative segment, address: CODE 00000A16 - 00000A1B (0x6 bytes), align: 0
  Segment part 77.            Intra module refs:   osal_start_system
           ENTRY                   ADDRESS         REF BY
           =====                   =======         ======
           osal_run_system::?relay
                                   00000A16 

    *************************************************************************

  FILE NAME : C:\ble\BLE-CC254x-1.4.1.43908\Projects\ble\SimpleBLEBroadcaster-usb\CC2540\CC2540USB\Obj\osal_bufmgr.r51
  PROGRAM MODULE, NAME : osal_bufmgr

  SEGMENTS IN THE MODULE
  ======================
XDATA_Z
  Relative segment, address: XDATA 00000415 - 00000416 (0x2 bytes), align: 0
  Segment part 7.             Intra module refs:   osal_bm_alloc
                                                   osal_bm_free
           LOCAL                   ADDRESS         
           =====                   =======         
           bm_list_ptr             00000415 
    -------------------------------------------------------------------------
<BANKED_CODE,XDATA_ROM_C_FLASH> 1 (was BANKED_CODE)
  Relative segment, address: CODE 0000BDF2 - 0000BE58 (0x67 bytes), align: 0
  Segment part 8.             Intra module refs:   osal_bm_alloc::?relay
           ENTRY                   ADDRESS         REF BY
           =====                   =======         ======
           osal_bm_alloc           0000BDF2 
               calls direct
               XSTACK = 00000000 ( 0000000E )
    -------------------------------------------------------------------------
<BANKED_CODE,XDATA_ROM_C_FLASH> 1 (was BANKED_CODE)
  Relative segment, address: CODE 0000BE59 - 0000BF15 (0xbd bytes), align: 0
  Segment part 10.            Intra module refs:   osal_bm_free::?relay
           ENTRY                   ADDRESS         REF BY
           =====                   =======         ======
           osal_bm_free            0000BE59 
               calls direct
               XSTACK = 00000000 ( 0000000D )
    -------------------------------------------------------------------------
BANK_RELAYS
  Relative segment, address: CODE 00000A1C - 00000A21 (0x6 bytes), align: 0
  Segment part 9.
           ENTRY                   ADDRESS         REF BY
           =====                   =======         ======
           osal_bm_alloc::?relay   00000A1C        LL_TX_bm_alloc (ll)
    -------------------------------------------------------------------------
BANK_RELAYS
  Relative segment, address: CODE 00000A22 - 00000A27 (0x6 bytes), align: 0
  Segment part 11.
           ENTRY                   ADDRESS         REF BY
           =====                   =======         ======
           osal_bm_free::?relay    00000A22        hciProcessCtrlToHost (hci_tl)
                                                   hciProcessHostToCtrlData (hci_tl)

    *************************************************************************

  FILE NAME : C:\ble\BLE-CC254x-1.4.1.43908\Projects\ble\SimpleBLEBroadcaster-usb\CC2540\CC2540USB\Obj\osal_cbtimer.r51
  PROGRAM MODULE, NAME : osal_cbtimer

  SEGMENTS IN THE MODULE
  ======================
XDATA_I
  Relative segment, address: XDATA 000010F1 - 000010F2 (0x2 bytes), align: 0
  Segment part 7.             Intra module refs:   osal_CbTimerInit
                                                   osal_CbTimerProcessEvent
           ENTRY                   ADDRESS         REF BY
           =====                   =======         ======
           baseTaskID              000010F1 
    -------------------------------------------------------------------------
XDATA_Z
  Relative segment, address: XDATA 00000417 - 00000452 (0x3c bytes), align: 0
  Segment part 9.             Intra module refs:   osal_CbTimerInit
                                                   osal_CbTimerProcessEvent
           ENTRY                   ADDRESS         REF BY
           =====                   =======         ======
           cbTimers                00000417 
    -------------------------------------------------------------------------
<BANKED_CODE,XDATA_ROM_C_FLASH> 1 (was BANKED_CODE)
  Relative segment, address: CODE 0000BA03 - 0000BA35 (0x33 bytes), align: 0
  Segment part 10.            Intra module refs:   osal_CbTimerInit::?relay
           ENTRY                   ADDRESS         REF BY
           =====                   =======         ======
           osal_CbTimerInit        0000BA03 
               calls direct
               XSTACK = 00000000 ( 00000009 )
    -------------------------------------------------------------------------
<BANKED_CODE,XDATA_ROM_C_FLASH> 1 (was BANKED_CODE)
  Relative segment, address: CODE 0000BA36 - 0000BB67 (0x132 bytes), align: 0
  Segment part 12.            Intra module refs:   osal_CbTimerProcessEvent::?relay
           ENTRY                   ADDRESS         REF BY
           =====                   =======         ======
           osal_CbTimerProcessEvent
                                   0000BA36 
               calls direct
               XSTACK = 00000000 ( 00000012 )
    -------------------------------------------------------------------------
XDATA_ID
  Relative segment, address: CODE 000001CD - 000001CE (0x2 bytes), align: 0
  Segment part 8.             Intra module refs:   baseTaskID
    -------------------------------------------------------------------------
BANK_RELAYS
  Relative segment, address: CODE 00000A28 - 00000A2D (0x6 bytes), align: 0
  Segment part 11.
           ENTRY                   ADDRESS         REF BY
           =====                   =======         ======
           osal_CbTimerInit::?relay
                                   00000A28        osalInitTasks (OSAL_SimpleBLEBroadcaster)
    -------------------------------------------------------------------------
BANK_RELAYS
  Relative segment, address: CODE 00000A2E - 00000A33 (0x6 bytes), align: 0
  Segment part 13.
           ENTRY                   ADDRESS         REF BY
           =====                   =======         ======
           osal_CbTimerProcessEvent::?relay
                                   00000A2E        tasksArr (OSAL_SimpleBLEBroadcaster)

    *************************************************************************

  FILE NAME : C:\ble\BLE-CC254x-1.4.1.43908\Projects\ble\SimpleBLEBroadcaster-usb\CC2540\CC2540USB\Obj\OSAL_ClockBLE.r51
  PROGRAM MODULE, NAME : OSAL_ClockBLE

  SEGMENTS IN THE MODULE
  ======================
XDATA_Z
  Relative segment, address: XDATA 00000453 - 00000454 (0x2 bytes), align: 0
  Segment part 6.             Intra module refs:   osalTimeUpdate
           LOCAL                   ADDRESS         
           =====                   =======         
           previousLLTimerTick     00000453 
    -------------------------------------------------------------------------
XDATA_Z
  Relative segment, address: XDATA 00000455 - 00000456 (0x2 bytes), align: 0
  Segment part 7.             Intra module refs:   osalTimeUpdate
           LOCAL                   ADDRESS         
           =====                   =======         
           remUsTicks              00000455 
    -------------------------------------------------------------------------
XDATA_Z
  Relative segment, address: XDATA 00000457 - 00000458 (0x2 bytes), align: 0
  Segment part 8.             Intra module refs:   osalClockUpdate
           LOCAL                   ADDRESS         
           =====                   =======         
           timeMSec                00000457 
    -------------------------------------------------------------------------
XDATA_Z
  Relative segment, address: XDATA 00000459 - 0000045C (0x4 bytes), align: 0
  Segment part 9.             Intra module refs:   osalClockUpdate
           ENTRY                   ADDRESS         REF BY
           =====                   =======         ======
           OSAL_timeSeconds        00000459 
    -------------------------------------------------------------------------
<BANKED_CODE,XDATA_ROM_C_FLASH> 1 (was BANKED_CODE)
  Relative segment, address: CODE 0000BCB8 - 0000BD95 (0xde bytes), align: 0
  Segment part 13.            Intra module refs:   osalTimeUpdate::?relay
           ENTRY                   ADDRESS         REF BY
           =====                   =======         ======
           osalTimeUpdate          0000BCB8 
               calls direct
               XSTACK = 00000000 ( 0000000E )
    -------------------------------------------------------------------------
<BANKED_CODE,XDATA_ROM_C_FLASH> 1 (was BANKED_CODE)
  Relative segment, address: CODE 0000BD96 - 0000BDF1 (0x5c bytes), align: 0
  Segment part 15.            Intra module refs:   osalClockUpdate::?relay
           LOCAL                   ADDRESS         
           =====                   =======         
           osalClockUpdate         0000BD96 
               XSTACK = 0000000E ( 0000000C )
    -------------------------------------------------------------------------
BANK_RELAYS
  Relative segment, address: CODE 00000A34 - 00000A39 (0x6 bytes), align: 0
  Segment part 14.
           ENTRY                   ADDRESS         REF BY
           =====                   =======         ======
           osalTimeUpdate::?relay
                                   00000A34        llScheduleTask (ll_scheduler)
                                                   osal_run_system (OSAL)
    -------------------------------------------------------------------------
BANK_RELAYS
  Relative segment, address: CODE 00000A3A - 00000A3F (0x6 bytes), align: 0
  Segment part 16.            Intra module refs:   osalTimeUpdate
           LOCAL                   ADDRESS         
           =====                   =======         
           osalClockUpdate::?relay
                                   00000A3A 

    *************************************************************************

  FILE NAME : C:\ble\BLE-CC254x-1.4.1.43908\Projects\ble\SimpleBLEBroadcaster-usb\CC2540\CC2540USB\Obj\OSAL_Memory.r51
  PROGRAM MODULE, NAME : OSAL_Memory

  SEGMENTS IN THE MODULE
  ======================
XDATA_Z
  Relative segment, address: XDATA 0000045D - 00000FB0 (0xb54 bytes), align: 0
  Segment part 7.             Intra module refs:   osal_mem_alloc
                                                   osal_mem_free
                                                   osal_mem_init
           LOCAL                   ADDRESS         
           =====                   =======         
           theHeap                 0000045D 
    -------------------------------------------------------------------------
XDATA_Z
  Relative segment, address: XDATA 00000FB1 - 00000FB2 (0x2 bytes), align: 0
  Segment part 8.             Intra module refs:   osal_mem_alloc
                                                   osal_mem_free
                                                   osal_mem_init
                                                   osal_mem_kick
           LOCAL                   ADDRESS         
           =====                   =======         
           ff1                     00000FB1 
    -------------------------------------------------------------------------
XDATA_Z
  Relative segment, address: XDATA 00000FB3 - 00000FB3 (0x1 bytes), align: 0
  Segment part 9.             Intra module refs:   osal_mem_alloc
                                                   osal_mem_kick
           LOCAL                   ADDRESS         
           =====                   =======         
           osalMemStat             00000FB3 
    -------------------------------------------------------------------------
<BANKED_CODE,XDATA_ROM_C_FLASH> 1 (was BANKED_CODE)
  Relative segment, address: CODE 0000A8A0 - 0000A8E4 (0x45 bytes), align: 0
  Segment part 10.            Intra module refs:   osal_mem_init::?relay
           ENTRY                   ADDRESS         REF BY
           =====                   =======         ======
           osal_mem_init           0000A8A0 
               ISTACK = 00000000 ( 00000002 )
    -------------------------------------------------------------------------
<BANKED_CODE,XDATA_ROM_C_FLASH> 1 (was BANKED_CODE)
  Relative segment, address: CODE 0000A8E5 - 0000A931 (0x4d bytes), align: 0
  Segment part 12.            Intra module refs:   osal_mem_kick::?relay
           ENTRY                   ADDRESS         REF BY
           =====                   =======         ======
           osal_mem_kick           0000A8E5 
               calls direct
               XSTACK = 00000000 ( 0000000C )
    -------------------------------------------------------------------------
<BANKED_CODE,XDATA_ROM_C_FLASH> 1 (was BANKED_CODE)
  Relative segment, address: CODE 0000A932 - 0000AAFA (0x1c9 bytes), align: 0
  Segment part 14.            Intra module refs:   osal_mem_alloc::?relay
           ENTRY                   ADDRESS         REF BY
           =====                   =======         ======
           osal_mem_alloc          0000A932 
               XSTACK = 0000000C ( 0000000F )
    -------------------------------------------------------------------------
<BANKED_CODE,XDATA_ROM_C_FLASH> 1 (was BANKED_CODE)
  Relative segment, address: CODE 0000AAFB - 0000AB79 (0x7f bytes), align: 0
  Segment part 16.            Intra module refs:   osal_mem_free::?relay
           ENTRY                   ADDRESS         REF BY
           =====                   =======         ======
           osal_mem_free           0000AAFB 
               calls direct
               XSTACK = 0000000C ( 0000000B )
    -------------------------------------------------------------------------
BANK_RELAYS
  Relative segment, address: CODE 00000A40 - 00000A45 (0x6 bytes), align: 0
  Segment part 11.
           ENTRY                   ADDRESS         REF BY
           =====                   =======         ======
           osal_mem_init::?relay   00000A40        osal_init_system (OSAL)
    -------------------------------------------------------------------------
BANK_RELAYS
  Relative segment, address: CODE 00000A46 - 00000A4B (0x6 bytes), align: 0
  Segment part 13.
           ENTRY                   ADDRESS         REF BY
           =====                   =======         ======
           osal_mem_kick::?relay   00000A46        osal_init_system (OSAL)
    -------------------------------------------------------------------------
BANK_RELAYS
  Relative segment, address: CODE 00000A4C - 00000A51 (0x6 bytes), align: 0
  Segment part 15.            Intra module refs:   osal_mem_kick
           ENTRY                   ADDRESS         REF BY
           =====                   =======         ======
           osal_mem_alloc::?relay
                                   00000A4C        GAP_MakeDiscoverable (gap_peridevmgr)
                                                   GAP_PeriDevMgrInit (gap_peridevmgr)
                                                   osalAddTimer (OSAL_Timers)
                                                   osalInitTasks (OSAL_SimpleBLEBroadcaster)
                                                   osal_bm_alloc (osal_bufmgr)
                                                   osal_msg_allocate (OSAL)
    -------------------------------------------------------------------------
BANK_RELAYS
  Relative segment, address: CODE 00000A52 - 00000A57 (0x6 bytes), align: 0
  Segment part 17.            Intra module refs:   osal_mem_kick
           ENTRY                   ADDRESS         REF BY
           =====                   =======         ======
           osal_mem_free::?relay   00000A52        GAP_PeriDevMgrInit (gap_peridevmgr)
                                                   gapFreeAdvertState (gap_peridevmgr)
                                                   osalTimerUpdate (OSAL_Timers)
                                                   osal_bm_free (osal_bufmgr)
                                                   osal_msg_deallocate (OSAL)

    *************************************************************************

  FILE NAME : C:\ble\BLE-CC254x-1.4.1.43908\Projects\ble\SimpleBLEBroadcaster-usb\CC2540\CC2540USB\Obj\OSAL_PwrMgr.r51
  PROGRAM MODULE, NAME : OSAL_PwrMgr

  SEGMENTS IN THE MODULE
  ======================
XDATA_Z
  Relative segment, address: XDATA 00000FB4 - 00000FBA (0x7 bytes), align: 0
  Segment part 7.             Intra module refs:   osal_pwrmgr_device
                                                   osal_pwrmgr_init
                                                   osal_pwrmgr_task_state
           ENTRY                   ADDRESS         REF BY
           =====                   =======         ======
           pwrmgr_attribute        00000FB4 
    -------------------------------------------------------------------------
<BANKED_CODE,XDATA_ROM_C_FLASH> 1 (was BANKED_CODE)
  Relative segment, address: CODE 0000C426 - 0000C440 (0x1b bytes), align: 0
  Segment part 8.             Intra module refs:   osal_pwrmgr_init::?relay
           ENTRY                   ADDRESS         REF BY
           =====                   =======         ======
           osal_pwrmgr_init        0000C426 
               ISTACK = 00000000 ( 00000002 )
    -------------------------------------------------------------------------
<BANKED_CODE,XDATA_ROM_C_FLASH> 1 (was BANKED_CODE)
  Relative segment, address: CODE 0000C441 - 0000C450 (0x10 bytes), align: 0
  Segment part 10.            Intra module refs:   osal_pwrmgr_device::?relay
           ENTRY                   ADDRESS         REF BY
           =====                   =======         ======
           osal_pwrmgr_device      0000C441 
               ISTACK = 00000000 ( 00000002 )
    -------------------------------------------------------------------------
<BANKED_CODE,XDATA_ROM_C_FLASH> 1 (was BANKED_CODE)
  Relative segment, address: CODE 0000C451 - 0000C4B5 (0x65 bytes), align: 0
  Segment part 12.            Intra module refs:   osal_pwrmgr_task_state::?relay
           ENTRY                   ADDRESS         REF BY
           =====                   =======         ======
           osal_pwrmgr_task_state
                                   0000C451 
               XSTACK = 00000000 ( 0000000A )
    -------------------------------------------------------------------------
BANK_RELAYS
  Relative segment, address: CODE 00000A58 - 00000A5D (0x6 bytes), align: 0
  Segment part 9.
           ENTRY                   ADDRESS         REF BY
           =====                   =======         ======
           osal_pwrmgr_init::?relay
                                   00000A58        osal_init_system (OSAL)
    -------------------------------------------------------------------------
BANK_RELAYS
  Relative segment, address: CODE 00000A5E - 00000A63 (0x6 bytes), align: 0
  Segment part 11.
           ENTRY                   ADDRESS         REF BY
           =====                   =======         ======
           osal_pwrmgr_device::?relay
                                   00000A5E        LL_ProcessEvent (ll)
    -------------------------------------------------------------------------
BANK_RELAYS
  Relative segment, address: CODE 00000A64 - 00000A69 (0x6 bytes), align: 0
  Segment part 13.
           ENTRY                   ADDRESS         REF BY
           =====                   =======         ======
           osal_pwrmgr_task_state::?relay
                                   00000A64        LL_Init (ll)
                                                   LL_ProcessEvent (ll)
                                                   LL_SetAdvControl (ll)
                                                   llFreeTask (ll_scheduler)

    *************************************************************************

  FILE NAME : C:\ble\BLE-CC254x-1.4.1.43908\Projects\ble\SimpleBLEBroadcaster-usb\CC2540\CC2540USB\Obj\OSAL_SimpleBLEBroadcaster.r51
  PROGRAM MODULE, NAME : OSAL_SimpleBLEBroadcaster

  SEGMENTS IN THE MODULE
  ======================
<XDATA_ROM_C> 1 (was XDATA_ROM_C)
  Relative segment, address: CONST 00008F6C - 00008F7B (0x10 bytes), align: 0
  Segment part 6.
           ENTRY                   ADDRESS         REF BY
           =====                   =======         ======
           tasksArr                00008F6C        osal_run_system (OSAL)
    -------------------------------------------------------------------------
<XDATA_ROM_C> 1 (was XDATA_ROM_C)
  Relative segment, address: CONST 00008F96 - 00008F96 (0x1 bytes), align: 0
  Segment part 7.             Intra module refs:   osalInitTasks
           ENTRY                   ADDRESS         REF BY
           =====                   =======         ======
           tasksCnt                00008F96        osal_clear_event (OSAL)
                                                   osal_msg_enqueue_push (OSAL)
                                                   osal_pwrmgr_task_state (OSAL_PwrMgr)
                                                   osal_run_system (OSAL)
                                                   osal_set_event (OSAL)
    -------------------------------------------------------------------------
XDATA_Z
  Relative segment, address: XDATA 00000FBB - 00000FBC (0x2 bytes), align: 0
  Segment part 8.             Intra module refs:   osalInitTasks
           ENTRY                   ADDRESS         REF BY
           =====                   =======         ======
           tasksEvents             00000FBB        osal_clear_event (OSAL)
                                                   osal_run_system (OSAL)
                                                   osal_set_event (OSAL)
    -------------------------------------------------------------------------
<BANKED_CODE,XDATA_ROM_C_FLASH> 1 (was BANKED_CODE)
  Relative segment, address: CODE 0000C4B6 - 0000C540 (0x8b bytes), align: 0
  Segment part 9.             Intra module refs:   osalInitTasks::?relay
           ENTRY                   ADDRESS         REF BY
           =====                   =======         ======
           osalInitTasks           0000C4B6 
               calls direct
               XSTACK = 00000000 ( 00000009 )
    -------------------------------------------------------------------------
BANK_RELAYS
  Relative segment, address: CODE 00000A6A - 00000A6F (0x6 bytes), align: 0
  Segment part 10.
           ENTRY                   ADDRESS         REF BY
           =====                   =======         ======
           osalInitTasks::?relay   00000A6A        osal_init_system (OSAL)
    -------------------------------------------------------------------------
<BANKED_CODE,XDATA_ROM_C_FLASH> 1 (was XDATA_ROM_C_FLASH)
  Relative segment, address: CODE 00008F6C - 00008F7B (0x10 bytes), align: 0
  Segment part 11.            Intra module refs:   tasksArr
    -------------------------------------------------------------------------
<BANKED_CODE,XDATA_ROM_C_FLASH> 1 (was XDATA_ROM_C_FLASH)
  Relative segment, address: CODE 00008F96 - 00008F96 (0x1 bytes), align: 0
  Segment part 12.            Intra module refs:   tasksCnt

    *************************************************************************

  FILE NAME : C:\ble\BLE-CC254x-1.4.1.43908\Projects\ble\SimpleBLEBroadcaster-usb\CC2540\CC2540USB\Obj\osal_snv.r51
  PROGRAM MODULE, NAME : osal_snv

  SEGMENTS IN THE MODULE
  ======================
BLENV_ADDRESS_SPACE
  Relative segment, address: CODE 0003E800 - 0003F7FF (0x1000 bytes), align: 0
  Segment part 6.             Intra module refs:   activePg
           ENTRY                   ADDRESS         REF BY
           =====                   =======         ======
           _nvBuf                  0003E800 
    -------------------------------------------------------------------------
XDATA_Z
  Relative segment, address: XDATA 00000FBD - 00000FBD (0x1 bytes), align: 0
  Segment part 7.             Intra module refs:   findOffset
                                                   initNV
                                                   osal_snv_read
                                                   osal_snv_write
                                                   setActivePage
                                                   setXferPage
                                                   xferItem
           LOCAL                   ADDRESS         
           =====                   =======         
           activePg                00000FBD 
    -------------------------------------------------------------------------
XDATA_Z
  Relative segment, address: XDATA 00000FBE - 00000FBF (0x2 bytes), align: 0
  Segment part 8.             Intra module refs:   compactPage
                                                   findOffset
                                                   initNV
                                                   osal_snv_read
                                                   osal_snv_write
           LOCAL                   ADDRESS         
           =====                   =======         
           pgOff                   00000FBE 
    -------------------------------------------------------------------------
XDATA_Z
  Relative segment, address: XDATA 00000FC0 - 00000FC0 (0x1 bytes), align: 0
  Segment part 9.             Intra module refs:   compactPage
                                                   erasePage
                                                   initNV
                                                   osal_snv_write
                                                   setActivePage
                                                   verifyWordM
                                                   writeWord
                                                   writeWordM
           LOCAL                   ADDRESS         
           =====                   =======         
           failF                   00000FC0 
    -------------------------------------------------------------------------
<BANKED_CODE,CODE_C> 1 (was BANKED_CODE)
  Relative segment, address: CODE 0000354E - 00003629 (0xdc bytes), align: 0
  Segment part 14.            Intra module refs:   initNV::?relay
           LOCAL                   ADDRESS         
           =====                   =======         
           initNV                  0000354E 
               calls direct
               XSTACK = 00000000 ( 00000012 )
    -------------------------------------------------------------------------
<BANKED_CODE,CODE_C> 1 (was BANKED_CODE)
  Relative segment, address: CODE 0000362A - 00003670 (0x47 bytes), align: 0
  Segment part 16.            Intra module refs:   setActivePage::?relay
           LOCAL                   ADDRESS         
           =====                   =======         
           setActivePage           0000362A 
               calls direct
               XSTACK = 00000014 ( 0000000D )
    -------------------------------------------------------------------------
<BANKED_CODE,CODE_C> 1 (was BANKED_CODE)
  Relative segment, address: CODE 00003671 - 000036AD (0x3d bytes), align: 0
  Segment part 18.            Intra module refs:   setXferPage::?relay
           LOCAL                   ADDRESS         
           =====                   =======         
           setXferPage             00003671 
               calls direct
               XSTACK = 00000014 ( 0000000D )
    -------------------------------------------------------------------------
<BANKED_CODE,CODE_C> 1 (was BANKED_CODE)
  Relative segment, address: CODE 000036AE - 0000371B (0x6e bytes), align: 0
  Segment part 20.            Intra module refs:   erasePage::?relay
           LOCAL                   ADDRESS         
           =====                   =======         
           erasePage               000036AE 
               calls direct
               XSTACK = 00000014 ( 0000000F )
    -------------------------------------------------------------------------
<BANKED_CODE,CODE_C> 1 (was BANKED_CODE)
  Relative segment, address: CODE 0000371C - 00003775 (0x5a bytes), align: 0
  Segment part 22.            Intra module refs:   cleanErasedPage::?relay
           LOCAL                   ADDRESS         
           =====                   =======         
           cleanErasedPage         0000371C 
               calls direct
               XSTACK = 00000010 ( 0000000F )
    -------------------------------------------------------------------------
<BANKED_CODE,CODE_C> 1 (was BANKED_CODE)
  Relative segment, address: CODE 00003776 - 000037E5 (0x70 bytes), align: 0
  Segment part 24.            Intra module refs:   findOffset::?relay
           LOCAL                   ADDRESS         
           =====                   =======         
           findOffset              00003776 
               calls direct
               XSTACK = 00000010 ( 00000012 )
    -------------------------------------------------------------------------
<BANKED_CODE,CODE_C> 1 (was BANKED_CODE)
  Relative segment, address: CODE 000037E6 - 000038B8 (0xd3 bytes), align: 0
  Segment part 26.            Intra module refs:   findItem::?relay
           LOCAL                   ADDRESS         
           =====                   =======         
           findItem                000037E6 
               calls direct
               XSTACK = 00000014 ( 00000012 )
    -------------------------------------------------------------------------
<BANKED_CODE,CODE_C> 1 (was BANKED_CODE)
  Relative segment, address: CODE 000038B9 - 000039A7 (0xef bytes), align: 0
  Segment part 28.            Intra module refs:   writeItem::?relay
           LOCAL                   ADDRESS         
           =====                   =======         
           writeItem               000038B9 
               calls direct
               XSTACK = 00000017 ( 00000015 )
    -------------------------------------------------------------------------
<BANKED_CODE,CODE_C> 1 (was BANKED_CODE)
  Relative segment, address: CODE 000039A8 - 00003A1E (0x77 bytes), align: 0
  Segment part 30.            Intra module refs:   xferItem::?relay
           LOCAL                   ADDRESS         
           =====                   =======         
           xferItem                000039A8 
               calls direct
               XSTACK = 00000016 ( 00000018 )
    -------------------------------------------------------------------------
<BANKED_CODE,CODE_C> 1 (was BANKED_CODE)
  Relative segment, address: CODE 00003A1F - 00003BBD (0x19f bytes), align: 0
  Segment part 32.            Intra module refs:   compactPage::?relay
           LOCAL                   ADDRESS         
           =====                   =======         
           compactPage             00003A1F 
               calls direct
               XSTACK = 00000014 ( 00000016 )
    -------------------------------------------------------------------------
<BANKED_CODE,CODE_C> 1 (was BANKED_CODE)
  Relative segment, address: CODE 00003BBE - 00003C4A (0x8d bytes), align: 0
  Segment part 34.            Intra module refs:   verifyWordM::?relay
           LOCAL                   ADDRESS         
           =====                   =======         
           verifyWordM             00003BBE 
               calls direct
               XSTACK = 00000013 ( 00000016 )
    -------------------------------------------------------------------------
<BANKED_CODE,CODE_C> 1 (was BANKED_CODE)
  Relative segment, address: CODE 00003C4B - 00003CBD (0x73 bytes), align: 0
  Segment part 36.            Intra module refs:   writeWord::?relay
           LOCAL                   ADDRESS         
           =====                   =======         
           writeWord               00003C4B 
               calls direct
               XSTACK = 00000016 ( 00000014 )
    -------------------------------------------------------------------------
<BANKED_CODE,CODE_C> 1 (was BANKED_CODE)
  Relative segment, address: CODE 00003CBE - 00003D39 (0x7c bytes), align: 0
  Segment part 38.            Intra module refs:   writeWordM::?relay
           LOCAL                   ADDRESS         
           =====                   =======         
           writeWordM              00003CBE 
               calls direct
               XSTACK = 00000015 ( 00000014 )
    -------------------------------------------------------------------------
<BANKED_CODE,CODE_C> 1 (was BANKED_CODE)
  Relative segment, address: CODE 00003D3A - 00003D53 (0x1a bytes), align: 0
  Segment part 40.            Intra module refs:   osal_snv_init::?relay
           ENTRY                   ADDRESS         REF BY
           =====                   =======         ======
           osal_snv_init           00003D3A 
               calls direct
               ISTACK = 00000000 ( 00000002 )
    -------------------------------------------------------------------------
<BANKED_CODE,CODE_C> 1 (was BANKED_CODE)
  Relative segment, address: CODE 00003D54 - 00003E78 (0x125 bytes), align: 0
  Segment part 42.            Intra module refs:   osal_snv_write::?relay
           ENTRY                   ADDRESS         REF BY
           =====                   =======         ======
           osal_snv_write          00003D54 
               calls direct
               XSTACK = 00000000 ( 00000017 )
    -------------------------------------------------------------------------
<BANKED_CODE,CODE_C> 1 (was BANKED_CODE)
  Relative segment, address: CODE 00003E79 - 00003ED2 (0x5a bytes), align: 0
  Segment part 44.            Intra module refs:   osal_snv_read::?relay
           ENTRY                   ADDRESS         REF BY
           =====                   =======         ======
           osal_snv_read           00003E79 
               calls direct
               XSTACK = 00000000 ( 00000010 )
    -------------------------------------------------------------------------
<XDATA_ROM_C> 1 (was XDATA_ROM_C)
  Relative segment, address: CONST 00008FD4 - 00008FD7 (0x4 bytes), align: 0
  Segment part 10.            Intra module refs:   initNV
           ENTRY                   ADDRESS         REF BY
           =====                   =======         ======
           __Constant_100000       00008FD4 
    -------------------------------------------------------------------------
<XDATA_ROM_C> 1 (was XDATA_ROM_C)
  Relative segment, address: CONST 00008FD8 - 00008FDB (0x4 bytes), align: 0
  Segment part 11.            Intra module refs:   findOffset
                                                   llSetT2OVFC2Event2 (ll_timer2)
           ENTRY                   ADDRESS         REF BY
           =====                   =======         ======
           __Constant_ffffffff     00008FD8 
    -------------------------------------------------------------------------
<XDATA_ROM_C> 1 (was XDATA_ROM_C)
  Relative segment, address: CONST 00008FDC - 00008FDF (0x4 bytes), align: 0
  Segment part 13.            Intra module refs:   llScheduler (ll_scheduler)
           ENTRY                   ADDRESS         REF BY
           =====                   =======         ======
           __Constant_800          00008FDC 
    -------------------------------------------------------------------------
BANK_RELAYS
  Relative segment, address: CODE 00000A70 - 00000A75 (0x6 bytes), align: 0
  Segment part 15.            Intra module refs:   osal_snv_init
           LOCAL                   ADDRESS         
           =====                   =======         
           initNV::?relay          00000A70 
    -------------------------------------------------------------------------
BANK_RELAYS
  Relative segment, address: CODE 00000A76 - 00000A7B (0x6 bytes), align: 0
  Segment part 17.            Intra module refs:   compactPage
                                                   initNV
           LOCAL                   ADDRESS         
           =====                   =======         
           setActivePage::?relay   00000A76 
    -------------------------------------------------------------------------
BANK_RELAYS
  Relative segment, address: CODE 00000A7C - 00000A81 (0x6 bytes), align: 0
  Segment part 19.            Intra module refs:   osal_snv_write
           LOCAL                   ADDRESS         
           =====                   =======         
           setXferPage::?relay     00000A7C 
    -------------------------------------------------------------------------
BANK_RELAYS
  Relative segment, address: CODE 00000A82 - 00000A87 (0x6 bytes), align: 0
  Segment part 21.            Intra module refs:   cleanErasedPage
                                                   compactPage
                                                   initNV
           LOCAL                   ADDRESS         
           =====                   =======         
           erasePage::?relay       00000A82 
    -------------------------------------------------------------------------
BANK_RELAYS
  Relative segment, address: CODE 00000A88 - 00000A8D (0x6 bytes), align: 0
  Segment part 23.            Intra module refs:   initNV
           LOCAL                   ADDRESS         
           =====                   =======         
           cleanErasedPage::?relay
                                   00000A88 
    -------------------------------------------------------------------------
BANK_RELAYS
  Relative segment, address: CODE 00000A8E - 00000A93 (0x6 bytes), align: 0
  Segment part 25.            Intra module refs:   initNV
           LOCAL                   ADDRESS         
           =====                   =======         
           findOffset::?relay      00000A8E 
    -------------------------------------------------------------------------
BANK_RELAYS
  Relative segment, address: CODE 00000A94 - 00000A99 (0x6 bytes), align: 0
  Segment part 27.            Intra module refs:   compactPage
                                                   osal_snv_read
                                                   osal_snv_write
           LOCAL                   ADDRESS         
           =====                   =======         
           findItem::?relay        00000A94 
    -------------------------------------------------------------------------
BANK_RELAYS
  Relative segment, address: CODE 00000A9A - 00000A9F (0x6 bytes), align: 0
  Segment part 29.            Intra module refs:   osal_snv_write
           LOCAL                   ADDRESS         
           =====                   =======         
           writeItem::?relay       00000A9A 
    -------------------------------------------------------------------------
BANK_RELAYS
  Relative segment, address: CODE 00000AA0 - 00000AA5 (0x6 bytes), align: 0
  Segment part 31.            Intra module refs:   compactPage
           LOCAL                   ADDRESS         
           =====                   =======         
           xferItem::?relay        00000AA0 
    -------------------------------------------------------------------------
BANK_RELAYS
  Relative segment, address: CODE 00000AA6 - 00000AAB (0x6 bytes), align: 0
  Segment part 33.            Intra module refs:   initNV
                                                   osal_snv_write
           LOCAL                   ADDRESS         
           =====                   =======         
           compactPage::?relay     00000AA6 
    -------------------------------------------------------------------------
BANK_RELAYS
  Relative segment, address: CODE 00000AAC - 00000AB1 (0x6 bytes), align: 0
  Segment part 35.            Intra module refs:   writeWord
                                                   writeWordM
           LOCAL                   ADDRESS         
           =====                   =======         
           verifyWordM::?relay     00000AAC 
    -------------------------------------------------------------------------
BANK_RELAYS
  Relative segment, address: CODE 00000AB2 - 00000AB7 (0x6 bytes), align: 0
  Segment part 37.            Intra module refs:   setActivePage
                                                   setXferPage
                                                   writeItem
                                                   xferItem
           LOCAL                   ADDRESS         
           =====                   =======         
           writeWord::?relay       00000AB2 
    -------------------------------------------------------------------------
BANK_RELAYS
  Relative segment, address: CODE 00000AB8 - 00000ABD (0x6 bytes), align: 0
  Segment part 39.            Intra module refs:   writeItem
           LOCAL                   ADDRESS         
           =====                   =======         
           writeWordM::?relay      00000AB8 
    -------------------------------------------------------------------------
BANK_RELAYS
  Relative segment, address: CODE 00000ABE - 00000AC3 (0x6 bytes), align: 0
  Segment part 41.
           ENTRY                   ADDRESS         REF BY
           =====                   =======         ======
           osal_snv_init::?relay   00000ABE        SimpleBLEBroadcaster_Init (simpleBLEBroadcaster)
                                                   main (SimpleBLEBroadcaster_Main)
    -------------------------------------------------------------------------
BANK_RELAYS
  Relative segment, address: CODE 00000AC4 - 00000AC9 (0x6 bytes), align: 0
  Segment part 43.
           ENTRY                   ADDRESS         REF BY
           =====                   =======         ======
           osal_snv_write::?relay
                                   00000AC4        Application_UpdateAdv (simpleBLEBroadcaster)
                                                   Application_UpdateRsp (simpleBLEBroadcaster)
    -------------------------------------------------------------------------
BANK_RELAYS
  Relative segment, address: CODE 00000ACA - 00000ACF (0x6 bytes), align: 0
  Segment part 45.
           ENTRY                   ADDRESS         REF BY
           =====                   =======         ======
           osal_snv_read::?relay   00000ACA        SimpleBLEBroadcaster_Init (simpleBLEBroadcaster)
    -------------------------------------------------------------------------
<BANKED_CODE,XDATA_ROM_C_FLASH> 1 (was XDATA_ROM_C_FLASH)
  Relative segment, address: CODE 00008FD4 - 00008FD7 (0x4 bytes), align: 0
  Segment part 48.            Intra module refs:   __Constant_100000
    -------------------------------------------------------------------------
<BANKED_CODE,XDATA_ROM_C_FLASH> 1 (was XDATA_ROM_C_FLASH)
  Relative segment, address: CODE 00008FD8 - 00008FDB (0x4 bytes), align: 0
  Segment part 49.            Intra module refs:   __Constant_ffffffff
    -------------------------------------------------------------------------
<BANKED_CODE,XDATA_ROM_C_FLASH> 1 (was XDATA_ROM_C_FLASH)
  Relative segment, address: CODE 00008FDC - 00008FDF (0x4 bytes), align: 0
  Segment part 51.            Intra module refs:   __Constant_800

    *************************************************************************

  FILE NAME : C:\ble\BLE-CC254x-1.4.1.43908\Projects\ble\SimpleBLEBroadcaster-usb\CC2540\CC2540USB\Obj\OSAL_Timers.r51
  PROGRAM MODULE, NAME : OSAL_Timers

  SEGMENTS IN THE MODULE
  ======================
XDATA_Z
  Relative segment, address: XDATA 00000FC1 - 00000FC2 (0x2 bytes), align: 0
  Segment part 7.             Intra module refs:   osalAddTimer
                                                   osalFindTimer
                                                   osalTimerUpdate
           ENTRY                   ADDRESS         REF BY
           =====                   =======         ======
           timerHead               00000FC1 
    -------------------------------------------------------------------------
XDATA_Z
  Relative segment, address: XDATA 00000FC3 - 00000FC6 (0x4 bytes), align: 0
  Segment part 8.             Intra module refs:   osalTimerInit
                                                   osalTimerUpdate
                                                   osal_GetSystemClock
           LOCAL                   ADDRESS         
           =====                   =======         
           osal_systemClock        00000FC3 
    -------------------------------------------------------------------------
<BANKED_CODE,CODE_C> 1 (was BANKED_CODE)
  Relative segment, address: CODE 00006C48 - 00006C67 (0x20 bytes), align: 0
  Segment part 9.             Intra module refs:   osalTimerInit::?relay
           ENTRY                   ADDRESS         REF BY
           =====                   =======         ======
           osalTimerInit           00006C48 
               XSTACK = 00000000 ( 00000009 )
    -------------------------------------------------------------------------
<BANKED_CODE,CODE_C> 1 (was BANKED_CODE)
  Relative segment, address: CODE 00006C68 - 00006D6D (0x106 bytes), align: 0
  Segment part 11.            Intra module refs:   osalAddTimer::?relay
           ENTRY                   ADDRESS         REF BY
           =====                   =======         ======
           osalAddTimer            00006C68 
               calls direct
               XSTACK = 00000016 ( 00000014 )
               ISTACK = 00000000 ( 00000001 )
    -------------------------------------------------------------------------
<BANKED_CODE,CODE_C> 1 (was BANKED_CODE)
  Relative segment, address: CODE 00006D6E - 00006DB9 (0x4c bytes), align: 0
  Segment part 13.            Intra module refs:   osalFindTimer::?relay
           ENTRY                   ADDRESS         REF BY
           =====                   =======         ======
           osalFindTimer           00006D6E 
               XSTACK = 00000014 ( 00000009 )
    -------------------------------------------------------------------------
<BANKED_CODE,CODE_C> 1 (was BANKED_CODE)
  Relative segment, address: CODE 00006DBA - 00006DD9 (0x20 bytes), align: 0
  Segment part 15.            Intra module refs:   osalDeleteTimer::?relay
           ENTRY                   ADDRESS         REF BY
           =====                   =======         ======
           osalDeleteTimer         00006DBA 
               XSTACK = 0000000E ( 00000000 )
               ISTACK = 00000000 ( 00000002 )
    -------------------------------------------------------------------------
<BANKED_CODE,CODE_C> 1 (was BANKED_CODE)
  Relative segment, address: CODE 00006DDA - 00006E2C (0x53 bytes), align: 0
  Segment part 17.            Intra module refs:   osal_start_timerEx::?relay
           ENTRY                   ADDRESS         REF BY
           =====                   =======         ======
           osal_start_timerEx      00006DDA 
               calls direct, is indirectly called
               XSTACK = 00000004 ( 00000016 )
    -------------------------------------------------------------------------
<BANKED_CODE,CODE_C> 1 (was BANKED_CODE)
  Relative segment, address: CODE 00006E2D - 00006E99 (0x6d bytes), align: 0
  Segment part 19.            Intra module refs:   osal_start_reload_timer::?relay
           ENTRY                   ADDRESS         REF BY
           =====                   =======         ======
           osal_start_reload_timer
                                   00006E2D 
               calls direct
               XSTACK = 00000004 ( 00000016 )
    -------------------------------------------------------------------------
<BANKED_CODE,CODE_C> 1 (was BANKED_CODE)
  Relative segment, address: CODE 00006E9A - 00006EDF (0x46 bytes), align: 0
  Segment part 21.            Intra module refs:   osal_stop_timerEx::?relay
           ENTRY                   ADDRESS         REF BY
           =====                   =======         ======
           osal_stop_timerEx       00006E9A 
               calls direct
               XSTACK = 00000000 ( 0000000E )
    -------------------------------------------------------------------------
<BANKED_CODE,CODE_C> 1 (was BANKED_CODE)
  Relative segment, address: CODE 00006EE0 - 00006F43 (0x64 bytes), align: 0
  Segment part 23.            Intra module refs:   osal_get_timeoutEx::?relay
           ENTRY                   ADDRESS         REF BY
           =====                   =======         ======
           osal_get_timeoutEx      00006EE0 
               calls direct
               XSTACK = 00000000 ( 00000014 )
    -------------------------------------------------------------------------
<BANKED_CODE,CODE_C> 1 (was BANKED_CODE)
  Relative segment, address: CODE 00006F44 - 000071EF (0x2ac bytes), align: 0
  Segment part 27.            Intra module refs:   osalTimerUpdate::?relay
           ENTRY                   ADDRESS         REF BY
           =====                   =======         ======
           osalTimerUpdate         00006F44 
               calls direct
               XSTACK = 00000000 ( 0000001A )
    -------------------------------------------------------------------------
<BANKED_CODE,CODE_C> 1 (was BANKED_CODE)
  Relative segment, address: CODE 000071F0 - 00007200 (0x11 bytes), align: 0
  Segment part 29.            Intra module refs:   osal_GetSystemClock::?relay
           ENTRY                   ADDRESS         REF BY
           =====                   =======         ======
           osal_GetSystemClock     000071F0 
               ISTACK = 00000000 ( 00000002 )
    -------------------------------------------------------------------------
BANK_RELAYS
  Relative segment, address: CODE 00000AD0 - 00000AD5 (0x6 bytes), align: 0
  Segment part 10.
           ENTRY                   ADDRESS         REF BY
           =====                   =======         ======
           osalTimerInit::?relay   00000AD0        osal_init_system (OSAL)
    -------------------------------------------------------------------------
BANK_RELAYS
  Relative segment, address: CODE 00000AD6 - 00000ADB (0x6 bytes), align: 0
  Segment part 12.            Intra module refs:   osal_start_reload_timer
                                                   osal_start_timerEx
           ENTRY                   ADDRESS         REF BY
           =====                   =======         ======
           osalAddTimer::?relay    00000AD6 
    -------------------------------------------------------------------------
BANK_RELAYS
  Relative segment, address: CODE 00000ADC - 00000AE1 (0x6 bytes), align: 0
  Segment part 14.            Intra module refs:   osalAddTimer
                                                   osal_get_timeoutEx
                                                   osal_stop_timerEx
           ENTRY                   ADDRESS         REF BY
           =====                   =======         ======
           osalFindTimer::?relay   00000ADC 
    -------------------------------------------------------------------------
BANK_RELAYS
  Relative segment, address: CODE 00000AE2 - 00000AE7 (0x6 bytes), align: 0
  Segment part 16.            Intra module refs:   osal_stop_timerEx
           ENTRY                   ADDRESS         REF BY
           =====                   =======         ======
           osalDeleteTimer::?relay
                                   00000AE2 
    -------------------------------------------------------------------------
BANK_RELAYS
  Relative segment, address: CODE 00000AE8 - 00000AED (0x6 bytes), align: 0
  Segment part 18.
           ENTRY                   ADDRESS         REF BY
           =====                   =======         ======
           osal_start_timerEx::?relay
                                   00000AE8        HalLedUpdate (hal_led)
                                                   LL_EXT_ResetSystem (ll)
                                                   LL_ProcessEvent (ll)
                                                   gapProcessAdvertisingEvt (gap_peridevmgr)
                                                   gapRole_ProcessGAPMsg (broadcaster)
                                                   gapWriteAdvEnableStatus (gap_peridevmgr)
                                                   llScheduleTask (ll_scheduler)
    -------------------------------------------------------------------------
BANK_RELAYS
  Relative segment, address: CODE 00000AEE - 00000AF3 (0x6 bytes), align: 0
  Segment part 20.
           ENTRY                   ADDRESS         REF BY
           =====                   =======         ======
           osal_start_reload_timer::?relay
                                   00000AEE        GAP_MakeDiscoverable (gap_peridevmgr)
                                                   gapProcessRandomAddrComplete (gap_configmgr)
                                                   gapWriteAdvEnableStatus (gap_peridevmgr)
    -------------------------------------------------------------------------
BANK_RELAYS
  Relative segment, address: CODE 00000AF4 - 00000AF9 (0x6 bytes), align: 0
  Segment part 22.
           ENTRY                   ADDRESS         REF BY
           =====                   =======         ======
           osal_stop_timerEx::?relay
                                   00000AF4        GAP_EndDiscoverable (gap_peridevmgr)
                                                   HalLedBlink (hal_led)
                                                   LL_SetAdvControl (ll)
                                                   gapProcessAdvertisingEvt (gap_peridevmgr)
                                                   llT2OVFC1_ISR (ll_isr)
    -------------------------------------------------------------------------
BANK_RELAYS
  Relative segment, address: CODE 00000AFA - 00000AFF (0x6 bytes), align: 0
  Segment part 24.
           ENTRY                   ADDRESS         REF BY
           =====                   =======         ======
           osal_get_timeoutEx::?relay
                                   00000AFA        gapRole_ProcessGAPMsg (broadcaster)
                                                   osal_CbTimerProcessEvent (osal_cbtimer)
    -------------------------------------------------------------------------
BANK_RELAYS
  Relative segment, address: CODE 00000B00 - 00000B05 (0x6 bytes), align: 0
  Segment part 28.
           ENTRY                   ADDRESS         REF BY
           =====                   =======         ======
           osalTimerUpdate::?relay
                                   00000B00        osalTimeUpdate (OSAL_ClockBLE)
    -------------------------------------------------------------------------
BANK_RELAYS
  Relative segment, address: CODE 00000B06 - 00000B0B (0x6 bytes), align: 0
  Segment part 30.
           ENTRY                   ADDRESS         REF BY
           =====                   =======         ======
           osal_GetSystemClock::?relay
                                   00000B06        HalLedBlink (hal_led)
                                                   HalLedUpdate (hal_led)

    *************************************************************************

  FILE NAME : C:\ble\BLE-CC254x-1.4.1.43908\Projects\ble\SimpleBLEBroadcaster-usb\CC2540\CC2540USB\Obj\serialInterface.r51
  PROGRAM MODULE, NAME : serialInterface

  SEGMENTS IN THE MODULE
  ======================
XDATA_Z
  Relative segment, address: XDATA 00000FC7 - 00000FC7 (0x1 bytes), align: 0
  Segment part 6.             Intra module refs:   SerialInterface_Init
                                                   SerialInterface_ProcessEvent
                                                   cSerialPacketParser
                                                   parseCmd
           ENTRY                   ADDRESS         REF BY
           =====                   =======         ======
           serialInterface_TaskID
                                   00000FC7 
    -------------------------------------------------------------------------
XDATA_Z
  Relative segment, address: XDATA 00000FC8 - 00000FE8 (0x21 bytes), align: 0
  Segment part 7.             Intra module refs:   cSerialPacketParser
                                                   parseCmd
           LOCAL                   ADDRESS         
           =====                   =======         
           rxSerialPkt             00000FC8 
    -------------------------------------------------------------------------
XDATA_Z
  Relative segment, address: XDATA 00000FE9 - 00000FED (0x5 bytes), align: 0
  Segment part 8.             Intra module refs:   parseCmd
                                                   sendSerialEvt
           LOCAL                   ADDRESS         
           =====                   =======         
           txSerialPkt             00000FE9 
    -------------------------------------------------------------------------
XDATA_Z
  Relative segment, address: XDATA 00000FEE - 00000FEE (0x1 bytes), align: 0
  Segment part 9.             Intra module refs:   cSerialPacketParser
                                                   parseCmd
           LOCAL                   ADDRESS         
           =====                   =======         
           cmd_len                 00000FEE 
    -------------------------------------------------------------------------
<BANKED_CODE,XDATA_ROM_C_FLASH> 1 (was BANKED_CODE)
  Relative segment, address: CODE 00009C15 - 00009C2C (0x18 bytes), align: 0
  Segment part 13.            Intra module refs:   SerialInterface_Init::?relay
           ENTRY                   ADDRESS         REF BY
           =====                   =======         ======
           SerialInterface_Init    00009C15 
               calls direct
               XSTACK = 00000000 ( 00000009 )
    -------------------------------------------------------------------------
<BANKED_CODE,XDATA_ROM_C_FLASH> 1 (was BANKED_CODE)
  Relative segment, address: CODE 00009C2D - 00009CD6 (0xaa bytes), align: 0
  Segment part 15.            Intra module refs:   SerialInterface_ProcessEvent::?relay
           ENTRY                   ADDRESS         REF BY
           =====                   =======         ======
           SerialInterface_ProcessEvent
                                   00009C2D 
               calls direct
               XSTACK = 00000000 ( 0000000E )
    -------------------------------------------------------------------------
<BANKED_CODE,XDATA_ROM_C_FLASH> 1 (was BANKED_CODE)
  Relative segment, address: CODE 00009CD7 - 00009CD9 (0x3 bytes), align: 0
  Segment part 17.            Intra module refs:   SerialInterface_ProcessOSALMsg::?relay
           LOCAL                   ADDRESS         
           =====                   =======         
           SerialInterface_ProcessOSALMsg
                                   00009CD7 
               XSTACK = 0000000E ( 00000000 )
    -------------------------------------------------------------------------
<BANKED_CODE,XDATA_ROM_C_FLASH> 1 (was BANKED_CODE)
  Relative segment, address: CODE 00009CDA - 00009E18 (0x13f bytes), align: 0
  Segment part 19.            Intra module refs:   cSerialPacketParser::?relay
           ENTRY                   ADDRESS         REF BY
           =====                   =======         ======
           cSerialPacketParser     00009CDA 
               calls direct, is indirectly called
               XSTACK = 00000000 ( 00000010 )
    -------------------------------------------------------------------------
XDATA_Z
  Relative segment, address: XDATA 00000FEF - 00000FEF (0x1 bytes), align: 0
  Segment part 10.            Intra module refs:   cSerialPacketParser
           LOCAL                   ADDRESS         
           =====                   =======         
           cSerialPacketParser::pktState
                                   00000FEF 
    -------------------------------------------------------------------------
XDATA_Z
  Relative segment, address: XDATA 00000FF0 - 00000FF0 (0x1 bytes), align: 0
  Segment part 11.            Intra module refs:   cSerialPacketParser
           LOCAL                   ADDRESS         
           =====                   =======         
           cSerialPacketParser::cmd_identifier
                                   00000FF0 
    -------------------------------------------------------------------------
XDATA_Z
  Relative segment, address: XDATA 00000FF1 - 00000FF1 (0x1 bytes), align: 0
  Segment part 12.            Intra module refs:   cSerialPacketParser
           LOCAL                   ADDRESS         
           =====                   =======         
           cSerialPacketParser::cmd_opcode
                                   00000FF1 
    -------------------------------------------------------------------------
<BANKED_CODE,XDATA_ROM_C_FLASH> 1 (was BANKED_CODE)
  Relative segment, address: CODE 00009E19 - 00009F31 (0x119 bytes), align: 0
  Segment part 21.            Intra module refs:   parseCmd::?relay
           ENTRY                   ADDRESS         REF BY
           =====                   =======         ======
           parseCmd                00009E19 
               calls direct
               XSTACK = 0000000E ( 00000009 )
    -------------------------------------------------------------------------
<BANKED_CODE,XDATA_ROM_C_FLASH> 1 (was BANKED_CODE)
  Relative segment, address: CODE 00009F32 - 00009F57 (0x26 bytes), align: 0
  Segment part 23.            Intra module refs:   sendSerialEvt::?relay
           ENTRY                   ADDRESS         REF BY
           =====                   =======         ======
           sendSerialEvt           00009F32 
               calls direct
               XSTACK = 0000000E ( 00000009 )
    -------------------------------------------------------------------------
<BANKED_CODE,XDATA_ROM_C_FLASH> 1 (was BANKED_CODE)
  Relative segment, address: CODE 00009F58 - 00009F89 (0x32 bytes), align: 0
  Segment part 25.            Intra module refs:   SerialDebug_process::?relay
           LOCAL                   ADDRESS         
           =====                   =======         
           SerialDebug_process     00009F58 
               calls direct
               XSTACK = 0000000E ( 00000009 )
    -------------------------------------------------------------------------
BANK_RELAYS
  Relative segment, address: CODE 00000B0C - 00000B11 (0x6 bytes), align: 0
  Segment part 14.
           ENTRY                   ADDRESS         REF BY
           =====                   =======         ======
           SerialInterface_Init::?relay
                                   00000B0C        osalInitTasks (OSAL_SimpleBLEBroadcaster)
    -------------------------------------------------------------------------
BANK_RELAYS
  Relative segment, address: CODE 00000B12 - 00000B17 (0x6 bytes), align: 0
  Segment part 16.
           ENTRY                   ADDRESS         REF BY
           =====                   =======         ======
           SerialInterface_ProcessEvent::?relay
                                   00000B12        tasksArr (OSAL_SimpleBLEBroadcaster)
    -------------------------------------------------------------------------
BANK_RELAYS
  Relative segment, address: CODE 00000B18 - 00000B1D (0x6 bytes), align: 0
  Segment part 18.            Intra module refs:   SerialInterface_ProcessEvent
           LOCAL                   ADDRESS         
           =====                   =======         
           SerialInterface_ProcessOSALMsg::?relay
                                   00000B18 
    -------------------------------------------------------------------------
BANK_RELAYS
  Relative segment, address: CODE 00000B1E - 00000B23 (0x6 bytes), align: 0
  Segment part 20.            Intra module refs:   SerialInterface_Init
           ENTRY                   ADDRESS         REF BY
           =====                   =======         ======
           cSerialPacketParser::?relay
                                   00000B1E 
    -------------------------------------------------------------------------
BANK_RELAYS
  Relative segment, address: CODE 00000B24 - 00000B29 (0x6 bytes), align: 0
  Segment part 22.            Intra module refs:   SerialInterface_ProcessEvent
           ENTRY                   ADDRESS         REF BY
           =====                   =======         ======
           parseCmd::?relay        00000B24 
    -------------------------------------------------------------------------
BANK_RELAYS
  Relative segment, address: CODE 00000B2A - 00000B2F (0x6 bytes), align: 0
  Segment part 24.            Intra module refs:   SerialInterface_ProcessEvent
           ENTRY                   ADDRESS         REF BY
           =====                   =======         ======
           sendSerialEvt::?relay   00000B2A 
    -------------------------------------------------------------------------
BANK_RELAYS
  Relative segment, address: CODE 00000B30 - 00000B35 (0x6 bytes), align: 0
  Segment part 26.            Intra module refs:   SerialInterface_ProcessEvent
           LOCAL                   ADDRESS         
           =====                   =======         
           SerialDebug_process::?relay
                                   00000B30 

    *************************************************************************

  FILE NAME : C:\ble\BLE-CC254x-1.4.1.43908\Projects\ble\SimpleBLEBroadcaster-usb\CC2540\CC2540USB\Obj\simpleBLEBroadcaster.r51
  PROGRAM MODULE, NAME : simpleBLEBroadcaster

  SEGMENTS IN THE MODULE
  ======================
XDATA_Z
  Relative segment, address: XDATA 00000FF2 - 00000FF2 (0x1 bytes), align: 0
  Segment part 6.             Intra module refs:   SimpleBLEBroadcaster_Init
                                                   SimpleBLEBroadcaster_ProcessEvent
           LOCAL                   ADDRESS         
           =====                   =======         
           simpleBLEBroadcaster_TaskID
                                   00000FF2 
    -------------------------------------------------------------------------
XDATA_Z
  Relative segment, address: XDATA 00000FF3 - 00001010 (0x1e bytes), align: 0
  Segment part 7.             Intra module refs:   Application_UpdateRsp
                                                   SimpleBLEBroadcaster_Init
           LOCAL                   ADDRESS         
           =====                   =======         
           scanRspData             00000FF3 
    -------------------------------------------------------------------------
XDATA_I
  Relative segment, address: XDATA 000010F3 - 0000110B (0x19 bytes), align: 0
  Segment part 8.             Intra module refs:   SimpleBLEBroadcaster_Init
           LOCAL                   ADDRESS         
           =====                   =======         
           def_scanRspData         000010F3 
    -------------------------------------------------------------------------
XDATA_Z
  Relative segment, address: XDATA 00001011 - 0000102E (0x1e bytes), align: 0
  Segment part 10.            Intra module refs:   Application_UpdateAdv
                                                   SimpleBLEBroadcaster_Init
           LOCAL                   ADDRESS         
           =====                   =======         
           advertData              00001011 
    -------------------------------------------------------------------------
XDATA_I
  Relative segment, address: XDATA 0000110C - 00001113 (0x8 bytes), align: 0
  Segment part 11.            Intra module refs:   SimpleBLEBroadcaster_Init
           LOCAL                   ADDRESS         
           =====                   =======         
           def_advertData          0000110C 
    -------------------------------------------------------------------------
XDATA_I
  Relative segment, address: XDATA 00001114 - 00001117 (0x4 bytes), align: 0
  Segment part 14.            Intra module refs:   SimpleBLEBroadcaster_ProcessEvent
           LOCAL                   ADDRESS         
           =====                   =======         
           simpleBLEBroadcaster_BroadcasterCBs
                                   00001114 
    -------------------------------------------------------------------------
<BANKED_CODE,XDATA_ROM_C_FLASH> 1 (was BANKED_CODE)
  Relative segment, address: CODE 00009F8A - 0000A0B3 (0x12a bytes), align: 0
  Segment part 16.            Intra module refs:   SimpleBLEBroadcaster_Init::?relay
           ENTRY                   ADDRESS         REF BY
           =====                   =======         ======
           SimpleBLEBroadcaster_Init
                                   00009F8A 
               calls direct
               XSTACK = 00000000 ( 00000012 )
    -------------------------------------------------------------------------
<BANKED_CODE,XDATA_ROM_C_FLASH> 1 (was BANKED_CODE)
  Relative segment, address: CODE 0000A0B4 - 0000A123 (0x70 bytes), align: 0
  Segment part 18.            Intra module refs:   SimpleBLEBroadcaster_ProcessEvent::?relay
           ENTRY                   ADDRESS         REF BY
           =====                   =======         ======
           SimpleBLEBroadcaster_ProcessEvent
                                   0000A0B4 
               calls direct
               XSTACK = 00000000 ( 0000000E )
    -------------------------------------------------------------------------
<BANKED_CODE,XDATA_ROM_C_FLASH> 1 (was BANKED_CODE)
  Relative segment, address: CODE 0000A124 - 0000A126 (0x3 bytes), align: 0
  Segment part 20.            Intra module refs:   simpleBLEBroadcaster_ProcessOSALMsg::?relay
           LOCAL                   ADDRESS         
           =====                   =======         
           simpleBLEBroadcaster_ProcessOSALMsg
                                   0000A124 
               XSTACK = 0000000E ( 00000000 )
    -------------------------------------------------------------------------
<BANKED_CODE,XDATA_ROM_C_FLASH> 1 (was BANKED_CODE)
  Relative segment, address: CODE 0000A127 - 0000A161 (0x3b bytes), align: 0
  Segment part 22.            Intra module refs:   peripheralStateNotificationCB::?relay
           LOCAL                   ADDRESS         
           =====                   =======         
           peripheralStateNotificationCB
                                   0000A127 
               calls direct, is indirectly called
               XSTACK = 00000000 ( 0000000F )
    -------------------------------------------------------------------------
<BANKED_CODE,XDATA_ROM_C_FLASH> 1 (was BANKED_CODE)
  Relative segment, address: CODE 0000A162 - 0000A1A8 (0x47 bytes), align: 0
  Segment part 24.            Intra module refs:   Application_StartAdvertise::?relay
           ENTRY                   ADDRESS         REF BY
           =====                   =======         ======
           Application_StartAdvertise
                                   0000A162 
               calls direct
               XSTACK = 00000000 ( 00000001 )
               ISTACK = 00000000 ( 00000002 )
    -------------------------------------------------------------------------
<BANKED_CODE,XDATA_ROM_C_FLASH> 1 (was BANKED_CODE)
  Relative segment, address: CODE 0000A1A9 - 0000A1F1 (0x49 bytes), align: 0
  Segment part 26.            Intra module refs:   Application_StopAdvertise::?relay
           ENTRY                   ADDRESS         REF BY
           =====                   =======         ======
           Application_StopAdvertise
                                   0000A1A9 
               calls direct
               XSTACK = 00000000 ( 00000001 )
               ISTACK = 00000000 ( 00000002 )
    -------------------------------------------------------------------------
<BANKED_CODE,XDATA_ROM_C_FLASH> 1 (was BANKED_CODE)
  Relative segment, address: CODE 0000A1F2 - 0000A236 (0x45 bytes), align: 0
  Segment part 28.            Intra module refs:   Application_UpdateAdv::?relay
           ENTRY                   ADDRESS         REF BY
           =====                   =======         ======
           Application_UpdateAdv   0000A1F2 
               calls direct
               XSTACK = 00000000 ( 0000000E )
    -------------------------------------------------------------------------
<BANKED_CODE,XDATA_ROM_C_FLASH> 1 (was BANKED_CODE)
  Relative segment, address: CODE 0000A237 - 0000A2A2 (0x6c bytes), align: 0
  Segment part 30.            Intra module refs:   Application_UpdateRsp::?relay
           ENTRY                   ADDRESS         REF BY
           =====                   =======         ======
           Application_UpdateRsp   0000A237 
               calls direct
               XSTACK = 00000000 ( 0000000E )
    -------------------------------------------------------------------------
XDATA_ID
  Relative segment, address: CODE 000001CF - 000001E7 (0x19 bytes), align: 0
  Segment part 9.             Intra module refs:   def_scanRspData
    -------------------------------------------------------------------------
XDATA_ID
  Relative segment, address: CODE 000001E8 - 000001EF (0x8 bytes), align: 0
  Segment part 12.            Intra module refs:   def_advertData
    -------------------------------------------------------------------------
XDATA_ID
  Relative segment, address: CODE 000001F0 - 000001F3 (0x4 bytes), align: 0
  Segment part 15.            Intra module refs:   simpleBLEBroadcaster_BroadcasterCBs
    -------------------------------------------------------------------------
BANK_RELAYS
  Relative segment, address: CODE 00000B36 - 00000B3B (0x6 bytes), align: 0
  Segment part 17.
           ENTRY                   ADDRESS         REF BY
           =====                   =======         ======
           SimpleBLEBroadcaster_Init::?relay
                                   00000B36        osalInitTasks (OSAL_SimpleBLEBroadcaster)
    -------------------------------------------------------------------------
BANK_RELAYS
  Relative segment, address: CODE 00000B3C - 00000B41 (0x6 bytes), align: 0
  Segment part 19.
           ENTRY                   ADDRESS         REF BY
           =====                   =======         ======
           SimpleBLEBroadcaster_ProcessEvent::?relay
                                   00000B3C        tasksArr (OSAL_SimpleBLEBroadcaster)
    -------------------------------------------------------------------------
BANK_RELAYS
  Relative segment, address: CODE 00000B42 - 00000B47 (0x6 bytes), align: 0
  Segment part 21.            Intra module refs:   SimpleBLEBroadcaster_ProcessEvent
           LOCAL                   ADDRESS         
           =====                   =======         
           simpleBLEBroadcaster_ProcessOSALMsg::?relay
                                   00000B42 
    -------------------------------------------------------------------------
BANK_RELAYS
  Relative segment, address: CODE 00000B48 - 00000B4D (0x6 bytes), align: 0
  Segment part 23.            Intra module refs:   Segment part 15
           LOCAL                   ADDRESS         
           =====                   =======         
           peripheralStateNotificationCB::?relay
                                   00000B48 
    -------------------------------------------------------------------------
BANK_RELAYS
  Relative segment, address: CODE 00000B4E - 00000B53 (0x6 bytes), align: 0
  Segment part 25.
           ENTRY                   ADDRESS         REF BY
           =====                   =======         ======
           Application_StartAdvertise::?relay
                                   00000B4E        parseCmd (serialInterface)
    -------------------------------------------------------------------------
BANK_RELAYS
  Relative segment, address: CODE 00000B54 - 00000B59 (0x6 bytes), align: 0
  Segment part 27.
           ENTRY                   ADDRESS         REF BY
           =====                   =======         ======
           Application_StopAdvertise::?relay
                                   00000B54        parseCmd (serialInterface)
    -------------------------------------------------------------------------
BANK_RELAYS
  Relative segment, address: CODE 00000B5A - 00000B5F (0x6 bytes), align: 0
  Segment part 29.
           ENTRY                   ADDRESS         REF BY
           =====                   =======         ======
           Application_UpdateAdv::?relay
                                   00000B5A        parseCmd (serialInterface)
    -------------------------------------------------------------------------
BANK_RELAYS
  Relative segment, address: CODE 00000B60 - 00000B65 (0x6 bytes), align: 0
  Segment part 31.
           ENTRY                   ADDRESS         REF BY
           =====                   =======         ======
           Application_UpdateRsp::?relay
                                   00000B60        parseCmd (serialInterface)

    *************************************************************************

  FILE NAME : C:\ble\BLE-CC254x-1.4.1.43908\Projects\ble\SimpleBLEBroadcaster-usb\CC2540\CC2540USB\Obj\SimpleBLEBroadcaster_Main.r51
  PROGRAM MODULE, NAME : SimpleBLEBroadcaster_Main

  SEGMENTS IN THE MODULE
  ======================
<BANKED_CODE,XDATA_ROM_C_FLASH> 1 (was BANKED_CODE)
  Relative segment, address: CODE 0000C541 - 0000C595 (0x55 bytes), align: 0
  Segment part 11.
           ENTRY                   ADDRESS         REF BY
           =====                   =======         ======
           main                    0000C541        ?call_main (?cmain)
               calls direct

    *************************************************************************

  FILE NAME : C:\ble\BLE-CC254x-1.4.1.43908\Projects\ble\SimpleBLEBroadcaster-usb\CC2540\CC2540USB\Obj\usb_cdc_descriptor.r51
  LIBRARY MODULE, NAME : usb_descriptor

  SEGMENTS IN THE MODULE
  ======================
RCODE
  Relative segment, address: CODE 00000C32 - 00000C8E (0x5d bytes), align: 0
  Segment part 0. ROOT 
           ENTRY                   ADDRESS         REF BY
           =====                   =======         ======
           usbDescStart            00000C32        Segment part 7 (usb_firmware_library_config)
           usbDescEnd              00000C87        Segment part 7 (usb_firmware_library_config)
           usbDescLut              00000C87        Segment part 7 (usb_firmware_library_config)
           usbDescLutEnd           00000C87        Segment part 7 (usb_firmware_library_config)
           usbDblbufLut            00000C87        Segment part 7 (usb_firmware_library_config)
           usbDblbufLutEnd         00000C8F        Segment part 7 (usb_firmware_library_config)
           LOCAL                   ADDRESS         
           =====                   =======         
           deviceDesc              00000C32 
           deviceDescEnd           00000C44 
           config1LengthStart      00000C44 
           configDesc              00000C44 
           configDescEnd           00000C4D 
           config1LengthEnd        00000C87 
           interface0Desc          00000C4D 
           interface0DescEnd       00000C56 
           headerFunctionalDesc    00000C56 
           headerFunctionalDescEnd
                                   00000C5B 
           absCtrlManFuncDesc      00000C5B 
           absCtrlManFuncDescEnd   00000C5F 
           unionFunctionalDesc     00000C5F 
           unionFunctionalDescEnd
                                   00000C64 
           callMngFuncDesc         00000C64 
           callMngFuncDescEnd      00000C69 
           endpoint0Desc           00000C69 
           endpoint0DescEnd        00000C70 
           interface1Desc          00000C70 
           interface1DescEnd       00000C79 
           endpoint1Desc           00000C79 
           endpoint1DescEnd        00000C80 
           endpoint2Desc           00000C80 
           endpoint2DescEnd        00000C87 

    *************************************************************************

  FILE NAME : C:\ble\BLE-CC254x-1.4.1.43908\Projects\ble\SimpleBLEBroadcaster-usb\CC2540\CC2540USB\Obj\usb_cdc_hooks.r51
  PROGRAM MODULE, NAME : usb_cdc_hooks

  SEGMENTS IN THE MODULE
  ======================
XDATA_Z
  Relative segment, address: XDATA 0000102F - 00001035 (0x7 bytes), align: 0
  Segment part 6.             Intra module refs:   usbcrHookProcessIn
                                                   usbcrHookProcessOut
           ENTRY                   ADDRESS         REF BY
           =====                   =======         ======
           currentLineCoding       0000102F        HalUARTInitUSB (hal_uart)
    -------------------------------------------------------------------------
<BANKED_CODE,XDATA_ROM_C_FLASH> 1 (was BANKED_CODE)
  Relative segment, address: CODE 0000C109 - 0000C153 (0x4b bytes), align: 0
  Segment part 7.             Intra module refs:   usbcrHookProcessOut::?relay
           ENTRY                   ADDRESS         REF BY
           =====                   =======         ======
           usbcrHookProcessOut     0000C109 
               is indirectly called
               ISTACK = 00000000 ( 00000002 )
    -------------------------------------------------------------------------
<BANKED_CODE,XDATA_ROM_C_FLASH> 1 (was BANKED_CODE)
  Relative segment, address: CODE 0000C154 - 0000C192 (0x3f bytes), align: 0
  Segment part 9.             Intra module refs:   usbcrHookProcessIn::?relay
           ENTRY                   ADDRESS         REF BY
           =====                   =======         ======
           usbcrHookProcessIn      0000C154 
               is indirectly called
               ISTACK = 00000000 ( 00000002 )
    -------------------------------------------------------------------------
<BANKED_CODE,XDATA_ROM_C_FLASH> 1 (was BANKED_CODE)
  Relative segment, address: CODE 0000C193 - 0000C1A3 (0x11 bytes), align: 0
  Segment part 11.            Intra module refs:   usbvrHookProcessOut::?relay
           ENTRY                   ADDRESS         REF BY
           =====                   =======         ======
           usbvrHookProcessOut     0000C193 
               is indirectly called
               ISTACK = 00000000 ( 00000002 )
    -------------------------------------------------------------------------
<BANKED_CODE,XDATA_ROM_C_FLASH> 1 (was BANKED_CODE)
  Relative segment, address: CODE 0000C1A4 - 0000C1B4 (0x11 bytes), align: 0
  Segment part 13.            Intra module refs:   usbvrHookProcessIn::?relay
           ENTRY                   ADDRESS         REF BY
           =====                   =======         ======
           usbvrHookProcessIn      0000C1A4 
               is indirectly called
               ISTACK = 00000000 ( 00000002 )
    -------------------------------------------------------------------------
<BANKED_CODE,XDATA_ROM_C_FLASH> 1 (was BANKED_CODE)
  Relative segment, address: CODE 0000C1B5 - 0000C1C5 (0x11 bytes), align: 0
  Segment part 19.            Intra module refs:   usbsrHookClearFeature::?relay
           ENTRY                   ADDRESS         REF BY
           =====                   =======         ======
           usbsrHookClearFeature   0000C1B5 
               ISTACK = 00000000 ( 00000002 )
    -------------------------------------------------------------------------
<BANKED_CODE,XDATA_ROM_C_FLASH> 1 (was BANKED_CODE)
  Relative segment, address: CODE 0000C1C6 - 0000C1D6 (0x11 bytes), align: 0
  Segment part 21.            Intra module refs:   usbsrHookSetFeature::?relay
           ENTRY                   ADDRESS         REF BY
           =====                   =======         ======
           usbsrHookSetFeature     0000C1C6 
               ISTACK = 00000000 ( 00000002 )
    -------------------------------------------------------------------------
<BANKED_CODE,XDATA_ROM_C_FLASH> 1 (was BANKED_CODE)
  Relative segment, address: CODE 0000C1D7 - 0000C1F6 (0x20 bytes), align: 0
  Segment part 25.            Intra module refs:   usbsrHookProcessEvent::?relay
           ENTRY                   ADDRESS         REF BY
           =====                   =======         ======
           usbsrHookProcessEvent   0000C1D7 
    -------------------------------------------------------------------------
<BANKED_CODE,XDATA_ROM_C_FLASH> 1 (was BANKED_CODE)
  Relative segment, address: CODE 0000C1F7 - 0000C1F9 (0x3 bytes), align: 0
  Segment part 27.            Intra module refs:   usbirqHookProcessEvents::?relay
           ENTRY                   ADDRESS         REF BY
           =====                   =======         ======
           usbirqHookProcessEvents
                                   0000C1F7 
    -------------------------------------------------------------------------
BANK_RELAYS
  Relative segment, address: CODE 00000B66 - 00000B6B (0x6 bytes), align: 0
  Segment part 8.
           ENTRY                   ADDRESS         REF BY
           =====                   =======         ======
           usbcrHookProcessOut::?relay
                                   00000B66        usbfwSetupHandler (usb_framework)
    -------------------------------------------------------------------------
BANK_RELAYS
  Relative segment, address: CODE 00000B6C - 00000B71 (0x6 bytes), align: 0
  Segment part 10.
           ENTRY                   ADDRESS         REF BY
           =====                   =======         ======
           usbcrHookProcessIn::?relay
                                   00000B6C        usbfwSetupHandler (usb_framework)
    -------------------------------------------------------------------------
BANK_RELAYS
  Relative segment, address: CODE 00000B72 - 00000B77 (0x6 bytes), align: 0
  Segment part 12.
           ENTRY                   ADDRESS         REF BY
           =====                   =======         ======
           usbvrHookProcessOut::?relay
                                   00000B72        usbfwSetupHandler (usb_framework)
    -------------------------------------------------------------------------
BANK_RELAYS
  Relative segment, address: CODE 00000B78 - 00000B7D (0x6 bytes), align: 0
  Segment part 14.
           ENTRY                   ADDRESS         REF BY
           =====                   =======         ======
           usbvrHookProcessIn::?relay
                                   00000B78        usbfwSetupHandler (usb_framework)
    -------------------------------------------------------------------------
BANK_RELAYS
  Relative segment, address: CODE 00000B7E - 00000B83 (0x6 bytes), align: 0
  Segment part 20.
           ENTRY                   ADDRESS         REF BY
           =====                   =======         ======
           usbsrHookClearFeature::?relay
                                   00000B7E        usbsrClearFeature (usb_standard_requests)
    -------------------------------------------------------------------------
BANK_RELAYS
  Relative segment, address: CODE 00000B84 - 00000B89 (0x6 bytes), align: 0
  Segment part 22.
           ENTRY                   ADDRESS         REF BY
           =====                   =======         ======
           usbsrHookSetFeature::?relay
                                   00000B84        usbsrSetFeature (usb_standard_requests)
    -------------------------------------------------------------------------
BANK_RELAYS
  Relative segment, address: CODE 00000B8A - 00000B8F (0x6 bytes), align: 0
  Segment part 26.
           ENTRY                   ADDRESS         REF BY
           =====                   =======         ======
           usbsrHookProcessEvent::?relay
                                   00000B8A        ChangeFeature (usb_standard_requests)
                                                   usbsrSetConfiguration (usb_standard_requests)
                                                   usbsrSetInterface (usb_standard_requests)
    -------------------------------------------------------------------------
BANK_RELAYS
  Relative segment, address: CODE 00000B90 - 00000B95 (0x6 bytes), align: 0
  Segment part 28.
           ENTRY                   ADDRESS         REF BY
           =====                   =======         ======
           usbirqHookProcessEvents::?relay
                                   00000B90        usbirqHandler (usb_interrupt)

    *************************************************************************

  FILE NAME : C:\ble\BLE-CC254x-1.4.1.43908\Projects\ble\SimpleBLEBroadcaster-usb\CC2540\CC2540USB\Obj\usb_descriptor_parser.r51
  PROGRAM MODULE, NAME : usb_descriptor_parser

  SEGMENTS IN THE MODULE
  ======================
XDATA_Z
  Relative segment, address: XDATA 00001036 - 00001037 (0x2 bytes), align: 0
  Segment part 6.             Intra module refs:   usbdpFindNext
                                                   usbdpInit
           LOCAL                   ADDRESS         
           =====                   =======         
           usbdpData               00001036 
    -------------------------------------------------------------------------
<XDATA_ROM_C> 1 (was XDATA_ROM_C)
  Relative segment, address: CONST 00008FE0 - 00008FE3 (0x4 bytes), align: 0
  Segment part 7.             Intra module refs:   usbdpGetStringDesc
           LOCAL                   ADDRESS         
           =====                   =======         
           languageId              00008FE0 
    -------------------------------------------------------------------------
<XDATA_ROM_C> 1 (was XDATA_ROM_C)
  Relative segment, address: CONST 00008F24 - 00008F47 (0x24 bytes), align: 0
  Segment part 8.             Intra module refs:   usbdpGetStringDesc
           LOCAL                   ADDRESS         
           =====                   =======         
           manufacturer            00008F24 
    -------------------------------------------------------------------------
<XDATA_ROM_C> 1 (was XDATA_ROM_C)
  Relative segment, address: CONST 00008F48 - 00008F6B (0x24 bytes), align: 0
  Segment part 9.             Intra module refs:   usbdpGetStringDesc
           LOCAL                   ADDRESS         
           =====                   =======         
           product                 00008F48 
    -------------------------------------------------------------------------
XDATA_I
  Relative segment, address: XDATA 00001118 - 00001141 (0x2a bytes), align: 0
  Segment part 10.            Intra module refs:   usbdpGetStringDesc
           LOCAL                   ADDRESS         
           =====                   =======         
           serialNumber            00001118 
    -------------------------------------------------------------------------
<BANKED_CODE,CODE_C> 1 (was BANKED_CODE)
  Relative segment, address: CODE 00007CA9 - 00007CC3 (0x1b bytes), align: 0
  Segment part 12.            Intra module refs:   usbdpInit::?relay
           ENTRY                   ADDRESS         REF BY
           =====                   =======         ======
           usbdpInit               00007CA9 
               XSTACK = 0000000C ( 00000000 )
               ISTACK = 00000000 ( 00000002 )
    -------------------------------------------------------------------------
<BANKED_CODE,CODE_C> 1 (was BANKED_CODE)
  Relative segment, address: CODE 00007CC4 - 00007D64 (0xa1 bytes), align: 0
  Segment part 14.            Intra module refs:   usbdpFindNext::?relay
           ENTRY                   ADDRESS         REF BY
           =====                   =======         ======
           usbdpFindNext           00007CC4 
               XSTACK = 0000000E ( 00000000 )
               ISTACK = 00000000 ( 00000002 )
    -------------------------------------------------------------------------
<BANKED_CODE,CODE_C> 1 (was BANKED_CODE)
  Relative segment, address: CODE 00007D65 - 00007D79 (0x15 bytes), align: 0
  Segment part 16.            Intra module refs:   usbdpGetDeviceDesc::?relay
           ENTRY                   ADDRESS         REF BY
           =====                   =======         ======
           usbdpGetDeviceDesc      00007D65 
               calls direct
               ISTACK = 00000000 ( 00000002 )
    -------------------------------------------------------------------------
<BANKED_CODE,CODE_C> 1 (was BANKED_CODE)
  Relative segment, address: CODE 00007D7A - 00007DC0 (0x47 bytes), align: 0
  Segment part 18.            Intra module refs:   usbdpGetConfigurationDesc::?relay
           ENTRY                   ADDRESS         REF BY
           =====                   =======         ======
           usbdpGetConfigurationDesc
                                   00007D7A 
               calls direct
               XSTACK = 0000000E ( 0000000C )
    -------------------------------------------------------------------------
<BANKED_CODE,CODE_C> 1 (was BANKED_CODE)
  Relative segment, address: CODE 00007DC1 - 00007E07 (0x47 bytes), align: 0
  Segment part 20.            Intra module refs:   usbdpGetInterfaceDesc::?relay
           ENTRY                   ADDRESS         REF BY
           =====                   =======         ======
           usbdpGetInterfaceDesc   00007DC1 
               calls direct
               XSTACK = 00000000 ( 0000000E )
    -------------------------------------------------------------------------
<BANKED_CODE,CODE_C> 1 (was BANKED_CODE)
  Relative segment, address: CODE 00007E08 - 00007FD7 (0x1d0 bytes), align: 0
  Segment part 22.            Intra module refs:   usbdpGetStringDesc::?relay
           ENTRY                   ADDRESS         REF BY
           =====                   =======         ======
           usbdpGetStringDesc      00007E08 
               XSTACK = 00000000 ( 00000014 )
               ISTACK = 00000000 ( 00000001 )
    -------------------------------------------------------------------------
XDATA_ID
  Relative segment, address: CODE 000001F4 - 0000021D (0x2a bytes), align: 0
  Segment part 11.            Intra module refs:   serialNumber
    -------------------------------------------------------------------------
BANK_RELAYS
  Relative segment, address: CODE 00000B96 - 00000B9B (0x6 bytes), align: 0
  Segment part 13.            Intra module refs:   usbdpGetConfigurationDesc
                                                   usbdpGetDeviceDesc
           ENTRY                   ADDRESS         REF BY
           =====                   =======         ======
           usbdpInit::?relay       00000B96 
    -------------------------------------------------------------------------
BANK_RELAYS
  Relative segment, address: CODE 00000B9C - 00000BA1 (0x6 bytes), align: 0
  Segment part 15.            Intra module refs:   usbdpGetConfigurationDesc
                                                   usbdpGetDeviceDesc
                                                   usbdpGetInterfaceDesc
           ENTRY                   ADDRESS         REF BY
           =====                   =======         ======
           usbdpFindNext::?relay   00000B9C        ConfigureEndpoints (usb_standard_requests)
                                                   usbsrSetConfiguration (usb_standard_requests)
    -------------------------------------------------------------------------
BANK_RELAYS
  Relative segment, address: CODE 00000BA2 - 00000BA7 (0x6 bytes), align: 0
  Segment part 17.
           ENTRY                   ADDRESS         REF BY
           =====                   =======         ======
           usbdpGetDeviceDesc::?relay
                                   00000BA2        usbsrGetDescriptor (usb_standard_requests)
    -------------------------------------------------------------------------
BANK_RELAYS
  Relative segment, address: CODE 00000BA8 - 00000BAD (0x6 bytes), align: 0
  Segment part 19.            Intra module refs:   usbdpGetInterfaceDesc
           ENTRY                   ADDRESS         REF BY
           =====                   =======         ======
           usbdpGetConfigurationDesc::?relay
                                   00000BA8        usbfwInit (usb_framework)
                                                   usbsrGetDescriptor (usb_standard_requests)
                                                   usbsrSetConfiguration (usb_standard_requests)
    -------------------------------------------------------------------------
BANK_RELAYS
  Relative segment, address: CODE 00000BAE - 00000BB3 (0x6 bytes), align: 0
  Segment part 21.
           ENTRY                   ADDRESS         REF BY
           =====                   =======         ======
           usbdpGetInterfaceDesc::?relay
                                   00000BAE        usbsrSetInterface (usb_standard_requests)
    -------------------------------------------------------------------------
BANK_RELAYS
  Relative segment, address: CODE 00000BB4 - 00000BB9 (0x6 bytes), align: 0
  Segment part 23.
           ENTRY                   ADDRESS         REF BY
           =====                   =======         ======
           usbdpGetStringDesc::?relay
                                   00000BB4        usbsrGetDescriptor (usb_standard_requests)
    -------------------------------------------------------------------------
<BANKED_CODE,XDATA_ROM_C_FLASH> 1 (was XDATA_ROM_C_FLASH)
  Relative segment, address: CODE 00008FE0 - 00008FE3 (0x4 bytes), align: 0
  Segment part 24.            Intra module refs:   languageId
    -------------------------------------------------------------------------
<BANKED_CODE,XDATA_ROM_C_FLASH> 1 (was XDATA_ROM_C_FLASH)
  Relative segment, address: CODE 00008F24 - 00008F47 (0x24 bytes), align: 0
  Segment part 25.            Intra module refs:   manufacturer
    -------------------------------------------------------------------------
<BANKED_CODE,XDATA_ROM_C_FLASH> 1 (was XDATA_ROM_C_FLASH)
  Relative segment, address: CODE 00008F48 - 00008F6B (0x24 bytes), align: 0
  Segment part 26.            Intra module refs:   product

    *************************************************************************

  FILE NAME : C:\ble\BLE-CC254x-1.4.1.43908\Projects\ble\SimpleBLEBroadcaster-usb\CC2540\CC2540USB\Obj\usb_firmware_library_config.r51
  PROGRAM MODULE, NAME : usb_firmware_library_config

  SEGMENTS IN THE MODULE
  ======================
XDATA_I
  Relative segment, address: XDATA 00001142 - 0000114D (0xc bytes), align: 0
  Segment part 6.
           ENTRY                   ADDRESS         REF BY
           =====                   =======         ======
           usbDescriptorMarker     00001142        ConfigureEndpoints (usb_standard_requests)
                                                   usbdpFindNext (usb_descriptor_parser)
                                                   usbdpInit (usb_descriptor_parser)
                                                   usbsrGetDescriptor (usb_standard_requests)
    -------------------------------------------------------------------------
XDATA_ID
  Relative segment, address: CODE 0000021E - 00000229 (0xc bytes), align: 0
  Segment part 7.             Intra module refs:   usbDescriptorMarker

    *************************************************************************

  FILE NAME : C:\ble\BLE-CC254x-1.4.1.43908\Projects\ble\SimpleBLEBroadcaster-usb\CC2540\CC2540USB\Obj\usb_framework.r51
  PROGRAM MODULE, NAME : usb_framework

  SEGMENTS IN THE MODULE
  ======================
XDATA_Z
  Relative segment, address: XDATA 00001038 - 0000104B (0x14 bytes), align: 0
  Segment part 6.             Intra module refs:   usbfwInit
                                                   usbfwResetHandler
                                                   usbfwSetAllEpStatus
                                                   usbfwSetupHandler
           ENTRY                   ADDRESS         REF BY
           =====                   =======         ======
           usbfwData               00001038        ChangeFeature (usb_standard_requests)
                                                   ConfigureEndpoints (usb_standard_requests)
                                                   usbcrHookProcessIn (usb_cdc_hooks)
                                                   usbcrHookProcessOut (usb_cdc_hooks)
                                                   usbsrGetConfiguration (usb_standard_requests)
                                                   usbsrGetDescriptor (usb_standard_requests)
                                                   usbsrGetInterface (usb_standard_requests)
                                                   usbsrGetStatus (usb_standard_requests)
                                                   usbsrHookClearFeature (usb_cdc_hooks)
                                                   usbsrHookSetFeature (usb_cdc_hooks)
                                                   usbsrSetAddress (usb_standard_requests)
                                                   usbsrSetConfiguration (usb_standard_requests)
                                                   usbsrSetInterface (usb_standard_requests)
                                                   usbvrHookProcessIn (usb_cdc_hooks)
                                                   usbvrHookProcessOut (usb_cdc_hooks)
    -------------------------------------------------------------------------
XDATA_Z
  Relative segment, address: XDATA 0000104C - 00001050 (0x5 bytes), align: 0
  Segment part 7.             Intra module refs:   usbfwSetupHandler
           ENTRY                   ADDRESS         REF BY
           =====                   =======         ======
           usbSetupData            0000104C        usbcrHookProcessIn (usb_cdc_hooks)
                                                   usbcrHookProcessOut (usb_cdc_hooks)
                                                   usbsrGetConfiguration (usb_standard_requests)
                                                   usbsrGetDescriptor (usb_standard_requests)
                                                   usbsrGetInterface (usb_standard_requests)
                                                   usbsrGetStatus (usb_standard_requests)
    -------------------------------------------------------------------------
XDATA_Z
  Relative segment, address: XDATA 00001051 - 00001058 (0x8 bytes), align: 0
  Segment part 8.             Intra module refs:   usbfwSetupHandler
           ENTRY                   ADDRESS         REF BY
           =====                   =======         ======
           usbSetupHeader          00001051        ChangeFeature (usb_standard_requests)
                                                   usbcrHookProcessIn (usb_cdc_hooks)
                                                   usbcrHookProcessOut (usb_cdc_hooks)
                                                   usbsrGetConfiguration (usb_standard_requests)
                                                   usbsrGetDescriptor (usb_standard_requests)
                                                   usbsrGetInterface (usb_standard_requests)
                                                   usbsrGetStatus (usb_standard_requests)
                                                   usbsrSetAddress (usb_standard_requests)
                                                   usbsrSetConfiguration (usb_standard_requests)
                                                   usbsrSetInterface (usb_standard_requests)
    -------------------------------------------------------------------------
DATA_Z
  Relative segment, address: DATA 00000023 - 00000024 (0x2 bytes), align: 0
  Segment part 9.             Intra module refs:   usbfwResetHandler
                                                   usbfwSetupHandler
           LOCAL                   ADDRESS         
           =====                   =======         
           ProcessFunc             00000023 
    -------------------------------------------------------------------------
<BANKED_CODE,XDATA_ROM_C_FLASH> 1 (was BANKED_CODE)
  Relative segment, address: CODE 0000945B - 000094AB (0x51 bytes), align: 0
  Segment part 10.            Intra module refs:   usbfwInit::?relay
           ENTRY                   ADDRESS         REF BY
           =====                   =======         ======
           usbfwInit               0000945B 
               calls direct
               XSTACK = 00000000 ( 0000000A )
    -------------------------------------------------------------------------
<BANKED_CODE,XDATA_ROM_C_FLASH> 1 (was BANKED_CODE)
  Relative segment, address: CODE 000094AC - 000094D3 (0x28 bytes), align: 0
  Segment part 12.            Intra module refs:   usbfwResetHandler::?relay
           ENTRY                   ADDRESS         REF BY
           =====                   =======         ======
           usbfwResetHandler       000094AC 
               calls direct
               ISTACK = 00000000 ( 00000002 )
    -------------------------------------------------------------------------
<BANKED_CODE,XDATA_ROM_C_FLASH> 1 (was BANKED_CODE)
  Relative segment, address: CODE 000094D4 - 00009783 (0x2b0 bytes), align: 0
  Segment part 14.            Intra module refs:   usbfwSetupHandler::?relay
           ENTRY                   ADDRESS         REF BY
           =====                   =======         ======
           usbfwSetupHandler       000094D4 
               calls direct
               XSTACK = 00000000 ( 00000012 )
    -------------------------------------------------------------------------
<BANKED_CODE,XDATA_ROM_C_FLASH> 1 (was BANKED_CODE)
  Relative segment, address: CODE 00009784 - 000097CC (0x49 bytes), align: 0
  Segment part 16.            Intra module refs:   usbfwSetAllEpStatus::?relay
           ENTRY                   ADDRESS         REF BY
           =====                   =======         ======
           usbfwSetAllEpStatus     00009784 
               ISTACK = 00000000 ( 00000003 )
    -------------------------------------------------------------------------
<BANKED_CODE,XDATA_ROM_C_FLASH> 1 (was BANKED_CODE)
  Relative segment, address: CODE 000097CD - 0000980D (0x41 bytes), align: 0
  Segment part 18.            Intra module refs:   usbfwReadFifo::?relay
           ENTRY                   ADDRESS         REF BY
           =====                   =======         ======
           usbfwReadFifo           000097CD 
               XSTACK = 00000012 ( 0000000B )
               ISTACK = 00000000 ( 00000001 )
    -------------------------------------------------------------------------
<BANKED_CODE,XDATA_ROM_C_FLASH> 1 (was BANKED_CODE)
  Relative segment, address: CODE 0000980E - 0000984E (0x41 bytes), align: 0
  Segment part 20.            Intra module refs:   usbfwWriteFifo::?relay
           ENTRY                   ADDRESS         REF BY
           =====                   =======         ======
           usbfwWriteFifo          0000980E 
               XSTACK = 00000012 ( 0000000B )
               ISTACK = 00000000 ( 00000001 )
    -------------------------------------------------------------------------
BANK_RELAYS
  Relative segment, address: CODE 00000BBA - 00000BBF (0x6 bytes), align: 0
  Segment part 11.
           ENTRY                   ADDRESS         REF BY
           =====                   =======         ======
           usbfwInit::?relay       00000BBA        HalUARTInitUSB (hal_uart)
    -------------------------------------------------------------------------
BANK_RELAYS
  Relative segment, address: CODE 00000BC0 - 00000BC5 (0x6 bytes), align: 0
  Segment part 13.
           ENTRY                   ADDRESS         REF BY
           =====                   =======         ======
           usbfwResetHandler::?relay
                                   00000BC0        halUartPollEvt (hal_uart)
    -------------------------------------------------------------------------
BANK_RELAYS
  Relative segment, address: CODE 00000BC6 - 00000BCB (0x6 bytes), align: 0
  Segment part 15.
           ENTRY                   ADDRESS         REF BY
           =====                   =======         ======
           usbfwSetupHandler::?relay
                                   00000BC6        halUartPollEvt (hal_uart)
    -------------------------------------------------------------------------
BANK_RELAYS
  Relative segment, address: CODE 00000BCC - 00000BD1 (0x6 bytes), align: 0
  Segment part 17.            Intra module refs:   usbfwResetHandler
           ENTRY                   ADDRESS         REF BY
           =====                   =======         ======
           usbfwSetAllEpStatus::?relay
                                   00000BCC        usbsrSetConfiguration (usb_standard_requests)
    -------------------------------------------------------------------------
BANK_RELAYS
  Relative segment, address: CODE 00000BD2 - 00000BD7 (0x6 bytes), align: 0
  Segment part 19.            Intra module refs:   usbfwSetupHandler
           ENTRY                   ADDRESS         REF BY
           =====                   =======         ======
           usbfwReadFifo::?relay   00000BD2 
    -------------------------------------------------------------------------
BANK_RELAYS
  Relative segment, address: CODE 00000BD8 - 00000BDD (0x6 bytes), align: 0
  Segment part 21.            Intra module refs:   usbfwSetupHandler
           ENTRY                   ADDRESS         REF BY
           =====                   =======         ======
           usbfwWriteFifo::?relay
                                   00000BD8 

    *************************************************************************

  FILE NAME : C:\ble\BLE-CC254x-1.4.1.43908\Projects\ble\SimpleBLEBroadcaster-usb\CC2540\CC2540USB\Obj\usb_interrupt.r51
  PROGRAM MODULE, NAME : usb_interrupt

  SEGMENTS IN THE MODULE
  ======================
DATA_Z
  Relative segment, address: DATA 00000025 - 00000029 (0x5 bytes), align: 0
  Segment part 12.            Intra module refs:   usbirqHandler
                                                   usbirqInit
           ENTRY                   ADDRESS         REF BY
           =====                   =======         ======
           usbirqData              00000025        halUartPollEvt (hal_uart)
    -------------------------------------------------------------------------
SFR_AN
  Relative segment, address: DATA 0000008B - 0000008B (0x1 bytes), align: 0
  Segment part 1. ROOT        Intra module refs:   usbirqHandler
                                                   usbirqInit
           ENTRY                   ADDRESS         REF BY
           =====                   =======         ======
           P2IFG                   0000008B 
    -------------------------------------------------------------------------
SFR_AN
  Relative segment, address: DATA 000000AC - 000000AC (0x1 bytes), align: 0
  Segment part 4. ROOT        Intra module refs:   LL_EXT_MapPmIoPort (ll)
                                                   usbirqInit
           ENTRY                   ADDRESS         REF BY
           =====                   =======         ======
           P2IEN                   000000AC 
    -------------------------------------------------------------------------
SFR_AN
  Relative segment, address: DATA 000000E8 - 000000E8 (0x1 bytes), align: 0
  Segment part 5. ROOT        Intra module refs:   usbirqHandler
                                                   usbirqInit
           ENTRY                   ADDRESS         REF BY
           =====                   =======         ======
           _A_IRCON2               000000E8 
           LOCAL                   ADDRESS         
           =====                   =======         
           IRCON2                  000000E8 
    -------------------------------------------------------------------------
<BANKED_CODE,XDATA_ROM_C_FLASH> 1 (was BANKED_CODE)
  Relative segment, address: CODE 0000C5EA - 0000C634 (0x4b bytes), align: 0
  Segment part 13.            Intra module refs:   usbirqInit::?relay
           ENTRY                   ADDRESS         REF BY
           =====                   =======         ======
           usbirqInit              0000C5EA 
               XSTACK = 00000000 ( 0000000A )
    -------------------------------------------------------------------------
NEAR_CODE
  Relative segment, address: CODE 000016E8 - 000017A5 (0xbe bytes), align: 0
  Segment part 15.            Intra module refs:   usbirqHandler::??INTVEC 51
           ENTRY                   ADDRESS         REF BY
           =====                   =======         ======
           usbirqHandler           000016E8 
               interrupt function
               calls direct
               XSTACK = 00000000 ( 0000000F )
    -------------------------------------------------------------------------
INTVEC
  Common segment, address: CODE 00000000 - 00000035 (0x36 bytes), align: 0
  Segment part 6. ROOT 
           ENTRY                   ADDRESS         REF BY
           =====                   =======         ======
           usbirqHandler::??INTVEC 51
                                   00000033 
    -------------------------------------------------------------------------
BANK_RELAYS
  Relative segment, address: CODE 00000BDE - 00000BE3 (0x6 bytes), align: 0
  Segment part 14.
           ENTRY                   ADDRESS         REF BY
           =====                   =======         ======
           usbirqInit::?relay      00000BDE        HalUARTInitUSB (hal_uart)

    *************************************************************************

  FILE NAME : C:\ble\BLE-CC254x-1.4.1.43908\Projects\ble\SimpleBLEBroadcaster-usb\CC2540\CC2540USB\Obj\usb_standard_requests.r51
  PROGRAM MODULE, NAME : usb_standard_requests

  SEGMENTS IN THE MODULE
  ======================
<BANKED_CODE,CODE_C> 1 (was BANKED_CODE)
  Relative segment, address: CODE 00002AE0 - 00002C42 (0x163 bytes), align: 0
  Segment part 7.             Intra module refs:   usbsrGetStatus::?relay
           ENTRY                   ADDRESS         REF BY
           =====                   =======         ======
           usbsrGetStatus          00002AE0 
               ISTACK = 00000000 ( 00000002 )
    -------------------------------------------------------------------------
XDATA_Z
  Relative segment, address: XDATA 00001059 - 0000105A (0x2 bytes), align: 0
  Segment part 6.             Intra module refs:   usbsrGetStatus
           LOCAL                   ADDRESS         
           =====                   =======         
           usbsrGetStatus::status
                                   00001059 
    -------------------------------------------------------------------------
<BANKED_CODE,CODE_C> 1 (was BANKED_CODE)
  Relative segment, address: CODE 00002C43 - 00002D83 (0x141 bytes), align: 0
  Segment part 9.             Intra module refs:   ChangeFeature::?relay
           LOCAL                   ADDRESS         
           =====                   =======         
           ChangeFeature           00002C43 
               calls direct
               XSTACK = 00000000 ( 00000009 )
               ISTACK = 00000000 ( 00000001 )
    -------------------------------------------------------------------------
<BANKED_CODE,CODE_C> 1 (was BANKED_CODE)
  Relative segment, address: CODE 00002D84 - 00002D99 (0x16 bytes), align: 0
  Segment part 11.            Intra module refs:   usbsrClearFeature::?relay
           ENTRY                   ADDRESS         REF BY
           =====                   =======         ======
           usbsrClearFeature       00002D84 
               calls direct
               ISTACK = 00000000 ( 00000002 )
    -------------------------------------------------------------------------
<BANKED_CODE,CODE_C> 1 (was BANKED_CODE)
  Relative segment, address: CODE 00002D9A - 00002DAF (0x16 bytes), align: 0
  Segment part 13.            Intra module refs:   usbsrSetFeature::?relay
           ENTRY                   ADDRESS         REF BY
           =====                   =======         ======
           usbsrSetFeature         00002D9A 
               calls direct
               ISTACK = 00000000 ( 00000002 )
    -------------------------------------------------------------------------
<BANKED_CODE,CODE_C> 1 (was BANKED_CODE)
  Relative segment, address: CODE 00002DB0 - 00002E22 (0x73 bytes), align: 0
  Segment part 15.            Intra module refs:   usbsrSetAddress::?relay
           ENTRY                   ADDRESS         REF BY
           =====                   =======         ======
           usbsrSetAddress         00002DB0 
               ISTACK = 00000000 ( 00000002 )
    -------------------------------------------------------------------------
<BANKED_CODE,CODE_C> 1 (was BANKED_CODE)
  Relative segment, address: CODE 00002E23 - 00003140 (0x31e bytes), align: 0
  Segment part 17.            Intra module refs:   usbsrGetDescriptor::?relay
           ENTRY                   ADDRESS         REF BY
           =====                   =======         ======
           usbsrGetDescriptor      00002E23 
               calls direct
               XSTACK = 00000000 ( 0000000B )
               ISTACK = 00000000 ( 00000002 )
    -------------------------------------------------------------------------
<BANKED_CODE,CODE_C> 1 (was BANKED_CODE)
  Relative segment, address: CODE 00003141 - 000032DA (0x19a bytes), align: 0
  Segment part 19.            Intra module refs:   ConfigureEndpoints::?relay
           LOCAL                   ADDRESS         
           =====                   =======         
           ConfigureEndpoints      00003141 
               calls direct
               XSTACK = 0000000E ( 00000014 )
    -------------------------------------------------------------------------
<BANKED_CODE,CODE_C> 1 (was BANKED_CODE)
  Relative segment, address: CODE 000032DB - 00003331 (0x57 bytes), align: 0
  Segment part 21.            Intra module refs:   usbsrGetConfiguration::?relay
           ENTRY                   ADDRESS         REF BY
           =====                   =======         ======
           usbsrGetConfiguration   000032DB 
               ISTACK = 00000000 ( 00000002 )
    -------------------------------------------------------------------------
<BANKED_CODE,CODE_C> 1 (was BANKED_CODE)
  Relative segment, address: CODE 00003332 - 00003441 (0x110 bytes), align: 0
  Segment part 23.            Intra module refs:   usbsrSetConfiguration::?relay
           ENTRY                   ADDRESS         REF BY
           =====                   =======         ======
           usbsrSetConfiguration   00003332 
               calls direct
               XSTACK = 00000000 ( 0000000E )
    -------------------------------------------------------------------------
<BANKED_CODE,CODE_C> 1 (was BANKED_CODE)
  Relative segment, address: CODE 00003442 - 000034AC (0x6b bytes), align: 0
  Segment part 25.            Intra module refs:   usbsrGetInterface::?relay
           ENTRY                   ADDRESS         REF BY
           =====                   =======         ======
           usbsrGetInterface       00003442 
               XSTACK = 00000000 ( 0000000B )
    -------------------------------------------------------------------------
<BANKED_CODE,CODE_C> 1 (was BANKED_CODE)
  Relative segment, address: CODE 000034AD - 0000354D (0xa1 bytes), align: 0
  Segment part 27.            Intra module refs:   usbsrSetInterface::?relay
           ENTRY                   ADDRESS         REF BY
           =====                   =======         ======
           usbsrSetInterface       000034AD 
               calls direct
               XSTACK = 00000000 ( 0000000A )
               ISTACK = 00000000 ( 00000001 )
    -------------------------------------------------------------------------
BANK_RELAYS
  Relative segment, address: CODE 00000BE4 - 00000BE9 (0x6 bytes), align: 0
  Segment part 8.
           ENTRY                   ADDRESS         REF BY
           =====                   =======         ======
           usbsrGetStatus::?relay
                                   00000BE4        usbfwSetupHandler (usb_framework)
    -------------------------------------------------------------------------
BANK_RELAYS
  Relative segment, address: CODE 00000BEA - 00000BEF (0x6 bytes), align: 0
  Segment part 10.            Intra module refs:   usbsrClearFeature
                                                   usbsrSetFeature
           LOCAL                   ADDRESS         
           =====                   =======         
           ChangeFeature::?relay   00000BEA 
    -------------------------------------------------------------------------
BANK_RELAYS
  Relative segment, address: CODE 00000BF0 - 00000BF5 (0x6 bytes), align: 0
  Segment part 12.
           ENTRY                   ADDRESS         REF BY
           =====                   =======         ======
           usbsrClearFeature::?relay
                                   00000BF0        usbfwSetupHandler (usb_framework)
    -------------------------------------------------------------------------
BANK_RELAYS
  Relative segment, address: CODE 00000BF6 - 00000BFB (0x6 bytes), align: 0
  Segment part 14.
           ENTRY                   ADDRESS         REF BY
           =====                   =======         ======
           usbsrSetFeature::?relay
                                   00000BF6        usbfwSetupHandler (usb_framework)
    -------------------------------------------------------------------------
BANK_RELAYS
  Relative segment, address: CODE 00000BFC - 00000C01 (0x6 bytes), align: 0
  Segment part 16.
           ENTRY                   ADDRESS         REF BY
           =====                   =======         ======
           usbsrSetAddress::?relay
                                   00000BFC        usbfwSetupHandler (usb_framework)
    -------------------------------------------------------------------------
BANK_RELAYS
  Relative segment, address: CODE 00000C02 - 00000C07 (0x6 bytes), align: 0
  Segment part 18.
           ENTRY                   ADDRESS         REF BY
           =====                   =======         ======
           usbsrGetDescriptor::?relay
                                   00000C02        usbfwSetupHandler (usb_framework)
    -------------------------------------------------------------------------
BANK_RELAYS
  Relative segment, address: CODE 00000C08 - 00000C0D (0x6 bytes), align: 0
  Segment part 20.            Intra module refs:   usbsrSetConfiguration
                                                   usbsrSetInterface
           LOCAL                   ADDRESS         
           =====                   =======         
           ConfigureEndpoints::?relay
                                   00000C08 
    -------------------------------------------------------------------------
BANK_RELAYS
  Relative segment, address: CODE 00000C0E - 00000C13 (0x6 bytes), align: 0
  Segment part 22.
           ENTRY                   ADDRESS         REF BY
           =====                   =======         ======
           usbsrGetConfiguration::?relay
                                   00000C0E        usbfwSetupHandler (usb_framework)
    -------------------------------------------------------------------------
BANK_RELAYS
  Relative segment, address: CODE 00000C14 - 00000C19 (0x6 bytes), align: 0
  Segment part 24.
           ENTRY                   ADDRESS         REF BY
           =====                   =======         ======
           usbsrSetConfiguration::?relay
                                   00000C14        usbfwSetupHandler (usb_framework)
    -------------------------------------------------------------------------
BANK_RELAYS
  Relative segment, address: CODE 00000C1A - 00000C1F (0x6 bytes), align: 0
  Segment part 26.
           ENTRY                   ADDRESS         REF BY
           =====                   =======         ======
           usbsrGetInterface::?relay
                                   00000C1A        usbfwSetupHandler (usb_framework)
    -------------------------------------------------------------------------
BANK_RELAYS
  Relative segment, address: CODE 00000C20 - 00000C25 (0x6 bytes), align: 0
  Segment part 28.
           ENTRY                   ADDRESS         REF BY
           =====                   =======         ======
           usbsrSetInterface::?relay
                                   00000C20        usbfwSetupHandler (usb_framework)

    *************************************************************************

  FILE NAME : C:\ble\BLE-CC254x-1.4.1.43908\Projects\ble\SimpleBLEBroadcaster-usb\CC2540\CC2540USB\Obj\usb_suspend.r51
  PROGRAM MODULE, NAME : usb_suspend

  SEGMENTS IN THE MODULE
  ======================

    *************************************************************************

  FILE NAME : C:\Program Files\IAR Systems\Embedded Workbench 7.2\8051\LIB\CLIB\cl-pli-blxd-1e16x01.r51
  LIBRARY MODULE, NAME : ?cexit

  SEGMENTS IN THE MODULE
  ======================
CSTART
  Relative segment, address: CODE 00000091 - 00000095 (0x5 bytes), align: 0
  Segment part 0.
           ENTRY                   ADDRESS         REF BY
           =====                   =======         ======
           exit                    00000091        ?call_main (?cmain)
           ?C_EXIT                 00000091 
           ?ROM_MONITOR_NOPS       00000091 

    -------------------------------------------------------------------------
  LIBRARY MODULE, NAME : ?cmain

  SEGMENTS IN THE MODULE
  ======================
CSTART
  Relative segment, address: CODE 00000096, align: 0
  Segment part 5.
           ENTRY                   ADDRESS         REF BY
           =====                   =======         ======
           ?cmain                  00000096        Segment part 13 (CSTARTUP)
               calls direct
    -------------------------------------------------------------------------
CSTART
  Relative segment, address: CODE 00000096 - 0000009E (0x9 bytes), align: 0
  Segment part 6.
           ENTRY                   ADDRESS         REF BY
           =====                   =======         ======
           __low_level_init_call   00000096        __low_level_init (hal_startup)
    -------------------------------------------------------------------------
CSTART
  Relative segment, address: CODE 0000009F - 000000AC (0xe bytes), align: 0
  Segment part 10.
           ENTRY                   ADDRESS         REF BY
           =====                   =======         ======
           __INIT_DATA_Z           0000009F        ProcessFunc (usb_framework)
                                                   Segment part 1 (ll_halt)
                                                   usbirqData (usb_interrupt)
    -------------------------------------------------------------------------
CSTART
  Relative segment, address: CODE 000000AD - 000000BA (0xe bytes), align: 0
  Segment part 12.
           ENTRY                   ADDRESS         REF BY
           =====                   =======         ======
           __INIT_IDATA_Z          000000AD        myPC (ll)
    -------------------------------------------------------------------------
CSTART
  Relative segment, address: CODE 000000BB - 000000CA (0x10 bytes), align: 0
  Segment part 16.
           ENTRY                   ADDRESS         REF BY
           =====                   =======         ======
           __INIT_XDATA_Z          000000BB        HalLedState (hal_led)
                                                   HalLedStatusControl (hal_led)
                                                   Hal_TaskID (hal_drivers)
                                                   LL_TaskID (ll)
                                                   OSAL_timeSeconds (OSAL_ClockBLE)
                                                   OnboardKeyIntEnable (OnBoard)
                                                   Segment part 10 (gap_peridevmgr)
                                                   Segment part 10 (gap_simpletask)
                                                   Segment part 11 (gap_peridevmgr)
                                                   Segment part 12 (gap_configmgr)
                                                   Segment part 13 (hci_tl)
                                                   Segment part 14 (hci_tl)
                                                   Segment part 15 (gap_configmgr)
                                                   Segment part 15 (hci_tl)
                                                   Segment part 16 (hci_tl)
                                                   Segment part 8 (ll_scheduler)
                                                   Segment part 9 (gap_peridevmgr)
                                                   activePg (osal_snv)
                                                   adcRef (hal_adc)
                                                   advInfo (ll)
                                                   advertData (simpleBLEBroadcaster)
                                                   bleEvtMask (hci_event)
                                                   bm_list_ptr (osal_bufmgr)
                                                   buildInfo (ll)
                                                   cSerialPacketParser::cmd_identifier (serialInterface)
                                                   cSerialPacketParser::cmd_opcode (serialInterface)
                                                   cSerialPacketParser::pktState (serialInterface)
                                                   cbTimers (osal_cbtimer)
                                                   clkDivOnHalt (ll)
                                                   cmd_len (serialInterface)
                                                   ctrlToHostEnable (hci)
                                                   currentLineCoding (usb_cdc_hooks)
                                                   dcdcData (ll)
                                                   deviceFeatureSet (ll)
                                                   dmaCh0 (hal_dma)
                                                   dmaCh1234 (hal_dma)
                                                   dtmInfo (ll)
                                                   extendRfRange (ll)
                                                   failF (osal_snv)
                                                   ff1 (OSAL_Memory)
                                                   gapAutoAdvPrivateAddrChange (gap_configmgr)
                                                   gapDeviceAddrMode (gap_configmgr)
                                                   gapPrivateAddrChangeTimeout (gap_configmgr)
                                                   gapProfileRole (gap_configmgr)
                                                   gapRole_AdvChanMap (broadcaster)
                                                   gapRole_AdvDirectAddr (broadcaster)
                                                   gapRole_AdvDirectType (broadcaster)
                                                   gapRole_AdvEventType (broadcaster)
                                                   gapRole_AdvFilterPolicy (broadcaster)
                                                   gapRole_ScanRspData (broadcaster)
                                                   gapRole_ScanRspDataLen (broadcaster)
                                                   gapRole_TaskID (broadcaster)
                                                   gapRole_bdAddr (broadcaster)
                                                   gapRole_profileRole (broadcaster)
                                                   gapRole_state (broadcaster)
                                                   gapTaskID (gap_simpletask)
                                                   halUartRxH (hal_uart)
                                                   halUartRxT (hal_uart)
                                                   halUartTxH (hal_uart)
                                                   halUartTxT (hal_uart)
                                                   haltDuringRf (ll)
                                                   hciExtTaskID (hci_tl)
                                                   hciGapTaskID (hci_tl)
                                                   hciL2capTaskID (hci_tl)
                                                   hciPTMenabled (hci)
                                                   hciSmpTaskID (hci_tl)
                                                   hciTaskID (hci_tl)
                                                   hciTestTaskID (hci_tl)
                                                   llState (ll)
                                                   maxTxPwrForDTM (ll)
                                                   numHostBufs (hci)
                                                   numWLEntries (phy)
                                                   nvInUse (ll)
                                                   osalMemStat (OSAL_Memory)
                                                   osal_qHead (OSAL)
                                                   osal_systemClock (OSAL_Timers)
                                                   ownPublicAddr (ll)
                                                   ownRandomAddr (ll)
                                                   ownSavedPublicAddr (ll)
                                                   pGapAdvertState (gap_devmgr)
                                                   pGapRoles_AppCGs (broadcaster)
                                                   pHciEvtMask (hci_event)
                                                   pHciEvtMask2 (hci_event_PATCH)
                                                   pfnPeripheralCBs (gap_simpletask)
                                                   pgOff (osal_snv)
                                                   postRfOperations (ll)
                                                   preBlinkState (hal_led)
                                                   previousLLTimerTick (OSAL_ClockBLE)
                                                   pwrmgr_attribute (OSAL_PwrMgr)
                                                   remUsTicks (OSAL_ClockBLE)
                                                   rssiCorrection (ll)
                                                   rxFifoFlowCtrl (ll)
                                                   rxSerialPkt (serialInterface)
                                                   rxShdw (hal_uart)
                                                   rxTick (hal_uart)
                                                   scanRspData (simpleBLEBroadcaster)
                                                   serialInterface_TaskID (serialInterface)
                                                   simpleBLEBroadcaster_TaskID (simpleBLEBroadcaster)
                                                   sleepDelay (ll)
                                                   taskEndCause (ll)
                                                   tasksEvents (OSAL_SimpleBLEBroadcaster)
                                                   theHeap (OSAL_Memory)
                                                   timeMSec (OSAL_ClockBLE)
                                                   timerHead (OSAL_Timers)
                                                   trngCounter (ll)
                                                   txSerialPkt (serialInterface)
                                                   usbCB (hal_uart)
                                                   usbSetupData (usb_framework)
                                                   usbSetupHeader (usb_framework)
                                                   usbTxMT (hal_uart)
                                                   usbdpData (usb_descriptor_parser)
                                                   usbfwData (usb_framework)
                                                   usbsrGetStatus::status (usb_standard_requests)
                                                   verInfo (ll)
    -------------------------------------------------------------------------
CSTART
  Relative segment, address: CODE 000000CB - 000000F0 (0x26 bytes), align: 0
  Segment part 33.
           ENTRY                   ADDRESS         REF BY
           =====                   =======         ======
           __INIT_XDATA_I          000000CB        Segment part 12 (gap_peridevmgr)
                                                   Segment part 13 (gap_configmgr)
                                                   Segment part 6 (gap_peridevmgr)
                                                   activeTaskID (OSAL)
                                                   baseTaskID (osal_cbtimer)
                                                   def_advertData (simpleBLEBroadcaster)
                                                   def_scanRspData (simpleBLEBroadcaster)
                                                   gapAppTaskID (gap_configmgr)
                                                   gapRole_AdvEnabled (broadcaster)
                                                   gapRole_AdvertData (broadcaster)
                                                   gapRole_AdvertDataLen (broadcaster)
                                                   gapRole_AdvertOffTime (broadcaster)
                                                   gapUnwantedTaskID (gap_simpletask)
                                                   registeredKeysTaskID (OnBoard)
                                                   serialNumber (usb_descriptor_parser)
                                                   simpleBLEBroadcaster_BroadcasterCBs (simpleBLEBroadcaster)
                                                   taskEndCauses (ll)
                                                   taskErrorEndCauses (ll)
                                                   usbDescriptorMarker (usb_firmware_library_config)
    -------------------------------------------------------------------------
CSTART
  Relative segment, address: CODE 000000F1, align: 0
  Segment part 37.            Intra module refs:   __low_level_init_call
    -------------------------------------------------------------------------
CSTART
  Relative segment, address: CODE 000000F1 - 00000106 (0x16 bytes), align: 0
  Segment part 38.            Intra module refs:   ?cmain
           ENTRY                   ADDRESS         REF BY
           =====                   =======         ======
           ?call_main              000000F1 

    -------------------------------------------------------------------------
  LIBRARY MODULE, NAME : CSTARTUP

  SEGMENTS IN THE MODULE
  ======================
REGISTERS
  Relative segment, address: DATA 00000000, align: 0
  Segment part 0.             Intra module refs:   Segment part 6
           ENTRY                   ADDRESS         REF BY
           =====                   =======         ======
           ?REGISTERS              00000000 
    -------------------------------------------------------------------------
ISTACK
  Relative segment, address: IDATA 00000040, align: 0
  Segment part 1.             Intra module refs:   Segment part 6
           ENTRY                   ADDRESS         REF BY
           =====                   =======         ======
           ?ISTACK_START           00000040 
    -------------------------------------------------------------------------
XSTACK
  Relative segment, address: XDATA 00000001, align: 0
  Segment part 3.             Intra module refs:   ?RESET_XSP
           ENTRY                   ADDRESS         REF BY
           =====                   =======         ======
           ?XSTACK_START           00000001 
    -------------------------------------------------------------------------
INTVEC
  Common segment, address: CODE 00000000 - 00000002 (0x3 bytes), align: 0
  Segment part 5. ROOT        Intra module refs:   Segment part 6
    -------------------------------------------------------------------------
CSTART
  Relative segment, address: CODE 00000107 - 0000010C (0x6 bytes), align: 0
  Segment part 6. ROOT        Intra module refs:   Segment part 5
           ENTRY                   ADDRESS         REF BY
           =====                   =======         ======
           __program_start         00000107        Absolute parts (?ABS_ENTRY_MOD)
           ?RESET_SP               0000010A 
    -------------------------------------------------------------------------
CSTART
  Relative segment, address: CODE 0000010D - 00000112 (0x6 bytes), align: 0
  Segment part 8.
           ENTRY                   ADDRESS         REF BY
           =====                   =======         ======
           ?RESET_XSP              0000010D        ?XSP (VIRTUAL_REGISTERS)
    -------------------------------------------------------------------------
CSTART
  Relative segment, address: CODE 00000113 - 00000115 (0x3 bytes), align: 0
  Segment part 9.
           ENTRY                   ADDRESS         REF BY
           =====                   =======         ======
           ?RESET_CODE_BANK        00000113        Absolute parts (?BANKED_CODE_SUPPORT)
    -------------------------------------------------------------------------
CSTART
  Relative segment, address: CODE 00000116 - 00000118 (0x3 bytes), align: 0
  Segment part 13.            Intra module refs:   Absolute parts

    -------------------------------------------------------------------------
  LIBRARY MODULE, NAME : VIRTUAL_REGISTERS

  SEGMENTS IN THE MODULE
  ======================
BREG
  Relative segment, address: BIT 00000020.0 - 00000020.7 (0x8 bits), align: 0
  Segment part 0.
           ENTRY                   ADDRESS         REF BY
           =====                   =======         ======
           ?B0                     00000020.0      Absolute parts (CSTARTUP)
    -------------------------------------------------------------------------
VREG
  Relative segment, address: DATA 00000008 - 00000008 (0x1 bytes), align: 0
  Segment part 1.             Intra module refs:   ?V1
           ENTRY                   ADDRESS         REF BY
           =====                   =======         ======
           ?V0                     00000008        ?BANKED_ENTER_XDATA (?BANKED_ENTER_XDATA)
                                                   ?BANKED_LEAVE_XDATA (?BANKED_LEAVE_XDATA)
                                                   ?FUNC_ENTER_XDATA (?FUNC_ENTER_XDATA)
                                                   ?FUNC_LEAVE_XDATA (?FUNC_LEAVE_XDATA)
                                                   ?INTERRUPT_ENTER_XSP (?INTERRUPT_ENTER_XSP)
                                                   ?INTERRUPT_LEAVE_XSP (?INTERRUPT_LEAVE_XSP)
                                                   ?UL_GE_X (?UL_GE_X)
                                                   Application_UpdateAdv (simpleBLEBroadcaster)
                                                   Application_UpdateRsp (simpleBLEBroadcaster)
                                                   ConfigureEndpoints (usb_standard_requests)
                                                   GAPRole_GetParameter (broadcaster)
                                                   GAPRole_ProcessEvent (broadcaster)
                                                   GAPRole_SetParameter (broadcaster)
                                                   GAP_DeviceInit (gap)
                                                   GAP_MakeDiscoverable (gap_peridevmgr)
                                                   GAP_ProcessEvent (gap_simpletask)
                                                   GAP_UpdateAdvertisingData (gap_peridevmgr)
                                                   HCI_CommandCompleteEvent (hci_event)
                                                   HCI_EXT_DecryptCmd (hci)
                                                   HCI_LE_EncryptCmd (hci)
                                                   HCI_LE_SetAdvParamCmd (hci)
                                                   HCI_LE_TransmitterTestCmd (hci)
                                                   HCI_ProcessEvent (hci_tl)
                                                   HCI_ReadLocalVersionInfoCmd (hci)
                                                   HCI_ReverseBytes (hci_data)
                                                   HCI_SendCommandCompleteEvent (hci_event)
                                                   HCI_SetEventMaskCmd (hci)
                                                   HCI_SetEventMaskPage2Cmd (hci_PATCH)
                                                   HCI_VendorSpecifcCommandCompleteEvent (hci_event_PATCH)
                                                   HalFlashRead (hal_flash)
                                                   HalFlashWrite (hal_flash)
                                                   HalLedBlink (hal_led)
                                                   HalLedSet (hal_led)
                                                   HalLedUpdate (hal_led)
                                                   HalUARTOpen (hal_uart)
                                                   HalUARTRead (hal_uart)
                                                   HalUARTWrite (hal_uart)
                                                   Hal_ProcessEvent (hal_drivers)
                                                   LL_AddWhiteListDevice (ll)
                                                   LL_DirectTestEnd (ll)
                                                   LL_DirectTestTxTest (ll)
                                                   LL_ENC_AES128_Decrypt (ll_enc)
                                                   LL_ENC_AES128_Encrypt (ll_enc)
                                                   LL_ENC_GenerateTrueRandNum (ll_enc)
                                                   LL_EXT_Decrypt (ll)
                                                   LL_EXT_ExtendRfRange (ll)
                                                   LL_EXT_MapPmIoPort (ll)
                                                   LL_EXT_SaveFreqTune (ll)
                                                   LL_EXT_SetBDADDR (ll)
                                                   LL_EXT_SetRxGain (ll)
                                                   LL_EXT_SetTxPower (ll)
                                                   LL_Encrypt (ll)
                                                   LL_Init (ll)
                                                   LL_ProcessEvent (ll)
                                                   LL_Rand (ll)
                                                   LL_RandCback (hci)
                                                   LL_RemoveWhiteListDevice (ll)
                                                   LL_SetAdvControl (ll)
                                                   LL_SetAdvData (ll)
                                                   LL_SetAdvParam (ll)
                                                   LL_SetScanRspData (ll)
                                                   LL_TX_bm_alloc (ll)
                                                   NPI_ReadTransport (npi)
                                                   NPI_WriteTransport (npi)
                                                   OnBoard_KeyCallback (OnBoard)
                                                   OnBoard_SendKeys (OnBoard)
                                                   PHY_AddWlEntry (phy)
                                                   PHY_ClearBlacklistIndex (phy)
                                                   PHY_RemoveWlEntry (phy)
                                                   PHY_SetBlacklistIndex (phy)
                                                   PHY_SetCRCInit (phy)
                                                   PHY_SetSyncWord (phy)
                                                   RF_NormalIsr (ll_isr)
                                                   Segment part 131 (hci_tl)
                                                   Segment part 134 (ll)
                                                   Segment part 146 (ll)
                                                   Segment part 16 (ll_advEndCauses)
                                                   Segment part 20 (ll_advEndCauses)
                                                   Segment part 26 (ll_scheduler)
                                                   Segment part 37 (hci)
                                                   Segment part 37 (hci_tl)
                                                   Segment part 38 (hci_tl)
                                                   Segment part 43 (hci_tl)
                                                   Segment part 65 (gap_configmgr)
                                                   Segment part 65 (ll_common)
                                                   Segment part 79 (hci_tl)
                                                   SerialInterface_ProcessEvent (serialInterface)
                                                   SimpleBLEBroadcaster_Init (simpleBLEBroadcaster)
                                                   SimpleBLEBroadcaster_ProcessEvent (simpleBLEBroadcaster)
                                                   cSerialPacketParser (serialInterface)
                                                   cleanErasedPage (osal_snv)
                                                   compactPage (osal_snv)
                                                   erasePage (osal_snv)
                                                   findItem (osal_snv)
                                                   findOffset (osal_snv)
                                                   gapFindADType (gap_devmgr)
                                                   gapPeriProcessHCICmdCompleteEvt (gap_peridevmgr)
                                                   gapProcessAdvertisingEvt (gap_peridevmgr)
                                                   gapProcessHCICmdCompleteEvt (gap_simpletask)
                                                   gapProcessRandomAddrComplete (gap_configmgr)
                                                   gapReadBD_ADDRStatus (gap_configmgr)
                                                   gapReadBufSizeCmdStatus (gap_configmgr)
                                                   gapRole_ProcessGAPMsg (broadcaster)
                                                   gapRole_SetupGAP (broadcaster)
                                                   gapSendDeviceInitDoneEvent (gap_configmgr)
                                                   gapSendMakeDiscEvent (gap_peridevmgr)
                                                   gapSetAdvParams (gap_peridevmgr)
                                                   gapWriteAdvDataStatus (gap_peridevmgr)
                                                   gapWriteAdvEnableStatus (gap_peridevmgr)
                                                   halUartPollRx (hal_uart)
                                                   hciExtDecrypt (hci_tl)
                                                   hciLEEncrypt (hci_tl)
                                                   hciLESetAdvParam (hci_tl)
                                                   hciProcessCtrlToHost (hci_tl)
                                                   hciProcessHostToCtrlCmd (hci_tl)
                                                   hciSerialPacketParser (hci_tl)
                                                   initNV (osal_snv)
                                                   isLimitedDiscoverableMode (gap_peridevmgr)
                                                   ll24BitTimeCompare (ll_timer2)
                                                   ll24BitTimeDelta (ll_timer2)
                                                   llDiscoverableAdvEvt_TaskEndOk (ll_advEndCauses)
                                                   llFindNextSecTask (ll_scheduler)
                                                   llFindTxPowerSettings (ll_common)
                                                   llNonConnAdvEvt_TaskEndOk (ll_advEndCauses)
                                                   llScheduleTask (ll_scheduler)
                                                   llScheduler (ll_scheduler)
                                                   llSetT2OVFC2Event2 (ll_timer2)
                                                   memcpy (?memcpy)
                                                   osalAddTimer (OSAL_Timers)
                                                   osalClockUpdate (OSAL_ClockBLE)
                                                   osalTimeUpdate (OSAL_ClockBLE)
                                                   osalTimerUpdate (OSAL_Timers)
                                                   osal_CbTimerProcessEvent (osal_cbtimer)
                                                   osal_bm_alloc (osal_bufmgr)
                                                   osal_bm_free (osal_bufmgr)
                                                   osal_clear_event (OSAL)
                                                   osal_get_timeoutEx (OSAL_Timers)
                                                   osal_mem_alloc (OSAL_Memory)
                                                   osal_mem_free (OSAL_Memory)
                                                   osal_mem_kick (OSAL_Memory)
                                                   osal_memcmp (OSAL)
                                                   osal_memcpy (OSAL)
                                                   osal_memset (OSAL)
                                                   osal_msg_allocate (OSAL)
                                                   osal_msg_deallocate (OSAL)
                                                   osal_msg_enqueue (OSAL)
                                                   osal_msg_enqueue_push (OSAL)
                                                   osal_msg_extract (OSAL)
                                                   osal_msg_push_front (OSAL)
                                                   osal_msg_receive (OSAL)
                                                   osal_msg_send (OSAL)
                                                   osal_pwrmgr_task_state (OSAL_PwrMgr)
                                                   osal_run_system (OSAL)
                                                   osal_snv_read (osal_snv)
                                                   osal_snv_write (osal_snv)
                                                   osal_start_reload_timer (OSAL_Timers)
                                                   osal_start_timerEx (OSAL_Timers)
                                                   osal_stop_timerEx (OSAL_Timers)
                                                   phyFindWlEntry (phy)
                                                   usbdpGetConfigurationDesc (usb_descriptor_parser)
                                                   usbdpGetInterfaceDesc (usb_descriptor_parser)
                                                   usbdpGetStringDesc (usb_descriptor_parser)
                                                   usbfwInit (usb_framework)
                                                   usbfwReadFifo (usb_framework)
                                                   usbfwSetupHandler (usb_framework)
                                                   usbfwWriteFifo (usb_framework)
                                                   usbirqHandler (usb_interrupt)
                                                   usbirqInit (usb_interrupt)
                                                   usbsrGetDescriptor (usb_standard_requests)
                                                   usbsrGetInterface (usb_standard_requests)
                                                   usbsrSetConfiguration (usb_standard_requests)
                                                   usbsrSetInterface (usb_standard_requests)
                                                   verifyWordM (osal_snv)
                                                   writeItem (osal_snv)
                                                   writeWord (osal_snv)
                                                   writeWordM (osal_snv)
                                                   xferItem (osal_snv)
    -------------------------------------------------------------------------
VREG
  Relative segment, address: DATA 00000009 - 00000009 (0x1 bytes), align: 0
  Segment part 2.             Intra module refs:   ?V2
           ENTRY                   ADDRESS         REF BY
           =====                   =======         ======
           ?V1                     00000009        Application_UpdateRsp (simpleBLEBroadcaster)
                                                   ConfigureEndpoints (usb_standard_requests)
                                                   GAPRole_ProcessEvent (broadcaster)
                                                   GAPRole_SetParameter (broadcaster)
                                                   GAP_DeviceInit (gap)
                                                   GAP_ProcessEvent (gap_simpletask)
                                                   GAP_UpdateAdvertisingData (gap_peridevmgr)
                                                   HCI_CommandCompleteEvent (hci_event)
                                                   HCI_EXT_DecryptCmd (hci)
                                                   HCI_LE_EncryptCmd (hci)
                                                   HCI_ProcessEvent (hci_tl)
                                                   HCI_ReadLocalVersionInfoCmd (hci)
                                                   HCI_ReverseBytes (hci_data)
                                                   HCI_SendCommandCompleteEvent (hci_event)
                                                   HCI_SetEventMaskCmd (hci)
                                                   HCI_SetEventMaskPage2Cmd (hci_PATCH)
                                                   HCI_VendorSpecifcCommandCompleteEvent (hci_event_PATCH)
                                                   HalFlashRead (hal_flash)
                                                   HalLedBlink (hal_led)
                                                   HalLedSet (hal_led)
                                                   HalLedUpdate (hal_led)
                                                   HalUARTRead (hal_uart)
                                                   HalUARTWrite (hal_uart)
                                                   Hal_ProcessEvent (hal_drivers)
                                                   LL_DirectTestEnd (ll)
                                                   LL_ENC_GenerateTrueRandNum (ll_enc)
                                                   LL_EXT_Decrypt (ll)
                                                   LL_EXT_ExtendRfRange (ll)
                                                   LL_EXT_MapPmIoPort (ll)
                                                   LL_EXT_SaveFreqTune (ll)
                                                   LL_EXT_SetBDADDR (ll)
                                                   LL_EXT_SetRxGain (ll)
                                                   LL_EXT_SetTxPower (ll)
                                                   LL_Encrypt (ll)
                                                   LL_Init (ll)
                                                   LL_ProcessEvent (ll)
                                                   LL_RandCback (hci)
                                                   LL_SetAdvControl (ll)
                                                   LL_SetAdvData (ll)
                                                   LL_SetScanRspData (ll)
                                                   LL_TX_bm_alloc (ll)
                                                   NPI_ReadTransport (npi)
                                                   NPI_WriteTransport (npi)
                                                   OnBoard_SendKeys (OnBoard)
                                                   PHY_AddWlEntry (phy)
                                                   PHY_ClearBlacklistIndex (phy)
                                                   PHY_RemoveWlEntry (phy)
                                                   PHY_SetBlacklistIndex (phy)
                                                   PHY_SetCRCInit (phy)
                                                   PHY_SetSyncWord (phy)
                                                   RF_NormalIsr (ll_isr)
                                                   Segment part 131 (hci_tl)
                                                   Segment part 134 (ll)
                                                   Segment part 146 (ll)
                                                   Segment part 16 (ll_advEndCauses)
                                                   Segment part 26 (ll_scheduler)
                                                   Segment part 37 (hci_tl)
                                                   Segment part 38 (hci_tl)
                                                   Segment part 43 (hci_tl)
                                                   Segment part 65 (ll_common)
                                                   SerialInterface_ProcessEvent (serialInterface)
                                                   SimpleBLEBroadcaster_ProcessEvent (simpleBLEBroadcaster)
                                                   cSerialPacketParser (serialInterface)
                                                   compactPage (osal_snv)
                                                   findItem (osal_snv)
                                                   findOffset (osal_snv)
                                                   gapFindADType (gap_devmgr)
                                                   gapPeriProcessHCICmdCompleteEvt (gap_peridevmgr)
                                                   gapProcessAdvertisingEvt (gap_peridevmgr)
                                                   gapProcessHCICmdCompleteEvt (gap_simpletask)
                                                   gapReadBD_ADDRStatus (gap_configmgr)
                                                   gapReadBufSizeCmdStatus (gap_configmgr)
                                                   gapRole_ProcessGAPMsg (broadcaster)
                                                   gapRole_SetupGAP (broadcaster)
                                                   gapSendMakeDiscEvent (gap_peridevmgr)
                                                   gapSetAdvParams (gap_peridevmgr)
                                                   gapWriteAdvDataStatus (gap_peridevmgr)
                                                   gapWriteAdvEnableStatus (gap_peridevmgr)
                                                   halUartPollRx (hal_uart)
                                                   hciExtDecrypt (hci_tl)
                                                   hciLEEncrypt (hci_tl)
                                                   hciLESetAdvParam (hci_tl)
                                                   hciProcessCtrlToHost (hci_tl)
                                                   hciProcessHostToCtrlCmd (hci_tl)
                                                   hciSerialPacketParser (hci_tl)
                                                   initNV (osal_snv)
                                                   isLimitedDiscoverableMode (gap_peridevmgr)
                                                   ll24BitTimeCompare (ll_timer2)
                                                   ll24BitTimeDelta (ll_timer2)
                                                   llDiscoverableAdvEvt_TaskEndOk (ll_advEndCauses)
                                                   llFindNextSecTask (ll_scheduler)
                                                   llFindTxPowerSettings (ll_common)
                                                   llNonConnAdvEvt_TaskEndOk (ll_advEndCauses)
                                                   llScheduleTask (ll_scheduler)
                                                   llScheduler (ll_scheduler)
                                                   llSetT2OVFC2Event2 (ll_timer2)
                                                   memcpy (?memcpy)
                                                   osalAddTimer (OSAL_Timers)
                                                   osalClockUpdate (OSAL_ClockBLE)
                                                   osalTimeUpdate (OSAL_ClockBLE)
                                                   osalTimerUpdate (OSAL_Timers)
                                                   osal_CbTimerProcessEvent (osal_cbtimer)
                                                   osal_bm_free (osal_bufmgr)
                                                   osal_get_timeoutEx (OSAL_Timers)
                                                   osal_mem_alloc (OSAL_Memory)
                                                   osal_mem_free (OSAL_Memory)
                                                   osal_memcmp (OSAL)
                                                   osal_memcpy (OSAL)
                                                   osal_memset (OSAL)
                                                   osal_msg_allocate (OSAL)
                                                   osal_msg_deallocate (OSAL)
                                                   osal_msg_enqueue_push (OSAL)
                                                   osal_msg_extract (OSAL)
                                                   osal_msg_receive (OSAL)
                                                   osal_pwrmgr_task_state (OSAL_PwrMgr)
                                                   osal_run_system (OSAL)
                                                   osal_snv_read (osal_snv)
                                                   osal_snv_write (osal_snv)
                                                   osal_start_reload_timer (OSAL_Timers)
                                                   osal_start_timerEx (OSAL_Timers)
                                                   osal_stop_timerEx (OSAL_Timers)
                                                   phyFindWlEntry (phy)
                                                   usbdpGetConfigurationDesc (usb_descriptor_parser)
                                                   usbdpGetInterfaceDesc (usb_descriptor_parser)
                                                   usbdpGetStringDesc (usb_descriptor_parser)
                                                   usbfwInit (usb_framework)
                                                   usbfwReadFifo (usb_framework)
                                                   usbfwWriteFifo (usb_framework)
                                                   usbirqHandler (usb_interrupt)
                                                   usbirqInit (usb_interrupt)
                                                   usbsrGetDescriptor (usb_standard_requests)
                                                   usbsrGetInterface (usb_standard_requests)
                                                   usbsrSetConfiguration (usb_standard_requests)
                                                   usbsrSetInterface (usb_standard_requests)
                                                   verifyWordM (osal_snv)
                                                   writeItem (osal_snv)
                                                   writeWord (osal_snv)
                                                   writeWordM (osal_snv)
                                                   xferItem (osal_snv)
    -------------------------------------------------------------------------
VREG
  Relative segment, address: DATA 0000000A - 0000000A (0x1 bytes), align: 0
  Segment part 3.             Intra module refs:   ?V3
           ENTRY                   ADDRESS         REF BY
           =====                   =======         ======
           ?V2                     0000000A        Application_UpdateAdv (simpleBLEBroadcaster)
                                                   Application_UpdateRsp (simpleBLEBroadcaster)
                                                   ConfigureEndpoints (usb_standard_requests)
                                                   GAPRole_GetParameter (broadcaster)
                                                   GAPRole_ProcessEvent (broadcaster)
                                                   GAPRole_SetParameter (broadcaster)
                                                   GAP_DeviceInit (gap)
                                                   GAP_MakeDiscoverable (gap_peridevmgr)
                                                   GAP_ProcessEvent (gap_simpletask)
                                                   GAP_UpdateAdvertisingData (gap_peridevmgr)
                                                   HCI_CommandCompleteEvent (hci_event)
                                                   HCI_ReverseBytes (hci_data)
                                                   HCI_SendCommandCompleteEvent (hci_event)
                                                   HCI_VendorSpecifcCommandCompleteEvent (hci_event_PATCH)
                                                   HalFlashRead (hal_flash)
                                                   HalFlashWrite (hal_flash)
                                                   HalLedBlink (hal_led)
                                                   HalLedSet (hal_led)
                                                   HalLedUpdate (hal_led)
                                                   HalUARTRead (hal_uart)
                                                   HalUARTWrite (hal_uart)
                                                   Hal_ProcessEvent (hal_drivers)
                                                   LL_ENC_GenerateTrueRandNum (ll_enc)
                                                   LL_EXT_ExtendRfRange (ll)
                                                   LL_EXT_SaveFreqTune (ll)
                                                   LL_EXT_SetBDADDR (ll)
                                                   LL_EXT_SetRxGain (ll)
                                                   LL_EXT_SetTxPower (ll)
                                                   LL_Init (ll)
                                                   LL_ProcessEvent (ll)
                                                   LL_Rand (ll)
                                                   LL_SetAdvControl (ll)
                                                   OnBoard_SendKeys (OnBoard)
                                                   PHY_AddWlEntry (phy)
                                                   PHY_SetSyncWord (phy)
                                                   RF_NormalIsr (ll_isr)
                                                   Segment part 16 (ll_advEndCauses)
                                                   Segment part 34 (hci_tl)
                                                   Segment part 35 (hci_tl)
                                                   Segment part 36 (hci_tl)
                                                   Segment part 41 (hci_tl)
                                                   Segment part 42 (hci_tl)
                                                   Segment part 46 (hci_tl)
                                                   Segment part 50 (hci_event)
                                                   SerialInterface_ProcessEvent (serialInterface)
                                                   SimpleBLEBroadcaster_Init (simpleBLEBroadcaster)
                                                   SimpleBLEBroadcaster_ProcessEvent (simpleBLEBroadcaster)
                                                   cSerialPacketParser (serialInterface)
                                                   cleanErasedPage (osal_snv)
                                                   compactPage (osal_snv)
                                                   erasePage (osal_snv)
                                                   findItem (osal_snv)
                                                   findOffset (osal_snv)
                                                   gapFindADType (gap_devmgr)
                                                   gapProcessAdvertisingEvt (gap_peridevmgr)
                                                   gapProcessHCICmdCompleteEvt (gap_simpletask)
                                                   gapProcessRandomAddrComplete (gap_configmgr)
                                                   gapRole_ProcessGAPMsg (broadcaster)
                                                   gapSendDeviceInitDoneEvent (gap_configmgr)
                                                   gapSetAdvParams (gap_peridevmgr)
                                                   gapWriteAdvEnableStatus (gap_peridevmgr)
                                                   halUartPollRx (hal_uart)
                                                   hciProcessCtrlToHost (hci_tl)
                                                   hciProcessHostToCtrlCmd (hci_tl)
                                                   hciSerialPacketParser (hci_tl)
                                                   initNV (osal_snv)
                                                   ll24BitTimeCompare (ll_timer2)
                                                   ll24BitTimeDelta (ll_timer2)
                                                   llDiscoverableAdvEvt_TaskEndOk (ll_advEndCauses)
                                                   llFindNextSecTask (ll_scheduler)
                                                   llFindTxPowerSettings (ll_common)
                                                   llNonConnAdvEvt_TaskEndOk (ll_advEndCauses)
                                                   llScheduleTask (ll_scheduler)
                                                   llScheduler (ll_scheduler)
                                                   llSetT2OVFC2Event2 (ll_timer2)
                                                   osalAddTimer (OSAL_Timers)
                                                   osalClockUpdate (OSAL_ClockBLE)
                                                   osalTimeUpdate (OSAL_ClockBLE)
                                                   osalTimerUpdate (OSAL_Timers)
                                                   osal_CbTimerProcessEvent (osal_cbtimer)
                                                   osal_bm_alloc (osal_bufmgr)
                                                   osal_bm_free (osal_bufmgr)
                                                   osal_get_timeoutEx (OSAL_Timers)
                                                   osal_mem_alloc (OSAL_Memory)
                                                   osal_mem_free (OSAL_Memory)
                                                   osal_mem_kick (OSAL_Memory)
                                                   osal_memcmp (OSAL)
                                                   osal_memcpy (OSAL)
                                                   osal_memset (OSAL)
                                                   osal_msg_allocate (OSAL)
                                                   osal_msg_receive (OSAL)
                                                   osal_run_system (OSAL)
                                                   osal_snv_read (osal_snv)
                                                   osal_snv_write (osal_snv)
                                                   osal_start_reload_timer (OSAL_Timers)
                                                   osal_start_timerEx (OSAL_Timers)
                                                   osal_stop_timerEx (OSAL_Timers)
                                                   phyFindWlEntry (phy)
                                                   usbdpGetConfigurationDesc (usb_descriptor_parser)
                                                   usbdpGetInterfaceDesc (usb_descriptor_parser)
                                                   usbdpGetStringDesc (usb_descriptor_parser)
                                                   usbfwReadFifo (usb_framework)
                                                   usbfwWriteFifo (usb_framework)
                                                   usbsrGetDescriptor (usb_standard_requests)
                                                   usbsrGetInterface (usb_standard_requests)
                                                   usbsrSetConfiguration (usb_standard_requests)
                                                   verifyWordM (osal_snv)
                                                   writeItem (osal_snv)
                                                   writeWord (osal_snv)
                                                   writeWordM (osal_snv)
                                                   xferItem (osal_snv)
    -------------------------------------------------------------------------
VREG
  Relative segment, address: DATA 0000000B - 0000000B (0x1 bytes), align: 0
  Segment part 4.             Intra module refs:   ?V4
           ENTRY                   ADDRESS         REF BY
           =====                   =======         ======
           ?V3                     0000000B        Application_UpdateAdv (simpleBLEBroadcaster)
                                                   Application_UpdateRsp (simpleBLEBroadcaster)
                                                   ConfigureEndpoints (usb_standard_requests)
                                                   GAPRole_GetParameter (broadcaster)
                                                   GAPRole_SetParameter (broadcaster)
                                                   GAP_DeviceInit (gap)
                                                   GAP_MakeDiscoverable (gap_peridevmgr)
                                                   GAP_ProcessEvent (gap_simpletask)
                                                   GAP_UpdateAdvertisingData (gap_peridevmgr)
                                                   HCI_CommandCompleteEvent (hci_event)
                                                   HCI_ReverseBytes (hci_data)
                                                   HCI_SendCommandCompleteEvent (hci_event)
                                                   HCI_VendorSpecifcCommandCompleteEvent (hci_event_PATCH)
                                                   HalFlashRead (hal_flash)
                                                   HalFlashWrite (hal_flash)
                                                   HalLedBlink (hal_led)
                                                   HalLedUpdate (hal_led)
                                                   LL_ENC_GenerateTrueRandNum (ll_enc)
                                                   LL_EXT_ExtendRfRange (ll)
                                                   LL_EXT_SaveFreqTune (ll)
                                                   LL_EXT_SetBDADDR (ll)
                                                   LL_Init (ll)
                                                   LL_ProcessEvent (ll)
                                                   LL_Rand (ll)
                                                   LL_SetAdvControl (ll)
                                                   OnBoard_SendKeys (OnBoard)
                                                   PHY_AddWlEntry (phy)
                                                   PHY_SetSyncWord (phy)
                                                   RF_NormalIsr (ll_isr)
                                                   Segment part 16 (ll_advEndCauses)
                                                   Segment part 34 (hci_tl)
                                                   Segment part 35 (hci_tl)
                                                   Segment part 36 (hci_tl)
                                                   Segment part 40 (hci_tl)
                                                   Segment part 41 (hci_tl)
                                                   Segment part 46 (hci_tl)
                                                   SimpleBLEBroadcaster_Init (simpleBLEBroadcaster)
                                                   cleanErasedPage (osal_snv)
                                                   compactPage (osal_snv)
                                                   erasePage (osal_snv)
                                                   findItem (osal_snv)
                                                   findOffset (osal_snv)
                                                   gapFindADType (gap_devmgr)
                                                   gapProcessAdvertisingEvt (gap_peridevmgr)
                                                   gapProcessHCICmdCompleteEvt (gap_simpletask)
                                                   gapProcessRandomAddrComplete (gap_configmgr)
                                                   gapRole_ProcessGAPMsg (broadcaster)
                                                   gapSendDeviceInitDoneEvent (gap_configmgr)
                                                   gapSetAdvParams (gap_peridevmgr)
                                                   gapWriteAdvEnableStatus (gap_peridevmgr)
                                                   hciProcessCtrlToHost (hci_tl)
                                                   hciProcessHostToCtrlCmd (hci_tl)
                                                   hciSerialPacketParser (hci_tl)
                                                   initNV (osal_snv)
                                                   ll24BitTimeCompare (ll_timer2)
                                                   ll24BitTimeDelta (ll_timer2)
                                                   llDiscoverableAdvEvt_TaskEndOk (ll_advEndCauses)
                                                   llFindNextSecTask (ll_scheduler)
                                                   llFindTxPowerSettings (ll_common)
                                                   llNonConnAdvEvt_TaskEndOk (ll_advEndCauses)
                                                   llScheduleTask (ll_scheduler)
                                                   llScheduler (ll_scheduler)
                                                   llSetT2OVFC2Event2 (ll_timer2)
                                                   osalAddTimer (OSAL_Timers)
                                                   osalClockUpdate (OSAL_ClockBLE)
                                                   osalTimeUpdate (OSAL_ClockBLE)
                                                   osalTimerUpdate (OSAL_Timers)
                                                   osal_CbTimerProcessEvent (osal_cbtimer)
                                                   osal_bm_alloc (osal_bufmgr)
                                                   osal_bm_free (osal_bufmgr)
                                                   osal_get_timeoutEx (OSAL_Timers)
                                                   osal_mem_alloc (OSAL_Memory)
                                                   osal_mem_kick (OSAL_Memory)
                                                   osal_memcmp (OSAL)
                                                   osal_memcpy (OSAL)
                                                   osal_msg_allocate (OSAL)
                                                   osal_msg_receive (OSAL)
                                                   osal_snv_read (osal_snv)
                                                   osal_snv_write (osal_snv)
                                                   osal_start_reload_timer (OSAL_Timers)
                                                   osal_start_timerEx (OSAL_Timers)
                                                   osal_stop_timerEx (OSAL_Timers)
                                                   usbdpGetConfigurationDesc (usb_descriptor_parser)
                                                   usbdpGetStringDesc (usb_descriptor_parser)
                                                   verifyWordM (osal_snv)
                                                   writeItem (osal_snv)
                                                   writeWord (osal_snv)
                                                   writeWordM (osal_snv)
    -------------------------------------------------------------------------
VREG
  Relative segment, address: DATA 0000000C - 0000000C (0x1 bytes), align: 0
  Segment part 5.             Intra module refs:   ?V5
           ENTRY                   ADDRESS         REF BY
           =====                   =======         ======
           ?V4                     0000000C        ConfigureEndpoints (usb_standard_requests)
                                                   GAPRole_GetParameter (broadcaster)
                                                   GAPRole_ProcessEvent (broadcaster)
                                                   GAPRole_SetParameter (broadcaster)
                                                   GAP_UpdateAdvertisingData (gap_peridevmgr)
                                                   HCI_CommandCompleteEvent (hci_event)
                                                   HCI_SendCommandCompleteEvent (hci_event)
                                                   HCI_VendorSpecifcCommandCompleteEvent (hci_event_PATCH)
                                                   HalFlashRead (hal_flash)
                                                   HalLedBlink (hal_led)
                                                   HalLedUpdate (hal_led)
                                                   Hal_ProcessEvent (hal_drivers)
                                                   LL_EXT_ExtendRfRange (ll)
                                                   LL_EXT_SetBDADDR (ll)
                                                   LL_EXT_SetRxGain (ll)
                                                   LL_EXT_SetTxPower (ll)
                                                   PHY_SetCRCInit (phy)
                                                   PHY_SetSyncWord (phy)
                                                   Segment part 16 (ll_advEndCauses)
                                                   Segment part 20 (ll_advEndCauses)
                                                   Segment part 46 (gap_peridevmgr)
                                                   SerialInterface_ProcessEvent (serialInterface)
                                                   SimpleBLEBroadcaster_ProcessEvent (simpleBLEBroadcaster)
                                                   cSerialPacketParser (serialInterface)
                                                   compactPage (osal_snv)
                                                   gapFindADType (gap_devmgr)
                                                   gapRole_ProcessGAPMsg (broadcaster)
                                                   gapSetAdvParams (gap_peridevmgr)
                                                   gapWriteAdvEnableStatus (gap_peridevmgr)
                                                   hciProcessHostToCtrlCmd (hci_tl)
                                                   hciSerialPacketParser (hci_tl)
                                                   ll24BitTimeCompare (ll_timer2)
                                                   ll24BitTimeDelta (ll_timer2)
                                                   llDiscoverableAdvEvt_TaskEndOk (ll_advEndCauses)
                                                   llFindNextSecTask (ll_scheduler)
                                                   llFindTxPowerSettings (ll_common)
                                                   llNonConnAdvEvt_TaskEndOk (ll_advEndCauses)
                                                   llScheduleTask (ll_scheduler)
                                                   llScheduler (ll_scheduler)
                                                   osalAddTimer (OSAL_Timers)
                                                   osalTimeUpdate (OSAL_ClockBLE)
                                                   osalTimerUpdate (OSAL_Timers)
                                                   osal_CbTimerProcessEvent (osal_cbtimer)
                                                   osal_bm_alloc (osal_bufmgr)
                                                   osal_bm_free (osal_bufmgr)
                                                   osal_get_timeoutEx (OSAL_Timers)
                                                   osal_mem_alloc (OSAL_Memory)
                                                   osal_memcmp (OSAL)
                                                   osal_msg_receive (OSAL)
                                                   osal_run_system (OSAL)
                                                   osal_snv_read (osal_snv)
                                                   osal_snv_write (osal_snv)
                                                   osal_start_reload_timer (OSAL_Timers)
                                                   osal_start_timerEx (OSAL_Timers)
                                                   osal_stop_timerEx (OSAL_Timers)
                                                   usbdpGetInterfaceDesc (usb_descriptor_parser)
                                                   usbfwSetupHandler (usb_framework)
                                                   usbsrSetConfiguration (usb_standard_requests)
                                                   verifyWordM (osal_snv)
                                                   writeItem (osal_snv)
                                                   writeWord (osal_snv)
                                                   writeWordM (osal_snv)
                                                   xferItem (osal_snv)
    -------------------------------------------------------------------------
VREG
  Relative segment, address: DATA 0000000D - 0000000D (0x1 bytes), align: 0
  Segment part 6.             Intra module refs:   ?V6
           ENTRY                   ADDRESS         REF BY
           =====                   =======         ======
           ?V5                     0000000D        ConfigureEndpoints (usb_standard_requests)
                                                   GAPRole_GetParameter (broadcaster)
                                                   GAPRole_ProcessEvent (broadcaster)
                                                   GAPRole_SetParameter (broadcaster)
                                                   HCI_CommandCompleteEvent (hci_event)
                                                   HCI_SendCommandCompleteEvent (hci_event)
                                                   HCI_VendorSpecifcCommandCompleteEvent (hci_event_PATCH)
                                                   HalLedBlink (hal_led)
                                                   HalLedUpdate (hal_led)
                                                   Hal_ProcessEvent (hal_drivers)
                                                   LL_EXT_ExtendRfRange (ll)
                                                   LL_EXT_SetRxGain (ll)
                                                   LL_EXT_SetTxPower (ll)
                                                   PHY_SetCRCInit (phy)
                                                   PHY_SetSyncWord (phy)
                                                   Segment part 20 (ll_advEndCauses)
                                                   SerialInterface_ProcessEvent (serialInterface)
                                                   SimpleBLEBroadcaster_ProcessEvent (simpleBLEBroadcaster)
                                                   cSerialPacketParser (serialInterface)
                                                   gapFindADType (gap_devmgr)
                                                   gapRole_ProcessGAPMsg (broadcaster)
                                                   gapSetAdvParams (gap_peridevmgr)
                                                   gapWriteAdvEnableStatus (gap_peridevmgr)
                                                   hciProcessHostToCtrlCmd (hci_tl)
                                                   hciSerialPacketParser (hci_tl)
                                                   ll24BitTimeCompare (ll_timer2)
                                                   ll24BitTimeDelta (ll_timer2)
                                                   llDiscoverableAdvEvt_TaskEndOk (ll_advEndCauses)
                                                   llFindNextSecTask (ll_scheduler)
                                                   llFindTxPowerSettings (ll_common)
                                                   llNonConnAdvEvt_TaskEndOk (ll_advEndCauses)
                                                   llScheduleTask (ll_scheduler)
                                                   llScheduler (ll_scheduler)
                                                   osalAddTimer (OSAL_Timers)
                                                   osalTimeUpdate (OSAL_ClockBLE)
                                                   osalTimerUpdate (OSAL_Timers)
                                                   osal_CbTimerProcessEvent (osal_cbtimer)
                                                   osal_bm_alloc (osal_bufmgr)
                                                   osal_get_timeoutEx (OSAL_Timers)
                                                   osal_mem_alloc (OSAL_Memory)
                                                   osal_memcmp (OSAL)
                                                   osal_msg_receive (OSAL)
                                                   osal_run_system (OSAL)
                                                   osal_snv_read (osal_snv)
                                                   osal_snv_write (osal_snv)
                                                   osal_start_reload_timer (OSAL_Timers)
                                                   osal_start_timerEx (OSAL_Timers)
                                                   osal_stop_timerEx (OSAL_Timers)
                                                   usbdpGetInterfaceDesc (usb_descriptor_parser)
                                                   usbfwSetupHandler (usb_framework)
                                                   usbsrSetConfiguration (usb_standard_requests)
                                                   writeItem (osal_snv)
                                                   writeWord (osal_snv)
                                                   writeWordM (osal_snv)
                                                   xferItem (osal_snv)
    -------------------------------------------------------------------------
VREG
  Relative segment, address: DATA 0000000E - 0000000E (0x1 bytes), align: 0
  Segment part 7.             Intra module refs:   ?V7
           ENTRY                   ADDRESS         REF BY
           =====                   =======         ======
           ?V6                     0000000E        ConfigureEndpoints (usb_standard_requests)
                                                   GAPRole_SetParameter (broadcaster)
                                                   GAP_UpdateAdvertisingData (gap_peridevmgr)
                                                   HCI_CommandCompleteEvent (hci_event)
                                                   HCI_VendorSpecifcCommandCompleteEvent (hci_event_PATCH)
                                                   HalLedUpdate (hal_led)
                                                   LL_EXT_ExtendRfRange (ll)
                                                   LL_EXT_SetRxGain (ll)
                                                   LL_EXT_SetTxPower (ll)
                                                   PHY_SetCRCInit (phy)
                                                   PHY_SetSyncWord (phy)
                                                   Segment part 20 (ll_advEndCauses)
                                                   cSerialPacketParser (serialInterface)
                                                   compactPage (osal_snv)
                                                   gapFindADType (gap_devmgr)
                                                   gapRole_ProcessGAPMsg (broadcaster)
                                                   gapWriteAdvEnableStatus (gap_peridevmgr)
                                                   hciProcessHostToCtrlCmd (hci_tl)
                                                   ll24BitTimeCompare (ll_timer2)
                                                   ll24BitTimeDelta (ll_timer2)
                                                   llDiscoverableAdvEvt_TaskEndOk (ll_advEndCauses)
                                                   llFindNextSecTask (ll_scheduler)
                                                   llFindTxPowerSettings (ll_common)
                                                   llNonConnAdvEvt_TaskEndOk (ll_advEndCauses)
                                                   llScheduleTask (ll_scheduler)
                                                   llScheduler (ll_scheduler)
                                                   osalAddTimer (OSAL_Timers)
                                                   osalTimerUpdate (OSAL_Timers)
                                                   osal_CbTimerProcessEvent (osal_cbtimer)
                                                   osal_get_timeoutEx (OSAL_Timers)
                                                   osal_mem_alloc (OSAL_Memory)
                                                   osal_memcmp (OSAL)
                                                   osal_snv_write (osal_snv)
                                                   osal_start_reload_timer (OSAL_Timers)
                                                   osal_start_timerEx (OSAL_Timers)
                                                   usbfwSetupHandler (usb_framework)
                                                   verifyWordM (osal_snv)
                                                   writeItem (osal_snv)
                                                   writeWord (osal_snv)
                                                   writeWordM (osal_snv)
                                                   xferItem (osal_snv)
    -------------------------------------------------------------------------
VREG
  Relative segment, address: DATA 0000000F - 0000000F (0x1 bytes), align: 0
  Segment part 8.             Intra module refs:   ?V8
           ENTRY                   ADDRESS         REF BY
           =====                   =======         ======
           ?V7                     0000000F        ConfigureEndpoints (usb_standard_requests)
                                                   GAPRole_SetParameter (broadcaster)
                                                   GAP_UpdateAdvertisingData (gap_peridevmgr)
                                                   HCI_CommandCompleteEvent (hci_event)
                                                   HalLedUpdate (hal_led)
                                                   LL_EXT_ExtendRfRange (ll)
                                                   LL_EXT_SetRxGain (ll)
                                                   LL_EXT_SetTxPower (ll)
                                                   PHY_SetCRCInit (phy)
                                                   PHY_SetSyncWord (phy)
                                                   Segment part 20 (ll_advEndCauses)
                                                   cSerialPacketParser (serialInterface)
                                                   compactPage (osal_snv)
                                                   gapRole_ProcessGAPMsg (broadcaster)
                                                   gapWriteAdvEnableStatus (gap_peridevmgr)
                                                   ll24BitTimeCompare (ll_timer2)
                                                   ll24BitTimeDelta (ll_timer2)
                                                   llDiscoverableAdvEvt_TaskEndOk (ll_advEndCauses)
                                                   llFindNextSecTask (ll_scheduler)
                                                   llNonConnAdvEvt_TaskEndOk (ll_advEndCauses)
                                                   llScheduleTask (ll_scheduler)
                                                   llScheduler (ll_scheduler)
                                                   osalTimerUpdate (OSAL_Timers)
                                                   osal_get_timeoutEx (OSAL_Timers)
                                                   osal_snv_write (osal_snv)
                                                   osal_start_reload_timer (OSAL_Timers)
                                                   osal_start_timerEx (OSAL_Timers)
                                                   verifyWordM (osal_snv)
                                                   writeItem (osal_snv)
                                                   writeWord (osal_snv)
                                                   writeWordM (osal_snv)
                                                   xferItem (osal_snv)
    -------------------------------------------------------------------------
VREG
  Relative segment, address: DATA 00000010 - 00000010 (0x1 bytes), align: 0
  Segment part 9.             Intra module refs:   ?V9
           ENTRY                   ADDRESS         REF BY
           =====                   =======         ======
           ?V8                     00000010        ConfigureEndpoints (usb_standard_requests)
                                                   GAPRole_SetParameter (broadcaster)
                                                   GAP_UpdateAdvertisingData (gap_peridevmgr)
                                                   HCI_CommandCompleteEvent (hci_event)
                                                   HCI_VendorSpecifcCommandCompleteEvent (hci_event_PATCH)
                                                   HalLedUpdate (hal_led)
                                                   ll24BitTimeDelta (ll_timer2)
                                                   llFindNextSecTask (ll_scheduler)
                                                   llFindTxPowerSettings (ll_common)
                                                   osalAddTimer (OSAL_Timers)
                                                   osalTimerUpdate (OSAL_Timers)
                                                   osal_CbTimerProcessEvent (osal_cbtimer)
                                                   osal_get_timeoutEx (OSAL_Timers)
                                                   osal_snv_write (osal_snv)
                                                   osal_start_reload_timer (OSAL_Timers)
                                                   osal_start_timerEx (OSAL_Timers)
                                                   writeWord (osal_snv)
                                                   writeWordM (osal_snv)
                                                   xferItem (osal_snv)
    -------------------------------------------------------------------------
VREG
  Relative segment, address: DATA 00000011 - 00000011 (0x1 bytes), align: 0
  Segment part 10.            Intra module refs:   ?V10
           ENTRY                   ADDRESS         REF BY
           =====                   =======         ======
           ?V9                     00000011        GAPRole_SetParameter (broadcaster)
                                                   GAP_UpdateAdvertisingData (gap_peridevmgr)
                                                   HCI_CommandCompleteEvent (hci_event)
                                                   HCI_VendorSpecifcCommandCompleteEvent (hci_event_PATCH)
                                                   HalLedUpdate (hal_led)
                                                   ll24BitTimeDelta (ll_timer2)
                                                   llFindNextSecTask (ll_scheduler)
                                                   llFindTxPowerSettings (ll_common)
                                                   osalAddTimer (OSAL_Timers)
                                                   osalTimerUpdate (OSAL_Timers)
                                                   osal_CbTimerProcessEvent (osal_cbtimer)
                                                   osal_get_timeoutEx (OSAL_Timers)
                                                   osal_snv_write (osal_snv)
                                                   osal_start_reload_timer (OSAL_Timers)
                                                   osal_start_timerEx (OSAL_Timers)
                                                   writeWord (osal_snv)
                                                   writeWordM (osal_snv)
                                                   xferItem (osal_snv)
    -------------------------------------------------------------------------
VREG
  Relative segment, address: DATA 00000012 - 00000012 (0x1 bytes), align: 0
  Segment part 11.            Intra module refs:   ?V11
           ENTRY                   ADDRESS         REF BY
           =====                   =======         ======
           ?V10                    00000012        ConfigureEndpoints (usb_standard_requests)
                                                   HalLedUpdate (hal_led)
                                                   ll24BitTimeDelta (ll_timer2)
                                                   osalAddTimer (OSAL_Timers)
                                                   osalTimerUpdate (OSAL_Timers)
                                                   osal_get_timeoutEx (OSAL_Timers)
    -------------------------------------------------------------------------
VREG
  Relative segment, address: DATA 00000013 - 00000013 (0x1 bytes), align: 0
  Segment part 12.            Intra module refs:   ?V12
           ENTRY                   ADDRESS         REF BY
           =====                   =======         ======
           ?V11                    00000013        ConfigureEndpoints (usb_standard_requests)
                                                   HalLedUpdate (hal_led)
                                                   ll24BitTimeDelta (ll_timer2)
                                                   osalAddTimer (OSAL_Timers)
                                                   osalTimerUpdate (OSAL_Timers)
                                                   osal_get_timeoutEx (OSAL_Timers)
    -------------------------------------------------------------------------
VREG
  Relative segment, address: DATA 00000014 - 00000014 (0x1 bytes), align: 0
  Segment part 13.            Intra module refs:   ?V13
           ENTRY                   ADDRESS         REF BY
           =====                   =======         ======
           ?V12                    00000014        HalLedUpdate (hal_led)
                                                   osalTimerUpdate (OSAL_Timers)
    -------------------------------------------------------------------------
VREG
  Relative segment, address: DATA 00000015 - 00000015 (0x1 bytes), align: 0
  Segment part 14.            Intra module refs:   ?V14
           ENTRY                   ADDRESS         REF BY
           =====                   =======         ======
           ?V13                    00000015        HalLedUpdate (hal_led)
                                                   osalTimerUpdate (OSAL_Timers)
    -------------------------------------------------------------------------
VREG
  Relative segment, address: DATA 00000016 - 00000016 (0x1 bytes), align: 0
  Segment part 15.            Intra module refs:   ?V15
           ENTRY                   ADDRESS         REF BY
           =====                   =======         ======
           ?V14                    00000016        HalLedUpdate (hal_led)
    -------------------------------------------------------------------------
VREG
  Relative segment, address: DATA 00000017 - 00000017 (0x1 bytes), align: 0
  Segment part 16.
           ENTRY                   ADDRESS         REF BY
           =====                   =======         ======
           ?V15                    00000017        HalLedUpdate (hal_led)
    -------------------------------------------------------------------------
XSP
  Relative segment, address: DATA 00000018 - 00000019 (0x2 bytes), align: 0
  Segment part 34.
           ENTRY                   ADDRESS         REF BY
           =====                   =======         ======
           ?XSP                    00000018        ?ADD_XSTACK_DISP0_8 (?ADD_XSTACK_DISP8)
                                                   ?ALLOC_XSTACK8 (?ALLOC_XSTACK8)
                                                   ?BANKED_ENTER_XDATA (?BANKED_ENTER_XDATA)
                                                   ?BANKED_LEAVE_XDATA (?BANKED_LEAVE_XDATA)
                                                   ?DEALLOC_XSTACK8 (?DEALLOC_XSTACK8)
                                                   ?FUNC_ENTER_XDATA (?FUNC_ENTER_XDATA)
                                                   ?FUNC_LEAVE_XDATA (?FUNC_LEAVE_XDATA)
                                                   ?INTERRUPT_ENTER_XSP (?INTERRUPT_ENTER_XSP)
                                                   ?INTERRUPT_LEAVE_XSP (?INTERRUPT_LEAVE_XSP)
                                                   ?PUSH_XSTACK8_X (?PUSH_XSTACK8_X)
                                                   ?RESET_XSP (CSTARTUP)
                                                   ?XSTACK_DISP0_8 (?XSTACK_DISP8)
                                                   ?XSTACK_DISP100_8 (?XSTACK_DISP8_RP)
                                                   ?XSTACK_DISP101_8 (?XSTACK_DISP8_RP)
                                                   ?XSTACK_DISP102_8 (?XSTACK_DISP8_RP)
                                                   Application_StartAdvertise (simpleBLEBroadcaster)
                                                   Application_StopAdvertise (simpleBLEBroadcaster)
                                                   GAPRole_ProcessEvent (broadcaster)
                                                   HCI_EXT_BuildRevisionCmd (hci)
                                                   HCI_EXT_ClkDivOnHaltCmd (hci)
                                                   HCI_EXT_DeclareNvUsageCmd (hci)
                                                   HCI_EXT_DecryptCmd (hci)
                                                   HCI_EXT_DelaySleepCmd (hci_PATCH)
                                                   HCI_EXT_EndModemTestCmd (hci)
                                                   HCI_EXT_ExtendRfRangeCmd (hci)
                                                   HCI_EXT_HaltDuringRfCmd (hci)
                                                   HCI_EXT_MapPmIoPortCmd (hci)
                                                   HCI_EXT_ModemHopTestTxCmd (hci)
                                                   HCI_EXT_ModemTestRxCmd (hci)
                                                   HCI_EXT_ModemTestTxCmd (hci)
                                                   HCI_EXT_ResetSystemCmd (hci_PATCH)
                                                   HCI_EXT_SaveFreqTuneCmd (hci)
                                                   HCI_EXT_SetBDADDRCmd (hci)
                                                   HCI_EXT_SetFreqTuneCmd (hci)
                                                   HCI_EXT_SetLocalSupportedFeaturesCmd (hci)
                                                   HCI_EXT_SetMaxDtmTxPowerCmd (hci)
                                                   HCI_EXT_SetRxGainCmd (hci)
                                                   HCI_EXT_SetTxPowerCmd (hci)
                                                   HCI_LE_EncryptCmd (hci)
                                                   HCI_LE_RandCmd (hci)
                                                   HCI_LE_ReadBufSizeCmd (hci_PATCH)
                                                   HCI_LE_ReadLocalSupportedFeaturesCmd (hci)
                                                   HCI_LE_ReadSupportedStatesCmd (hci)
                                                   HCI_LE_SetEventMaskCmd (hci)
                                                   HCI_LE_SetRandomAddressCmd (hci)
                                                   HCI_LE_TestEndCmd (hci)
                                                   HCI_ReadLocalSupportedFeaturesCmd (hci)
                                                   HCI_ReadRssiCmd (hci)
                                                   HCI_ResetCmd (hci_PATCH)
                                                   HCI_SetEventMaskCmd (hci)
                                                   HCI_SetEventMaskPage2Cmd (hci_PATCH)
                                                   HalLedUpdate (hal_led)
                                                   LL_DirectTestEndDoneCback (hci_event)
                                                   LL_EXT_ExtendRfRangeCback (hci)
                                                   LL_EXT_SaveFreqTune (ll)
                                                   LL_EXT_SetRxGainCback (hci)
                                                   LL_EXT_SetTxPowerCback (hci)
                                                   LL_RandCback (hci)
                                                   LL_ReadLocalVersionInfo (ll)
                                                   NPI_InitTransport (npi)
                                                   PHY_RawGetRxData (phy)
                                                   Segment part 21 (hci_PATCH)
                                                   Segment part 35 (ll_timer2)
                                                   Segment part 38 (ll_timer2)
                                                   Segment part 40 (ll_timer2)
                                                   Segment part 41 (ll_timer2)
                                                   Segment part 47 (hci)
                                                   Segment part 49 (hci)
                                                   Segment part 49 (ll_timer2)
                                                   Segment part 54 (hci)
                                                   Segment part 55 (ll_timer2)
                                                   Segment part 63 (ll_timer2)
                                                   Segment part 81 (hci)
                                                   SimpleBLEBroadcaster_Init (simpleBLEBroadcaster)
                                                   cleanErasedPage (osal_snv)
                                                   compactPage (osal_snv)
                                                   erasePage (osal_snv)
                                                   findItem (osal_snv)
                                                   findOffset (osal_snv)
                                                   hciProcessHostToCtrlCmd (hci_tl)
                                                   initNV (osal_snv)
                                                   llFindTxPowerSettings (ll_common)
                                                   llProcessPostRfOps (ll_common)
                                                   llSetT2Delta (ll_timer2)
                                                   llSetT2OVFC2Event2 (ll_timer2)
                                                   ll_McuPrecisionCount (ll_timer2)
                                                   memset (?memset)
                                                   osalTimerUpdate (OSAL_Timers)
                                                   osal_snv_write (osal_snv)
                                                   peripheralStateNotificationCB (simpleBLEBroadcaster)
                                                   setActivePage (osal_snv)
                                                   setXferPage (osal_snv)
                                                   usbdpGetStringDesc (usb_descriptor_parser)
                                                   writeItem (osal_snv)
                                                   xferItem (osal_snv)

    -------------------------------------------------------------------------
  LIBRARY MODULE, NAME : ?BANKED_CODE_SUPPORT

  SEGMENTS IN THE MODULE
  ======================
CSTART
  Relative segment, address: CODE 00000119 - 00000136 (0x1e bytes), align: 0
  Segment part 0.
           ENTRY                   ADDRESS         REF BY
           =====                   =======         ======
           ?BCALL_FF               00000119        ?call_main (?cmain)
           ?BRET_FF                0000011F        ?BANKED_LEAVE_XDATA (?BANKED_LEAVE_XDATA)
                                                   Application_StartAdvertise (simpleBLEBroadcaster)
                                                   Application_StopAdvertise (simpleBLEBroadcaster)
                                                   GAP_NumActiveConnections (gap_simpletask)
                                                   HalAdcInit (hal_adc)
                                                   HalAesInit (hal_aes)
                                                   HalDmaInit (hal_dma)
                                                   HalDriverInit (hal_drivers)
                                                   HalFlashErase (hal_flash)
                                                   HalKeyConfig (hal_key)
                                                   HalLedInit (hal_led)
                                                   HalLedOnOff (hal_led)
                                                   HalUARTInit (hal_uart)
                                                   HalUARTOpenUSB (hal_uart)
                                                   HalUARTPoll (hal_uart)
                                                   HalUARTPollUSB (hal_uart)
                                                   HalUARTRxAvailUSB (hal_uart)
                                                   HalUARTTx (hal_uart)
                                                   Hal_Init (hal_drivers)
                                                   Hal_ProcessPoll (hal_drivers)
                                                   LL_DirectTestEndDoneCback (hci_event)
                                                   LL_ENC_StartAES (ll_enc)
                                                   NPI_GetMaxRxBufSize (npi)
                                                   NPI_RxBufLen (npi)
                                                   PHY_Command (phy)
                                                   PHY_GetWlSize (phy)
                                                   Segment part 104 (hci_tl)
                                                   Segment part 184 (phy)
                                                   Segment part 25 (hci_PATCH)
                                                   Segment part 32 (gap_simpletask)
                                                   Segment part 32 (ll_enc)
                                                   Segment part 33 (gap_peridevmgr)
                                                   Segment part 38 (ll_scheduler)
                                                   Segment part 41 (gap_configmgr)
                                                   Segment part 44 (ll_timer2)
                                                   Segment part 60 (ll_common)
                                                   Segment part 73 (ll)
                                                   Segment part 74 (ll_timer2)
                                                   Segment part 95 (hci)
                                                   SerialInterface_ProcessOSALMsg (serialInterface)
                                                   aesDmaInit (hal_aes)
                                                   gapValidADType (gap_devmgr)
                                                   halAssertHandler (hal_assert)
                                                   halUartPollEvt (hal_uart)
                                                   hciInitEventMasks (hci_event_PATCH)
                                                   llAdvEvt_TaskAbort (ll_advEndCauses)
                                                   llClearRfInts (ll_common)
                                                   llUnexpectedEndCauseHandler (ll_errorEndCauses)
                                                   main (SimpleBLEBroadcaster_Main)
                                                   memset (?memset)
                                                   osalDeleteTimer (OSAL_Timers)
                                                   osal_GetSystemClock (OSAL_Timers)
                                                   osal_init_system (OSAL)
                                                   osal_int_disable (OSAL)
                                                   osal_mem_init (OSAL_Memory)
                                                   osal_pwrmgr_device (OSAL_PwrMgr)
                                                   osal_pwrmgr_init (OSAL_PwrMgr)
                                                   osal_snv_init (osal_snv)
                                                   simpleBLEBroadcaster_ProcessOSALMsg (simpleBLEBroadcaster)
                                                   usbcrHookProcessIn (usb_cdc_hooks)
                                                   usbcrHookProcessOut (usb_cdc_hooks)
                                                   usbdpFindNext (usb_descriptor_parser)
                                                   usbdpGetDeviceDesc (usb_descriptor_parser)
                                                   usbdpInit (usb_descriptor_parser)
                                                   usbfwResetHandler (usb_framework)
                                                   usbfwSetAllEpStatus (usb_framework)
                                                   usbirqHookProcessEvents (usb_cdc_hooks)
                                                   usbsrClearFeature (usb_standard_requests)
                                                   usbsrGetConfiguration (usb_standard_requests)
                                                   usbsrGetStatus (usb_standard_requests)
                                                   usbsrHookClearFeature (usb_cdc_hooks)
                                                   usbsrHookProcessEvent (usb_cdc_hooks)
                                                   usbsrHookSetFeature (usb_cdc_hooks)
                                                   usbsrSetAddress (usb_standard_requests)
                                                   usbsrSetFeature (usb_standard_requests)
                                                   usbvrHookProcessIn (usb_cdc_hooks)
                                                   usbvrHookProcessOut (usb_cdc_hooks)
           ?BDISPATCH_FF           00000122        Application_StartAdvertise::?relay (simpleBLEBroadcaster)
                                                   Application_StopAdvertise::?relay (simpleBLEBroadcaster)
                                                   Application_UpdateAdv::?relay (simpleBLEBroadcaster)
                                                   Application_UpdateRsp::?relay (simpleBLEBroadcaster)
                                                   ChangeFeature::?relay (usb_standard_requests)
                                                   ConfigureEndpoints::?relay (usb_standard_requests)
                                                   GAPRole_GetParameter::?relay (broadcaster)
                                                   GAPRole_Init::?relay (broadcaster)
                                                   GAPRole_ProcessEvent::?relay (broadcaster)
                                                   GAPRole_SetParameter::?relay (broadcaster)
                                                   GAPRole_StartDevice::?relay (broadcaster)
                                                   GAP_DeviceInit::?relay (gap)
                                                   GAP_EndDiscoverable::?relay (gap_peridevmgr)
                                                   GAP_GetParamValue::?relay (gap_configmgr)
                                                   GAP_Init::?relay (gap_simpletask)
                                                   GAP_MakeDiscoverable::?relay (gap_peridevmgr)
                                                   GAP_NumActiveConnections::?relay (gap_simpletask)
                                                   GAP_ParamsInit::?relay (gap_configmgr)
                                                   GAP_PeriDevMgrInit::?relay (gap_peridevmgr)
                                                   GAP_ProcessEvent::?relay (gap_simpletask)
                                                   GAP_RegisterForMsgs::?relay (gap_simpletask)
                                                   GAP_SetParamValue::?relay (gap_configmgr)
                                                   GAP_UpdateAdvertisingData::?relay (gap_peridevmgr)
                                                   HCI_CommandCompleteEvent::?relay (hci_event)
                                                   HCI_EXT_BuildRevisionCmd::?relay (hci)
                                                   HCI_EXT_ClkDivOnHaltCmd::?relay (hci)
                                                   HCI_EXT_DeclareNvUsageCmd::?relay (hci)
                                                   HCI_EXT_DecryptCmd::?relay (hci)
                                                   HCI_EXT_DelaySleepCmd::?relay (hci_PATCH)
                                                   HCI_EXT_EndModemTestCmd::?relay (hci)
                                                   HCI_EXT_ExtendRfRangeCmd::?relay (hci)
                                                   HCI_EXT_HaltDuringRfCmd::?relay (hci)
                                                   HCI_EXT_MapPmIoPortCmd::?relay (hci)
                                                   HCI_EXT_ModemHopTestTxCmd::?relay (hci)
                                                   HCI_EXT_ModemTestRxCmd::?relay (hci)
                                                   HCI_EXT_ModemTestTxCmd::?relay (hci)
                                                   HCI_EXT_ResetSystemCmd::?relay (hci_PATCH)
                                                   HCI_EXT_SaveFreqTuneCmd::?relay (hci)
                                                   HCI_EXT_SetBDADDRCmd::?relay (hci)
                                                   HCI_EXT_SetFreqTuneCmd::?relay (hci)
                                                   HCI_EXT_SetLocalSupportedFeaturesCmd::?relay (hci)
                                                   HCI_EXT_SetMaxDtmTxPowerCmd::?relay (hci)
                                                   HCI_EXT_SetRxGainCmd::?relay (hci)
                                                   HCI_EXT_SetTxPowerCmd::?relay (hci)
                                                   HCI_GAPTaskRegister::?relay (hci_tl)
                                                   HCI_Init::?relay (hci_tl)
                                                   HCI_LE_AddWhiteListCmd::?relay (hci)
                                                   HCI_LE_ClearWhiteListCmd::?relay (hci)
                                                   HCI_LE_EncryptCmd::?relay (hci)
                                                   HCI_LE_RandCmd::?relay (hci)
                                                   HCI_LE_ReadAdvChanTxPowerCmd::?relay (hci)
                                                   HCI_LE_ReadBufSizeCmd::?relay (hci_PATCH)
                                                   HCI_LE_ReadLocalSupportedFeaturesCmd::?relay (hci)
                                                   HCI_LE_ReadSupportedStatesCmd::?relay (hci)
                                                   HCI_LE_ReadWhiteListSizeCmd::?relay (hci)
                                                   HCI_LE_ReceiverTestCmd::?relay (hci)
                                                   HCI_LE_RemoveWhiteListCmd::?relay (hci)
                                                   HCI_LE_SetAdvDataCmd::?relay (hci)
                                                   HCI_LE_SetAdvEnableCmd::?relay (hci)
                                                   HCI_LE_SetAdvParamCmd::?relay (hci)
                                                   HCI_LE_SetEventMaskCmd::?relay (hci)
                                                   HCI_LE_SetRandomAddressCmd::?relay (hci)
                                                   HCI_LE_SetScanRspDataCmd::?relay (hci)
                                                   HCI_LE_TestEndCmd::?relay (hci)
                                                   HCI_LE_TransmitterTestCmd::?relay (hci)
                                                   HCI_ProcessEvent::?relay (hci_tl)
                                                   HCI_ReadBDADDRCmd::?relay (hci)
                                                   HCI_ReadLocalSupportedCommandsCmd::?relay (hci_PATCH)
                                                   HCI_ReadLocalSupportedFeaturesCmd::?relay (hci)
                                                   HCI_ReadLocalVersionInfoCmd::?relay (hci)
                                                   HCI_ReadRssiCmd::?relay (hci)
                                                   HCI_ResetCmd::?relay (hci_PATCH)
                                                   HCI_ReverseBytes::?relay (hci_data)
                                                   HCI_SendCommandCompleteEvent::?relay (hci_event)
                                                   HCI_SetEventMaskCmd::?relay (hci)
                                                   HCI_SetEventMaskPage2Cmd::?relay (hci_PATCH)
                                                   HCI_VendorSpecifcCommandCompleteEvent::?relay (hci_event_PATCH)
                                                   HCI_bm_alloc::?relay (hci)
                                                   HalAdcInit::?relay (hal_adc)
                                                   HalAesInit::?relay (hal_aes)
                                                   HalDmaInit::?relay (hal_dma)
                                                   HalDriverInit::?relay (hal_drivers)
                                                   HalFlashErase::?relay (hal_flash)
                                                   HalFlashRead::?relay (hal_flash)
                                                   HalFlashWrite::?relay (hal_flash)
                                                   HalKeyConfig::?relay (hal_key)
                                                   HalLedBlink::?relay (hal_led)
                                                   HalLedInit::?relay (hal_led)
                                                   HalLedOnOff::?relay (hal_led)
                                                   HalLedSet::?relay (hal_led)
                                                   HalLedUpdate::?relay (hal_led)
                                                   HalUARTInit::?relay (hal_uart)
                                                   HalUARTInitUSB::?relay (hal_uart)
                                                   HalUARTOpen::?relay (hal_uart)
                                                   HalUARTOpenUSB::?relay (hal_uart)
                                                   HalUARTPoll::?relay (hal_uart)
                                                   HalUARTPollUSB::?relay (hal_uart)
                                                   HalUARTRead::?relay (hal_uart)
                                                   HalUARTRx::?relay (hal_uart)
                                                   HalUARTRxAvailUSB::?relay (hal_uart)
                                                   HalUARTTx::?relay (hal_uart)
                                                   HalUARTWrite::?relay (hal_uart)
                                                   Hal_Init::?relay (hal_drivers)
                                                   Hal_ProcessEvent::?relay (hal_drivers)
                                                   Hal_ProcessPoll::?relay (hal_drivers)
                                                   Hal_UART_RxBufLen::?relay (hal_uart)
                                                   InitBoard::?relay (OnBoard)
                                                   LL_AddWhiteListDevice::?relay (ll)
                                                   LL_ClearWhiteList::?relay (ll)
                                                   LL_DirectTestEnd::?relay (ll)
                                                   LL_DirectTestEndDoneCback::?relay (hci_event)
                                                   LL_DirectTestRxTest::?relay (ll)
                                                   LL_DirectTestTxTest::?relay (ll)
                                                   LL_ENC_AES128_Decrypt::?relay (ll_enc)
                                                   LL_ENC_AES128_Encrypt::?relay (ll_enc)
                                                   LL_ENC_GeneratePseudoRandNum::?relay (ll_enc)
                                                   LL_ENC_GenerateTrueRandNum::?relay (ll_enc)
                                                   LL_ENC_InitAesDMA::?relay (ll_enc)
                                                   LL_ENC_LoadKey::?relay (ll_enc)
                                                   LL_ENC_SetupCryptoDMA::?relay (ll_enc)
                                                   LL_ENC_SetupLoadDMA::?relay (ll_enc)
                                                   LL_ENC_StartAES::?relay (ll_enc)
                                                   LL_EXT_BuildRevision::?relay (ll)
                                                   LL_EXT_ClkDivOnHalt::?relay (ll)
                                                   LL_EXT_DeclareNvUsage::?relay (ll)
                                                   LL_EXT_Decrypt::?relay (ll)
                                                   LL_EXT_EndModemTest::?relay (ll)
                                                   LL_EXT_ExtendRfRange::?relay (ll)
                                                   LL_EXT_ExtendRfRangeCback::?relay (hci)
                                                   LL_EXT_HaltDuringRf::?relay (ll)
                                                   LL_EXT_MapPmIoPort::?relay (ll)
                                                   LL_EXT_ModemHopTestTx::?relay (ll)
                                                   LL_EXT_ModemTestRx::?relay (ll)
                                                   LL_EXT_ModemTestTx::?relay (ll)
                                                   LL_EXT_ResetSystem::?relay (ll)
                                                   LL_EXT_SaveFreqTune::?relay (ll)
                                                   LL_EXT_SetBDADDR::?relay (ll)
                                                   LL_EXT_SetFreqTune::?relay (ll)
                                                   LL_EXT_SetLocalSupportedFeatures::?relay (ll)
                                                   LL_EXT_SetMaxDtmTxPower::?relay (ll)
                                                   LL_EXT_SetRxGain::?relay (ll)
                                                   LL_EXT_SetRxGainCback::?relay (hci)
                                                   LL_EXT_SetTxPower::?relay (ll)
                                                   LL_EXT_SetTxPowerCback::?relay (hci)
                                                   LL_Encrypt::?relay (ll)
                                                   LL_Init::?relay (ll)
                                                   LL_ProcessEvent::?relay (ll)
                                                   LL_Rand::?relay (ll)
                                                   LL_RandCback::?relay (hci)
                                                   LL_ReadAdvChanTxPower::?relay (ll)
                                                   LL_ReadBDADDR::?relay (ll)
                                                   LL_ReadLocalSupportedFeatures::?relay (ll)
                                                   LL_ReadLocalVersionInfo::?relay (ll)
                                                   LL_ReadRssi::?relay (ll)
                                                   LL_ReadSupportedStates::?relay (ll)
                                                   LL_ReadWlSize::?relay (ll)
                                                   LL_RemoveWhiteListDevice::?relay (ll)
                                                   LL_Reset::?relay (ll)
                                                   LL_SetAdvControl::?relay (ll)
                                                   LL_SetAdvData::?relay (ll)
                                                   LL_SetAdvParam::?relay (ll)
                                                   LL_SetRandomAddress::?relay (ll)
                                                   LL_SetScanRspData::?relay (ll)
                                                   LL_TX_bm_alloc::?relay (ll)
                                                   NPI_GetMaxRxBufSize::?relay (npi)
                                                   NPI_InitTransport::?relay (npi)
                                                   NPI_ReadTransport::?relay (npi)
                                                   NPI_RxBufLen::?relay (npi)
                                                   NPI_WriteTransport::?relay (npi)
                                                   OnBoard_KeyCallback::?relay (OnBoard)
                                                   OnBoard_SendKeys::?relay (OnBoard)
                                                   PHY_AddWlEntry::?relay (phy)
                                                   PHY_ClearAllRegsAndFifos::?relay (phy)
                                                   PHY_ClearBlacklist::?relay (phy)
                                                   PHY_ClearBlacklistIndex::?relay (phy)
                                                   PHY_ClearSavedWhiteList::?relay (phy)
                                                   PHY_ClearWhitelist::?relay (phy)
                                                   PHY_Command::?relay (phy)
                                                   PHY_ConfigWhitener::?relay (phy)
                                                   PHY_ConfigureAppendRfStatus::?relay (phy)
                                                   PHY_ConfigureFifoDataProcessing::?relay (phy)
                                                   PHY_ConfigureMD::?relay (phy)
                                                   PHY_GetAdvChans::?relay (phy)
                                                   PHY_GetEndCause::?relay (phy)
                                                   PHY_GetWlSize::?relay (phy)
                                                   PHY_Init::?relay (phy)
                                                   PHY_LoadNR::?relay (phy)
                                                   PHY_RawGetNumTxPkts::?relay (phy)
                                                   PHY_RawGetRxData::?relay (phy)
                                                   PHY_RawRxInit::?relay (phy)
                                                   PHY_RawTxInit::?relay (phy)
                                                   PHY_RemoveWlEntry::?relay (phy)
                                                   PHY_Reset::?relay (phy)
                                                   PHY_SetAdvChans::?relay (phy)
                                                   PHY_SetAdvWlPolicy::?relay (phy)
                                                   PHY_SetBlacklistIndex::?relay (phy)
                                                   PHY_SetCRCInit::?relay (phy)
                                                   PHY_SetEndConnection::?relay (phy)
                                                   PHY_SetFifoConfig::?relay (phy)
                                                   PHY_SetOwnAddr::?relay (phy)
                                                   PHY_SetRfFreq::?relay (phy)
                                                   PHY_SetSyncWord::?relay (phy)
                                                   PHY_VerifyNR::?relay (phy)
                                                   SerialDebug_process::?relay (serialInterface)
                                                   SerialInterface_Init::?relay (serialInterface)
                                                   SerialInterface_ProcessEvent::?relay (serialInterface)
                                                   SerialInterface_ProcessOSALMsg::?relay (serialInterface)
                                                   SimpleBLEBroadcaster_Init::?relay (simpleBLEBroadcaster)
                                                   SimpleBLEBroadcaster_ProcessEvent::?relay (simpleBLEBroadcaster)
                                                   aesDmaInit::?relay (hal_aes)
                                                   cSerialPacketParser::?relay (serialInterface)
                                                   cleanErasedPage::?relay (osal_snv)
                                                   compactPage::?relay (osal_snv)
                                                   erasePage::?relay (osal_snv)
                                                   findItem::?relay (osal_snv)
                                                   findOffset::?relay (osal_snv)
                                                   gapAddAddrAdj::?relay (gap_configmgr)
                                                   gapFindADType::?relay (gap_devmgr)
                                                   gapFreeAdvertState::?relay (gap_peridevmgr)
                                                   gapPeriProcessHCICmdCompleteEvt::?relay (gap_peridevmgr)
                                                   gapProcessAdvertisingEvt::?relay (gap_peridevmgr)
                                                   gapProcessHCICmdCompleteEvt::?relay (gap_simpletask)
                                                   gapProcessRandomAddrComplete::?relay (gap_configmgr)
                                                   gapReadBD_ADDRStatus::?relay (gap_configmgr)
                                                   gapReadBufSizeCmdStatus::?relay (gap_configmgr)
                                                   gapRegisterPeripheral::?relay (gap_simpletask)
                                                   gapRole_ProcessGAPMsg::?relay (broadcaster)
                                                   gapRole_ProcessOSALMsg::?relay (broadcaster)
                                                   gapRole_SetupGAP::?relay (broadcaster)
                                                   gapSendDeviceInitDoneEvent::?relay (gap_configmgr)
                                                   gapSendMakeDiscEvent::?relay (gap_peridevmgr)
                                                   gapSetAdvParams::?relay (gap_peridevmgr)
                                                   gapSetAdvParamsStatus::?relay (gap_peridevmgr)
                                                   gapValidADType::?relay (gap_devmgr)
                                                   gapWriteAdvDataStatus::?relay (gap_peridevmgr)
                                                   gapWriteAdvEnableStatus::?relay (gap_peridevmgr)
                                                   halAssertHandler::?relay (hal_assert)
                                                   halUartPollEvt::?relay (hal_uart)
                                                   halUartPollRx::?relay (hal_uart)
                                                   halUartPollTx::?relay (hal_uart)
                                                   hciExtBuildRevision::?relay (hci_tl)
                                                   hciExtClkDivOnHalt::?relay (hci_tl)
                                                   hciExtDeclareNvUsage::?relay (hci_tl)
                                                   hciExtDecrypt::?relay (hci_tl)
                                                   hciExtDelaySleep::?relay (hci_tl)
                                                   hciExtEndModemTest::?relay (hci_tl)
                                                   hciExtExtendRfRange::?relay (hci_tl)
                                                   hciExtHaltDuringRf::?relay (hci_tl)
                                                   hciExtMapPmIoPort::?relay (hci_tl)
                                                   hciExtModemHopTestTx::?relay (hci_tl)
                                                   hciExtModemTestTx::?relay (hci_tl)
                                                   hciExtModemtestRx::?relay (hci_tl)
                                                   hciExtResetSystem::?relay (hci_tl)
                                                   hciExtSaveFreqTune::?relay (hci_tl)
                                                   hciExtSetBDADDR::?relay (hci_tl)
                                                   hciExtSetFreqTune::?relay (hci_tl)
                                                   hciExtSetLocalSupportedFeatures::?relay (hci_tl)
                                                   hciExtSetMaxDtmTxPower::?relay (hci_tl)
                                                   hciExtSetRxGain::?relay (hci_tl)
                                                   hciExtSetTxPower::?relay (hci_tl)
                                                   hciInitEventMasks::?relay (hci_event_PATCH)
                                                   hciLEAddWhiteList::?relay (hci_tl)
                                                   hciLEClearWhiteList::?relay (hci_tl)
                                                   hciLEEncrypt::?relay (hci_tl)
                                                   hciLERand::?relay (hci_tl)
                                                   hciLEReadAdvChanTxPower::?relay (hci_tl)
                                                   hciLEReadBufSize::?relay (hci_tl)
                                                   hciLEReadLocalSupportedFeatures::?relay (hci_tl)
                                                   hciLEReadSupportedStates::?relay (hci_tl)
                                                   hciLEReadWhiteListSize::?relay (hci_tl)
                                                   hciLEReceiverTest::?relay (hci_tl)
                                                   hciLERemoveWhiteList::?relay (hci_tl)
                                                   hciLESetAdvData::?relay (hci_tl)
                                                   hciLESetAdvEnab::?relay (hci_tl)
                                                   hciLESetAdvParam::?relay (hci_tl)
                                                   hciLESetEventMask::?relay (hci_tl)
                                                   hciLESetRandomAddr::?relay (hci_tl)
                                                   hciLESetScanRspData::?relay (hci_tl)
                                                   hciLETestEnd::?relay (hci_tl)
                                                   hciLETransmitterTest::?relay (hci_tl)
                                                   hciProcessCtrlToHost::?relay (hci_tl)
                                                   hciProcessHostToCtrlCmd::?relay (hci_tl)
                                                   hciProcessHostToCtrlData::?relay (hci_tl)
                                                   hciReadBDADDR::?relay (hci_tl)
                                                   hciReadLocalSupportedCommands::?relay (hci_tl)
                                                   hciReadLocalSupportedFeatures::?relay (hci_tl)
                                                   hciReadLocalVersionInfo::?relay (hci_tl)
                                                   hciReadRssi::?relay (hci_tl)
                                                   hciReset::?relay (hci_tl)
                                                   hciSerialPacketParser::?relay (hci_tl)
                                                   hciSetEventMask::?relay (hci_tl)
                                                   hciSetEventMaskPage2::?relay (hci_tl)
                                                   initNV::?relay (osal_snv)
                                                   isLimitedDiscoverableMode::?relay (gap_peridevmgr)
                                                   llAdvEvt_TaskAbort::?relay (ll_advEndCauses)
                                                   llAllocTask::?relay (ll_scheduler)
                                                   llCheckWhiteListUsage::?relay (ll_common)
                                                   llClearRfInts::?relay (ll_common)
                                                   llClearSetInts::?relay (ll_common)
                                                   llDisableRfInts::?relay (ll_common)
                                                   llDisableT2E1::?relay (ll_timer2)
                                                   llDisableT2Ints::?relay (ll_timer2)
                                                   llDisableT2IntsEvts::?relay (ll_timer2)
                                                   llDiscoverableAdvEvt_TaskEndOk::?relay (ll_advEndCauses)
                                                   llEnableRfInts::?relay (ll_common)
                                                   llExtendRfRange::?relay (ll_common)
                                                   llFindNextSecTask::?relay (ll_scheduler)
                                                   llFindTxPowerSettings::?relay (ll_common)
                                                   llFreeTask::?relay (ll_scheduler)
                                                   llGetCurrentTask::?relay (ll_scheduler)
                                                   llGetCurrentTime::?relay (ll_timer2)
                                                   llGetNumTasks::?relay (ll_scheduler)
                                                   llGetTask::?relay (ll_scheduler)
                                                   llGetTaskState::?relay (ll_scheduler)
                                                   llGetTxPower::?relay (ll_common)
                                                   llInitFeatureSet::?relay (ll_common)
                                                   llInitTimer2::?relay (ll_timer2)
                                                   llNonConnAdvEvt_TaskEndOk::?relay (ll_advEndCauses)
                                                   llProcessPostRfOps::?relay (ll_common)
                                                   llRfInit::?relay (ll_common)
                                                   llScheduleTask::?relay (ll_scheduler)
                                                   llScheduler::?relay (ll_scheduler)
                                                   llSchedulerInit::?relay (ll_scheduler)
                                                   llSetFreqTune::?relay (ll_common)
                                                   llSetRxGain::?relay (ll_common)
                                                   llSetT2C1Event1::?relay (ll_timer2)
                                                   llSetT2Delta::?relay (ll_timer2)
                                                   llSetT2OVFC1Event1::?relay (ll_timer2)
                                                   llSetT2OVFC1Timeout::?relay (ll_timer2)
                                                   llSetT2OVFC2Event2::?relay (ll_timer2)
                                                   llSetTxPower::?relay (ll_common)
                                                   llSetupAdv::?relay (ll_common)
                                                   llSetupNonConnectableAdvEvt::?relay (ll_common)
                                                   llSetupScannableAdvEvt::?relay (ll_common)
                                                   llStartAdvSetup::?relay (ll_common)
                                                   llStartTimer2::?relay (ll_timer2)
                                                   llStopTimer2::?relay (ll_timer2)
                                                   llUnexpectedEndCauseHandler::?relay (ll_errorEndCauses)
                                                   ll_McuPrecisionCount::?relay (ll_timer2)
                                                   memcpy::?relay (?memcpy)
                                                   memset::?relay (?memset)
                                                   osalAddTimer::?relay (OSAL_Timers)
                                                   osalClockUpdate::?relay (OSAL_ClockBLE)
                                                   osalDeleteTimer::?relay (OSAL_Timers)
                                                   osalFindTimer::?relay (OSAL_Timers)
                                                   osalInitTasks::?relay (OSAL_SimpleBLEBroadcaster)
                                                   osalTimeUpdate::?relay (OSAL_ClockBLE)
                                                   osalTimerInit::?relay (OSAL_Timers)
                                                   osalTimerUpdate::?relay (OSAL_Timers)
                                                   osal_CbTimerInit::?relay (osal_cbtimer)
                                                   osal_CbTimerProcessEvent::?relay (osal_cbtimer)
                                                   osal_GetSystemClock::?relay (OSAL_Timers)
                                                   osal_bm_alloc::?relay (osal_bufmgr)
                                                   osal_bm_free::?relay (osal_bufmgr)
                                                   osal_clear_event::?relay (OSAL)
                                                   osal_get_timeoutEx::?relay (OSAL_Timers)
                                                   osal_init_system::?relay (OSAL)
                                                   osal_int_disable::?relay (OSAL)
                                                   osal_mem_alloc::?relay (OSAL_Memory)
                                                   osal_mem_free::?relay (OSAL_Memory)
                                                   osal_mem_init::?relay (OSAL_Memory)
                                                   osal_mem_kick::?relay (OSAL_Memory)
                                                   osal_memcmp::?relay (OSAL)
                                                   osal_memcpy::?relay (OSAL)
                                                   osal_memset::?relay (OSAL)
                                                   osal_msg_allocate::?relay (OSAL)
                                                   osal_msg_deallocate::?relay (OSAL)
                                                   osal_msg_enqueue::?relay (OSAL)
                                                   osal_msg_enqueue_push::?relay (OSAL)
                                                   osal_msg_extract::?relay (OSAL)
                                                   osal_msg_push::?relay (OSAL)
                                                   osal_msg_push_front::?relay (OSAL)
                                                   osal_msg_receive::?relay (OSAL)
                                                   osal_msg_send::?relay (OSAL)
                                                   osal_pwrmgr_device::?relay (OSAL_PwrMgr)
                                                   osal_pwrmgr_init::?relay (OSAL_PwrMgr)
                                                   osal_pwrmgr_task_state::?relay (OSAL_PwrMgr)
                                                   osal_run_system::?relay (OSAL)
                                                   osal_set_event::?relay (OSAL)
                                                   osal_snv_init::?relay (osal_snv)
                                                   osal_snv_read::?relay (osal_snv)
                                                   osal_snv_write::?relay (osal_snv)
                                                   osal_start_reload_timer::?relay (OSAL_Timers)
                                                   osal_start_system::?relay (OSAL)
                                                   osal_start_timerEx::?relay (OSAL_Timers)
                                                   osal_stop_timerEx::?relay (OSAL_Timers)
                                                   parseCmd::?relay (serialInterface)
                                                   peripheralStateNotificationCB::?relay (simpleBLEBroadcaster)
                                                   phyFindWlEntry::?relay (phy)
                                                   sendSerialEvt::?relay (serialInterface)
                                                   setActivePage::?relay (osal_snv)
                                                   setXferPage::?relay (osal_snv)
                                                   simpleBLEBroadcaster_ProcessOSALMsg::?relay (simpleBLEBroadcaster)
                                                   usbcrHookProcessIn::?relay (usb_cdc_hooks)
                                                   usbcrHookProcessOut::?relay (usb_cdc_hooks)
                                                   usbdpFindNext::?relay (usb_descriptor_parser)
                                                   usbdpGetConfigurationDesc::?relay (usb_descriptor_parser)
                                                   usbdpGetDeviceDesc::?relay (usb_descriptor_parser)
                                                   usbdpGetInterfaceDesc::?relay (usb_descriptor_parser)
                                                   usbdpGetStringDesc::?relay (usb_descriptor_parser)
                                                   usbdpInit::?relay (usb_descriptor_parser)
                                                   usbfwInit::?relay (usb_framework)
                                                   usbfwReadFifo::?relay (usb_framework)
                                                   usbfwResetHandler::?relay (usb_framework)
                                                   usbfwSetAllEpStatus::?relay (usb_framework)
                                                   usbfwSetupHandler::?relay (usb_framework)
                                                   usbfwWriteFifo::?relay (usb_framework)
                                                   usbirqHookProcessEvents::?relay (usb_cdc_hooks)
                                                   usbirqInit::?relay (usb_interrupt)
                                                   usbsrClearFeature::?relay (usb_standard_requests)
                                                   usbsrGetConfiguration::?relay (usb_standard_requests)
                                                   usbsrGetDescriptor::?relay (usb_standard_requests)
                                                   usbsrGetInterface::?relay (usb_standard_requests)
                                                   usbsrGetStatus::?relay (usb_standard_requests)
                                                   usbsrHookClearFeature::?relay (usb_cdc_hooks)
                                                   usbsrHookProcessEvent::?relay (usb_cdc_hooks)
                                                   usbsrHookSetFeature::?relay (usb_cdc_hooks)
                                                   usbsrSetAddress::?relay (usb_standard_requests)
                                                   usbsrSetConfiguration::?relay (usb_standard_requests)
                                                   usbsrSetFeature::?relay (usb_standard_requests)
                                                   usbsrSetInterface::?relay (usb_standard_requests)
                                                   usbvrHookProcessIn::?relay (usb_cdc_hooks)
                                                   usbvrHookProcessOut::?relay (usb_cdc_hooks)
                                                   verifyWordM::?relay (osal_snv)
                                                   writeItem::?relay (osal_snv)
                                                   writeWord::?relay (osal_snv)
                                                   writeWordM::?relay (osal_snv)
                                                   xferItem::?relay (osal_snv)

    -------------------------------------------------------------------------
  LIBRARY MODULE, NAME : ?L_EQ_X

  SEGMENTS IN THE MODULE
  ======================
RCODE
  Relative segment, address: CODE 00000C8F - 00000CA3 (0x15 bytes), align: 0
  Segment part 1.
           ENTRY                   ADDRESS         REF BY
           =====                   =======         ======
           ?L_EQ_X                 00000C8F        findOffset (osal_snv)
                                                   initNV (osal_snv)
                                                   llSetT2OVFC2Event2 (ll_timer2)

    -------------------------------------------------------------------------
  LIBRARY MODULE, NAME : ?UL_GT

  SEGMENTS IN THE MODULE
  ======================
RCODE
  Relative segment, address: CODE 00000CA4 - 00000CB3 (0x10 bytes), align: 0
  Segment part 1.
           ENTRY                   ADDRESS         REF BY
           =====                   =======         ======
           ?UL_GT                  00000CA4        ll24BitTimeCompare (ll_timer2)
                                                   ll24BitTimeDelta (ll_timer2)

    -------------------------------------------------------------------------
  LIBRARY MODULE, NAME : ?UL_GT_X

  SEGMENTS IN THE MODULE
  ======================
RCODE
  Relative segment, address: CODE 00000CB4 - 00000CC3 (0x10 bytes), align: 0
  Segment part 1.
           ENTRY                   ADDRESS         REF BY
           =====                   =======         ======
           ?UL_GT_X                00000CB4        osalTimerUpdate (OSAL_Timers)

    -------------------------------------------------------------------------
  LIBRARY MODULE, NAME : ?UL_GE_X

  SEGMENTS IN THE MODULE
  ======================
RCODE
  Relative segment, address: CODE 00000CC4 - 00000CE2 (0x1f bytes), align: 0
  Segment part 1.
           ENTRY                   ADDRESS         REF BY
           =====                   =======         ======
           ?UL_GE_X                00000CC4        HalLedUpdate (hal_led)
                                                   LL_EXT_ExtendRfRange (ll)
                                                   LL_EXT_SetRxGain (ll)
                                                   LL_EXT_SetTxPower (ll)
                                                   ll24BitTimeCompare (ll_timer2)

    -------------------------------------------------------------------------
  LIBRARY MODULE, NAME : ?G_EQ

  SEGMENTS IN THE MODULE
  ======================
RCODE
  Relative segment, address: CODE 00000CE3 - 00000CED (0xb bytes), align: 0
  Segment part 0.
           ENTRY                   ADDRESS         REF BY
           =====                   =======         ======
           ?G_EQ                   00000CE3        usbsrGetDescriptor (usb_standard_requests)

    -------------------------------------------------------------------------
  LIBRARY MODULE, NAME : ?C_GPTR_LOAD

  SEGMENTS IN THE MODULE
  ======================
RCODE
  Relative segment, address: CODE 00000CEE - 00000D07 (0x1a bytes), align: 0
  Segment part 0.
           ENTRY                   ADDRESS         REF BY
           =====                   =======         ======
           ?C_GPTR_LOAD            00000CEE        usbfwWriteFifo (usb_framework)
                                                   usbsrGetDescriptor (usb_standard_requests)

    -------------------------------------------------------------------------
  LIBRARY MODULE, NAME : ?C_GPTR_STORE

  SEGMENTS IN THE MODULE
  ======================
RCODE
  Relative segment, address: CODE 00000D08 - 00000D1D (0x16 bytes), align: 0
  Segment part 0.
           ENTRY                   ADDRESS         REF BY
           =====                   =======         ======
           ?C_GPTR_STORE           00000D08        usbfwReadFifo (usb_framework)

    -------------------------------------------------------------------------
  LIBRARY MODULE, NAME : ?L_MUL

  SEGMENTS IN THE MODULE
  ======================
RCODE
  Relative segment, address: CODE 00000D1E - 00000D20 (0x3 bytes), align: 0
  Segment part 0.
           ENTRY                   ADDRESS         REF BY
           =====                   =======         ======
           ?L_MUL                  00000D1E        HalLedUpdate (hal_led)
                                                   gapWriteAdvEnableStatus (gap_peridevmgr)
                                                   llScheduleTask (ll_scheduler)
    -------------------------------------------------------------------------
RCODE
  Relative segment, address: CODE 00000D21 - 00000D9D (0x7d bytes), align: 0
  Segment part 1.             Intra module refs:   ?L_MUL
           ENTRY                   ADDRESS         REF BY
           =====                   =======         ======
           ?L_MUL_REW              00000D21 

    -------------------------------------------------------------------------
  LIBRARY MODULE, NAME : ?UL_DIV_MOD

  SEGMENTS IN THE MODULE
  ======================
RCODE
  Relative segment, address: CODE 00000D9E - 00000E0C (0x6f bytes), align: 0
  Segment part 1.
           ENTRY                   ADDRESS         REF BY
           =====                   =======         ======
           ?UL_DIV_MOD             00000D9E        HalLedUpdate (hal_led)

    -------------------------------------------------------------------------
  LIBRARY MODULE, NAME : ?UL_SHR

  SEGMENTS IN THE MODULE
  ======================
RCODE
  Relative segment, address: CODE 00000E0D - 00000E11 (0x5 bytes), align: 0
  Segment part 1.             Intra module refs:   Segment part 2
           ENTRY                   ADDRESS         REF BY
           =====                   =======         ======
           ?UL_SHR                 00000E0D        llFindTxPowerSettings (ll_common)
                                                   llScheduleTask (ll_scheduler)
    -------------------------------------------------------------------------
RCODE
  Relative segment, address: CODE 00000E12 - 00000E25 (0x14 bytes), align: 0
  Segment part 2.             Intra module refs:   ?UL_SHR

    -------------------------------------------------------------------------
  LIBRARY MODULE, NAME : ?L_ADD

  SEGMENTS IN THE MODULE
  ======================
RCODE
  Relative segment, address: CODE 00000E26 - 00000E38 (0x13 bytes), align: 0
  Segment part 1.
           ENTRY                   ADDRESS         REF BY
           =====                   =======         ======
           ?L_ADD                  00000E26        HalLedUpdate (hal_led)
                                                   ll24BitTimeDelta (ll_timer2)
                                                   llDiscoverableAdvEvt_TaskEndOk (ll_advEndCauses)
                                                   llNonConnAdvEvt_TaskEndOk (ll_advEndCauses)

    -------------------------------------------------------------------------
  LIBRARY MODULE, NAME : ?L_ADD_X

  SEGMENTS IN THE MODULE
  ======================
RCODE
  Relative segment, address: CODE 00000E39 - 00000E4B (0x13 bytes), align: 0
  Segment part 1.
           ENTRY                   ADDRESS         REF BY
           =====                   =======         ======
           ?L_ADD_X                00000E39        LL_SetAdvControl (ll)
                                                   llDiscoverableAdvEvt_TaskEndOk (ll_advEndCauses)
                                                   llFindNextSecTask (ll_scheduler)
                                                   llNonConnAdvEvt_TaskEndOk (ll_advEndCauses)
                                                   llScheduler (ll_scheduler)

    -------------------------------------------------------------------------
  LIBRARY MODULE, NAME : ?L_ADD_TO_X

  SEGMENTS IN THE MODULE
  ======================
RCODE
  Relative segment, address: CODE 00000E4C - 00000E5E (0x13 bytes), align: 0
  Segment part 1.
           ENTRY                   ADDRESS         REF BY
           =====                   =======         ======
           ?L_ADD_TO_X             00000E4C        osalClockUpdate (OSAL_ClockBLE)
                                                   osalTimerUpdate (OSAL_Timers)

    -------------------------------------------------------------------------
  LIBRARY MODULE, NAME : ?L_SUB

  SEGMENTS IN THE MODULE
  ======================
RCODE
  Relative segment, address: CODE 00000E5F - 00000E72 (0x14 bytes), align: 0
  Segment part 1.
           ENTRY                   ADDRESS         REF BY
           =====                   =======         ======
           ?L_SUB                  00000E5F        ll24BitTimeCompare (ll_timer2)
                                                   ll24BitTimeDelta (ll_timer2)

    -------------------------------------------------------------------------
  LIBRARY MODULE, NAME : ?L_SUB_FROM_X

  SEGMENTS IN THE MODULE
  ======================
RCODE
  Relative segment, address: CODE 00000E73 - 00000E86 (0x14 bytes), align: 0
  Segment part 1.
           ENTRY                   ADDRESS         REF BY
           =====                   =======         ======
           ?L_SUB_FROM_X           00000E73        osalTimerUpdate (OSAL_Timers)

    -------------------------------------------------------------------------
  LIBRARY MODULE, NAME : ?L_AND_X

  SEGMENTS IN THE MODULE
  ======================
RCODE
  Relative segment, address: CODE 00000E87 - 00000E99 (0x13 bytes), align: 0
  Segment part 1.
           ENTRY                   ADDRESS         REF BY
           =====                   =======         ======
           ?L_AND_X                00000E87        LL_SetAdvControl (ll)
                                                   ll24BitTimeCompare (ll_timer2)
                                                   ll24BitTimeDelta (ll_timer2)
                                                   llDiscoverableAdvEvt_TaskEndOk (ll_advEndCauses)
                                                   llNonConnAdvEvt_TaskEndOk (ll_advEndCauses)
                                                   llScheduler (ll_scheduler)

    -------------------------------------------------------------------------
  LIBRARY MODULE, NAME : ?L_IOR_X

  SEGMENTS IN THE MODULE
  ======================
RCODE
  Relative segment, address: CODE 00000E9A - 00000EAC (0x13 bytes), align: 0
  Segment part 1.
           ENTRY                   ADDRESS         REF BY
           =====                   =======         ======
           ?L_IOR_X                00000E9A        LL_EXT_SaveFreqTune (ll)

    -------------------------------------------------------------------------
  LIBRARY MODULE, NAME : ?L_MOV_X

  SEGMENTS IN THE MODULE
  ======================
RCODE
  Relative segment, address: CODE 00000EAD - 00000EBB (0xf bytes), align: 0
  Segment part 0.
           ENTRY                   ADDRESS         REF BY
           =====                   =======         ======
           ?L_MOV_X                00000EAD        HalLedUpdate (hal_led)
                                                   LL_EXT_SaveFreqTune (ll)
                                                   findOffset (osal_snv)
                                                   gapWriteAdvEnableStatus (gap_peridevmgr)
                                                   initNV (osal_snv)
                                                   ll24BitTimeCompare (ll_timer2)
                                                   ll24BitTimeDelta (ll_timer2)
                                                   llFindNextSecTask (ll_scheduler)
                                                   llFindTxPowerSettings (ll_common)
                                                   llScheduleTask (ll_scheduler)
                                                   llScheduler (ll_scheduler)
                                                   llSetT2OVFC2Event2 (ll_timer2)
                                                   osalAddTimer (OSAL_Timers)
                                                   osalTimerUpdate (OSAL_Timers)
                                                   osal_get_timeoutEx (OSAL_Timers)
                                                   osal_start_reload_timer (OSAL_Timers)
                                                   osal_start_timerEx (OSAL_Timers)

    -------------------------------------------------------------------------
  LIBRARY MODULE, NAME : ?L_MOV_TO_X

  SEGMENTS IN THE MODULE
  ======================
RCODE
  Relative segment, address: CODE 00000EBC - 00000ECA (0xf bytes), align: 0
  Segment part 2.
           ENTRY                   ADDRESS         REF BY
           =====                   =======         ======
           ?L_MOV_TO_X             00000EBC        HalLedUpdate (hal_led)
                                                   LL_EXT_SaveFreqTune (ll)
                                                   LL_SetAdvControl (ll)
                                                   llDiscoverableAdvEvt_TaskEndOk (ll_advEndCauses)
                                                   llNonConnAdvEvt_TaskEndOk (ll_advEndCauses)
                                                   llScheduler (ll_scheduler)
                                                   osalAddTimer (OSAL_Timers)
                                                   osalTimerUpdate (OSAL_Timers)
                                                   osal_start_reload_timer (OSAL_Timers)

    -------------------------------------------------------------------------
  LIBRARY MODULE, NAME : ?XLOAD_R2345

  SEGMENTS IN THE MODULE
  ======================
RCODE
  Relative segment, address: CODE 00000ECB - 00000ED6 (0xc bytes), align: 0
  Segment part 0.
           ENTRY                   ADDRESS         REF BY
           =====                   =======         ======
           ?XLOAD_R2345            00000ECB        LL_DirectTestRxTest (ll)
                                                   LL_DirectTestTxTest (ll)
                                                   LL_EXT_ExtendRfRange (ll)
                                                   LL_EXT_ModemHopTestTx (ll)
                                                   LL_EXT_ModemTestRx (ll)
                                                   LL_EXT_ModemTestTx (ll)
                                                   LL_EXT_SetRxGain (ll)
                                                   LL_EXT_SetTxPower (ll)
                                                   LL_Reset (ll)
                                                   Segment part 41 (ll_timer2)
                                                   llFindNextSecTask (ll_scheduler)
                                                   llScheduleTask (ll_scheduler)
                                                   llScheduler (ll_scheduler)
                                                   llSetupAdv (ll_common)
                                                   osal_GetSystemClock (OSAL_Timers)

    -------------------------------------------------------------------------
  LIBRARY MODULE, NAME : ?XLOAD_R0123

  SEGMENTS IN THE MODULE
  ======================
RCODE
  Relative segment, address: CODE 00000ED7 - 00000EE2 (0xc bytes), align: 0
  Segment part 0.
           ENTRY                   ADDRESS         REF BY
           =====                   =======         ======
           ?XLOAD_R0123            00000ED7        initNV (osal_snv)
                                                   osalTimerUpdate (OSAL_Timers)

    -------------------------------------------------------------------------
  LIBRARY MODULE, NAME : ?XSTORE_R0123

  SEGMENTS IN THE MODULE
  ======================
RCODE
  Relative segment, address: CODE 00000EE3 - 00000EEE (0xc bytes), align: 0
  Segment part 0.
           ENTRY                   ADDRESS         REF BY
           =====                   =======         ======
           ?XSTORE_R0123           00000EE3        HalLedBlink (hal_led)
                                                   llAllocTask (ll_scheduler)
                                                   osalTimerUpdate (OSAL_Timers)

    -------------------------------------------------------------------------
  LIBRARY MODULE, NAME : ?MOVE_LONG8_XDATA_IDATA

  SEGMENTS IN THE MODULE
  ======================
RCODE
  Relative segment, address: CODE 00000EEF - 00000EFB (0xd bytes), align: 0
  Segment part 0.
           ENTRY                   ADDRESS         REF BY
           =====                   =======         ======
           ?MOVE_LONG8_XDATA_IDATA
                                   00000EEF        ?PUSH_XSTACK_I (?PUSH_XSTACK_I)

    -------------------------------------------------------------------------
  LIBRARY MODULE, NAME : ?MOVE_LONG8_XDATA_XDATA

  SEGMENTS IN THE MODULE
  ======================
RCODE
  Relative segment, address: CODE 00000EFC - 00000F1C (0x21 bytes), align: 0
  Segment part 0.
           ENTRY                   ADDRESS         REF BY
           =====                   =======         ======
           ?MOVE_LONG8_XDATA_XDATA
                                   00000EFC        ?PUSH_XSTACK8_X (?PUSH_XSTACK8_X)
                                                   HCI_LE_ReadSupportedStatesCmd (hci)
                                                   HCI_ReadLocalSupportedFeaturesCmd (hci)
                                                   llFindTxPowerSettings (ll_common)

    -------------------------------------------------------------------------
  LIBRARY MODULE, NAME : ?S_DIV_MOD

  SEGMENTS IN THE MODULE
  ======================
RCODE
  Relative segment, address: CODE 00000F1D - 00000F5D (0x41 bytes), align: 0
  Segment part 0.
           ENTRY                   ADDRESS         REF BY
           =====                   =======         ======
           ?S_DIV_MOD              00000F56        osal_snv_write (osal_snv)
                                                   usbdpGetStringDesc (usb_descriptor_parser)
    -------------------------------------------------------------------------
RCODE
  Relative segment, address: CODE 00000F5E - 00000FB6 (0x59 bytes), align: 0
  Segment part 1.             Intra module refs:   ?S_DIV_MOD
           ENTRY                   ADDRESS         REF BY
           =====                   =======         ======
           ?US_DIV_MOD             00000F5E        osalClockUpdate (OSAL_ClockBLE)
                                                   osalTimeUpdate (OSAL_ClockBLE)
                                                   usbdpGetStringDesc (usb_descriptor_parser)

    -------------------------------------------------------------------------
  LIBRARY MODULE, NAME : ?SS_SHR

  SEGMENTS IN THE MODULE
  ======================
RCODE
  Relative segment, address: CODE 00000FB7 - 00000FB9 (0x3 bytes), align: 0
  Segment part 1.             Intra module refs:   Segment part 2
           ENTRY                   ADDRESS         REF BY
           =====                   =======         ======
           ?SS_SHR                 00000FB7        phyFindWlEntry (phy)
    -------------------------------------------------------------------------
RCODE
  Relative segment, address: CODE 00000FBA - 00000FC6 (0xd bytes), align: 0
  Segment part 2.             Intra module refs:   ?SS_SHR

    -------------------------------------------------------------------------
  LIBRARY MODULE, NAME : ?US_SHR

  SEGMENTS IN THE MODULE
  ======================
RCODE
  Relative segment, address: CODE 00000FC7 - 00000FC9 (0x3 bytes), align: 0
  Segment part 1.             Intra module refs:   Segment part 2
           ENTRY                   ADDRESS         REF BY
           =====                   =======         ======
           ?US_SHR                 00000FC7        ConfigureEndpoints (usb_standard_requests)
                                                   LL_Init (ll)
                                                   LL_TX_bm_alloc (ll)
                                                   RF_NormalIsr (ll_isr)
                                                   hciSerialPacketParser (hci_tl)
                                                   osalTimeUpdate (OSAL_ClockBLE)
                                                   osal_CbTimerProcessEvent (osal_cbtimer)
                                                   usbirqHandler (usb_interrupt)
                                                   usbirqInit (usb_interrupt)
                                                   usbsrGetDescriptor (usb_standard_requests)
                                                   writeItem (osal_snv)
                                                   writeWord (osal_snv)
                                                   writeWordM (osal_snv)
    -------------------------------------------------------------------------
RCODE
  Relative segment, address: CODE 00000FCA - 00000FD5 (0xc bytes), align: 0
  Segment part 2.             Intra module refs:   ?US_SHR

    -------------------------------------------------------------------------
  LIBRARY MODULE, NAME : ?S_SHL

  SEGMENTS IN THE MODULE
  ======================
RCODE
  Relative segment, address: CODE 00000FD6 - 00000FD8 (0x3 bytes), align: 0
  Segment part 0.
           ENTRY                   ADDRESS         REF BY
           =====                   =======         ======
           ?S_SHL                  00000FD6        ConfigureEndpoints (usb_standard_requests)
                                                   LL_EXT_MapPmIoPort (ll)
                                                   LL_TX_bm_alloc (ll)
                                                   PHY_AddWlEntry (phy)
                                                   PHY_ClearBlacklistIndex (phy)
                                                   PHY_RemoveWlEntry (phy)
                                                   PHY_SetBlacklistIndex (phy)
                                                   hciProcessHostToCtrlCmd (hci_tl)
                                                   llFindTxPowerSettings (ll_common)
                                                   osal_CbTimerProcessEvent (osal_cbtimer)
                                                   osal_pwrmgr_task_state (OSAL_PwrMgr)
                                                   phyFindWlEntry (phy)
                                                   usbirqHandler (usb_interrupt)
                                                   writeWord (osal_snv)
                                                   writeWordM (osal_snv)
    -------------------------------------------------------------------------
RCODE
  Relative segment, address: CODE 00000FD9 - 00000FDB (0x3 bytes), align: 0
  Segment part 1.             Intra module refs:   Segment part 2
           ENTRY                   ADDRESS         REF BY
           =====                   =======         ======
           ?S_SHL_REW              00000FD9 
    -------------------------------------------------------------------------
RCODE
  Relative segment, address: CODE 00000FDC - 00000FE8 (0xd bytes), align: 0
  Segment part 2.             Intra module refs:   ?S_SHL
                                                   ?S_SHL_REW

    -------------------------------------------------------------------------
  LIBRARY MODULE, NAME : ?ALLOC_XSTACK8

  SEGMENTS IN THE MODULE
  ======================
RCODE
  Relative segment, address: CODE 00000FE9 - 00000FFE (0x16 bytes), align: 0
  Segment part 0.
           ENTRY                   ADDRESS         REF BY
           =====                   =======         ======
           ?ALLOC_XSTACK8          00000FE9        Application_StartAdvertise (simpleBLEBroadcaster)
                                                   Application_StopAdvertise (simpleBLEBroadcaster)
                                                   GAPRole_ProcessEvent (broadcaster)
                                                   HCI_EXT_BuildRevisionCmd (hci)
                                                   HCI_EXT_ClkDivOnHaltCmd (hci)
                                                   HCI_EXT_DeclareNvUsageCmd (hci)
                                                   HCI_EXT_DecryptCmd (hci)
                                                   HCI_EXT_DelaySleepCmd (hci_PATCH)
                                                   HCI_EXT_EndModemTestCmd (hci)
                                                   HCI_EXT_ExtendRfRangeCmd (hci)
                                                   HCI_EXT_HaltDuringRfCmd (hci)
                                                   HCI_EXT_MapPmIoPortCmd (hci)
                                                   HCI_EXT_ModemHopTestTxCmd (hci)
                                                   HCI_EXT_ModemTestRxCmd (hci)
                                                   HCI_EXT_ModemTestTxCmd (hci)
                                                   HCI_EXT_ResetSystemCmd (hci_PATCH)
                                                   HCI_EXT_SaveFreqTuneCmd (hci)
                                                   HCI_EXT_SetBDADDRCmd (hci)
                                                   HCI_EXT_SetFreqTuneCmd (hci)
                                                   HCI_EXT_SetLocalSupportedFeaturesCmd (hci)
                                                   HCI_EXT_SetMaxDtmTxPowerCmd (hci)
                                                   HCI_EXT_SetRxGainCmd (hci)
                                                   HCI_EXT_SetTxPowerCmd (hci)
                                                   HCI_LE_AddWhiteListCmd (hci)
                                                   HCI_LE_ClearWhiteListCmd (hci)
                                                   HCI_LE_EncryptCmd (hci)
                                                   HCI_LE_RandCmd (hci)
                                                   HCI_LE_ReadAdvChanTxPowerCmd (hci)
                                                   HCI_LE_ReadBufSizeCmd (hci_PATCH)
                                                   HCI_LE_ReadLocalSupportedFeaturesCmd (hci)
                                                   HCI_LE_ReadSupportedStatesCmd (hci)
                                                   HCI_LE_ReadWhiteListSizeCmd (hci)
                                                   HCI_LE_ReceiverTestCmd (hci)
                                                   HCI_LE_RemoveWhiteListCmd (hci)
                                                   HCI_LE_SetAdvDataCmd (hci)
                                                   HCI_LE_SetAdvEnableCmd (hci)
                                                   HCI_LE_SetAdvParamCmd (hci)
                                                   HCI_LE_SetEventMaskCmd (hci)
                                                   HCI_LE_SetRandomAddressCmd (hci)
                                                   HCI_LE_SetScanRspDataCmd (hci)
                                                   HCI_LE_TestEndCmd (hci)
                                                   HCI_LE_TransmitterTestCmd (hci)
                                                   HCI_ReadBDADDRCmd (hci)
                                                   HCI_ReadLocalSupportedFeaturesCmd (hci)
                                                   HCI_ReadLocalVersionInfoCmd (hci)
                                                   HCI_ReadRssiCmd (hci)
                                                   HCI_ResetCmd (hci_PATCH)
                                                   HCI_SetEventMaskCmd (hci)
                                                   HCI_SetEventMaskPage2Cmd (hci_PATCH)
                                                   HalLedUpdate (hal_led)
                                                   LL_DirectTestEndDoneCback (hci_event)
                                                   LL_EXT_ExtendRfRangeCback (hci)
                                                   LL_EXT_SaveFreqTune (ll)
                                                   LL_EXT_SetRxGainCback (hci)
                                                   LL_EXT_SetTxPowerCback (hci)
                                                   LL_RandCback (hci)
                                                   NPI_InitTransport (npi)
                                                   SimpleBLEBroadcaster_Init (simpleBLEBroadcaster)
                                                   cleanErasedPage (osal_snv)
                                                   compactPage (osal_snv)
                                                   erasePage (osal_snv)
                                                   findItem (osal_snv)
                                                   findOffset (osal_snv)
                                                   hciProcessHostToCtrlCmd (hci_tl)
                                                   initNV (osal_snv)
                                                   isLimitedDiscoverableMode (gap_peridevmgr)
                                                   llFindTxPowerSettings (ll_common)
                                                   llGetCurrentTime (ll_timer2)
                                                   llProcessPostRfOps (ll_common)
                                                   llSetT2C1Event1 (ll_timer2)
                                                   llSetT2Delta (ll_timer2)
                                                   llSetT2OVFC1Event1 (ll_timer2)
                                                   llSetT2OVFC1Timeout (ll_timer2)
                                                   llSetT2OVFC2Event2 (ll_timer2)
                                                   ll_McuPrecisionCount (ll_timer2)
                                                   osalTimerUpdate (OSAL_Timers)
                                                   osal_snv_write (osal_snv)
                                                   peripheralStateNotificationCB (simpleBLEBroadcaster)
                                                   setActivePage (osal_snv)
                                                   setXferPage (osal_snv)
                                                   usbdpGetStringDesc (usb_descriptor_parser)
                                                   verifyWordM (osal_snv)
                                                   writeItem (osal_snv)
                                                   xferItem (osal_snv)

    -------------------------------------------------------------------------
  LIBRARY MODULE, NAME : ?DEALLOC_XSTACK8

  SEGMENTS IN THE MODULE
  ======================
RCODE
  Relative segment, address: CODE 00000FFF - 00001019 (0x1b bytes), align: 0
  Segment part 0.
           ENTRY                   ADDRESS         REF BY
           =====                   =======         ======
           ?DEALLOC_XSTACK8        00000FFF        Application_StartAdvertise (simpleBLEBroadcaster)
                                                   Application_StopAdvertise (simpleBLEBroadcaster)
                                                   Application_UpdateAdv (simpleBLEBroadcaster)
                                                   Application_UpdateRsp (simpleBLEBroadcaster)
                                                   GAPRole_GetParameter (broadcaster)
                                                   GAPRole_ProcessEvent (broadcaster)
                                                   GAPRole_SetParameter (broadcaster)
                                                   GAP_MakeDiscoverable (gap_peridevmgr)
                                                   GAP_UpdateAdvertisingData (gap_peridevmgr)
                                                   HCI_CommandCompleteEvent (hci_event)
                                                   HCI_EXT_DecryptCmd (hci)
                                                   HCI_EXT_ResetSystemCmd (hci_PATCH)
                                                   HCI_LE_EncryptCmd (hci)
                                                   HCI_LE_SetAdvParamCmd (hci)
                                                   HCI_ReadLocalVersionInfoCmd (hci)
                                                   HCI_SendCommandCompleteEvent (hci_event)
                                                   HCI_SetEventMaskCmd (hci)
                                                   HCI_SetEventMaskPage2Cmd (hci_PATCH)
                                                   HCI_VendorSpecifcCommandCompleteEvent (hci_event_PATCH)
                                                   HalLedUpdate (hal_led)
                                                   LL_DirectTestEnd (ll)
                                                   LL_DirectTestEndDoneCback (hci_event)
                                                   LL_ENC_AES128_Decrypt (ll_enc)
                                                   LL_ENC_AES128_Encrypt (ll_enc)
                                                   LL_EXT_Decrypt (ll)
                                                   LL_EXT_ExtendRfRange (ll)
                                                   LL_EXT_ResetSystem (ll)
                                                   LL_EXT_SaveFreqTune (ll)
                                                   LL_EXT_SetRxGain (ll)
                                                   LL_EXT_SetTxPower (ll)
                                                   LL_Encrypt (ll)
                                                   LL_Init (ll)
                                                   LL_ProcessEvent (ll)
                                                   LL_RandCback (hci)
                                                   LL_SetAdvData (ll)
                                                   LL_SetScanRspData (ll)
                                                   NPI_InitTransport (npi)
                                                   Segment part 24 (hci_PATCH)
                                                   Segment part 43 (ll_timer2)
                                                   Segment part 62 (hci)
                                                   Segment part 83 (hci)
                                                   Segment part 94 (hci)
                                                   SimpleBLEBroadcaster_Init (simpleBLEBroadcaster)
                                                   cleanErasedPage (osal_snv)
                                                   compactPage (osal_snv)
                                                   erasePage (osal_snv)
                                                   findItem (osal_snv)
                                                   findOffset (osal_snv)
                                                   gapProcessAdvertisingEvt (gap_peridevmgr)
                                                   gapProcessRandomAddrComplete (gap_configmgr)
                                                   gapReadBD_ADDRStatus (gap_configmgr)
                                                   gapRole_ProcessGAPMsg (broadcaster)
                                                   gapRole_SetupGAP (broadcaster)
                                                   gapSendDeviceInitDoneEvent (gap_configmgr)
                                                   gapSetAdvParams (gap_peridevmgr)
                                                   gapWriteAdvEnableStatus (gap_peridevmgr)
                                                   hciLESetAdvParam (hci_tl)
                                                   hciProcessHostToCtrlCmd (hci_tl)
                                                   initNV (osal_snv)
                                                   isLimitedDiscoverableMode (gap_peridevmgr)
                                                   llFindNextSecTask (ll_scheduler)
                                                   llFindTxPowerSettings (ll_common)
                                                   llProcessPostRfOps (ll_common)
                                                   llScheduleTask (ll_scheduler)
                                                   llScheduler (ll_scheduler)
                                                   llSetT2OVFC2Event2 (ll_timer2)
                                                   osalTimerUpdate (OSAL_Timers)
                                                   osal_memset (OSAL)
                                                   osal_msg_receive (OSAL)
                                                   osal_snv_read (osal_snv)
                                                   osal_snv_write (osal_snv)
                                                   osal_start_reload_timer (OSAL_Timers)
                                                   osal_start_timerEx (OSAL_Timers)
                                                   peripheralStateNotificationCB (simpleBLEBroadcaster)
                                                   setActivePage (osal_snv)
                                                   setXferPage (osal_snv)
                                                   usbdpGetStringDesc (usb_descriptor_parser)
                                                   usbfwSetupHandler (usb_framework)
                                                   verifyWordM (osal_snv)
                                                   writeItem (osal_snv)
                                                   writeWord (osal_snv)
                                                   writeWordM (osal_snv)
                                                   xferItem (osal_snv)

    -------------------------------------------------------------------------
  LIBRARY MODULE, NAME : ?ADD_XSTACK_DISP8

  SEGMENTS IN THE MODULE
  ======================
RCODE
  Relative segment, address: CODE 0000101A - 00001034 (0x1b bytes), align: 0
  Segment part 1.
           ENTRY                   ADDRESS         REF BY
           =====                   =======         ======
           ?ADD_XSTACK_DISP0_8     0000101A        ?PUSH_XSTACK_I (?PUSH_XSTACK_I)

    -------------------------------------------------------------------------
  LIBRARY MODULE, NAME : ?XSTACK_DISP8

  SEGMENTS IN THE MODULE
  ======================
RCODE
  Relative segment, address: CODE 00001035 - 0000103E (0xa bytes), align: 0
  Segment part 1.
           ENTRY                   ADDRESS         REF BY
           =====                   =======         ======
           ?XSTACK_DISP0_8         00001035        GAPRole_ProcessEvent (broadcaster)
                                                   HCI_EXT_BuildRevisionCmd (hci)
                                                   HCI_EXT_ClkDivOnHaltCmd (hci)
                                                   HCI_EXT_DeclareNvUsageCmd (hci)
                                                   HCI_EXT_DecryptCmd (hci)
                                                   HCI_EXT_DelaySleepCmd (hci_PATCH)
                                                   HCI_EXT_EndModemTestCmd (hci)
                                                   HCI_EXT_ExtendRfRangeCmd (hci)
                                                   HCI_EXT_HaltDuringRfCmd (hci)
                                                   HCI_EXT_MapPmIoPortCmd (hci)
                                                   HCI_EXT_ModemHopTestTxCmd (hci)
                                                   HCI_EXT_ModemTestRxCmd (hci)
                                                   HCI_EXT_ModemTestTxCmd (hci)
                                                   HCI_EXT_ResetSystemCmd (hci_PATCH)
                                                   HCI_EXT_SaveFreqTuneCmd (hci)
                                                   HCI_EXT_SetBDADDRCmd (hci)
                                                   HCI_EXT_SetFreqTuneCmd (hci)
                                                   HCI_EXT_SetLocalSupportedFeaturesCmd (hci)
                                                   HCI_EXT_SetMaxDtmTxPowerCmd (hci)
                                                   HCI_EXT_SetRxGainCmd (hci)
                                                   HCI_EXT_SetTxPowerCmd (hci)
                                                   HCI_LE_EncryptCmd (hci)
                                                   HCI_LE_RandCmd (hci)
                                                   HCI_LE_ReadAdvChanTxPowerCmd (hci)
                                                   HCI_LE_ReadBufSizeCmd (hci_PATCH)
                                                   HCI_LE_ReadLocalSupportedFeaturesCmd (hci)
                                                   HCI_LE_ReadSupportedStatesCmd (hci)
                                                   HCI_LE_ReadWhiteListSizeCmd (hci)
                                                   HCI_LE_SetAdvParamCmd (hci)
                                                   HCI_LE_TestEndCmd (hci)
                                                   HCI_ReadBDADDRCmd (hci)
                                                   HCI_ReadLocalSupportedFeaturesCmd (hci)
                                                   HCI_ReadLocalVersionInfoCmd (hci)
                                                   HCI_ReadRssiCmd (hci)
                                                   HCI_SendCommandCompleteEvent (hci_event)
                                                   HalFlashRead (hal_flash)
                                                   HalFlashWrite (hal_flash)
                                                   HalLedUpdate (hal_led)
                                                   LL_DirectTestEndDoneCback (hci_event)
                                                   LL_ENC_AES128_Decrypt (ll_enc)
                                                   LL_ENC_AES128_Encrypt (ll_enc)
                                                   LL_ENC_SetupCryptoDMA (ll_enc)
                                                   LL_EXT_Decrypt (ll)
                                                   LL_EXT_ExtendRfRangeCback (hci)
                                                   LL_EXT_SetRxGainCback (hci)
                                                   LL_EXT_SetTxPowerCback (hci)
                                                   LL_Encrypt (ll)
                                                   LL_RandCback (hci)
                                                   LL_SetAdvParam (ll)
                                                   NPI_InitTransport (npi)
                                                   Segment part 40 (ll_timer2)
                                                   Segment part 41 (ll_timer2)
                                                   SimpleBLEBroadcaster_Init (simpleBLEBroadcaster)
                                                   compactPage (osal_snv)
                                                   findItem (osal_snv)
                                                   gapFindADType (gap_devmgr)
                                                   ll24BitTimeCompare (ll_timer2)
                                                   ll24BitTimeDelta (ll_timer2)
                                                   llFindTxPowerSettings (ll_common)
                                                   llSetT2C1Event1 (ll_timer2)
                                                   llSetT2Delta (ll_timer2)
                                                   llSetT2OVFC1Event1 (ll_timer2)
                                                   llSetT2OVFC1Timeout (ll_timer2)
                                                   llSetT2OVFC2Event2 (ll_timer2)
                                                   ll_McuPrecisionCount (ll_timer2)
                                                   memcpy (?memcpy)
                                                   osalAddTimer (OSAL_Timers)
                                                   osalTimerUpdate (OSAL_Timers)
                                                   osal_memcmp (OSAL)
                                                   osal_memcpy (OSAL)
                                                   osal_msg_extract (OSAL)
                                                   osal_start_reload_timer (OSAL_Timers)
                                                   osal_start_timerEx (OSAL_Timers)
                                                   usbdpGetStringDesc (usb_descriptor_parser)
                                                   usbfwReadFifo (usb_framework)
                                                   usbfwWriteFifo (usb_framework)
                                                   verifyWordM (osal_snv)
                                                   writeItem (osal_snv)
                                                   writeWordM (osal_snv)
                                                   xferItem (osal_snv)

    -------------------------------------------------------------------------
  LIBRARY MODULE, NAME : ?XSTACK_DISP8_RP

  SEGMENTS IN THE MODULE
  ======================
RCODE
  Relative segment, address: CODE 0000103F - 00001046 (0x8 bytes), align: 0
  Segment part 0.
           ENTRY                   ADDRESS         REF BY
           =====                   =======         ======
           ?XSTACK_DISP100_8       0000103F        HCI_ReadLocalVersionInfoCmd (hci)
    -------------------------------------------------------------------------
RCODE
  Relative segment, address: CODE 00001047 - 0000104E (0x8 bytes), align: 0
  Segment part 1.
           ENTRY                   ADDRESS         REF BY
           =====                   =======         ======
           ?XSTACK_DISP101_8       00001047        GAPRole_ProcessEvent (broadcaster)
                                                   HCI_ReadLocalVersionInfoCmd (hci)
                                                   isLimitedDiscoverableMode (gap_peridevmgr)
                                                   verifyWordM (osal_snv)
    -------------------------------------------------------------------------
RCODE
  Relative segment, address: CODE 0000104F - 00001056 (0x8 bytes), align: 0
  Segment part 2.
           ENTRY                   ADDRESS         REF BY
           =====                   =======         ======
           ?XSTACK_DISP102_8       0000104F        HCI_EXT_ExtendRfRangeCmd (hci)
                                                   HCI_EXT_SetRxGainCmd (hci)
                                                   HCI_EXT_SetTxPowerCmd (hci)
                                                   HCI_ReadLocalVersionInfoCmd (hci)
                                                   LL_EXT_SaveFreqTune (ll)
                                                   SimpleBLEBroadcaster_Init (simpleBLEBroadcaster)
                                                   cleanErasedPage (osal_snv)
                                                   compactPage (osal_snv)
                                                   erasePage (osal_snv)
                                                   findItem (osal_snv)
                                                   findOffset (osal_snv)
                                                   initNV (osal_snv)
                                                   llFindTxPowerSettings (ll_common)
                                                   osal_snv_write (osal_snv)
                                                   verifyWordM (osal_snv)
                                                   xferItem (osal_snv)

    -------------------------------------------------------------------------
  LIBRARY MODULE, NAME : ?CALL_IND

  SEGMENTS IN THE MODULE
  ======================
RCODE
  Relative segment, address: CODE 00001057 - 00001058 (0x2 bytes), align: 0
  Segment part 0.
           ENTRY                   ADDRESS         REF BY
           =====                   =======         ======
           ?CALL_IND               00001057        GAPRole_ProcessEvent (broadcaster)
                                                   GAP_ProcessEvent (gap_simpletask)
                                                   LL_ProcessEvent (ll)
                                                   gapProcessHCICmdCompleteEvt (gap_simpletask)
                                                   gapProcessRandomAddrComplete (gap_configmgr)
                                                   gapRole_ProcessGAPMsg (broadcaster)
                                                   halUartPollRx (hal_uart)
                                                   halUartPollTx (hal_uart)
                                                   hciProcessHostToCtrlCmd (hci_tl)
                                                   llScheduleTask (ll_scheduler)
                                                   osal_CbTimerProcessEvent (osal_cbtimer)
                                                   osal_run_system (OSAL)
                                                   usbfwSetupHandler (usb_framework)

    -------------------------------------------------------------------------
  LIBRARY MODULE, NAME : ?BANKED_ENTER_XDATA

  SEGMENTS IN THE MODULE
  ======================
RCODE
  Relative segment, address: CODE 00001059 - 000010C4 (0x6c bytes), align: 0
  Segment part 1.
           ENTRY                   ADDRESS         REF BY
           =====                   =======         ======
           ?BANKED_ENTER_XDATA     00001059        Application_UpdateAdv (simpleBLEBroadcaster)
                                                   Application_UpdateRsp (simpleBLEBroadcaster)
                                                   ChangeFeature (usb_standard_requests)
                                                   ConfigureEndpoints (usb_standard_requests)
                                                   GAPRole_GetParameter (broadcaster)
                                                   GAPRole_Init (broadcaster)
                                                   GAPRole_ProcessEvent (broadcaster)
                                                   GAPRole_SetParameter (broadcaster)
                                                   GAPRole_StartDevice (broadcaster)
                                                   GAP_DeviceInit (gap)
                                                   GAP_EndDiscoverable (gap_peridevmgr)
                                                   GAP_Init (gap_simpletask)
                                                   GAP_MakeDiscoverable (gap_peridevmgr)
                                                   GAP_ParamsInit (gap_configmgr)
                                                   GAP_PeriDevMgrInit (gap_peridevmgr)
                                                   GAP_ProcessEvent (gap_simpletask)
                                                   GAP_UpdateAdvertisingData (gap_peridevmgr)
                                                   HCI_CommandCompleteEvent (hci_event)
                                                   HCI_EXT_BuildRevisionCmd (hci)
                                                   HCI_EXT_ClkDivOnHaltCmd (hci)
                                                   HCI_EXT_DeclareNvUsageCmd (hci)
                                                   HCI_EXT_DecryptCmd (hci)
                                                   HCI_EXT_HaltDuringRfCmd (hci)
                                                   HCI_EXT_MapPmIoPortCmd (hci)
                                                   HCI_EXT_ModemTestRxCmd (hci)
                                                   HCI_EXT_ModemTestTxCmd (hci)
                                                   HCI_EXT_ResetSystemCmd (hci_PATCH)
                                                   HCI_EXT_SetFreqTuneCmd (hci)
                                                   HCI_EXT_SetMaxDtmTxPowerCmd (hci)
                                                   HCI_EXT_SetRxGainCmd (hci)
                                                   HCI_EXT_SetTxPowerCmd (hci)
                                                   HCI_Init (hci_tl)
                                                   HCI_LE_AddWhiteListCmd (hci)
                                                   HCI_LE_EncryptCmd (hci)
                                                   HCI_LE_ReceiverTestCmd (hci)
                                                   HCI_LE_RemoveWhiteListCmd (hci)
                                                   HCI_LE_SetAdvDataCmd (hci)
                                                   HCI_LE_SetAdvEnableCmd (hci)
                                                   HCI_LE_SetAdvParamCmd (hci)
                                                   HCI_LE_SetScanRspDataCmd (hci)
                                                   HCI_LE_TransmitterTestCmd (hci)
                                                   HCI_ProcessEvent (hci_tl)
                                                   HCI_ReadLocalVersionInfoCmd (hci)
                                                   HCI_ReadRssiCmd (hci)
                                                   HCI_ReverseBytes (hci_data)
                                                   HCI_SendCommandCompleteEvent (hci_event)
                                                   HCI_SetEventMaskCmd (hci)
                                                   HCI_SetEventMaskPage2Cmd (hci_PATCH)
                                                   HCI_VendorSpecifcCommandCompleteEvent (hci_event_PATCH)
                                                   HalFlashRead (hal_flash)
                                                   HalFlashWrite (hal_flash)
                                                   HalLedBlink (hal_led)
                                                   HalLedSet (hal_led)
                                                   HalLedUpdate (hal_led)
                                                   HalUARTInitUSB (hal_uart)
                                                   HalUARTOpen (hal_uart)
                                                   HalUARTRead (hal_uart)
                                                   HalUARTRx (hal_uart)
                                                   HalUARTWrite (hal_uart)
                                                   Hal_ProcessEvent (hal_drivers)
                                                   Hal_UART_RxBufLen (hal_uart)
                                                   InitBoard (OnBoard)
                                                   LL_AddWhiteListDevice (ll)
                                                   LL_DirectTestEnd (ll)
                                                   LL_DirectTestRxTest (ll)
                                                   LL_DirectTestTxTest (ll)
                                                   LL_ENC_AES128_Decrypt (ll_enc)
                                                   LL_ENC_AES128_Encrypt (ll_enc)
                                                   LL_ENC_GenerateTrueRandNum (ll_enc)
                                                   LL_ENC_SetupCryptoDMA (ll_enc)
                                                   LL_EXT_BuildRevision (ll)
                                                   LL_EXT_Decrypt (ll)
                                                   LL_EXT_ExtendRfRange (ll)
                                                   LL_EXT_MapPmIoPort (ll)
                                                   LL_EXT_ModemTestRx (ll)
                                                   LL_EXT_ModemTestTx (ll)
                                                   LL_EXT_ResetSystem (ll)
                                                   LL_EXT_SaveFreqTune (ll)
                                                   LL_EXT_SetBDADDR (ll)
                                                   LL_EXT_SetFreqTune (ll)
                                                   LL_EXT_SetRxGain (ll)
                                                   LL_EXT_SetTxPower (ll)
                                                   LL_Encrypt (ll)
                                                   LL_Init (ll)
                                                   LL_ProcessEvent (ll)
                                                   LL_Rand (ll)
                                                   LL_RandCback (hci)
                                                   LL_ReadAdvChanTxPower (ll)
                                                   LL_ReadWlSize (ll)
                                                   LL_RemoveWhiteListDevice (ll)
                                                   LL_SetAdvControl (ll)
                                                   LL_SetAdvData (ll)
                                                   LL_SetAdvParam (ll)
                                                   LL_SetScanRspData (ll)
                                                   LL_TX_bm_alloc (ll)
                                                   NPI_InitTransport (npi)
                                                   NPI_ReadTransport (npi)
                                                   NPI_WriteTransport (npi)
                                                   OnBoard_KeyCallback (OnBoard)
                                                   OnBoard_SendKeys (OnBoard)
                                                   PHY_AddWlEntry (phy)
                                                   PHY_ClearBlacklistIndex (phy)
                                                   PHY_RemoveWlEntry (phy)
                                                   PHY_SetBlacklistIndex (phy)
                                                   PHY_SetCRCInit (phy)
                                                   PHY_SetSyncWord (phy)
                                                   SerialDebug_process (serialInterface)
                                                   SerialInterface_Init (serialInterface)
                                                   SerialInterface_ProcessEvent (serialInterface)
                                                   SimpleBLEBroadcaster_Init (simpleBLEBroadcaster)
                                                   SimpleBLEBroadcaster_ProcessEvent (simpleBLEBroadcaster)
                                                   cSerialPacketParser (serialInterface)
                                                   cleanErasedPage (osal_snv)
                                                   compactPage (osal_snv)
                                                   erasePage (osal_snv)
                                                   findItem (osal_snv)
                                                   findOffset (osal_snv)
                                                   gapFindADType (gap_devmgr)
                                                   gapPeriProcessHCICmdCompleteEvt (gap_peridevmgr)
                                                   gapProcessAdvertisingEvt (gap_peridevmgr)
                                                   gapProcessHCICmdCompleteEvt (gap_simpletask)
                                                   gapProcessRandomAddrComplete (gap_configmgr)
                                                   gapReadBD_ADDRStatus (gap_configmgr)
                                                   gapReadBufSizeCmdStatus (gap_configmgr)
                                                   gapRole_ProcessGAPMsg (broadcaster)
                                                   gapRole_ProcessOSALMsg (broadcaster)
                                                   gapRole_SetupGAP (broadcaster)
                                                   gapSendDeviceInitDoneEvent (gap_configmgr)
                                                   gapSendMakeDiscEvent (gap_peridevmgr)
                                                   gapSetAdvParams (gap_peridevmgr)
                                                   gapSetAdvParamsStatus (gap_peridevmgr)
                                                   gapWriteAdvDataStatus (gap_peridevmgr)
                                                   gapWriteAdvEnableStatus (gap_peridevmgr)
                                                   halUartPollRx (hal_uart)
                                                   halUartPollTx (hal_uart)
                                                   hciExtDecrypt (hci_tl)
                                                   hciLEEncrypt (hci_tl)
                                                   hciLESetAdvParam (hci_tl)
                                                   hciProcessCtrlToHost (hci_tl)
                                                   hciProcessHostToCtrlCmd (hci_tl)
                                                   hciProcessHostToCtrlData (hci_tl)
                                                   hciSerialPacketParser (hci_tl)
                                                   initNV (osal_snv)
                                                   isLimitedDiscoverableMode (gap_peridevmgr)
                                                   llAllocTask (ll_scheduler)
                                                   llClearSetInts (ll_common)
                                                   llDiscoverableAdvEvt_TaskEndOk (ll_advEndCauses)
                                                   llFindNextSecTask (ll_scheduler)
                                                   llFindTxPowerSettings (ll_common)
                                                   llNonConnAdvEvt_TaskEndOk (ll_advEndCauses)
                                                   llScheduleTask (ll_scheduler)
                                                   llScheduler (ll_scheduler)
                                                   llSetT2OVFC2Event2 (ll_timer2)
                                                   llSetupNonConnectableAdvEvt (ll_common)
                                                   llSetupScannableAdvEvt (ll_common)
                                                   memcpy (?memcpy)
                                                   osalAddTimer (OSAL_Timers)
                                                   osalClockUpdate (OSAL_ClockBLE)
                                                   osalFindTimer (OSAL_Timers)
                                                   osalInitTasks (OSAL_SimpleBLEBroadcaster)
                                                   osalTimeUpdate (OSAL_ClockBLE)
                                                   osalTimerInit (OSAL_Timers)
                                                   osalTimerUpdate (OSAL_Timers)
                                                   osal_CbTimerInit (osal_cbtimer)
                                                   osal_CbTimerProcessEvent (osal_cbtimer)
                                                   osal_bm_alloc (osal_bufmgr)
                                                   osal_bm_free (osal_bufmgr)
                                                   osal_clear_event (OSAL)
                                                   osal_get_timeoutEx (OSAL_Timers)
                                                   osal_mem_alloc (OSAL_Memory)
                                                   osal_mem_free (OSAL_Memory)
                                                   osal_mem_kick (OSAL_Memory)
                                                   osal_memcmp (OSAL)
                                                   osal_memcpy (OSAL)
                                                   osal_memset (OSAL)
                                                   osal_msg_allocate (OSAL)
                                                   osal_msg_deallocate (OSAL)
                                                   osal_msg_enqueue (OSAL)
                                                   osal_msg_enqueue_push (OSAL)
                                                   osal_msg_extract (OSAL)
                                                   osal_msg_push (OSAL)
                                                   osal_msg_push_front (OSAL)
                                                   osal_msg_receive (OSAL)
                                                   osal_msg_send (OSAL)
                                                   osal_pwrmgr_task_state (OSAL_PwrMgr)
                                                   osal_run_system (OSAL)
                                                   osal_set_event (OSAL)
                                                   osal_snv_read (osal_snv)
                                                   osal_snv_write (osal_snv)
                                                   osal_start_reload_timer (OSAL_Timers)
                                                   osal_start_timerEx (OSAL_Timers)
                                                   osal_stop_timerEx (OSAL_Timers)
                                                   parseCmd (serialInterface)
                                                   peripheralStateNotificationCB (simpleBLEBroadcaster)
                                                   phyFindWlEntry (phy)
                                                   sendSerialEvt (serialInterface)
                                                   setActivePage (osal_snv)
                                                   setXferPage (osal_snv)
                                                   usbdpGetConfigurationDesc (usb_descriptor_parser)
                                                   usbdpGetInterfaceDesc (usb_descriptor_parser)
                                                   usbdpGetStringDesc (usb_descriptor_parser)
                                                   usbfwInit (usb_framework)
                                                   usbfwReadFifo (usb_framework)
                                                   usbfwSetupHandler (usb_framework)
                                                   usbfwWriteFifo (usb_framework)
                                                   usbirqInit (usb_interrupt)
                                                   usbsrGetDescriptor (usb_standard_requests)
                                                   usbsrGetInterface (usb_standard_requests)
                                                   usbsrSetConfiguration (usb_standard_requests)
                                                   usbsrSetInterface (usb_standard_requests)
                                                   verifyWordM (osal_snv)
                                                   writeItem (osal_snv)
                                                   writeWord (osal_snv)
                                                   writeWordM (osal_snv)
                                                   xferItem (osal_snv)

    -------------------------------------------------------------------------
  LIBRARY MODULE, NAME : ?FUNC_ENTER_XDATA

  SEGMENTS IN THE MODULE
  ======================
RCODE
  Relative segment, address: CODE 000010C5 - 0000112A (0x66 bytes), align: 0
  Segment part 1.
           ENTRY                   ADDRESS         REF BY
           =====                   =======         ======
           ?FUNC_ENTER_XDATA       000010C5        ll24BitTimeCompare (ll_timer2)
                                                   ll24BitTimeDelta (ll_timer2)
                                                   llT2OVFC1_ISR (ll_isr)

    -------------------------------------------------------------------------
  LIBRARY MODULE, NAME : ?BANKED_LEAVE_XDATA

  SEGMENTS IN THE MODULE
  ======================
RCODE
  Relative segment, address: CODE 0000112B - 00001170 (0x46 bytes), align: 0
  Segment part 1.
           ENTRY                   ADDRESS         REF BY
           =====                   =======         ======
           ?BANKED_LEAVE_XDATA     0000112B        Application_UpdateAdv (simpleBLEBroadcaster)
                                                   Application_UpdateRsp (simpleBLEBroadcaster)
                                                   ChangeFeature (usb_standard_requests)
                                                   ConfigureEndpoints (usb_standard_requests)
                                                   GAPRole_GetParameter (broadcaster)
                                                   GAPRole_Init (broadcaster)
                                                   GAPRole_ProcessEvent (broadcaster)
                                                   GAPRole_SetParameter (broadcaster)
                                                   GAPRole_StartDevice (broadcaster)
                                                   GAP_DeviceInit (gap)
                                                   GAP_Init (gap_simpletask)
                                                   GAP_UpdateAdvertisingData (gap_peridevmgr)
                                                   HCI_CommandCompleteEvent (hci_event)
                                                   HCI_EXT_ResetSystemCmd (hci_PATCH)
                                                   HCI_ReverseBytes (hci_data)
                                                   HCI_SetEventMaskPage2Cmd (hci_PATCH)
                                                   HCI_VendorSpecifcCommandCompleteEvent (hci_event_PATCH)
                                                   HalFlashRead (hal_flash)
                                                   HalFlashWrite (hal_flash)
                                                   HalLedBlink (hal_led)
                                                   HalLedSet (hal_led)
                                                   HalLedUpdate (hal_led)
                                                   HalUARTInitUSB (hal_uart)
                                                   HalUARTOpen (hal_uart)
                                                   HalUARTRead (hal_uart)
                                                   HalUARTRx (hal_uart)
                                                   HalUARTWrite (hal_uart)
                                                   Hal_ProcessEvent (hal_drivers)
                                                   Hal_UART_RxBufLen (hal_uart)
                                                   InitBoard (OnBoard)
                                                   LL_EXT_SetBDADDR (ll)
                                                   NPI_InitTransport (npi)
                                                   NPI_ReadTransport (npi)
                                                   NPI_WriteTransport (npi)
                                                   OnBoard_KeyCallback (OnBoard)
                                                   OnBoard_SendKeys (OnBoard)
                                                   Segment part 111 (phy)
                                                   Segment part 118 (ll)
                                                   Segment part 12 (ll_advEndCauses)
                                                   Segment part 124 (ll)
                                                   Segment part 137 (ll)
                                                   Segment part 17 (gap_simpletask)
                                                   Segment part 17 (ll_enc)
                                                   Segment part 18 (hci_event)
                                                   Segment part 19 (hci_tl)
                                                   Segment part 222 (phy)
                                                   Segment part 23 (ll_scheduler)
                                                   Segment part 25 (gap_configmgr)
                                                   Segment part 26 (ll_enc)
                                                   Segment part 33 (gap_configmgr)
                                                   Segment part 36 (gap_peridevmgr)
                                                   Segment part 43 (phy)
                                                   Segment part 48 (gap_configmgr)
                                                   Segment part 61 (gap_peridevmgr)
                                                   Segment part 62 (hci)
                                                   Segment part 64 (gap_peridevmgr)
                                                   Segment part 79 (phy)
                                                   Segment part 84 (hci)
                                                   Segment part 96 (ll)
                                                   Segment part 98 (hci_tl)
                                                   Segment part 98 (ll_common)
                                                   SerialDebug_process (serialInterface)
                                                   SerialInterface_Init (serialInterface)
                                                   SerialInterface_ProcessEvent (serialInterface)
                                                   SimpleBLEBroadcaster_Init (simpleBLEBroadcaster)
                                                   SimpleBLEBroadcaster_ProcessEvent (simpleBLEBroadcaster)
                                                   cSerialPacketParser (serialInterface)
                                                   cleanErasedPage (osal_snv)
                                                   compactPage (osal_snv)
                                                   erasePage (osal_snv)
                                                   findItem (osal_snv)
                                                   findOffset (osal_snv)
                                                   gapFindADType (gap_devmgr)
                                                   gapRole_ProcessGAPMsg (broadcaster)
                                                   gapRole_ProcessOSALMsg (broadcaster)
                                                   gapRole_SetupGAP (broadcaster)
                                                   gapSetAdvParams (gap_peridevmgr)
                                                   gapWriteAdvEnableStatus (gap_peridevmgr)
                                                   halUartPollRx (hal_uart)
                                                   halUartPollTx (hal_uart)
                                                   hciProcessCtrlToHost (hci_tl)
                                                   hciProcessHostToCtrlCmd (hci_tl)
                                                   hciSerialPacketParser (hci_tl)
                                                   initNV (osal_snv)
                                                   llAllocTask (ll_scheduler)
                                                   llFindNextSecTask (ll_scheduler)
                                                   llFindTxPowerSettings (ll_common)
                                                   llSetT2OVFC2Event2 (ll_timer2)
                                                   memcpy (?memcpy)
                                                   osalAddTimer (OSAL_Timers)
                                                   osalClockUpdate (OSAL_ClockBLE)
                                                   osalFindTimer (OSAL_Timers)
                                                   osalInitTasks (OSAL_SimpleBLEBroadcaster)
                                                   osalTimeUpdate (OSAL_ClockBLE)
                                                   osalTimerInit (OSAL_Timers)
                                                   osalTimerUpdate (OSAL_Timers)
                                                   osal_CbTimerInit (osal_cbtimer)
                                                   osal_CbTimerProcessEvent (osal_cbtimer)
                                                   osal_bm_alloc (osal_bufmgr)
                                                   osal_bm_free (osal_bufmgr)
                                                   osal_clear_event (OSAL)
                                                   osal_get_timeoutEx (OSAL_Timers)
                                                   osal_mem_alloc (OSAL_Memory)
                                                   osal_mem_free (OSAL_Memory)
                                                   osal_mem_kick (OSAL_Memory)
                                                   osal_memcmp (OSAL)
                                                   osal_memcpy (OSAL)
                                                   osal_memset (OSAL)
                                                   osal_msg_allocate (OSAL)
                                                   osal_msg_deallocate (OSAL)
                                                   osal_msg_enqueue (OSAL)
                                                   osal_msg_enqueue_push (OSAL)
                                                   osal_msg_extract (OSAL)
                                                   osal_msg_push (OSAL)
                                                   osal_msg_push_front (OSAL)
                                                   osal_msg_receive (OSAL)
                                                   osal_msg_send (OSAL)
                                                   osal_pwrmgr_task_state (OSAL_PwrMgr)
                                                   osal_run_system (OSAL)
                                                   osal_set_event (OSAL)
                                                   osal_snv_read (osal_snv)
                                                   osal_snv_write (osal_snv)
                                                   osal_start_reload_timer (OSAL_Timers)
                                                   osal_start_timerEx (OSAL_Timers)
                                                   osal_stop_timerEx (OSAL_Timers)
                                                   parseCmd (serialInterface)
                                                   peripheralStateNotificationCB (simpleBLEBroadcaster)
                                                   sendSerialEvt (serialInterface)
                                                   setActivePage (osal_snv)
                                                   setXferPage (osal_snv)
                                                   usbdpGetConfigurationDesc (usb_descriptor_parser)
                                                   usbdpGetInterfaceDesc (usb_descriptor_parser)
                                                   usbdpGetStringDesc (usb_descriptor_parser)
                                                   usbfwInit (usb_framework)
                                                   usbfwReadFifo (usb_framework)
                                                   usbfwSetupHandler (usb_framework)
                                                   usbfwWriteFifo (usb_framework)
                                                   usbirqInit (usb_interrupt)
                                                   usbsrGetDescriptor (usb_standard_requests)
                                                   usbsrGetInterface (usb_standard_requests)
                                                   usbsrSetConfiguration (usb_standard_requests)
                                                   usbsrSetInterface (usb_standard_requests)
                                                   verifyWordM (osal_snv)
                                                   writeItem (osal_snv)
                                                   writeWord (osal_snv)
                                                   writeWordM (osal_snv)
                                                   xferItem (osal_snv)

    -------------------------------------------------------------------------
  LIBRARY MODULE, NAME : ?FUNC_LEAVE_XDATA

  SEGMENTS IN THE MODULE
  ======================
RCODE
  Relative segment, address: CODE 00001171 - 000011B0 (0x40 bytes), align: 0
  Segment part 1.
           ENTRY                   ADDRESS         REF BY
           =====                   =======         ======
           ?FUNC_LEAVE_XDATA       00001171        Segment part 97 (ll_timer2)
                                                   ll24BitTimeDelta (ll_timer2)
                                                   llT2OVFC1_ISR (ll_isr)

    -------------------------------------------------------------------------
  LIBRARY MODULE, NAME : ?INTERRUPT_ENTER_XSP

  SEGMENTS IN THE MODULE
  ======================
RCODE
  Relative segment, address: CODE 000011B1 - 0000120F (0x5f bytes), align: 0
  Segment part 1.
           ENTRY                   ADDRESS         REF BY
           =====                   =======         ======
           ?INTERRUPT_ENTER_XSP    000011B1        RF_NormalIsr (ll_isr)
                                                   T2_Isr (ll_isr)
                                                   usbirqHandler (usb_interrupt)

    -------------------------------------------------------------------------
  LIBRARY MODULE, NAME : ?INTERRUPT_LEAVE_XSP

  SEGMENTS IN THE MODULE
  ======================
RCODE
  Relative segment, address: CODE 00001210 - 00001267 (0x58 bytes), align: 0
  Segment part 1.
           ENTRY                   ADDRESS         REF BY
           =====                   =======         ======
           ?INTERRUPT_LEAVE_XSP    00001210        RF_NormalIsr (ll_isr)
                                                   T2_Isr (ll_isr)
                                                   usbirqHandler (usb_interrupt)

    -------------------------------------------------------------------------
  LIBRARY MODULE, NAME : ?PUSH_XSTACK_I

  SEGMENTS IN THE MODULE
  ======================
RCODE
  Relative segment, address: CODE 00001268 - 0000126B (0x4 bytes), align: 0
  Segment part 0.
           ENTRY                   ADDRESS         REF BY
           =====                   =======         ======
           ?PUSH_XSTACK_I_FOUR     00001268        HalLedUpdate (hal_led)
                                                   LL_EXT_ExtendRfRange (ll)
                                                   LL_EXT_SetRxGain (ll)
                                                   LL_EXT_SetTxPower (ll)
                                                   LL_ProcessEvent (ll)
                                                   gapProcessAdvertisingEvt (gap_peridevmgr)
                                                   gapRole_ProcessGAPMsg (broadcaster)
                                                   gapWriteAdvEnableStatus (gap_peridevmgr)
                                                   llFindNextSecTask (ll_scheduler)
                                                   llScheduleTask (ll_scheduler)
                                                   llScheduler (ll_scheduler)
                                                   osal_start_reload_timer (OSAL_Timers)
                                                   osal_start_timerEx (OSAL_Timers)
    -------------------------------------------------------------------------
RCODE
  Relative segment, address: CODE 0000126C - 0000126F (0x4 bytes), align: 0
  Segment part 1.
           ENTRY                   ADDRESS         REF BY
           =====                   =======         ======
           ?PUSH_XSTACK_I_THREE    0000126C        usbfwSetupHandler (usb_framework)
    -------------------------------------------------------------------------
RCODE
  Relative segment, address: CODE 00001270 - 00001273 (0x4 bytes), align: 0
  Segment part 2.
           ENTRY                   ADDRESS         REF BY
           =====                   =======         ======
           ?PUSH_XSTACK_I_TWO      00001270        Application_UpdateAdv (simpleBLEBroadcaster)
                                                   Application_UpdateRsp (simpleBLEBroadcaster)
                                                   GAPRole_GetParameter (broadcaster)
                                                   GAPRole_ProcessEvent (broadcaster)
                                                   GAPRole_SetParameter (broadcaster)
                                                   GAP_MakeDiscoverable (gap_peridevmgr)
                                                   GAP_UpdateAdvertisingData (gap_peridevmgr)
                                                   HCI_CommandCompleteEvent (hci_event)
                                                   HCI_EXT_DecryptCmd (hci)
                                                   HCI_LE_EncryptCmd (hci)
                                                   HCI_ReadLocalVersionInfoCmd (hci)
                                                   HCI_SendCommandCompleteEvent (hci_event)
                                                   HCI_SetEventMaskCmd (hci)
                                                   HCI_SetEventMaskPage2Cmd (hci_PATCH)
                                                   HCI_VendorSpecifcCommandCompleteEvent (hci_event_PATCH)
                                                   LL_DirectTestEnd (ll)
                                                   LL_EXT_Decrypt (ll)
                                                   LL_EXT_SaveFreqTune (ll)
                                                   LL_Encrypt (ll)
                                                   LL_Init (ll)
                                                   LL_RandCback (hci)
                                                   LL_SetAdvData (ll)
                                                   LL_SetScanRspData (ll)
                                                   SimpleBLEBroadcaster_Init (simpleBLEBroadcaster)
                                                   cleanErasedPage (osal_snv)
                                                   compactPage (osal_snv)
                                                   erasePage (osal_snv)
                                                   findItem (osal_snv)
                                                   findOffset (osal_snv)
                                                   gapProcessRandomAddrComplete (gap_configmgr)
                                                   gapReadBD_ADDRStatus (gap_configmgr)
                                                   gapRole_ProcessGAPMsg (broadcaster)
                                                   gapRole_SetupGAP (broadcaster)
                                                   gapSendDeviceInitDoneEvent (gap_configmgr)
                                                   gapSetAdvParams (gap_peridevmgr)
                                                   hciLESetAdvParam (hci_tl)
                                                   initNV (osal_snv)
                                                   isLimitedDiscoverableMode (gap_peridevmgr)
                                                   llFindTxPowerSettings (ll_common)
                                                   osal_memset (OSAL)
                                                   osal_msg_receive (OSAL)
                                                   osal_snv_read (osal_snv)
                                                   osal_snv_write (osal_snv)
                                                   verifyWordM (osal_snv)
                                                   writeWord (osal_snv)
                                                   writeWordM (osal_snv)
                                                   xferItem (osal_snv)
    -------------------------------------------------------------------------
RCODE
  Relative segment, address: CODE 00001274 - 00001275 (0x2 bytes), align: 0
  Segment part 3.
           ENTRY                   ADDRESS         REF BY
           =====                   =======         ======
           ?PUSH_XSTACK_I_ONE      00001274        HCI_LE_SetAdvParamCmd (hci)
                                                   LL_ENC_AES128_Decrypt (ll_enc)
                                                   LL_ENC_AES128_Encrypt (ll_enc)
                                                   gapSetAdvParams (gap_peridevmgr)
                                                   hciLESetAdvParam (hci_tl)
                                                   writeItem (osal_snv)
                                                   writeWord (osal_snv)
                                                   writeWordM (osal_snv)
    -------------------------------------------------------------------------
RCODE
  Relative segment, address: CODE 00001276 - 00001282 (0xd bytes), align: 0
  Segment part 4.             Intra module refs:   ?PUSH_XSTACK_I_FOUR
                                                   ?PUSH_XSTACK_I_ONE
                                                   ?PUSH_XSTACK_I_THREE
                                                   ?PUSH_XSTACK_I_TWO
           ENTRY                   ADDRESS         REF BY
           =====                   =======         ======
           ?PUSH_XSTACK_I          00001276 

    -------------------------------------------------------------------------
  LIBRARY MODULE, NAME : ?PUSH_XSTACK8_X

  SEGMENTS IN THE MODULE
  ======================
RCODE
  Relative segment, address: CODE 00001283 - 00001286 (0x4 bytes), align: 0
  Segment part 1.
           ENTRY                   ADDRESS         REF BY
           =====                   =======         ======
           ?PUSH_XSTACK8_X_FOUR    00001283        GAP_MakeDiscoverable (gap_peridevmgr)
                                                   LL_EXT_ResetSystem (ll)
                                                   gapProcessRandomAddrComplete (gap_configmgr)
                                                   gapWriteAdvEnableStatus (gap_peridevmgr)
    -------------------------------------------------------------------------
RCODE
  Relative segment, address: CODE 00001287 - 0000128A (0x4 bytes), align: 0
  Segment part 2.
           ENTRY                   ADDRESS         REF BY
           =====                   =======         ======
           ?PUSH_XSTACK8_X_THREE   00001287        usbfwSetupHandler (usb_framework)
    -------------------------------------------------------------------------
RCODE
  Relative segment, address: CODE 0000128B - 0000128E (0x4 bytes), align: 0
  Segment part 3.
           ENTRY                   ADDRESS         REF BY
           =====                   =======         ======
           ?PUSH_XSTACK8_X_TWO     0000128B        HCI_LE_SetAdvParamCmd (hci)
    -------------------------------------------------------------------------
RCODE
  Relative segment, address: CODE 0000128F - 000012B7 (0x29 bytes), align: 0
  Segment part 5.             Intra module refs:   ?PUSH_XSTACK8_X_FOUR
                                                   ?PUSH_XSTACK8_X_THREE
                                                   ?PUSH_XSTACK8_X_TWO
           ENTRY                   ADDRESS         REF BY
           =====                   =======         ======
           ?PUSH_XSTACK8_X         0000128F 

    -------------------------------------------------------------------------
  LIBRARY MODULE, NAME : ?US_SWITCH_DENSE

  SEGMENTS IN THE MODULE
  ======================
RCODE
  Relative segment, address: CODE 000012B8 - 000012BE (0x7 bytes), align: 0
  Segment part 0.
           ENTRY                   ADDRESS         REF BY
           =====                   =======         ======
           ?US_SWITCH_DENSE        000012B8        GAPRole_GetParameter (broadcaster)
                                                   GAPRole_SetParameter (broadcaster)
                                                   gapPeriProcessHCICmdCompleteEvt (gap_peridevmgr)
           ?US_SD_CFI_INV_BEGINS   000012B8 
    -------------------------------------------------------------------------
RCODE
  Relative segment, address: CODE 000012BF - 000012FC (0x3e bytes), align: 0
  Segment part 2.             Intra module refs:   Segment part 0
    -------------------------------------------------------------------------
RCODE
  Relative segment, address: CODE 000012FD - 000012FD (0x1 bytes), align: 0
  Segment part 4.             Intra module refs:   Segment part 0
           ENTRY                   ADDRESS         REF BY
           =====                   =======         ======
           ?US_SD_CFI_INV_ENDS     000012FE 

    -------------------------------------------------------------------------
  LIBRARY MODULE, NAME : ?US_SWITCH_SPARSE

  SEGMENTS IN THE MODULE
  ======================
RCODE
  Relative segment, address: CODE 000012FE - 00001307 (0xa bytes), align: 0
  Segment part 0.
           ENTRY                   ADDRESS         REF BY
           =====                   =======         ======
           ?US_SWITCH_SPARSE       000012FE        gapProcessHCICmdCompleteEvt (gap_simpletask)
           ?US_SS_CFI_INV_BEGINS   000012FE 
    -------------------------------------------------------------------------
RCODE
  Relative segment, address: CODE 00001308 - 00001348 (0x41 bytes), align: 0
  Segment part 2.             Intra module refs:   Segment part 0
           ENTRY                   ADDRESS         REF BY
           =====                   =======         ======
           ?US_SWITCH_SPARSE_LEAVE
                                   0000133A        Segment part 0 (?US_JMP_IF_IN_RANGE)
                                                   Segment part 0 (?US_JMP_IF_VALUE)
    -------------------------------------------------------------------------
RCODE
  Relative segment, address: CODE 00001349 - 00001349 (0x1 bytes), align: 0
  Segment part 4.             Intra module refs:   Segment part 0
           ENTRY                   ADDRESS         REF BY
           =====                   =======         ======
           ?US_SS_CFI_INV_ENDS     0000134A 

    -------------------------------------------------------------------------
  LIBRARY MODULE, NAME : ?US_JMP_IF_IN_RANGE

  SEGMENTS IN THE MODULE
  ======================
RCODE
  Relative segment, address: CODE 0000134A - 00001388 (0x3f bytes), align: 0
  Segment part 0.
           ENTRY                   ADDRESS         REF BY
           =====                   =======         ======
           ?US_JMP_IF_IN_RANGE     0000134A        ?US_SWITCH_SPARSE_LEAVE (?US_SWITCH_SPARSE)
           ?US_JR_CFI_INV_BEGINS   0000134A 
           ?US_JR_CFI_INV_ENDS     00001389 

    -------------------------------------------------------------------------
  LIBRARY MODULE, NAME : ?US_JMP_IF_VALUE

  SEGMENTS IN THE MODULE
  ======================
RCODE
  Relative segment, address: CODE 00001389 - 000013B3 (0x2b bytes), align: 0
  Segment part 0.
           ENTRY                   ADDRESS         REF BY
           =====                   =======         ======
           ?US_JMP_IF_VALUE        00001389        ?US_SWITCH_SPARSE_LEAVE (?US_SWITCH_SPARSE)
           ?US_JMP_IF_VALUE_CFI_INV_BEGINS
                                   00001389 
           ?US_JMP_IF_VALUE_CFI_INV_ENDS
                                   000013B4 

    -------------------------------------------------------------------------
  LIBRARY MODULE, NAME : ?memcpy

  SEGMENTS IN THE MODULE
  ======================
<BANKED_CODE,XDATA_ROM_C_FLASH> 1 (was BANKED_CODE)
  Relative segment, address: CODE 0000C680 - 0000C6C5 (0x46 bytes), align: 0
  Segment part 6.             Intra module refs:   memcpy::?relay
           ENTRY                   ADDRESS         REF BY
           =====                   =======         ======
           memcpy                  0000C680 
               XSTACK = 00000002 ( 0000000A )
               ISTACK = 00000000 ( 00000001 )
    -------------------------------------------------------------------------
BANK_RELAYS
  Relative segment, address: CODE 00000C26 - 00000C2B (0x6 bytes), align: 0
  Segment part 7.
           ENTRY                   ADDRESS         REF BY
           =====                   =======         ======
           memcpy::?relay          00000C26        Application_UpdateAdv (simpleBLEBroadcaster)
                                                   Application_UpdateRsp (simpleBLEBroadcaster)
                                                   SimpleBLEBroadcaster_Init (simpleBLEBroadcaster)

    -------------------------------------------------------------------------
  LIBRARY MODULE, NAME : ?memset

  SEGMENTS IN THE MODULE
  ======================
<BANKED_CODE,XDATA_ROM_C_FLASH> 1 (was BANKED_CODE)
  Relative segment, address: CODE 0000C6C6 - 0000C6F1 (0x2c bytes), align: 0
  Segment part 6.             Intra module refs:   memset::?relay
           ENTRY                   ADDRESS         REF BY
           =====                   =======         ======
           memset                  0000C6C6 
               XSTACK = 00000002 ( 00000000 )
               ISTACK = 00000000 ( 00000002 )
    -------------------------------------------------------------------------
BANK_RELAYS
  Relative segment, address: CODE 00000C2C - 00000C31 (0x6 bytes), align: 0
  Segment part 7.
           ENTRY                   ADDRESS         REF BY
           =====                   =======         ======
           memset::?relay          00000C2C        Application_UpdateRsp (simpleBLEBroadcaster)
                                                   osal_memset (OSAL)




                ****************************************
                *                                      *
                *            MODULE SUMMARY            *
                *                                      *
                ****************************************

Module                         CODE      DATA      XDATA  IDATA    BIT  CONST
------                         ----      ----      -----  -----    ---  -----
                              (Rel)  (Rel)  (Abs)  (Rel)  (Rel)  (Rel)  (Rel)
?ADD_XSTACK_DISP8                27
?ALLOC_XSTACK8                   22
?BANKED_CODE_SUPPORT             30
?BANKED_ENTER_XDATA             108
?BANKED_LEAVE_XDATA              70
?CALL_IND                         2
?C_GPTR_LOAD                     26
?C_GPTR_STORE                    22
?DEALLOC_XSTACK8                 27
?FUNC_ENTER_XDATA               102
?FUNC_LEAVE_XDATA                64
?G_EQ                            11
?INTERRUPT_ENTER_XSP             95
?INTERRUPT_LEAVE_XSP             88
?L_ADD                           19
?L_ADD_TO_X                      19
?L_ADD_X                         19
?L_AND_X                         19
?L_EQ_X                          21
?L_IOR_X                         19
?L_MOV_TO_X                      15
?L_MOV_X                         15
?L_MUL                          128
?L_SUB                           20
?L_SUB_FROM_X                    20
?MOVE_LONG8_XDATA_IDATA          13
?MOVE_LONG8_XDATA_XDATA          33
?PUSH_XSTACK8_X                  53
?PUSH_XSTACK_I                   27
?SS_SHR                          16
?S_DIV_MOD                      154
?S_SHL                           19
?UL_DIV_MOD                     111
?UL_GE_X                         31
?UL_GT                           16
?UL_GT_X                         16
?UL_SHR                          25
?US_JMP_IF_IN_RANGE              63
?US_JMP_IF_VALUE                 43
?US_SHR                          15
?US_SWITCH_DENSE                 70
?US_SWITCH_SPARSE                76
?XLOAD_R0123                     12
?XLOAD_R2345                     12
?XSTACK_DISP8                    10
?XSTACK_DISP8_RP                 24
?XSTORE_R0123                    12
?cexit                            5
?cmain                          113
?memcpy                          76
?memset                          50
CSTARTUP                         18
  + common                        3
OSAL                          1 804                    3
OSAL_ClockBLE                   326                   10
OSAL_Memory                     754                2 903
OSAL_PwrMgr                     162                    7
OSAL_SimpleBLEBroadcaster       162                    2                   17
OSAL_Timers                   1 525                    6
OnBoard                         273                    2
SimpleBLEBroadcaster_Main        85
VIRTUAL_REGISTERS                       18                           8
broadcaster                   2 016                   88
gap                              81
gap_configmgr                   800                  106
  + shared                                                                  4
gap_devmgr                      179                    2
gap_peridevmgr                1 863                   13                    4
gap_simpletask                  537                    6
hal_adc                          23             4      1
  + shared                                      1
hal_aes                         741
  + shared                                      3
hal_assert                        9
  + shared                                      4
hal_dma                          35             4     40
hal_drivers                     207                    1
hal_flash                       791
  + shared                                      1
hal_key                           9
hal_led                       1 173                   39
  + shared                                      2                           4
hal_sleep                        37             2
  + shared                       46             6
  + common
hal_startup                      11
hal_uart                      1 056                  521
  + shared                                      1
hci                           2 666                    4                   18
hci_PATCH                       437                                        65
hci_data                         90
hci_event                       742                    9
hci_event_PATCH                 263                    8
hci_tl                        2 830                   12                  192
ll                            5 257             8    177      2            49
  + shared                                      2                          12
ll_advEndCauses                 590
ll_common                     1 673            10                          16
ll_constData                     12                                         4
ll_enc                          581             3
ll_errorEndCauses                 9
ll_halt                           7      2
ll_isr                          574
  + shared                      134            10
  + common
ll_scheduler                  1 399                   33                   12
ll_sleep                          4             1
  + shared                                                                  4
ll_timer2                     1 034             8
npi                             236
osal_bufmgr                     304                    2
osal_cbtimer                    371                   62
osal_snv                      6 641                    4                    4
  + shared                                                                  8
phy                           1 599                    1
phy_image                     3 582                                     3 582
serialInterface                 927                   43
simpleBLEBroadcaster            878                   98
usb_cdc_hooks                   289                    7
usb_descriptor                   93
usb_descriptor_parser           969                   44                   76
usb_firmware_library_config      12                   12
usb_framework                 1 048      2            33
usb_interrupt                   271      5
  + shared                       54             3
  + common
usb_standard_requests         2 736                    2
N/A (command line)                       8           640    192
N/A (alignment)                   1                                         1
----------                   ------     --     --  -----    ---      -  -----
Total:                       54 905     35     73  4 941    194      8  4 072
  + common                      134


                ****************************************
                *                                      *
                *      SEGMENTS IN ADDRESS ORDER       *
                *                                      *
                ****************************************


SEGMENT              SPACE    START ADDRESS   END ADDRESS     SIZE  TYPE  ALIGN
=======              =====    =============   ===========     ====  ====  =====
INTVEC               CODE          00000000 - 00000085          86   com    0
CSTART               CODE          00000086 - 00000136          B1   rel    0
BIT_ID               CODE               00000137                     dse    0
DATA_ID              CODE               00000137                     dse    0
IDATA_ID             CODE               00000137                     dse    0
IXDATA_ID            CODE               00000137                     dse    0
PDATA_ID             CODE               00000137                     dse    0
BDATA_ID             CODE               00000137                     dse    0
XDATA_ID             CODE          00000137 - 00000229          F3   rel    0
BANK_RELAYS          CODE          0000022A - 00000C31         A08   rel    0
RCODE                CODE          00000C32 - 000013B3         782   rel    0
CODE_N               CODE               000013B4                     dse    0
DIFUNCT              CODE               000013B4                     dse    0
NEAR_CODE            CODE          000013B4 - 000017A5         3F2   rel    2
<BANKED_CODE,CODE_C> 1
                     CODE          000017A8 - 00007FFD        6856   rel    2
<BANKED_CODE,XDATA_ROM_C_FLASH> 1
                     CODE          00008000 - 0000C702        4703   rel    2
BLENV_ADDRESS_SPACE
                     CODE          0003E800 - 0003F7FF        1000   rel    0
REGISTERS            DATA          00000000 - 00000007           8   rel    0
VREG                 DATA          00000008 - 00000017          10   rel    0
PSP                  DATA               00000018                     dse    0
XSP                  DATA          00000018 - 00000019           2   rel    0
DATA_I               DATA               0000001A                     dse    0
BREG                 BIT        00000020.0  -  00000020.7        8   rel    0
DATA_Z               DATA          00000021 - 00000029           9   rel    0
SFR_AN               DATA          00000080 - 00000080           1   rel    0
                     DATA          00000087 - 00000088           2 
                     DATA          0000008B - 0000008B           1 
                     DATA          0000008D - 0000008D           1 
                     DATA          00000090 - 00000091           2 
                     DATA          00000094 - 00000097           4 
                     DATA          0000009A - 000000A9          10 
                     DATA          000000AB - 000000AF           5 
                     DATA          000000B3 - 000000B4           2 
                     DATA          000000B6 - 000000B6           1 
                     DATA          000000B8 - 000000C0           9 
                     DATA          000000C3 - 000000C3           1 
                     DATA          000000C6 - 000000C7           2 
                     DATA          000000C9 - 000000C9           1 
                     DATA          000000D1 - 000000D7           7 
                     DATA          000000D9 - 000000DB           3 
                     DATA          000000E1 - 000000E5           5 
                     DATA          000000E8 - 000000E9           2 
                     DATA          000000F2 - 000000F2           1 
                     DATA          000000F2 - 000000F5           4 
                     DATA          000000FD - 000000FF           3 
XSTACK               XDATA         00000001 - 00000280         280   rel    0
XDATA_Z              XDATA         00000281 - 0000105A         DDA   rel    0
XDATA_I              XDATA         0000105B - 0000114D          F3   rel    0
<XDATA_N> 1          XDATA         0000114E - 0000134D         200   rel    0
<XDATA_ROM_C> 1      CONST         00008000 - 00008FE7         FE8   rel    2
IDATA_I              IDATA              0000002A                     dse    0
IDATA_Z              IDATA         0000002A - 0000002B           2   rel    0
ISTACK               IDATA         00000040 - 000000FF          C0   rel    0

                ****************************************
                *                                      *
                *        END OF CROSS REFERENCE        *
                *                                      *
                ****************************************

 55 039 bytes of CODE  memory
     35 bytes of DATA  memory (+ 73 absolute )
  4 941 bytes of XDATA memory
    194 bytes of IDATA memory
      8 bits  of BIT   memory
  4 072 bytes of CONST memory

Errors: none
Warnings: none

